 DiskCalculator

 Timestamp is 58f47260 (Mon Apr 17 15:44:32 2017)

 Preferred load address is 00400000

 Start         Length     Name                   Class
 0001:00000000 0006ab87H .text                   CODE
 0001:0006ab90 0000bd05H .text$x                 CODE
 0001:000768a0 0000199eH .text$yc                CODE
 0001:00078240 000010a0H .text$yd                CODE
 0002:00000000 00000104H .CRT$XCA                DATA
 0002:00000104 00000104H .CRT$XCAA               DATA
 0002:00000208 000001c2H .CRT$XCU                DATA
 0002:000003cc 00000104H .CRT$XCZ                DATA
 0002:000004d0 00000104H .CRT$XIA                DATA
 0002:000005d4 00000104H .CRT$XIAA               DATA
 0002:000006d8 00000104H .CRT$XIC                DATA
 0002:000007dc 00000104H .CRT$XIY                DATA
 0002:000008e0 00000104H .CRT$XIZ                DATA
 0002:000009f0 0000f373H .rdata                  DATA
 0002:0000fd64 0000019aH .rdata$debug            DATA
 0002:0000ff00 00002e51H .rdata$r                DATA
 0002:00012d60 00000786H .rdata$sxdata           DATA
 0002:000134e8 00000104H .rtc$IAA                DATA
 0002:000135ec 00000104H .rtc$IZZ                DATA
 0002:000136f0 00000104H .rtc$TAA                DATA
 0002:000137f4 00000104H .rtc$TZZ                DATA
 0002:000138f8 0000a862H .xdata$x                DATA
 0002:0001e160 00000180H .edata                  DATA
 0003:00000000 000011b8H .data                   DATA
 0003:000011b8 000006bcH .bss                    DATA
 0004:00000000 000000c8H .idata$2                DATA
 0004:000000c8 00000014H .idata$3                DATA
 0004:000000dc 000019fcH .idata$4                DATA
 0004:00001ad8 000019fcH .idata$5                DATA
 0004:000034d4 0000f460H .idata$6                DATA
 0005:00000000 00000434H .rsrc$01                DATA
 0005:00000440 00024293H .rsrc$02                DATA

  Address         Publics by Value              Rva+Base       Lib:Object

 0000:00000000       __except_list              00000000     <absolute>
 0000:0000015c       ___safe_se_handler_count   0000015c     <absolute>
 0000:00009876       __fltused                  00009876     <absolute>
 0000:00009876       __ldused                   00009876     <absolute>
 0000:00000000       ___ImageBase               00400000     <linker-defined>
 0001:00003820       ?qt_static_metacall@AboutDialog@@CAXPAVQObject@@W4Call@QMetaObject@@HPAPAX@Z 00404820 f   moc_AboutDialog.obj
 0001:00003890       ?metaObject@AboutDialog@@UBEPBUQMetaObject@@XZ 00404890 f   moc_AboutDialog.obj
 0001:000038d0       ?qt_metacast@AboutDialog@@UAEPAXPBD@Z 004048d0 f   moc_AboutDialog.obj
 0001:00003910       ?qt_metacall@AboutDialog@@UAEHW4Call@QMetaObject@@HPAPAX@Z 00404910 f   moc_AboutDialog.obj
 0001:00003970       ?signalCover@AboutDialog@@IAEXXZ 00404970 f   moc_AboutDialog.obj
 0001:000039a0       ?signalDiscover@AboutDialog@@IAEXXZ 004049a0 f   moc_AboutDialog.obj
 0001:00003a30       ?qt_noop@@YAXXZ            00404a30 f i moc_AboutDialog.obj
 0001:00003a40       ??C?$QScopedPointer@VQObjectData@@U?$QScopedPointerDeleter@VQObjectData@@@@@@QBEPAVQObjectData@@XZ 00404a40 f i moc_AboutDialog.obj
 0001:00003a60       ?qt_static_metacall@BandWidthPage@@CAXPAVQObject@@W4Call@QMetaObject@@HPAPAX@Z 00404a60 f   moc_BandWidthPage.obj
 0001:00003c80       ?metaObject@BandWidthPage@@UBEPBUQMetaObject@@XZ 00404c80 f   moc_BandWidthPage.obj
 0001:00003cc0       ?qt_metacast@BandWidthPage@@UAEPAXPBD@Z 00404cc0 f   moc_BandWidthPage.obj
 0001:00003d00       ?qt_metacall@BandWidthPage@@UAEHW4Call@QMetaObject@@HPAPAX@Z 00404d00 f   moc_BandWidthPage.obj
 0001:00003e20       ?qt_static_metacall@BaseDialog@aptui@@CAXPAVQObject@@W4Call@QMetaObject@@HPAPAX@Z 00404e20 f   moc_BaseDialog.obj
 0001:00004010       ?metaObject@BaseDialog@aptui@@UBEPBUQMetaObject@@XZ 00405010 f   moc_BaseDialog.obj
 0001:00004050       ?qt_metacast@BaseDialog@aptui@@UAEPAXPBD@Z 00405050 f   moc_BaseDialog.obj
 0001:00004090       ?qt_metacall@BaseDialog@aptui@@UAEHW4Call@QMetaObject@@HPAPAX@Z 00405090 f   moc_BaseDialog.obj
 0001:000040f0       ?signalAppButtonClicked@BaseDialog@aptui@@IAEXXZ 004050f0 f   moc_BaseDialog.obj
 0001:00004120       ?signalOptionButtonClicked@BaseDialog@aptui@@IAEXXZ 00405120 f   moc_BaseDialog.obj
 0001:00004150       ?signalMinButtonClicked@BaseDialog@aptui@@IAEXXZ 00405150 f   moc_BaseDialog.obj
 0001:00004180       ?signalMaxButtonClicked@BaseDialog@aptui@@IAEXXZ 00405180 f   moc_BaseDialog.obj
 0001:000041b0       ?signalCloseButtonClicked@BaseDialog@aptui@@IAEXXZ 004051b0 f   moc_BaseDialog.obj
 0001:000041e0       ?signalConfirmButtonClicked@BaseDialog@aptui@@IAEXXZ 004051e0 f   moc_BaseDialog.obj
 0001:00004210       ?signalCancelButtonClicked@BaseDialog@aptui@@IAEXXZ 00405210 f   moc_BaseDialog.obj
 0001:00004340       ?qt_static_metacall@BaseTitle@aptui@@CAXPAVQObject@@W4Call@QMetaObject@@HPAPAX@Z 00405340 f   moc_BaseTitle.obj
 0001:00004490       ?metaObject@BaseTitle@aptui@@UBEPBUQMetaObject@@XZ 00405490 f   moc_BaseTitle.obj
 0001:000044d0       ?qt_metacast@BaseTitle@aptui@@UAEPAXPBD@Z 004054d0 f   moc_BaseTitle.obj
 0001:00004510       ?qt_metacall@BaseTitle@aptui@@UAEHW4Call@QMetaObject@@HPAPAX@Z 00405510 f   moc_BaseTitle.obj
 0001:00004570       ?signalAppButtonClicked@BaseTitle@aptui@@IAEXXZ 00405570 f   moc_BaseTitle.obj
 0001:000045a0       ?signalOptionButtonClicked@BaseTitle@aptui@@IAEXXZ 004055a0 f   moc_BaseTitle.obj
 0001:000045d0       ?signalMinButtonClicked@BaseTitle@aptui@@IAEXXZ 004055d0 f   moc_BaseTitle.obj
 0001:00004600       ?signalMaxButtonClicked@BaseTitle@aptui@@IAEXXZ 00405600 f   moc_BaseTitle.obj
 0001:00004630       ?signalCloseButtonClicked@BaseTitle@aptui@@IAEXXZ 00405630 f   moc_BaseTitle.obj
 0001:00004720       ?qt_static_metacall@ButtonRadio@aptui@@CAXPAVQObject@@W4Call@QMetaObject@@HPAPAX@Z 00405720 f   moc_ButtonRadio.obj
 0001:00004730       ?metaObject@ButtonRadio@aptui@@UBEPBUQMetaObject@@XZ 00405730 f   moc_ButtonRadio.obj
 0001:00004770       ?qt_metacast@ButtonRadio@aptui@@UAEPAXPBD@Z 00405770 f   moc_ButtonRadio.obj
 0001:000047b0       ?qt_metacall@ButtonRadio@aptui@@UAEHW4Call@QMetaObject@@HPAPAX@Z 004057b0 f   moc_ButtonRadio.obj
 0001:00004820       ?qt_static_metacall@CapacityCalculation@@CAXPAVQObject@@W4Call@QMetaObject@@HPAPAX@Z 00405820 f   moc_CapacityCalculation.obj
 0001:00004890       ?metaObject@CapacityCalculation@@UBEPBUQMetaObject@@XZ 00405890 f   moc_CapacityCalculation.obj
 0001:000048d0       ?qt_metacast@CapacityCalculation@@UAEPAXPBD@Z 004058d0 f   moc_CapacityCalculation.obj
 0001:00004910       ?qt_metacall@CapacityCalculation@@UAEHW4Call@QMetaObject@@HPAPAX@Z 00405910 f   moc_CapacityCalculation.obj
 0001:00004970       ?signalClear@CapacityCalculation@@IAEXXZ 00405970 f   moc_CapacityCalculation.obj
 0001:000049a0       ?signalExport@CapacityCalculation@@IAEXXZ 004059a0 f   moc_CapacityCalculation.obj
 0001:00004a30       ?qt_static_metacall@CoverWidget@aptui@@CAXPAVQObject@@W4Call@QMetaObject@@HPAPAX@Z 00405a30 f   moc_CoverWidget.obj
 0001:00004a40       ?metaObject@CoverWidget@aptui@@UBEPBUQMetaObject@@XZ 00405a40 f   moc_CoverWidget.obj
 0001:00004a80       ?qt_metacast@CoverWidget@aptui@@UAEPAXPBD@Z 00405a80 f   moc_CoverWidget.obj
 0001:00004ac0       ?qt_metacall@CoverWidget@aptui@@UAEHW4Call@QMetaObject@@HPAPAX@Z 00405ac0 f   moc_CoverWidget.obj
 0001:00004b30       ?qt_static_metacall@DataCalculatorPage@@CAXPAVQObject@@W4Call@QMetaObject@@HPAPAX@Z 00405b30 f   moc_DataCalculatorPage.obj
 0001:00004ca0       ?metaObject@DataCalculatorPage@@UBEPBUQMetaObject@@XZ 00405ca0 f   moc_DataCalculatorPage.obj
 0001:00004ce0       ?qt_metacast@DataCalculatorPage@@UAEPAXPBD@Z 00405ce0 f   moc_DataCalculatorPage.obj
 0001:00004d20       ?qt_metacall@DataCalculatorPage@@UAEHW4Call@QMetaObject@@HPAPAX@Z 00405d20 f   moc_DataCalculatorPage.obj
 0001:00004d80       ?setDiskSize@DataCalculatorPage@@IAEXABVQString@@0@Z 00405d80 f   moc_DataCalculatorPage.obj
 0001:00004dc0       ?setTime@DataCalculatorPage@@IAEXABVQString@@00@Z 00405dc0 f   moc_DataCalculatorPage.obj
 0001:00004ec0       ?qt_static_metacall@DataDisplayPage@@CAXPAVQObject@@W4Call@QMetaObject@@HPAPAX@Z 00405ec0 f   moc_DataDisplayPage.obj
 0001:00004f10       ?metaObject@DataDisplayPage@@UBEPBUQMetaObject@@XZ 00405f10 f   moc_DataDisplayPage.obj
 0001:00004f50       ?qt_metacast@DataDisplayPage@@UAEPAXPBD@Z 00405f50 f   moc_DataDisplayPage.obj
 0001:00004f90       ?qt_metacall@DataDisplayPage@@UAEHW4Call@QMetaObject@@HPAPAX@Z 00405f90 f   moc_DataDisplayPage.obj
 0001:00005040       ?qt_static_metacall@DeviceAddPage@@CAXPAVQObject@@W4Call@QMetaObject@@HPAPAX@Z 00406040 f   moc_DeviceAddPage.obj
 0001:00005260       ?metaObject@DeviceAddPage@@UBEPBUQMetaObject@@XZ 00406260 f   moc_DeviceAddPage.obj
 0001:000052a0       ?qt_metacast@DeviceAddPage@@UAEPAXPBD@Z 004062a0 f   moc_DeviceAddPage.obj
 0001:000052e0       ?qt_metacall@DeviceAddPage@@UAEHW4Call@QMetaObject@@HPAPAX@Z 004062e0 f   moc_DeviceAddPage.obj
 0001:00005340       ?SignalDeviceChanged@DeviceAddPage@@IAEXN@Z 00406340 f   moc_DeviceAddPage.obj
 0001:00005380       ?SianalDeviceDelete@DeviceAddPage@@IAEXH@Z 00406380 f   moc_DeviceAddPage.obj
 0001:000053c0       ?SignalFramerateStandard@DeviceAddPage@@IAEXH@Z 004063c0 f   moc_DeviceAddPage.obj
 0001:00005400       ?signalCover@DeviceAddPage@@IAEXXZ 00406400 f   moc_DeviceAddPage.obj
 0001:00005430       ?signalDisvocer@DeviceAddPage@@IAEXXZ 00406430 f   moc_DeviceAddPage.obj
 0001:00005460       ?signalDeviceChangedToBandwith@DeviceAddPage@@IAEXAAVQString@@0000@Z 00406460 f   moc_DeviceAddPage.obj
 0001:000055d0       ??0Result@@QAE@ABU0@@Z     004065d0 f i moc_DeviceAddPage.obj
 0001:00005760       ??1?$QMap@_JUStructDeviceItem@NM_DiskCalculator@@@@QAE@XZ 00406760 f i moc_DeviceAddPage.obj
 0001:000057b0       ??4?$QMap@_JUStructDeviceItem@NM_DiskCalculator@@@@QAEAAV0@ABV0@@Z 004067b0 f i moc_DeviceAddPage.obj
 0001:00005850       ?freeData@?$QMap@_JUStructDeviceItem@NM_DiskCalculator@@@@AAEXPAUQMapData@@@Z 00406850 f i moc_DeviceAddPage.obj
 0001:000058e0       ??_GStructDeviceItem@NM_DiskCalculator@@QAEPAXI@Z 004068e0 f i moc_DeviceAddPage.obj
 0001:00005920       ??1StructDeviceItem@NM_DiskCalculator@@QAE@XZ 00406920 f i moc_DeviceAddPage.obj
 0001:00005a00       ?payload@?$QMap@_JUStructDeviceItem@NM_DiskCalculator@@@@CAHXZ 00406a00 f i moc_DeviceAddPage.obj
 0001:00005a10       ?concrete@?$QMap@_JUStructDeviceItem@NM_DiskCalculator@@@@CAPAU?$QMapNode@_JUStructDeviceItem@NM_DiskCalculator@@@@PAUNode@QMapData@@@Z 00406a10 f i moc_DeviceAddPage.obj
 0001:00005a30       ?detach_helper@?$QMap@_JUStructDeviceItem@NM_DiskCalculator@@@@AAEXXZ 00406a30 f i moc_DeviceAddPage.obj
 0001:00005bb0       ?alignment@?$QMap@_JUStructDeviceItem@NM_DiskCalculator@@@@CAHXZ 00406bb0 f i moc_DeviceAddPage.obj
 0001:00005bf0       ?node_create@?$QMap@_JUStructDeviceItem@NM_DiskCalculator@@@@AAEPAUNode@QMapData@@PAU3@QAPAU23@AB_JABUStructDeviceItem@NM_DiskCalculator@@@Z 00406bf0 f i moc_DeviceAddPage.obj
 0001:00005da0       ??2@YAPAXIPAX@Z            00406da0 f i moc_DeviceAddPage.obj
 0001:00005db0       ??3@YAXPAX0@Z              00406db0 f i moc_DeviceAddPage.obj
 0001:00005dc0       ??$qMax@I@@YAABIABI0@Z     00406dc0 f i moc_DeviceAddPage.obj
 0001:00005e00       ??0StructDeviceItem@NM_DiskCalculator@@QAE@ABU01@@Z 00406e00 f i moc_DeviceAddPage.obj
 0001:00005f60       ?qt_static_metacall@DeviceEditor@@CAXPAVQObject@@W4Call@QMetaObject@@HPAPAX@Z 00406f60 f   moc_DeviceEditor.obj
 0001:00006160       ?metaObject@DeviceEditor@@UBEPBUQMetaObject@@XZ 00407160 f   moc_DeviceEditor.obj
 0001:000061a0       ?qt_metacast@DeviceEditor@@UAEPAXPBD@Z 004071a0 f   moc_DeviceEditor.obj
 0001:000061e0       ?qt_metacall@DeviceEditor@@UAEHW4Call@QMetaObject@@HPAPAX@Z 004071e0 f   moc_DeviceEditor.obj
 0001:00006240       ?signalAddDevice@DeviceEditor@@IAEXABUStructDeviceItem@NM_DiskCalculator@@@Z 00407240 f   moc_DeviceEditor.obj
 0001:00006280       ?signalGetFrameStandard@DeviceEditor@@IAEXXZ 00407280 f   moc_DeviceEditor.obj
 0001:000062b0       ?signalAppStart@DeviceEditor@@IAEXXZ 004072b0 f   moc_DeviceEditor.obj
 0001:000062e0       ?signalCurrentFrameStandard@DeviceEditor@@IAEXH@Z 004072e0 f   moc_DeviceEditor.obj
 0001:00006410       ?qt_static_metacall@DeviceInfoManager@@CAXPAVQObject@@W4Call@QMetaObject@@HPAPAX@Z 00407410 f   moc_DeviceInfoManager.obj
 0001:00006420       ?metaObject@DeviceInfoManager@@UBEPBUQMetaObject@@XZ 00407420 f   moc_DeviceInfoManager.obj
 0001:00006460       ?qt_metacast@DeviceInfoManager@@UAEPAXPBD@Z 00407460 f   moc_DeviceInfoManager.obj
 0001:000064a0       ?qt_metacall@DeviceInfoManager@@UAEHW4Call@QMetaObject@@HPAPAX@Z 004074a0 f   moc_DeviceInfoManager.obj
 0001:00006510       ?qt_static_metacall@DeviceItemWidget@NM_DiskCalculator@@CAXPAVQObject@@W4Call@QMetaObject@@HPAPAX@Z 00407510 f   moc_DeviceItemWidget.obj
 0001:00006570       ?metaObject@DeviceItemWidget@NM_DiskCalculator@@UBEPBUQMetaObject@@XZ 00407570 f   moc_DeviceItemWidget.obj
 0001:000065b0       ?qt_metacast@DeviceItemWidget@NM_DiskCalculator@@UAEPAXPBD@Z 004075b0 f   moc_DeviceItemWidget.obj
 0001:000065f0       ?qt_metacall@DeviceItemWidget@NM_DiskCalculator@@UAEHW4Call@QMetaObject@@HPAPAX@Z 004075f0 f   moc_DeviceItemWidget.obj
 0001:00006650       ?signalDeleteClicked@DeviceItemWidget@NM_DiskCalculator@@IAEX_JH@Z 00407650 f   moc_DeviceItemWidget.obj
 0001:000066f0       ?qt_static_metacall@DiskCalculatorMainPage@@CAXPAVQObject@@W4Call@QMetaObject@@HPAPAX@Z 004076f0 f   moc_DiskCalculatorMainPage.obj
 0001:000068f0       ?metaObject@DiskCalculatorMainPage@@UBEPBUQMetaObject@@XZ 004078f0 f   moc_DiskCalculatorMainPage.obj
 0001:00006930       ?qt_metacast@DiskCalculatorMainPage@@UAEPAXPBD@Z 00407930 f   moc_DiskCalculatorMainPage.obj
 0001:00006970       ?qt_metacall@DiskCalculatorMainPage@@UAEHW4Call@QMetaObject@@HPAPAX@Z 00407970 f   moc_DiskCalculatorMainPage.obj
 0001:000069d0       ?signalGetHelp@DiskCalculatorMainPage@@IAEXXZ 004079d0 f   moc_DiskCalculatorMainPage.obj
 0001:00006a00       ?signalExportPdf@DiskCalculatorMainPage@@IAEXUResult@@@Z 00407a00 f   moc_DiskCalculatorMainPage.obj
 0001:00006b60       ??1Result@@QAE@XZ          00407b60 f i moc_DiskCalculatorMainPage.obj
 0001:00006c70       ?qt_static_metacall@CDlgAbout@aptui@@CAXPAVQObject@@W4Call@QMetaObject@@HPAPAX@Z 00407c70 f   moc_DlgAbout.obj
 0001:00006cd0       ?metaObject@CDlgAbout@aptui@@UBEPBUQMetaObject@@XZ 00407cd0 f   moc_DlgAbout.obj
 0001:00006d10       ?qt_metacast@CDlgAbout@aptui@@UAEPAXPBD@Z 00407d10 f   moc_DlgAbout.obj
 0001:00006d50       ?qt_metacall@CDlgAbout@aptui@@UAEHW4Call@QMetaObject@@HPAPAX@Z 00407d50 f   moc_DlgAbout.obj
 0001:00006db0       ?siganlBtn1Clicked@CDlgAbout@aptui@@IAEXXZ 00407db0 f   moc_DlgAbout.obj
 0001:00006de0       ?siganlBtn2Clicked@CDlgAbout@aptui@@IAEXXZ 00407de0 f   moc_DlgAbout.obj
 0001:00006e10       ?signalConerBtnClicked@CDlgAbout@aptui@@IAEXXZ 00407e10 f   moc_DlgAbout.obj
 0001:00006eb0       ?qt_static_metacall@Label@aptui@@CAXPAVQObject@@W4Call@QMetaObject@@HPAPAX@Z 00407eb0 f   moc_Label.obj
 0001:00006f20       ?metaObject@Label@aptui@@UBEPBUQMetaObject@@XZ 00407f20 f   moc_Label.obj
 0001:00006f60       ?qt_metacast@Label@aptui@@UAEPAXPBD@Z 00407f60 f   moc_Label.obj
 0001:00006fa0       ?qt_metacall@Label@aptui@@UAEHW4Call@QMetaObject@@HPAPAX@Z 00407fa0 f   moc_Label.obj
 0001:00007190       ?SignalDoubleClicked@Label@aptui@@IAEXXZ 00408190 f   moc_Label.obj
 0001:000071c0       ?SignalMouseClicked@Label@aptui@@IAEXXZ 004081c0 f   moc_Label.obj
 0001:000071f0       ?SignalMouseEnter@Label@aptui@@IAEXXZ 004081f0 f   moc_Label.obj
 0001:00007220       ?SignalMouseLeave@Label@aptui@@IAEXXZ 00408220 f   moc_Label.obj
 0001:00007250       ?qt_static_metacall@EditableLabel@aptui@@CAXPAVQObject@@W4Call@QMetaObject@@HPAPAX@Z 00408250 f   moc_Label.obj
 0001:00007290       ?metaObject@EditableLabel@aptui@@UBEPBUQMetaObject@@XZ 00408290 f   moc_Label.obj
 0001:000072d0       ?qt_metacast@EditableLabel@aptui@@UAEPAXPBD@Z 004082d0 f   moc_Label.obj
 0001:00007310       ?qt_metacall@EditableLabel@aptui@@UAEHW4Call@QMetaObject@@HPAPAX@Z 00408310 f   moc_Label.obj
 0001:00007370       ?qt_static_metacall@ColorLabel@aptui@@CAXPAVQObject@@W4Call@QMetaObject@@HPAPAX@Z 00408370 f   moc_Label.obj
 0001:000073b0       ?metaObject@ColorLabel@aptui@@UBEPBUQMetaObject@@XZ 004083b0 f   moc_Label.obj
 0001:000073f0       ?qt_metacast@ColorLabel@aptui@@UAEPAXPBD@Z 004083f0 f   moc_Label.obj
 0001:00007430       ?qt_metacall@ColorLabel@aptui@@UAEHW4Call@QMetaObject@@HPAPAX@Z 00408430 f   moc_Label.obj
 0001:00007610       ?qt_static_metacall@Line@aptui@@CAXPAVQObject@@W4Call@QMetaObject@@HPAPAX@Z 00408610 f   moc_Line.obj
 0001:00007620       ?metaObject@Line@aptui@@UBEPBUQMetaObject@@XZ 00408620 f   moc_Line.obj
 0001:00007660       ?qt_metacast@Line@aptui@@UAEPAXPBD@Z 00408660 f   moc_Line.obj
 0001:000076a0       ?qt_metacall@Line@aptui@@UAEHW4Call@QMetaObject@@HPAPAX@Z 004086a0 f   moc_Line.obj
 0001:00007710       ?qt_static_metacall@LineEditInterger@aptui@@CAXPAVQObject@@W4Call@QMetaObject@@HPAPAX@Z 00408710 f   moc_LineEditInterger.obj
 0001:00007720       ?metaObject@LineEditInterger@aptui@@UBEPBUQMetaObject@@XZ 00408720 f   moc_LineEditInterger.obj
 0001:00007760       ?qt_metacast@LineEditInterger@aptui@@UAEPAXPBD@Z 00408760 f   moc_LineEditInterger.obj
 0001:000077a0       ?qt_metacall@LineEditInterger@aptui@@UAEHW4Call@QMetaObject@@HPAPAX@Z 004087a0 f   moc_LineEditInterger.obj
 0001:00007810       ?qt_static_metacall@Menu@aptui@@CAXPAVQObject@@W4Call@QMetaObject@@HPAPAX@Z 00408810 f   moc_Menu.obj
 0001:00007820       ?metaObject@Menu@aptui@@UBEPBUQMetaObject@@XZ 00408820 f   moc_Menu.obj
 0001:00007860       ?qt_metacast@Menu@aptui@@UAEPAXPBD@Z 00408860 f   moc_Menu.obj
 0001:000078a0       ?qt_metacall@Menu@aptui@@UAEHW4Call@QMetaObject@@HPAPAX@Z 004088a0 f   moc_Menu.obj
 0001:000078e0       ?qt_static_metacall@CCustomStyle@Menu@aptui@@CAXPAVQObject@@W4Call@QMetaObject@@HPAPAX@Z 004088e0 f   moc_Menu.obj
 0001:000078f0       ?metaObject@CCustomStyle@Menu@aptui@@UBEPBUQMetaObject@@XZ 004088f0 f   moc_Menu.obj
 0001:00007930       ?qt_metacast@CCustomStyle@Menu@aptui@@UAEPAXPBD@Z 00408930 f   moc_Menu.obj
 0001:00007970       ?qt_metacall@CCustomStyle@Menu@aptui@@UAEHW4Call@QMetaObject@@HPAPAX@Z 00408970 f   moc_Menu.obj
 0001:00007a10       ?qt_static_metacall@MultiStatePushButton@aptui@@CAXPAVQObject@@W4Call@QMetaObject@@HPAPAX@Z 00408a10 f   moc_MultiStatePushButton.obj
 0001:00007a70       ?metaObject@MultiStatePushButton@aptui@@UBEPBUQMetaObject@@XZ 00408a70 f   moc_MultiStatePushButton.obj
 0001:00007ab0       ?qt_metacast@MultiStatePushButton@aptui@@UAEPAXPBD@Z 00408ab0 f   moc_MultiStatePushButton.obj
 0001:00007af0       ?qt_metacall@MultiStatePushButton@aptui@@UAEHW4Call@QMetaObject@@HPAPAX@Z 00408af0 f   moc_MultiStatePushButton.obj
 0001:00007c90       ?stateChanged@MultiStatePushButton@aptui@@IAEXVQString@@@Z 00408c90 f   moc_MultiStatePushButton.obj
 0001:00007dd0       ?qt_static_metacall@QtLocalPeer@SharedTools@@CAXPAVQObject@@W4Call@QMetaObject@@HPAPAX@Z 00408dd0 f   moc_qtlocalpeer.obj
 0001:00007e20       ?metaObject@QtLocalPeer@SharedTools@@UBEPBUQMetaObject@@XZ 00408e20 f   moc_qtlocalpeer.obj
 0001:00007e60       ?qt_metacast@QtLocalPeer@SharedTools@@UAEPAXPBD@Z 00408e60 f   moc_qtlocalpeer.obj
 0001:00007ea0       ?qt_metacall@QtLocalPeer@SharedTools@@UAEHW4Call@QMetaObject@@HPAPAX@Z 00408ea0 f   moc_qtlocalpeer.obj
 0001:00007f00       ?messageReceived@QtLocalPeer@SharedTools@@IAEXABVQString@@@Z 00408f00 f   moc_qtlocalpeer.obj
 0001:00007f90       ?qt_static_metacall@QtSingleApplication@SharedTools@@CAXPAVQObject@@W4Call@QMetaObject@@HPAPAX@Z 00408f90 f   moc_qtsingleapplication.obj
 0001:000080b0       ?metaObject@QtSingleApplication@SharedTools@@UBEPBUQMetaObject@@XZ 004090b0 f   moc_qtsingleapplication.obj
 0001:000080f0       ?qt_metacast@QtSingleApplication@SharedTools@@UAEPAXPBD@Z 004090f0 f   moc_qtsingleapplication.obj
 0001:00008130       ?qt_metacall@QtSingleApplication@SharedTools@@UAEHW4Call@QMetaObject@@HPAPAX@Z 00409130 f   moc_qtsingleapplication.obj
 0001:00008190       ?messageReceived@QtSingleApplication@SharedTools@@IAEXABVQString@@@Z 00409190 f   moc_qtsingleapplication.obj
 0001:000081d0       ?fileOpenRequest@QtSingleApplication@SharedTools@@IAEXABVQString@@@Z 004091d0 f   moc_qtsingleapplication.obj
 0001:000082b0       ?qt_static_metacall@QtSingleCoreApplication@SharedTools@@CAXPAVQObject@@W4Call@QMetaObject@@HPAPAX@Z 004092b0 f   moc_qtsinglecoreapplication.obj
 0001:00008360       ?metaObject@QtSingleCoreApplication@SharedTools@@UBEPBUQMetaObject@@XZ 00409360 f   moc_qtsinglecoreapplication.obj
 0001:000083a0       ?qt_metacast@QtSingleCoreApplication@SharedTools@@UAEPAXPBD@Z 004093a0 f   moc_qtsinglecoreapplication.obj
 0001:000083e0       ?qt_metacall@QtSingleCoreApplication@SharedTools@@UAEHW4Call@QMetaObject@@HPAPAX@Z 004093e0 f   moc_qtsinglecoreapplication.obj
 0001:00008440       ?messageReceived@QtSingleCoreApplication@SharedTools@@IAEXABVQString@@@Z 00409440 f   moc_qtsinglecoreapplication.obj
 0001:000084f0       ?qt_static_metacall@ScenceSelector@@CAXPAVQObject@@W4Call@QMetaObject@@HPAPAX@Z 004094f0 f   moc_ScenceSelector.obj
 0001:00008580       ?metaObject@ScenceSelector@@UBEPBUQMetaObject@@XZ 00409580 f   moc_ScenceSelector.obj
 0001:000085c0       ?qt_metacast@ScenceSelector@@UAEPAXPBD@Z 004095c0 f   moc_ScenceSelector.obj
 0001:00008600       ?qt_metacall@ScenceSelector@@UAEHW4Call@QMetaObject@@HPAPAX@Z 00409600 f   moc_ScenceSelector.obj
 0001:00008660       ?signalScenceChanged@ScenceSelector@@IAEXH@Z 00409660 f   moc_ScenceSelector.obj
 0001:000086a0       ?qt_static_metacall@ScenceQRaidoButton@ScenceSelector@@CAXPAVQObject@@W4Call@QMetaObject@@HPAPAX@Z 004096a0 f   moc_ScenceSelector.obj
 0001:000086f0       ?metaObject@ScenceQRaidoButton@ScenceSelector@@UBEPBUQMetaObject@@XZ 004096f0 f   moc_ScenceSelector.obj
 0001:00008730       ?qt_metacast@ScenceQRaidoButton@ScenceSelector@@UAEPAXPBD@Z 00409730 f   moc_ScenceSelector.obj
 0001:00008770       ?qt_metacall@ScenceQRaidoButton@ScenceSelector@@UAEHW4Call@QMetaObject@@HPAPAX@Z 00409770 f   moc_ScenceSelector.obj
 0001:000087d0       ?signalScenceButtonClick@ScenceQRaidoButton@ScenceSelector@@IAEXH@Z 004097d0 f   moc_ScenceSelector.obj
 0001:000088d0       ?OnScenceButtonClicked@ScenceQRaidoButton@ScenceSelector@@AAEXXZ 004098d0 f i moc_ScenceSelector.obj
 0001:000088f0       ?qt_static_metacall@SizeDisplayPage@@CAXPAVQObject@@W4Call@QMetaObject@@HPAPAX@Z 004098f0 f   moc_SizeDisplayPage.obj
 0001:00008930       ?metaObject@SizeDisplayPage@@UBEPBUQMetaObject@@XZ 00409930 f   moc_SizeDisplayPage.obj
 0001:00008970       ?qt_metacast@SizeDisplayPage@@UAEPAXPBD@Z 00409970 f   moc_SizeDisplayPage.obj
 0001:000089b0       ?qt_metacall@SizeDisplayPage@@UAEHW4Call@QMetaObject@@HPAPAX@Z 004099b0 f   moc_SizeDisplayPage.obj
 0001:00008a60       ?qt_static_metacall@Switch@aptui@@CAXPAVQObject@@W4Call@QMetaObject@@HPAPAX@Z 00409a60 f   moc_Switch.obj
 0001:00008b40       ?metaObject@Switch@aptui@@UBEPBUQMetaObject@@XZ 00409b40 f   moc_Switch.obj
 0001:00008b80       ?qt_metacast@Switch@aptui@@UAEPAXPBD@Z 00409b80 f   moc_Switch.obj
 0001:00008bc0       ?qt_metacall@Switch@aptui@@UAEHW4Call@QMetaObject@@HPAPAX@Z 00409bc0 f   moc_Switch.obj
 0001:00008d60       ?signalSwitch@Switch@aptui@@IAEX_N@Z 00409d60 f   moc_Switch.obj
 0001:00008da0       ?checkedChanged@Switch@aptui@@IAEXVQString@@@Z 00409da0 f   moc_Switch.obj
 0001:00008e20       ?signalON@Switch@aptui@@IAEXXZ 00409e20 f   moc_Switch.obj
 0001:00008e50       ?signalOFF@Switch@aptui@@IAEXXZ 00409e50 f   moc_Switch.obj
 0001:00008f80       ?qt_static_metacall@TabWidget@aptui@@CAXPAVQObject@@W4Call@QMetaObject@@HPAPAX@Z 00409f80 f   moc_TabWidget.obj
 0001:00008f90       ?metaObject@TabWidget@aptui@@UBEPBUQMetaObject@@XZ 00409f90 f   moc_TabWidget.obj
 0001:00008fd0       ?qt_metacast@TabWidget@aptui@@UAEPAXPBD@Z 00409fd0 f   moc_TabWidget.obj
 0001:00009010       ?qt_metacall@TabWidget@aptui@@UAEHW4Call@QMetaObject@@HPAPAX@Z 0040a010 f   moc_TabWidget.obj
 0001:00009080       ?qt_static_metacall@SystemMenu@aptui@@CAXPAVQObject@@W4Call@QMetaObject@@HPAPAX@Z 0040a080 f   moc_TitleMenu.obj
 0001:000090f0       ?metaObject@SystemMenu@aptui@@UBEPBUQMetaObject@@XZ 0040a0f0 f   moc_TitleMenu.obj
 0001:00009130       ?qt_metacast@SystemMenu@aptui@@UAEPAXPBD@Z 0040a130 f   moc_TitleMenu.obj
 0001:00009170       ?qt_metacall@SystemMenu@aptui@@UAEHW4Call@QMetaObject@@HPAPAX@Z 0040a170 f   moc_TitleMenu.obj
 0001:00009230       ?qt_static_metacall@ToolsApplication@apt@@CAXPAVQObject@@W4Call@QMetaObject@@HPAPAX@Z 0040a230 f   moc_ToolsApplication.obj
 0001:00009240       ?metaObject@ToolsApplication@apt@@UBEPBUQMetaObject@@XZ 0040a240 f   moc_ToolsApplication.obj
 0001:00009280       ?qt_metacast@ToolsApplication@apt@@UAEPAXPBD@Z 0040a280 f   moc_ToolsApplication.obj
 0001:000092c0       ?qt_metacall@ToolsApplication@apt@@UAEHW4Call@QMetaObject@@HPAPAX@Z 0040a2c0 f   moc_ToolsApplication.obj
 0001:00009330       ?qt_static_metacall@UpdateDialog@@CAXPAVQObject@@W4Call@QMetaObject@@HPAPAX@Z 0040a330 f   moc_UpdateDialog.obj
 0001:00009380       ?metaObject@UpdateDialog@@UBEPBUQMetaObject@@XZ 0040a380 f   moc_UpdateDialog.obj
 0001:000093c0       ?qt_metacast@UpdateDialog@@UAEPAXPBD@Z 0040a3c0 f   moc_UpdateDialog.obj
 0001:00009400       ?qt_metacall@UpdateDialog@@UAEHW4Call@QMetaObject@@HPAPAX@Z 0040a400 f   moc_UpdateDialog.obj
 0001:000094b0       ?qt_static_metacall@WarningDialog@NM_DiskCalculator@@CAXPAVQObject@@W4Call@QMetaObject@@HPAPAX@Z 0040a4b0 f   moc_WarningDialog.obj
 0001:00009500       ?metaObject@WarningDialog@NM_DiskCalculator@@UBEPBUQMetaObject@@XZ 0040a500 f   moc_WarningDialog.obj
 0001:00009540       ?qt_metacast@WarningDialog@NM_DiskCalculator@@UAEPAXPBD@Z 0040a540 f   moc_WarningDialog.obj
 0001:00009580       ?qt_metacall@WarningDialog@NM_DiskCalculator@@UAEHW4Call@QMetaObject@@HPAPAX@Z 0040a580 f   moc_WarningDialog.obj
 0001:000095e0       ?signalWarnClose@WarningDialog@NM_DiskCalculator@@IAEXXZ 0040a5e0 f   moc_WarningDialog.obj
 0001:00009660       ?qt_static_metacall@Widget@aptui@@CAXPAVQObject@@W4Call@QMetaObject@@HPAPAX@Z 0040a660 f   moc_Widget.obj
 0001:000096d0       ?metaObject@Widget@aptui@@UBEPBUQMetaObject@@XZ 0040a6d0 f   moc_Widget.obj
 0001:00009710       ?qt_metacast@Widget@aptui@@UAEPAXPBD@Z 0040a710 f   moc_Widget.obj
 0001:00009750       ?qt_metacall@Widget@aptui@@UAEHW4Call@QMetaObject@@HPAPAX@Z 0040a750 f   moc_Widget.obj
 0001:000097b0       ?signalDoubleClicked@Widget@aptui@@IAEXXZ 0040a7b0 f   moc_Widget.obj
 0001:000097e0       ?signalMouseClicked@Widget@aptui@@IAEXXZ 0040a7e0 f   moc_Widget.obj
 0001:00009810       ?signalMouseEnter@Widget@aptui@@IAEXXZ 0040a810 f   moc_Widget.obj
 0001:00009840       ?signalMouseLeave@Widget@aptui@@IAEXXZ 0040a840 f   moc_Widget.obj
 0001:000098f0       ?qt_static_metacall@WidgetDeviceListBorder@@CAXPAVQObject@@W4Call@QMetaObject@@HPAPAX@Z 0040a8f0 f   moc_WidgetDeviceListBorder.obj
 0001:00009900       ?metaObject@WidgetDeviceListBorder@@UBEPBUQMetaObject@@XZ 0040a900 f   moc_WidgetDeviceListBorder.obj
 0001:00009940       ?qt_metacast@WidgetDeviceListBorder@@UAEPAXPBD@Z 0040a940 f   moc_WidgetDeviceListBorder.obj
 0001:00009980       ?qt_metacall@WidgetDeviceListBorder@@UAEHW4Call@QMetaObject@@HPAPAX@Z 0040a980 f   moc_WidgetDeviceListBorder.obj
 0001:000099f0       ?qt_static_metacall@WindowTitle@aptui@@CAXPAVQObject@@W4Call@QMetaObject@@HPAPAX@Z 0040a9f0 f   moc_WindowTitle.obj
 0001:00009a80       ?metaObject@WindowTitle@aptui@@UBEPBUQMetaObject@@XZ 0040aa80 f   moc_WindowTitle.obj
 0001:00009ac0       ?qt_metacast@WindowTitle@aptui@@UAEPAXPBD@Z 0040aac0 f   moc_WindowTitle.obj
 0001:00009b00       ?qt_metacall@WindowTitle@aptui@@UAEHW4Call@QMetaObject@@HPAPAX@Z 0040ab00 f   moc_WindowTitle.obj
 0001:00009b60       ?signalCloseApp@WindowTitle@aptui@@IAEXXZ 0040ab60 f   moc_WindowTitle.obj
 0001:00009b90       ?signalSystemMenu@WindowTitle@aptui@@IAEXXZ 0040ab90 f   moc_WindowTitle.obj
 0001:00009c30       _main                      0040ac30 f   main.obj
 0001:0000a010       ??H@YA?BVQString@@ABV0@VQChar@@@Z 0040b010 f i main.obj
 0001:0000a0c0       ??H@YA?BVQString@@ABV0@PBD@Z 0040b0c0 f i main.obj
 0001:0000a1a0       ??0CCalculate@APT_DCS@@QAE@XZ 0040b1a0 f   Calculate.obj
 0001:0000a2a0       ??1CCalculate@APT_DCS@@QAE@XZ 0040b2a0 f   Calculate.obj
 0001:0000a320       ?SetVideoStandard@CCalculate@APT_DCS@@QAEXW4VideoStandard@2@@Z 0040b320 f   Calculate.obj
 0001:0000a340       ?SetDeviceType@CCalculate@APT_DCS@@QAEXW4DeviceType@2@@Z 0040b340 f   Calculate.obj
 0001:0000a360       ?CalBestBitRate@CCalculate@APT_DCS@@QAENW4DeviceType@2@W4Resolution@2@NW4ImageQuality@2@@Z 0040b360 f   Calculate.obj
 0001:0000a530       ?CalConstantBitRate@CCalculate@APT_DCS@@QAENW4DeviceType@2@ABVQString@@N@Z 0040b530 f   Calculate.obj
 0001:0000a630       ?CalTime@CCalculate@APT_DCS@@QAENNN@Z 0040b630 f   Calculate.obj
 0001:0000a680       ?CalDiskSize@CCalculate@APT_DCS@@QAENNH@Z 0040b680 f   Calculate.obj
 0001:0000a6d0       ?GetFramerate@CCalculate@APT_DCS@@AAEHN@Z 0040b6d0 f   Calculate.obj
 0001:0000a860       ?CalBandWidth@CCalculate@APT_DCS@@QAENNH@Z 0040b860 f   Calculate.obj
 0001:0000aa40       ??_GBitrateCalculate@APT_DCS@@QAEPAXI@Z 0040ba40 f i Calculate.obj
 0001:0000aa80       ?setConstantEncodingMode@BitrateConfig@APT_DCS@@QAEXABVQString@@@Z 0040ba80 f i Calculate.obj
 0001:0000aab0       ?setConstantEncodingMode@BitrateCalculate@APT_DCS@@QAEXABVQString@@@Z 0040bab0 f i Calculate.obj
 0001:0000aae0       ?qPow@@YANNN@Z             0040bae0 f i Calculate.obj
 0001:0000ab10       ??0CGenericDS@@QAE@XZ      0040bb10 f   GenericDS.obj
 0001:0000ab70       ??1CGenericDS@@QAE@XZ      0040bb70 f   GenericDS.obj
 0001:0000abd0       ?LoadXML@CGenericDS@@QAE_NABVQString@@@Z 0040bbd0 f   GenericDS.obj
 0001:0000ace0       ?SaveXML@CGenericDS@@QAE_NABVQString@@@Z 0040bce0 f   GenericDS.obj
 0001:0000ade0       ?GetChildrenCount@CGenericDS@@QBEHXZ 0040bde0 f   GenericDS.obj
 0001:0000aee0       ?GetChild@CGenericDS@@QBE?AV1@H@Z 0040bee0 f   GenericDS.obj
 0001:0000b0b0       ?GetChildByName@CGenericDS@@QBE?AV1@ABVQString@@@Z 0040c0b0 f   GenericDS.obj
 0001:0000b1e0       ?GetName@CGenericDS@@QBE?AVQString@@XZ 0040c1e0 f   GenericDS.obj
 0001:0000b210       ?CreateASRoot@CGenericDS@@QAE_NABVQString@@@Z 0040c210 f   GenericDS.obj
 0001:0000b340       ?CreateChild@CGenericDS@@QAE?AV1@ABVQString@@@Z 0040c340 f   GenericDS.obj
 0001:0000b450       ?SetValue@CGenericDS@@QAE_NABVQString@@@Z 0040c450 f   GenericDS.obj
 0001:0000b600       ?SetValue@CGenericDS@@QAE_NH@Z 0040c600 f   GenericDS.obj
 0001:0000b7f0       ?SetAttribute@CGenericDS@@QAE_NABVQString@@0@Z 0040c7f0 f   GenericDS.obj
 0001:0000b830       ?GetValue@CGenericDS@@QBE_NAAVQString@@@Z 0040c830 f   GenericDS.obj
 0001:0000b980       ?GetValue@CGenericDS@@QBE?AVQString@@XZ 0040c980 f   GenericDS.obj
 0001:0000ba10       ?GetAttribute@CGenericDS@@QBE?AVQString@@ABV2@0@Z 0040ca10 f   GenericDS.obj
 0001:0000ba50       ?DeleteChild@CGenericDS@@QAE?AV1@H@Z 0040ca50 f   GenericDS.obj
 0001:0000bb80       ?IsExistByName@CGenericDS@@QBE_NABVQString@@@Z 0040cb80 f   GenericDS.obj
 0001:0000c080       ??0CGenericDS@@QAE@ABV0@@Z 0040d080 f i GenericDS.obj
 0001:0000c110       ??U@YA?AV?$QFlags@W4OpenModeFlag@QIODevice@@@@W4OpenModeFlag@QIODevice@@0@Z 0040d110 f i GenericDS.obj
 0001:0000c140       ??0?$QFlags@W4OpenModeFlag@QIODevice@@@@QAE@W4OpenModeFlag@QIODevice@@@Z 0040d140 f i GenericDS.obj
 0001:0000c160       ??U?$QFlags@W4OpenModeFlag@QIODevice@@@@QBE?AV0@W4OpenModeFlag@QIODevice@@@Z 0040d160 f i GenericDS.obj
 0001:0000c190       ??0BitrateCalculate@APT_DCS@@QAE@XZ 0040d190 f   BitrateCalculate.obj
 0001:0000c2b0       ??1BitrateCalculate@APT_DCS@@QAE@XZ 0040d2b0 f   BitrateCalculate.obj
 0001:0000c3a0       ?constantbitrate@BitrateCalculate@APT_DCS@@QAEHABVQString@@HN@Z 0040d3a0 f   BitrateCalculate.obj
 0001:0000cca0       ?loadCSVConfig@BitrateCalculate@APT_DCS@@QAE_NXZ 0040dca0 f   BitrateCalculate.obj
 0001:0000cfe0       ?loadCSVConfig@BitrateCalculate@APT_DCS@@QAE_NABVQString@@AAV?$QVector@UConstantBitrateInfos@APT_DCS@@@@@Z 0040dfe0 f   BitrateCalculate.obj
 0001:0000d3a0       ?getConstantResolution@BitrateCalculate@APT_DCS@@QAE_NAAVQStringList@@HVQString@@@Z 0040e3a0 f   BitrateCalculate.obj
 0001:0000d4f0       ?getConstantResolution@BitrateCalculate@APT_DCS@@QAE_NAAVQStringList@@H@Z 0040e4f0 f   BitrateCalculate.obj
 0001:0000daa0       ??0ConstantBitrateInfos@APT_DCS@@QAE@XZ 0040eaa0 f i BitrateCalculate.obj
 0001:0000db20       ??1ConstantBitrateInfos@APT_DCS@@QAE@XZ 0040eb20 f i BitrateCalculate.obj
 0001:0000db90       ?push_back@?$QList@VQString@@@@QAEXABVQString@@@Z 0040eb90 f i BitrateCalculate.obj
 0001:0000dbb0       ??0?$QVector@N@@QAE@XZ     0040ebb0 f i BitrateCalculate.obj
 0001:0000dbe0       ??1?$QVector@N@@QAE@XZ     0040ebe0 f i BitrateCalculate.obj
 0001:0000dc30       ?size@?$QVector@N@@QBEHXZ  0040ec30 f i BitrateCalculate.obj
 0001:0000dc50       ?push_back@?$QVector@N@@QAEXABN@Z 0040ec50 f i BitrateCalculate.obj
 0001:0000dc70       ??0?$QMap@NH@@QAE@XZ       0040ec70 f i BitrateCalculate.obj
 0001:0000dca0       ??1?$QMap@NH@@QAE@XZ       0040eca0 f i BitrateCalculate.obj
 0001:0000dcf0       ??0?$QVector@UConstantBitrateInfos@APT_DCS@@@@QAE@XZ 0040ecf0 f i BitrateCalculate.obj
 0001:0000dd20       ??1?$QVector@UConstantBitrateInfos@APT_DCS@@@@QAE@XZ 0040ed20 f i BitrateCalculate.obj
 0001:0000dd70       ?size@?$QVector@UConstantBitrateInfos@APT_DCS@@@@QBEHXZ 0040ed70 f i BitrateCalculate.obj
 0001:0000dd90       ?push_back@?$QVector@UConstantBitrateInfos@APT_DCS@@@@QAEXABUConstantBitrateInfos@APT_DCS@@@Z 0040ed90 f i BitrateCalculate.obj
 0001:0000ddb0       ??0?$QMap@VQString@@V?$QVector@UConstantBitrateInfos@APT_DCS@@@@@@QAE@XZ 0040edb0 f i BitrateCalculate.obj
 0001:0000dde0       ??1?$QMap@VQString@@V?$QVector@UConstantBitrateInfos@APT_DCS@@@@@@QAE@XZ 0040ede0 f i BitrateCalculate.obj
 0001:0000de30       ??0?$QMap@VQString@@V?$QVector@UNetworkConnection@PublicData@@@@@@QAE@XZ 0040ee30 f i BitrateCalculate.obj
 0001:0000de60       ??1?$QMap@VQString@@V?$QVector@UNetworkConnection@PublicData@@@@@@QAE@XZ 0040ee60 f i BitrateCalculate.obj
 0001:0000deb0       ?size@?$QList@VQFileInfo@@@@QBEHXZ 0040eeb0 f i BitrateCalculate.obj
 0001:0000ded0       ??A?$QList@VQString@@@@QAEAAVQString@@H@Z 0040eed0 f i BitrateCalculate.obj
 0001:0000df10       ??A?$QMap@NH@@QAEAAHABN@Z  0040ef10 f i BitrateCalculate.obj
 0001:0000df90       ?insert@?$QMap@NH@@QAE?AViterator@1@ABNABH@Z 0040ef90 f i BitrateCalculate.obj
 0001:0000e030       ?freeData@?$QMap@NH@@AAEXPAUQMapData@@@Z 0040f030 f i BitrateCalculate.obj
 0001:0000e0a0       ??4?$QVector@UConstantBitrateInfos@APT_DCS@@@@QAEAAV0@ABV0@@Z 0040f0a0 f i BitrateCalculate.obj
 0001:0000e120       ??A?$QVector@UConstantBitrateInfos@APT_DCS@@@@QAEAAUConstantBitrateInfos@APT_DCS@@H@Z 0040f120 f i BitrateCalculate.obj
 0001:0000e150       ?append@?$QVector@UConstantBitrateInfos@APT_DCS@@@@QAEXABUConstantBitrateInfos@APT_DCS@@@Z 0040f150 f i BitrateCalculate.obj
 0001:0000e380       ?free@?$QVector@UConstantBitrateInfos@APT_DCS@@@@AAEXPAU?$QVectorTypedData@UConstantBitrateInfos@APT_DCS@@@@@Z 0040f380 f i BitrateCalculate.obj
 0001:0000e410       ??A?$QMap@VQString@@V?$QVector@UConstantBitrateInfos@APT_DCS@@@@@@QAEAAV?$QVector@UConstantBitrateInfos@APT_DCS@@@@ABVQString@@@Z 0040f410 f i BitrateCalculate.obj
 0001:0000e4f0       ?insert@?$QMap@VQString@@V?$QVector@UConstantBitrateInfos@APT_DCS@@@@@@QAE?AViterator@1@ABVQString@@ABV?$QVector@UConstantBitrateInfos@APT_DCS@@@@@Z 0040f4f0 f i BitrateCalculate.obj
 0001:0000e590       ?freeData@?$QMap@VQString@@V?$QVector@UConstantBitrateInfos@APT_DCS@@@@@@AAEXPAUQMapData@@@Z 0040f590 f i BitrateCalculate.obj
 0001:0000e630       ?freeData@?$QMap@VQString@@V?$QVector@UNetworkConnection@PublicData@@@@@@AAEXPAUQMapData@@@Z 0040f630 f i BitrateCalculate.obj
 0001:0000e6d0       ?clear@?$QVector@N@@QAEXXZ 0040f6d0 f i BitrateCalculate.obj
 0001:0000e760       ??A?$QVector@N@@QAEAANH@Z  0040f760 f i BitrateCalculate.obj
 0001:0000e790       ?append@?$QVector@N@@QAEXABN@Z 0040f790 f i BitrateCalculate.obj
 0001:0000e920       ?free@?$QVector@N@@AAEXPAU?$QVectorTypedData@N@@@Z 0040f920 f i BitrateCalculate.obj
 0001:0000e9a0       ??1?$QList@VQFileInfo@@@@QAE@XZ 0040f9a0 f i BitrateCalculate.obj
 0001:0000e9e0       ?at@?$QList@VQFileInfo@@@@QBEABVQFileInfo@@H@Z 0040f9e0 f i BitrateCalculate.obj
 0001:0000ea10       ??0ConstantBitrateInfos@APT_DCS@@QAE@ABU01@@Z 0040fa10 f i BitrateCalculate.obj
 0001:0000ea90       ??4ConstantBitrateInfos@APT_DCS@@QAEAAU01@ABU01@@Z 0040fa90 f i BitrateCalculate.obj
 0001:0000ead0       ??_GConstantBitrateInfos@APT_DCS@@QAEPAXI@Z 0040fad0 f i BitrateCalculate.obj
 0001:0000eb10       ??_G?$QVector@UConstantBitrateInfos@APT_DCS@@@@QAEPAXI@Z 0040fb10 f i BitrateCalculate.obj
 0001:0000eb50       ??_G?$QVector@UNetworkConnection@PublicData@@@@QAEPAXI@Z 0040fb50 f i BitrateCalculate.obj
 0001:0000eb90       ?detach@?$QList@VQString@@@@QAEXXZ 0040fb90 f i BitrateCalculate.obj
 0001:0000ebc0       ?data@?$QVector@N@@QAEPANXZ 0040fbc0 f i BitrateCalculate.obj
 0001:0000ebf0       ?sizeOfTypedData@?$QVector@N@@AAEHXZ 0040fbf0 f i BitrateCalculate.obj
 0001:0000ec10       ?alignOfTypedData@?$QVector@N@@ABEHXZ 0040fc10 f i BitrateCalculate.obj
 0001:0000ec50       ?payload@?$QMap@NH@@CAHXZ  0040fc50 f i BitrateCalculate.obj
 0001:0000ec60       ?concrete@?$QMap@NH@@CAPAU?$QMapNode@NH@@PAUNode@QMapData@@@Z 0040fc60 f i BitrateCalculate.obj
 0001:0000ec80       ??0?$QMap@NH@@QAE@ABV0@@Z  0040fc80 f i BitrateCalculate.obj
 0001:0000ecd0       ?detach@?$QMap@NH@@QAEXXZ  0040fcd0 f i BitrateCalculate.obj
 0001:0000ed10       ?data@?$QVector@UConstantBitrateInfos@APT_DCS@@@@QAEPAUConstantBitrateInfos@APT_DCS@@XZ 0040fd10 f i BitrateCalculate.obj
 0001:0000ed40       ?sizeOfTypedData@?$QVector@UConstantBitrateInfos@APT_DCS@@@@AAEHXZ 0040fd40 f i BitrateCalculate.obj
 0001:0000ed60       ?alignOfTypedData@?$QVector@UConstantBitrateInfos@APT_DCS@@@@ABEHXZ 0040fd60 f i BitrateCalculate.obj
 0001:0000eda0       ?payload@?$QMap@VQString@@V?$QVector@UConstantBitrateInfos@APT_DCS@@@@@@CAHXZ 0040fda0 f i BitrateCalculate.obj
 0001:0000edb0       ?concrete@?$QMap@VQString@@V?$QVector@UConstantBitrateInfos@APT_DCS@@@@@@CAPAU?$QMapNode@VQString@@V?$QVector@UConstantBitrateInfos@APT_DCS@@@@@@PAUNode@QMapData@@@Z 0040fdb0 f i BitrateCalculate.obj
 0001:0000edd0       ?detach@?$QMap@VQString@@V?$QVector@UConstantBitrateInfos@APT_DCS@@@@@@QAEXXZ 0040fdd0 f i BitrateCalculate.obj
 0001:0000ee10       ?payload@?$QMap@VQString@@V?$QVector@UNetworkConnection@PublicData@@@@@@CAHXZ 0040fe10 f i BitrateCalculate.obj
 0001:0000ee20       ?concrete@?$QMap@VQString@@V?$QVector@UNetworkConnection@PublicData@@@@@@CAPAU?$QMapNode@VQString@@V?$QVector@UNetworkConnection@PublicData@@@@@@PAUNode@QMapData@@@Z 0040fe20 f i BitrateCalculate.obj
 0001:0000ee40       ??0iterator@?$QMap@VQString@@V?$QVector@UConstantBitrateInfos@APT_DCS@@@@@@QAE@PAUNode@QMapData@@@Z 0040fe40 f i BitrateCalculate.obj
 0001:0000ee60       ??0iterator@?$QMap@NH@@QAE@PAUNode@QMapData@@@Z 0040fe60 f i BitrateCalculate.obj
 0001:0000ee80       ?free@?$QVectorTypedData@UConstantBitrateInfos@APT_DCS@@@@SAXPAU1@H@Z 0040fe80 f i BitrateCalculate.obj
 0001:0000eea0       ??1?$QVector@UNetworkConnection@PublicData@@@@QAE@XZ 0040fea0 f i BitrateCalculate.obj
 0001:0000eef0       ?free@?$QVectorTypedData@N@@SAXPAU1@H@Z 0040fef0 f i BitrateCalculate.obj
 0001:0000ef10       ?t@Node@?$QList@VQFileInfo@@@@QAEAAVQFileInfo@@XZ 0040ff10 f i BitrateCalculate.obj
 0001:0000ef40       ?detach@?$QVector@N@@QAEXXZ 0040ff40 f i BitrateCalculate.obj
 0001:0000ef70       ?detach@?$QVector@UConstantBitrateInfos@APT_DCS@@@@QAEXXZ 0040ff70 f i BitrateCalculate.obj
 0001:0000efa0       ??4?$QMap@NH@@QAEAAV0@ABV0@@Z 0040ffa0 f i BitrateCalculate.obj
 0001:0000f040       ?detach_helper@?$QMap@NH@@AAEXXZ 00410040 f i BitrateCalculate.obj
 0001:0000f1c0       ?mutableFindNode@?$QMap@NH@@ABEPAUNode@QMapData@@QAPAU23@ABN@Z 004101c0 f i BitrateCalculate.obj
 0001:0000f2b0       ?node_create@?$QMap@NH@@AAEPAUNode@QMapData@@PAU3@QAPAU23@ABNABH@Z 004102b0 f i BitrateCalculate.obj
 0001:0000f440       ?detach_helper@?$QVector@UConstantBitrateInfos@APT_DCS@@@@AAEXXZ 00410440 f i BitrateCalculate.obj
 0001:0000f470       ?realloc@?$QVector@UConstantBitrateInfos@APT_DCS@@@@AAEXHH@Z 00410470 f i BitrateCalculate.obj
 0001:0000fa40       ?detach_helper@?$QMap@VQString@@V?$QVector@UConstantBitrateInfos@APT_DCS@@@@@@AAEXXZ 00410a40 f i BitrateCalculate.obj
 0001:0000fbc0       ?mutableFindNode@?$QMap@VQString@@V?$QVector@UConstantBitrateInfos@APT_DCS@@@@@@ABEPAUNode@QMapData@@QAPAU23@ABVQString@@@Z 00410bc0 f i BitrateCalculate.obj
 0001:0000fcb0       ?node_create@?$QMap@VQString@@V?$QVector@UConstantBitrateInfos@APT_DCS@@@@@@AAEPAUNode@QMapData@@PAU3@QAPAU23@ABVQString@@ABV?$QVector@UConstantBitrateInfos@APT_DCS@@@@@Z 00410cb0 f i BitrateCalculate.obj
 0001:0000fe80       ?free@?$QVector@UNetworkConnection@PublicData@@@@AAEXPAU?$QVectorTypedData@UNetworkConnection@PublicData@@@@@Z 00410e80 f i BitrateCalculate.obj
 0001:0000ff10       ??4?$QVector@N@@QAEAAV0@ABV0@@Z 00410f10 f i BitrateCalculate.obj
 0001:0000ff90       ?detach_helper@?$QVector@N@@AAEXXZ 00410f90 f i BitrateCalculate.obj
 0001:0000ffc0       ?realloc@?$QVector@N@@AAEXHH@Z 00410fc0 f i BitrateCalculate.obj
 0001:000104f0       ?free@?$QList@VQFileInfo@@@@AAEXPAUData@QListData@@@Z 004114f0 f i BitrateCalculate.obj
 0001:00010540       ??_GNetworkConnection@PublicData@@QAEPAXI@Z 00411540 f i BitrateCalculate.obj
 0001:00010580       ??1NetworkConnection@PublicData@@QAE@XZ 00411580 f i BitrateCalculate.obj
 0001:000105a0       ?alignment@?$QMap@NH@@CAHXZ 004115a0 f i BitrateCalculate.obj
 0001:000105e0       ??0?$QVector@UConstantBitrateInfos@APT_DCS@@@@QAE@ABV0@@Z 004115e0 f i BitrateCalculate.obj
 0001:00010630       ?alignment@?$QMap@VQString@@V?$QVector@UConstantBitrateInfos@APT_DCS@@@@@@CAHXZ 00411630 f i BitrateCalculate.obj
 0001:00010670       ?alignOfTypedData@?$QVector@UNetworkConnection@PublicData@@@@ABEHXZ 00411670 f i BitrateCalculate.obj
 0001:000106b0       ?free@?$QVectorTypedData@UNetworkConnection@PublicData@@@@SAXPAU1@H@Z 004116b0 f i BitrateCalculate.obj
 0001:000106d0       ??$qMapLessThanKey@N@@YA_NABN0@Z 004116d0 f i BitrateCalculate.obj
 0001:00010710       ?malloc@?$QVector@UConstantBitrateInfos@APT_DCS@@@@AAEPAUQVectorData@@H@Z 00411710 f i BitrateCalculate.obj
 0001:00010770       ??$qMapLessThanKey@VQString@@@@YA_NABVQString@@0@Z 00411770 f i BitrateCalculate.obj
 0001:00010790       ?malloc@?$QVector@N@@AAEPAUQVectorData@@H@Z 00411790 f i BitrateCalculate.obj
 0001:000107f0       ?node_destruct@?$QList@VQFileInfo@@@@AAEXPAUNode@1@0@Z 004117f0 f i BitrateCalculate.obj
 0001:00010890       ??_GQFileInfo@@QAEPAXI@Z   00411890 f i BitrateCalculate.obj
 0001:000108d0       ??0QStringList@@QAE@XZ     004118d0 f i BitrateCalculate.obj
 0001:000108f0       ??6QStringList@@QAEAAV0@ABVQString@@@Z 004118f0 f i BitrateCalculate.obj
 0001:00010920       ??1QStringList@@QAE@XZ     00411920 f i BitrateCalculate.obj
 0001:00010940       ??0?$QList@VQString@@@@QAE@XZ 00411940 f i BitrateCalculate.obj
 0001:00010970       ??0?$QFlags@W4SortFlag@QDir@@@@QAE@W4SortFlag@QDir@@@Z 00411970 f i BitrateCalculate.obj
 0001:00010990       ??0?$QFlags@W4Filter@QDir@@@@QAE@W4Filter@QDir@@@Z 00411990 f i BitrateCalculate.obj
 0001:000109b0       ??$qMax@H@@YAABHABH0@Z     004119b0 f i BitrateCalculate.obj
 0001:000109f0       ??$qMin@H@@YAABHABH0@Z     004119f0 f i BitrateCalculate.obj
 0001:00010a30       ??1?$QList@VQString@@@@QAE@XZ 00411a30 f i BitrateCalculate.obj
 0001:00010a70       ?append@?$QList@VQString@@@@QAEXABVQString@@@Z 00411a70 f i BitrateCalculate.obj
 0001:00010c40       ?detach_helper@?$QList@VQString@@@@AAEXXZ 00411c40 f i BitrateCalculate.obj
 0001:00010c70       ?size@?$QList@VQString@@@@QBEHXZ 00411c70 f i BitrateCalculate.obj
 0001:00010c90       ?detach_helper_grow@?$QList@VQString@@@@AAEPAUNode@1@HH@Z 00411c90 f i BitrateCalculate.obj
 0001:00010e90       ?detach_helper@?$QList@VQString@@@@AAEXH@Z 00411e90 f i BitrateCalculate.obj
 0001:00010fb0       ?free@?$QList@VQString@@@@AAEXPAUData@QListData@@@Z 00411fb0 f i BitrateCalculate.obj
 0001:00011000       ?node_construct@?$QList@VQString@@@@AAEXPAUNode@1@ABVQString@@@Z 00412000 f i BitrateCalculate.obj
 0001:00011130       ?node_destruct@?$QList@VQString@@@@AAEXPAUNode@1@@Z 00412130 f i BitrateCalculate.obj
 0001:000111a0       ?node_copy@?$QList@VQString@@@@AAEXPAUNode@1@00@Z 004121a0 f i BitrateCalculate.obj
 0001:00011430       ??_GQString@@QAEPAXI@Z     00412430 f i BitrateCalculate.obj
 0001:00011470       ?t@Node@?$QList@VQString@@@@QAEAAVQString@@XZ 00412470 f i BitrateCalculate.obj
 0001:000114a0       ?node_destruct@?$QList@VQString@@@@AAEXPAUNode@1@0@Z 004124a0 f i BitrateCalculate.obj
 0001:00011540       ??0BitrateConfig@APT_DCS@@QAE@XZ 00412540 f   BitrateConfig.obj
 0001:00011850       ??1BitrateConfig@APT_DCS@@QAE@XZ 00412850 f   BitrateConfig.obj
 0001:00011960       ?loadConfig@BitrateConfig@APT_DCS@@QAE_NXZ 00412960 f   BitrateConfig.obj
 0001:00011fd0       ?getConstantConfig@BitrateConfig@APT_DCS@@QAE_NAAV?$QVector@UConstantBitrateInfo@APT_DCS@@@@H@Z 00412fd0 f   BitrateConfig.obj
 0001:00012020       ?getConstantResolution@BitrateConfig@APT_DCS@@QAE_NAAVQStringList@@HVQString@@@Z 00413020 f   BitrateConfig.obj
 0001:00012170       ?exportConstantConfig@BitrateConfig@APT_DCS@@QAE_NABVQString@@H@Z 00413170 f   BitrateConfig.obj
 0001:00012490       ?importConstantConfig@BitrateConfig@APT_DCS@@QAE_NABVQString@@H@Z 00413490 f   BitrateConfig.obj
 0001:00012910       ?constantbitrate@BitrateConfig@APT_DCS@@QAEHABVQString@@H@Z 00413910 f   BitrateConfig.obj
 0001:00012a20       ?getConstantResolution@BitrateConfig@APT_DCS@@QAE_NAAVQStringList@@H@Z 00413a20 f   BitrateConfig.obj
 0001:00012ad0       ?getScene@BitrateConfig@APT_DCS@@QAE_NAAV?$QVector@VQString@@@@@Z 00413ad0 f   BitrateConfig.obj
 0001:00012ce0       ?getSceneInfo@BitrateConfig@APT_DCS@@QAE_NABVQString@@AAUSceneInfo@2@@Z 00413ce0 f   BitrateConfig.obj
 0001:00012f80       ?getScenePic@BitrateConfig@APT_DCS@@QAE?AVQString@@ABV3@00@Z 00413f80 f   BitrateConfig.obj
 0001:000134c0       ?getSceneBitrate@BitrateConfig@APT_DCS@@QAEHABVQString@@00@Z 004144c0 f   BitrateConfig.obj
 0001:00013780       ?test@BitrateConfig@APT_DCS@@QAEXXZ 00414780 f   BitrateConfig.obj
 0001:000138f0       ?getConstantFrame@BitrateConfig@APT_DCS@@QAEXAAVQStringList@@H@Z 004148f0 f   BitrateConfig.obj
 0001:00013930       ?init@BitrateConfig@APT_DCS@@AAEXXZ 00414930 f   BitrateConfig.obj
 0001:00013940       ?getResolution@BitrateConfig@APT_DCS@@QAE_NABVQString@@AAVQStringList@@@Z 00414940 f   BitrateConfig.obj
 0001:00013bf0       ?getEncodingMode@BitrateConfig@APT_DCS@@QAE_NABVQString@@0AAVQStringList@@@Z 00414bf0 f   BitrateConfig.obj
 0001:00013eb0       ?getEncodingMode@BitrateConfig@APT_DCS@@QAEXAAVQStringList@@@Z 00414eb0 f   BitrateConfig.obj
 0001:00013ed0       ?loadCSVConfig@BitrateConfig@APT_DCS@@QAE_NXZ 00414ed0 f   BitrateConfig.obj
 0001:00014210       ?loadCSVConfig@BitrateConfig@APT_DCS@@QAE_NABVQString@@AAV?$QVector@UConstantBitrateInfo@APT_DCS@@@@@Z 00415210 f   BitrateConfig.obj
 0001:00014fa0       ??0ConstantBitrateInfo@APT_DCS@@QAE@XZ 00415fa0 f i BitrateConfig.obj
 0001:00014fd0       ??1ConstantBitrateInfo@APT_DCS@@QAE@XZ 00415fd0 f i BitrateConfig.obj
 0001:00014ff0       ??4CGenericDS@@QAEAAV0@ABV0@@Z 00415ff0 f i BitrateConfig.obj
 0001:00015030       ??0SceneInfo@APT_DCS@@QAE@XZ 00416030 f i BitrateConfig.obj
 0001:000150c0       ??1SceneInfo@APT_DCS@@QAE@XZ 004160c0 f i BitrateConfig.obj
 0001:00015140       ??4QStringList@@QAEAAV0@ABV0@@Z 00416140 f i BitrateConfig.obj
 0001:00015170       ??BQBool@@QBEPBXXZ         00416170 f i BitrateConfig.obj
 0001:00015190       ??0?$QVector@UConstantBitrateInfo@APT_DCS@@@@QAE@XZ 00416190 f i BitrateConfig.obj
 0001:000151c0       ??1?$QVector@UConstantBitrateInfo@APT_DCS@@@@QAE@XZ 004161c0 f i BitrateConfig.obj
 0001:00015210       ?size@?$QVector@UConstantBitrateInfo@APT_DCS@@@@QBEHXZ 00416210 f i BitrateConfig.obj
 0001:00015230       ?push_back@?$QVector@UConstantBitrateInfo@APT_DCS@@@@QAEXABUConstantBitrateInfo@APT_DCS@@@Z 00416230 f i BitrateConfig.obj
 0001:00015250       ??0?$QMap@VQString@@V?$QVector@UConstantBitrateInfo@APT_DCS@@@@@@QAE@XZ 00416250 f i BitrateConfig.obj
 0001:00015280       ??1?$QMap@VQString@@V?$QVector@UConstantBitrateInfo@APT_DCS@@@@@@QAE@XZ 00416280 f i BitrateConfig.obj
 0001:000152d0       ??0?$QVector@VQString@@@@QAE@XZ 004162d0 f i BitrateConfig.obj
 0001:00015300       ??1?$QVector@VQString@@@@QAE@XZ 00416300 f i BitrateConfig.obj
 0001:00015350       ?push_back@?$QVector@VQString@@@@QAEXABVQString@@@Z 00416350 f i BitrateConfig.obj
 0001:00015370       ??4?$QVector@UConstantBitrateInfo@APT_DCS@@@@QAEAAV0@ABV0@@Z 00416370 f i BitrateConfig.obj
 0001:000153f0       ?clear@?$QVector@UConstantBitrateInfo@APT_DCS@@@@QAEXXZ 004163f0 f i BitrateConfig.obj
 0001:00015480       ??A?$QVector@UConstantBitrateInfo@APT_DCS@@@@QAEAAUConstantBitrateInfo@APT_DCS@@H@Z 00416480 f i BitrateConfig.obj
 0001:000154b0       ?append@?$QVector@UConstantBitrateInfo@APT_DCS@@@@QAEXABUConstantBitrateInfo@APT_DCS@@@Z 004164b0 f i BitrateConfig.obj
 0001:000156e0       ?free@?$QVector@UConstantBitrateInfo@APT_DCS@@@@AAEXPAU?$QVectorTypedData@UConstantBitrateInfo@APT_DCS@@@@@Z 004166e0 f i BitrateConfig.obj
 0001:00015770       ??A?$QMap@VQString@@V?$QVector@UConstantBitrateInfo@APT_DCS@@@@@@QAEAAV?$QVector@UConstantBitrateInfo@APT_DCS@@@@ABVQString@@@Z 00416770 f i BitrateConfig.obj
 0001:00015850       ?insert@?$QMap@VQString@@V?$QVector@UConstantBitrateInfo@APT_DCS@@@@@@QAE?AViterator@1@ABVQString@@ABV?$QVector@UConstantBitrateInfo@APT_DCS@@@@@Z 00416850 f i BitrateConfig.obj
 0001:000158f0       ?freeData@?$QMap@VQString@@V?$QVector@UConstantBitrateInfo@APT_DCS@@@@@@AAEXPAUQMapData@@@Z 004168f0 f i BitrateConfig.obj
 0001:00015990       ??A?$QVector@VQString@@@@QAEAAVQString@@H@Z 00416990 f i BitrateConfig.obj
 0001:000159c0       ?append@?$QVector@VQString@@@@QAEXABVQString@@@Z 004169c0 f i BitrateConfig.obj
 0001:00015bf0       ?contains@?$QVector@VQString@@@@QBE_NABVQString@@@Z 00416bf0 f i BitrateConfig.obj
 0001:00015c70       ?free@?$QVector@VQString@@@@AAEXPAU?$QVectorTypedData@VQString@@@@@Z 00416c70 f i BitrateConfig.obj
 0001:00015d00       ??0ConstantBitrateInfo@APT_DCS@@QAE@ABU01@@Z 00416d00 f i BitrateConfig.obj
 0001:00015d40       ??4ConstantBitrateInfo@APT_DCS@@QAEAAU01@ABU01@@Z 00416d40 f i BitrateConfig.obj
 0001:00015d80       ??_GConstantBitrateInfo@APT_DCS@@QAEPAXI@Z 00416d80 f i BitrateConfig.obj
 0001:00015dc0       ??_G?$QVector@UConstantBitrateInfo@APT_DCS@@@@QAEPAXI@Z 00416dc0 f i BitrateConfig.obj
 0001:00015e00       ?data@?$QVector@UConstantBitrateInfo@APT_DCS@@@@QAEPAUConstantBitrateInfo@APT_DCS@@XZ 00416e00 f i BitrateConfig.obj
 0001:00015e30       ?sizeOfTypedData@?$QVector@UConstantBitrateInfo@APT_DCS@@@@AAEHXZ 00416e30 f i BitrateConfig.obj
 0001:00015e50       ?alignOfTypedData@?$QVector@UConstantBitrateInfo@APT_DCS@@@@ABEHXZ 00416e50 f i BitrateConfig.obj
 0001:00015e90       ?payload@?$QMap@VQString@@V?$QVector@UConstantBitrateInfo@APT_DCS@@@@@@CAHXZ 00416e90 f i BitrateConfig.obj
 0001:00015ea0       ?concrete@?$QMap@VQString@@V?$QVector@UConstantBitrateInfo@APT_DCS@@@@@@CAPAU?$QMapNode@VQString@@V?$QVector@UConstantBitrateInfo@APT_DCS@@@@@@PAUNode@QMapData@@@Z 00416ea0 f i BitrateConfig.obj
 0001:00015ec0       ?detach@?$QMap@VQString@@V?$QVector@UConstantBitrateInfo@APT_DCS@@@@@@QAEXXZ 00416ec0 f i BitrateConfig.obj
 0001:00015f00       ?data@?$QVector@VQString@@@@QAEPAVQString@@XZ 00416f00 f i BitrateConfig.obj
 0001:00015f30       ?sizeOfTypedData@?$QVector@VQString@@@@AAEHXZ 00416f30 f i BitrateConfig.obj
 0001:00015f50       ?alignOfTypedData@?$QVector@VQString@@@@ABEHXZ 00416f50 f i BitrateConfig.obj
 0001:00015f90       ??0iterator@?$QMap@VQString@@V?$QVector@UConstantBitrateInfo@APT_DCS@@@@@@QAE@PAUNode@QMapData@@@Z 00416f90 f i BitrateConfig.obj
 0001:00015fb0       ?free@?$QVectorTypedData@UConstantBitrateInfo@APT_DCS@@@@SAXPAU1@H@Z 00416fb0 f i BitrateConfig.obj
 0001:00015fd0       ?free@?$QVectorTypedData@VQString@@@@SAXPAU1@H@Z 00416fd0 f i BitrateConfig.obj
 0001:00015ff0       ?detach@?$QVector@UConstantBitrateInfo@APT_DCS@@@@QAEXXZ 00416ff0 f i BitrateConfig.obj
 0001:00016020       ?detach@?$QVector@VQString@@@@QAEXXZ 00417020 f i BitrateConfig.obj
 0001:00016050       ?detach_helper@?$QVector@UConstantBitrateInfo@APT_DCS@@@@AAEXXZ 00417050 f i BitrateConfig.obj
 0001:00016080       ?realloc@?$QVector@UConstantBitrateInfo@APT_DCS@@@@AAEXHH@Z 00417080 f i BitrateConfig.obj
 0001:00016650       ?detach_helper@?$QMap@VQString@@V?$QVector@UConstantBitrateInfo@APT_DCS@@@@@@AAEXXZ 00417650 f i BitrateConfig.obj
 0001:000167d0       ?mutableFindNode@?$QMap@VQString@@V?$QVector@UConstantBitrateInfo@APT_DCS@@@@@@ABEPAUNode@QMapData@@QAPAU23@ABVQString@@@Z 004177d0 f i BitrateConfig.obj
 0001:000168c0       ?node_create@?$QMap@VQString@@V?$QVector@UConstantBitrateInfo@APT_DCS@@@@@@AAEPAUNode@QMapData@@PAU3@QAPAU23@ABVQString@@ABV?$QVector@UConstantBitrateInfo@APT_DCS@@@@@Z 004178c0 f i BitrateConfig.obj
 0001:00016a90       ?detach_helper@?$QVector@VQString@@@@AAEXXZ 00417a90 f i BitrateConfig.obj
 0001:00016ac0       ?realloc@?$QVector@VQString@@@@AAEXHH@Z 00417ac0 f i BitrateConfig.obj
 0001:00017090       ??0?$QVector@UConstantBitrateInfo@APT_DCS@@@@QAE@ABV0@@Z 00418090 f i BitrateConfig.obj
 0001:000170e0       ?alignment@?$QMap@VQString@@V?$QVector@UConstantBitrateInfo@APT_DCS@@@@@@CAHXZ 004180e0 f i BitrateConfig.obj
 0001:00017120       ?malloc@?$QVector@UConstantBitrateInfo@APT_DCS@@@@AAEPAUQVectorData@@H@Z 00418120 f i BitrateConfig.obj
 0001:00017180       ?malloc@?$QVector@VQString@@@@AAEPAUQVectorData@@H@Z 00418180 f i BitrateConfig.obj
 0001:000171e0       ??H@YA?BVQString@@ABV0@0@Z 004181e0 f i BitrateConfig.obj
 0001:00017290       ?contains@QStringList@@QBE?AVQBool@@ABVQString@@W4CaseSensitivity@Qt@@@Z 00418290 f i BitrateConfig.obj
 0001:000172d0       ??6@YAAAVQTextStream@@AAV0@P6AAAV0@0@Z@Z 004182d0 f i BitrateConfig.obj
 0001:000172f0       ??4?$QList@VQString@@@@QAEAAV0@ABV0@@Z 004182f0 f i BitrateConfig.obj
 0001:00017380       ?clear@?$QList@VQString@@@@QAEXXZ 00418380 f i BitrateConfig.obj
 0001:00017410       ??0Configure@apt@@QAE@XZ   00418410 f   ConfigManager.obj
 0001:00017480       ??1Configure@apt@@UAE@XZ   00418480 f   ConfigManager.obj
 0001:000174f0       ?setKey@Configure@apt@@QAEXABVQString@@@Z 004184f0 f   ConfigManager.obj
 0001:00017510       ?setValue@Configure@apt@@QAEXABVQString@@@Z 00418510 f   ConfigManager.obj
 0001:00017530       ?set@Configure@apt@@QAEXABVQString@@0@Z 00418530 f   ConfigManager.obj
 0001:00017560       ??0ConfigureManager@apt@@AAE@XZ 00418560 f   ConfigManager.obj
 0001:000175f0       ??1ConfigureManager@apt@@UAE@XZ 004185f0 f   ConfigManager.obj
 0001:00017670       ?load@ConfigureManager@apt@@QAE_NABVQString@@@Z 00418670 f   ConfigManager.obj
 0001:00017870       ?save@ConfigureManager@apt@@QAE_NW4ConfigKey@12@ABVQString@@@Z 00418870 f   ConfigManager.obj
 0001:00017ac0       ?getConfigure@ConfigureManager@apt@@QBEPAVConfigure@2@W4ConfigKey@12@@Z 00418ac0 f   ConfigManager.obj
 0001:00017bc0       ?getLocaleCodec@ConfigureManager@apt@@QAEPAVQTextCodec@@XZ 00418bc0 f   ConfigManager.obj
 0001:00017be0       ?getLogSaveDay@ConfigureManager@apt@@QAEHXZ 00418be0 f   ConfigManager.obj
 0001:00017c00       ?getVersionType@ConfigureManager@apt@@QAEHXZ 00418c00 f   ConfigManager.obj
 0001:00017c30       ?getCurrentLanguage@ConfigureManager@apt@@QBE?AW4Language@TranslationLanguage@2@XZ 00418c30 f   ConfigManager.obj
 0001:00017c70       ?getSupportedLanguages@ConfigureManager@apt@@QBE?AV?$QList@W4Language@TranslationLanguage@apt@@@@XZ 00418c70 f   ConfigManager.obj
 0001:00017db0       ?keyToString@ConfigureManager@apt@@QBE?AVQString@@W4ConfigKey@12@@Z 00418db0 f   ConfigManager.obj
 0001:00017f10       ?clear@ConfigureManager@apt@@AAEXXZ 00418f10 f   ConfigManager.obj
 0001:00017f40       ?getIntValue@ConfigureManager@apt@@AAEHW4ConfigKey@12@@Z 00418f40 f   ConfigManager.obj
 0001:00017f90       ?getPingThreadCount@ConfigureManager@apt@@QAEHXZ 00418f90 f   ConfigManager.obj
 0001:00017fb0       ?getTaskThreadCount@ConfigureManager@apt@@QAEHXZ 00418fb0 f   ConfigManager.obj
 0001:00017fd0       ??0LanaguageManager@apt@@AAE@XZ 00418fd0 f   ConfigManager.obj
 0001:00018060       ??1LanaguageManager@apt@@UAE@XZ 00419060 f   ConfigManager.obj
 0001:000180e0       ?initialze@LanaguageManager@apt@@AAEXXZ 004190e0 f   ConfigManager.obj
 0001:000185a0       ?getLocale@LanaguageManager@apt@@QBE?AVQLocale@@XZ 004195a0 f   ConfigManager.obj
 0001:000185c0       ?getCurrentLanguage@LanaguageManager@apt@@QBE?AW4Language@TranslationLanguage@2@XZ 004195c0 f   ConfigManager.obj
 0001:00018a50       ??_EConfigure@apt@@UAEPAXI@Z 00419a50 f i ConfigManager.obj
 0001:00018a50       ??_GConfigure@apt@@UAEPAXI@Z 00419a50 f i ConfigManager.obj
 0001:00018a90       ??_GConfigureManager@apt@@UAEPAXI@Z 00419a90 f i ConfigManager.obj
 0001:00018a90       ??_EConfigureManager@apt@@UAEPAXI@Z 00419a90 f i ConfigManager.obj
 0001:00018ad0       ?key@Configure@apt@@QAE?AVQString@@XZ 00419ad0 f i ConfigManager.obj
 0001:00018b10       ?getValue@Configure@apt@@QBEABVQString@@XZ 00419b10 f i ConfigManager.obj
 0001:00018b30       ??_ELanaguageManager@apt@@UAEPAXI@Z 00419b30 f i ConfigManager.obj
 0001:00018b30       ??_GLanaguageManager@apt@@UAEPAXI@Z 00419b30 f i ConfigManager.obj
 0001:00018b70       ??_EQTranslator@@UAEPAXI@Z 00419b70 f i ConfigManager.obj
 0001:00018b70       ??_GQTranslator@@UAEPAXI@Z 00419b70 f i ConfigManager.obj
 0001:00018bb0       ??0?$CUiSingleton@VConfigureManager@apt@@@iVMSGUIToolkit@@IAE@XZ 00419bb0 f i ConfigManager.obj
 0001:00018bd0       ??1?$CUiSingleton@VConfigureManager@apt@@@iVMSGUIToolkit@@MAE@XZ 00419bd0 f i ConfigManager.obj
 0001:00018bf0       ??0?$QVector@PAVConfigure@apt@@@@QAE@XZ 00419bf0 f i ConfigManager.obj
 0001:00018c20       ??1?$QVector@PAVConfigure@apt@@@@QAE@XZ 00419c20 f i ConfigManager.obj
 0001:00018c70       ?constBegin@?$QVector@PAVConfigure@apt@@@@QBEPBQAVConfigure@apt@@XZ 00419c70 f i ConfigManager.obj
 0001:00018c90       ?constEnd@?$QVector@PAVConfigure@apt@@@@QBEPBQAVConfigure@apt@@XZ 00419c90 f i ConfigManager.obj
 0001:00018cc0       ??0?$CUiSingleton@VLanaguageManager@apt@@@iVMSGUIToolkit@@IAE@XZ 00419cc0 f i ConfigManager.obj
 0001:00018ce0       ??1?$CUiSingleton@VLanaguageManager@apt@@@iVMSGUIToolkit@@MAE@XZ 00419ce0 f i ConfigManager.obj
 0001:00018d00       ??0?$QVector@PAVQTranslator@@@@QAE@XZ 00419d00 f i ConfigManager.obj
 0001:00018d30       ??1?$QVector@PAVQTranslator@@@@QAE@XZ 00419d30 f i ConfigManager.obj
 0001:00018d80       ??0?$QList@W4Language@TranslationLanguage@apt@@@@QAE@XZ 00419d80 f i ConfigManager.obj
 0001:00018db0       ??0?$QList@W4Language@TranslationLanguage@apt@@@@QAE@ABV0@@Z 00419db0 f i ConfigManager.obj
 0001:00018e00       ??_E?$CUiSingleton@VConfigureManager@apt@@@iVMSGUIToolkit@@MAEPAXI@Z 00419e00 f i ConfigManager.obj
 0001:00018e00       ??_G?$CUiSingleton@VConfigureManager@apt@@@iVMSGUIToolkit@@MAEPAXI@Z 00419e00 f i ConfigManager.obj
 0001:00018e40       ??_E?$CUiSingleton@VLanaguageManager@apt@@@iVMSGUIToolkit@@MAEPAXI@Z 00419e40 f i ConfigManager.obj
 0001:00018e40       ??_G?$CUiSingleton@VLanaguageManager@apt@@@iVMSGUIToolkit@@MAEPAXI@Z 00419e40 f i ConfigManager.obj
 0001:00018e80       ?Instance@?$CUiSingleton@VConfigureManager@apt@@@iVMSGUIToolkit@@SAAAVConfigureManager@apt@@XZ 00419e80 f i ConfigManager.obj
 0001:00019030       ?clear@?$QVector@PAVConfigure@apt@@@@QAEXXZ 0041a030 f i ConfigManager.obj
 0001:000190c0       ?append@?$QVector@PAVConfigure@apt@@@@QAEXABQAVConfigure@apt@@@Z 0041a0c0 f i ConfigManager.obj
 0001:00019250       ?free@?$QVector@PAVConfigure@apt@@@@AAEXPAU?$QVectorTypedData@PAVConfigure@apt@@@@@Z 0041a250 f i ConfigManager.obj
 0001:000192d0       ?append@?$QVector@PAVQTranslator@@@@QAEXABQAVQTranslator@@@Z 0041a2d0 f i ConfigManager.obj
 0001:00019460       ?free@?$QVector@PAVQTranslator@@@@AAEXPAU?$QVectorTypedData@PAVQTranslator@@@@@Z 0041a460 f i ConfigManager.obj
 0001:000194e0       ??1?$QList@W4Language@TranslationLanguage@apt@@@@QAE@XZ 0041a4e0 f i ConfigManager.obj
 0001:00019520       ?append@?$QList@W4Language@TranslationLanguage@apt@@@@QAEXABW4Language@TranslationLanguage@apt@@@Z 0041a520 f i ConfigManager.obj
 0001:000196f0       ?detach_helper@?$QList@W4Language@TranslationLanguage@apt@@@@AAEXXZ 0041a6f0 f i ConfigManager.obj
 0001:00019720       ??$qDeleteAll@V?$QVector@PAVConfigure@apt@@@@@@YAXABV?$QVector@PAVConfigure@apt@@@@@Z 0041a720 f i ConfigManager.obj
 0001:00019750       ??$qDeleteAll@V?$QVector@PAVQTranslator@@@@@@YAXABV?$QVector@PAVQTranslator@@@@@Z 0041a750 f i ConfigManager.obj
 0001:00019780       ?begin@?$QVector@PAVConfigure@apt@@@@QBEPBQAVConfigure@apt@@XZ 0041a780 f i ConfigManager.obj
 0001:000197a0       ?end@?$QVector@PAVConfigure@apt@@@@QBEPBQAVConfigure@apt@@XZ 0041a7a0 f i ConfigManager.obj
 0001:000197d0       ?sizeOfTypedData@?$QVector@PAVConfigure@apt@@@@AAEHXZ 0041a7d0 f i ConfigManager.obj
 0001:000197f0       ?alignOfTypedData@?$QVector@PAVConfigure@apt@@@@ABEHXZ 0041a7f0 f i ConfigManager.obj
 0001:00019830       ?begin@?$QVector@PAVQTranslator@@@@QBEPBQAVQTranslator@@XZ 0041a830 f i ConfigManager.obj
 0001:00019850       ?end@?$QVector@PAVQTranslator@@@@QBEPBQAVQTranslator@@XZ 0041a850 f i ConfigManager.obj
 0001:00019880       ?sizeOfTypedData@?$QVector@PAVQTranslator@@@@AAEHXZ 0041a880 f i ConfigManager.obj
 0001:000198a0       ?alignOfTypedData@?$QVector@PAVQTranslator@@@@ABEHXZ 0041a8a0 f i ConfigManager.obj
 0001:000198e0       ?free@?$QVectorTypedData@PAVConfigure@apt@@@@SAXPAU1@H@Z 0041a8e0 f i ConfigManager.obj
 0001:00019900       ??0?$auto_ptr@VConfigureManager@apt@@@std@@QAE@PAVConfigureManager@apt@@@Z 0041a900 f i ConfigManager.obj
 0001:00019920       ??4?$auto_ptr@VConfigureManager@apt@@@std@@QAEAAV01@U?$auto_ptr_ref@VConfigureManager@apt@@@1@@Z 0041a920 f i ConfigManager.obj
 0001:00019960       ??1?$auto_ptr@VConfigureManager@apt@@@std@@QAE@XZ 0041a960 f i ConfigManager.obj
 0001:000199b0       ?get@?$auto_ptr@VConfigureManager@apt@@@std@@QBEPAVConfigureManager@apt@@XZ 0041a9b0 f i ConfigManager.obj
 0001:000199d0       ?free@?$QVectorTypedData@PAVQTranslator@@@@SAXPAU1@H@Z 0041a9d0 f i ConfigManager.obj
 0001:000199f0       ?reset@?$auto_ptr@VConfigureManager@apt@@@std@@QAEXPAVConfigureManager@apt@@@Z 0041a9f0 f i ConfigManager.obj
 0001:00019a60       ??$?BVConfigureManager@apt@@@?$auto_ptr@VConfigureManager@apt@@@std@@QAE?AU?$auto_ptr_ref@VConfigureManager@apt@@@1@XZ 0041aa60 f i ConfigManager.obj
 0001:00019ab0       ??4?$QVector@PAVConfigure@apt@@@@QAEAAV0@ABV0@@Z 0041aab0 f i ConfigManager.obj
 0001:00019b30       ?realloc@?$QVector@PAVConfigure@apt@@@@AAEXHH@Z 0041ab30 f i ConfigManager.obj
 0001:0001a060       ?realloc@?$QVector@PAVQTranslator@@@@AAEXHH@Z 0041b060 f i ConfigManager.obj
 0001:0001a590       ?detach_helper_grow@?$QList@W4Language@TranslationLanguage@apt@@@@AAEPAUNode@1@HH@Z 0041b590 f i ConfigManager.obj
 0001:0001a790       ?detach_helper@?$QList@W4Language@TranslationLanguage@apt@@@@AAEXH@Z 0041b790 f i ConfigManager.obj
 0001:0001a8b0       ?free@?$QList@W4Language@TranslationLanguage@apt@@@@AAEXPAUData@QListData@@@Z 0041b8b0 f i ConfigManager.obj
 0001:0001a900       ?node_construct@?$QList@W4Language@TranslationLanguage@apt@@@@AAEXPAUNode@1@ABW4Language@TranslationLanguage@apt@@@Z 0041b900 f i ConfigManager.obj
 0001:0001a9d0       ?node_destruct@?$QList@W4Language@TranslationLanguage@apt@@@@AAEXPAUNode@1@@Z 0041b9d0 f i ConfigManager.obj
 0001:0001aa10       ??$qDeleteAll@PBQAVConfigure@apt@@@@YAXPBQAVConfigure@apt@@0@Z 0041ba10 f i ConfigManager.obj
 0001:0001aa70       ??$qDeleteAll@PBQAVQTranslator@@@@YAXPBQAVQTranslator@@0@Z 0041ba70 f i ConfigManager.obj
 0001:0001aad0       ??0?$auto_ptr_ref@VConfigureManager@apt@@@std@@QAE@PAVConfigureManager@apt@@@Z 0041bad0 f i ConfigManager.obj
 0001:0001aaf0       ?detach_helper@?$QVector@PAVConfigure@apt@@@@AAEXXZ 0041baf0 f i ConfigManager.obj
 0001:0001ab20       ?malloc@?$QVector@PAVConfigure@apt@@@@AAEPAUQVectorData@@H@Z 0041bb20 f i ConfigManager.obj
 0001:0001ab80       ?malloc@?$QVector@PAVQTranslator@@@@AAEPAUQVectorData@@H@Z 0041bb80 f i ConfigManager.obj
 0001:0001abe0       ?node_destruct@?$QList@W4Language@TranslationLanguage@apt@@@@AAEXPAUNode@1@0@Z 0041bbe0 f i ConfigManager.obj
 0001:0001ac60       ?node_copy@?$QList@W4Language@TranslationLanguage@apt@@@@AAEXPAUNode@1@00@Z 0041bc60 f i ConfigManager.obj
 0001:0001aea0       ??0ToolsApplication@apt@@QAE@VQString@@AAHPAPAD@Z 0041bea0 f   ToolsApplication.obj
 0001:0001af10       ??1ToolsApplication@apt@@UAE@XZ 0041bf10 f   ToolsApplication.obj
 0001:0001af30       ?notify@ToolsApplication@apt@@UAE_NPAVQObject@@PAVQEvent@@@Z 0041bf30 f   ToolsApplication.obj
 0001:0001b270       ?initialize@ToolsApplication@apt@@QAE_NXZ 0041c270 f   ToolsApplication.obj
 0001:0001b5b0       ?release@ToolsApplication@apt@@QAEXXZ 0041c5b0 f   ToolsApplication.obj
 0001:0001b5c0       ?loadSkin@ToolsApplication@apt@@AAEXXZ 0041c5c0 f   ToolsApplication.obj
 0001:0001b710       ?loadFont@ToolsApplication@apt@@AAEXXZ 0041c710 f   ToolsApplication.obj
 0001:0001b7d0       ?loadStyle@ToolsApplication@apt@@AAEXXZ 0041c7d0 f   ToolsApplication.obj
 0001:0001b9b0       ?loadTranslator@ToolsApplication@apt@@AAEXXZ 0041c9b0 f   ToolsApplication.obj
 0001:0001bb20       ?initializeGuiToolkit@ToolsApplication@apt@@AAEXXZ 0041cb20 f   ToolsApplication.obj
 0001:0001bb60       ?releaseGuiToolkit@ToolsApplication@apt@@AAEXXZ 0041cb60 f   ToolsApplication.obj
 0001:0001bb70       ?loadConfigFile@ToolsApplication@apt@@AAEXXZ 0041cb70 f   ToolsApplication.obj
 0001:0001bbf0       ?legalResolution@ToolsApplication@apt@@AAE_NXZ 0041cbf0 f   ToolsApplication.obj
 0001:0001c020       ??_GToolsApplication@apt@@UAEPAXI@Z 0041d020 f i ToolsApplication.obj
 0001:0001c020       ??_EToolsApplication@apt@@UAEPAXI@Z 0041d020 f i ToolsApplication.obj
 0001:0001c060       ??1QtSingleApplication@SharedTools@@UAE@XZ 0041d060 f i ToolsApplication.obj
 0001:0001c0d0       ?tr@ToolsApplication@apt@@SA?AVQString@@PBD0@Z 0041d0d0 f i ToolsApplication.obj
 0001:0001c110       ?Instance@?$CUiSingleton@VLanaguageManager@apt@@@iVMSGUIToolkit@@SAAAVLanaguageManager@apt@@XZ 0041d110 f i ToolsApplication.obj
 0001:0001c2c0       ??$Load@PAUISkinPlugin@iVMS4200@@@CPluginFactory@iVMSGUIToolkit@@SAPAUISkinPlugin@iVMS4200@@ABVQString@@0@Z 0041d2c0 f i ToolsApplication.obj
 0001:0001c690       ??$qobject_cast@PAUISkinPlugin@iVMS4200@@@@YAPAUISkinPlugin@iVMS4200@@PAVQObject@@@Z 0041d690 f i ToolsApplication.obj
 0001:0001c6d0       ?removeOne@?$QList@VQString@@@@QAE_NABVQString@@@Z 0041d6d0 f i ToolsApplication.obj
 0001:0001c720       ?count@?$QList@VQString@@@@QBEHXZ 0041d720 f i ToolsApplication.obj
 0001:0001c740       ??0?$auto_ptr@VLanaguageManager@apt@@@std@@QAE@PAVLanaguageManager@apt@@@Z 0041d740 f i ToolsApplication.obj
 0001:0001c760       ??4?$auto_ptr@VLanaguageManager@apt@@@std@@QAEAAV01@U?$auto_ptr_ref@VLanaguageManager@apt@@@1@@Z 0041d760 f i ToolsApplication.obj
 0001:0001c7a0       ??1?$auto_ptr@VLanaguageManager@apt@@@std@@QAE@XZ 0041d7a0 f i ToolsApplication.obj
 0001:0001c7f0       ?get@?$auto_ptr@VLanaguageManager@apt@@@std@@QBEPAVLanaguageManager@apt@@XZ 0041d7f0 f i ToolsApplication.obj
 0001:0001c810       ?reset@?$auto_ptr@VLanaguageManager@apt@@@std@@QAEXPAVLanaguageManager@apt@@@Z 0041d810 f i ToolsApplication.obj
 0001:0001c880       ??$?BVLanaguageManager@apt@@@?$auto_ptr@VLanaguageManager@apt@@@std@@QAE?AU?$auto_ptr_ref@VLanaguageManager@apt@@@1@XZ 0041d880 f i ToolsApplication.obj
 0001:0001c8d0       ?removeAt@?$QList@VQString@@@@QAEXH@Z 0041d8d0 f i ToolsApplication.obj
 0001:0001c930       ?indexOf@?$QList@VQString@@@@QBEHABVQString@@H@Z 0041d930 f i ToolsApplication.obj
 0001:0001ca10       ??0?$auto_ptr_ref@VLanaguageManager@apt@@@std@@QAE@PAVLanaguageManager@apt@@@Z 0041da10 f i ToolsApplication.obj
 0001:0001ca30       ??0QLatin1Char@@QAE@D@Z    0041da30 f i ToolsApplication.obj
 0001:0001ca50       ?at@?$QList@VQString@@@@QBEABVQString@@H@Z 0041da50 f i ToolsApplication.obj
 0001:0001ca80       ??0DiskCalculatorMainPage@@QAE@PAVQWidget@@@Z 0041da80 f   DiskCalculatorMainPage.obj
 0001:0001cbc0       ?InitUi@DiskCalculatorMainPage@@AAE_NXZ 0041dbc0 f   DiskCalculatorMainPage.obj
 0001:0001d0a0       ?initConnections@DiskCalculatorMainPage@@QAEXXZ 0041e0a0 f   DiskCalculatorMainPage.obj
 0001:0001d360       ?setCover@DiskCalculatorMainPage@@AAEX_N@Z 0041e360 f   DiskCalculatorMainPage.obj
 0001:0001d3e0       ?enableCover@DiskCalculatorMainPage@@AAEXXZ 0041e3e0 f   DiskCalculatorMainPage.obj
 0001:0001d400       ?disableCover@DiskCalculatorMainPage@@AAEXXZ 0041e400 f   DiskCalculatorMainPage.obj
 0001:0001d420       ?getDeviceAddPage@DiskCalculatorMainPage@@QBEPBVQObject@@XZ 0041e420 f   DiskCalculatorMainPage.obj
 0001:0001d440       ?getDataDisplayPageTime@DiskCalculatorMainPage@@QBEPBVQObject@@XZ 0041e440 f   DiskCalculatorMainPage.obj
 0001:0001d460       ?getDataDisplayPageSize@DiskCalculatorMainPage@@QBEPBVQObject@@XZ 0041e460 f   DiskCalculatorMainPage.obj
 0001:0001d480       ?getDataCalculatorPage@DiskCalculatorMainPage@@QBEPBVQObject@@XZ 0041e480 f   DiskCalculatorMainPage.obj
 0001:0001d4a0       ?getCapacityCalculation@DiskCalculatorMainPage@@QBEPBVQObject@@XZ 0041e4a0 f   DiskCalculatorMainPage.obj
 0001:0001d4c0       ?getDeviceEditor@DiskCalculatorMainPage@@QBEPBVQObject@@XZ 0041e4c0 f   DiskCalculatorMainPage.obj
 0001:0001d4e0       ?getScenceSelector@DiskCalculatorMainPage@@QBEPBVQObject@@XZ 0041e4e0 f   DiskCalculatorMainPage.obj
 0001:0001d500       ??1DiskCalculatorMainPage@@UAE@XZ 0041e500 f   DiskCalculatorMainPage.obj
 0001:0001d540       ?resizeEvent@DiskCalculatorMainPage@@EAEXPAVQResizeEvent@@@Z 0041e540 f   DiskCalculatorMainPage.obj
 0001:0001d5a0       ?resizeAddBoarder@DiskCalculatorMainPage@@QAEXXZ 0041e5a0 f   DiskCalculatorMainPage.obj
 0001:0001d5b0       ?OnBtnSystemMenu@DiskCalculatorMainPage@@AAEXXZ 0041e5b0 f   DiskCalculatorMainPage.obj
 0001:0001d600       ?OnMenuHelpClicked@DiskCalculatorMainPage@@AAEXXZ 0041e600 f   DiskCalculatorMainPage.obj
 0001:0001d620       ?OnMenuUpdateClicked@DiskCalculatorMainPage@@AAEXXZ 0041e620 f   DiskCalculatorMainPage.obj
 0001:0001d720       ?closeEvent@DiskCalculatorMainPage@@MAEXPAVQCloseEvent@@@Z 0041e720 f   DiskCalculatorMainPage.obj
 0001:0001d8c0       ?keyPressEvent@DiskCalculatorMainPage@@EAEXPAVQKeyEvent@@@Z 0041e8c0 f   DiskCalculatorMainPage.obj
 0001:0001d8f0       ?onGetCalResults@DiskCalculatorMainPage@@AAEXXZ 0041e8f0 f   DiskCalculatorMainPage.obj
 0001:0001dd40       ?setupUi@Ui_DiskCalculatorMainPage@@QAEXPAVQMainWindow@@@Z 0041ed40 f i DiskCalculatorMainPage.obj
 0001:0001e7b0       ?retranslateUi@Ui_DiskCalculatorMainPage@@QAEXPAVQMainWindow@@@Z 0041f7b0 f i DiskCalculatorMainPage.obj
 0001:0001e860       ??_EQWidget@@UAEPAXI@Z     0041f860 f i DiskCalculatorMainPage.obj
 0001:0001e860       ??_GQWidget@@UAEPAXI@Z     0041f860 f i DiskCalculatorMainPage.obj
 0001:0001e8a0       ??_EQGridLayout@@UAEPAXI@Z 0041f8a0 f i DiskCalculatorMainPage.obj
 0001:0001e8a0       ??_GQGridLayout@@UAEPAXI@Z 0041f8a0 f i DiskCalculatorMainPage.obj
 0001:0001e8e0       ??_EQScrollArea@@UAEPAXI@Z 0041f8e0 f i DiskCalculatorMainPage.obj
 0001:0001e8e0       ??_GQScrollArea@@UAEPAXI@Z 0041f8e0 f i DiskCalculatorMainPage.obj
 0001:0001e920       ??_EQVBoxLayout@@UAEPAXI@Z 0041f920 f i DiskCalculatorMainPage.obj
 0001:0001e920       ??_GQVBoxLayout@@UAEPAXI@Z 0041f920 f i DiskCalculatorMainPage.obj
 0001:0001e960       ??_EDiskCalculatorMainPage@@UAEPAXI@Z 0041f960 f i DiskCalculatorMainPage.obj
 0001:0001e960       ??_GDiskCalculatorMainPage@@UAEPAXI@Z 0041f960 f i DiskCalculatorMainPage.obj
 0001:0001e9a0       ?tr@DiskCalculatorMainPage@@SA?AVQString@@PBD0@Z 0041f9a0 f i DiskCalculatorMainPage.obj
 0001:0001e9e0       ??U@YA?AV?$QFlags@W4WindowType@Qt@@@@W4WindowType@Qt@@0@Z 0041f9e0 f i DiskCalculatorMainPage.obj
 0001:0001ea10       ??_EQHBoxLayout@@UAEPAXI@Z 0041fa10 f i DiskCalculatorMainPage.obj
 0001:0001ea10       ??_GQHBoxLayout@@UAEPAXI@Z 0041fa10 f i DiskCalculatorMainPage.obj
 0001:0001ea50       ??0Result@@QAE@XZ          0041fa50 f i DiskCalculatorMainPage.obj
 0001:0001eb70       ??$castToQObject@VQObject@@@ShareFunction@@YAPAVQObject@@PAV1@@Z 0041fb70 f i DiskCalculatorMainPage.obj
 0001:0001eb90       ??$castToQObject@VCapacityCalculation@@@ShareFunction@@YAPAVQObject@@PAVCapacityCalculation@@@Z 0041fb90 f i DiskCalculatorMainPage.obj
 0001:0001ebb0       ??$castToQObject@VDeviceEditor@@@ShareFunction@@YAPAVQObject@@PAVDeviceEditor@@@Z 0041fbb0 f i DiskCalculatorMainPage.obj
 0001:0001ebd0       ??_EQWidget@@W7AEPAXI@Z    0041fbd0 f i DiskCalculatorMainPage.obj
 0001:0001ebe0       ??_EQVBoxLayout@@W7AEPAXI@Z 0041fbe0 f i DiskCalculatorMainPage.obj
 0001:0001ebf0       ??_EDiskCalculatorMainPage@@W7AEPAXI@Z 0041fbf0 f i DiskCalculatorMainPage.obj
 0001:0001ec00       ??_EQGridLayout@@W7AEPAXI@Z 0041fc00 f i DiskCalculatorMainPage.obj
 0001:0001ec10       ??_EQScrollArea@@W7AEPAXI@Z 0041fc10 f i DiskCalculatorMainPage.obj
 0001:0001ec20       ??_EQHBoxLayout@@W7AEPAXI@Z 0041fc20 f i DiskCalculatorMainPage.obj
 0001:0001ec30       ??G@YA?BVQPoint@@ABV0@0@Z  0041fc30 f i DiskCalculatorMainPage.obj
 0001:0001ec70       ??0?$QFlags@W4WindowType@Qt@@@@QAE@W4WindowType@Qt@@@Z 0041fc70 f i DiskCalculatorMainPage.obj
 0001:0001ec90       ??0?$QFlags@W4WindowType@Qt@@@@QAE@PAPAX@Z 0041fc90 f i DiskCalculatorMainPage.obj
 0001:0001ecb0       ??U?$QFlags@W4WindowType@Qt@@@@QBE?AV0@W4WindowType@Qt@@@Z 0041fcb0 f i DiskCalculatorMainPage.obj
 0001:0001ece0       ??0?$QFlags@W4AlignmentFlag@Qt@@@@QAE@PAPAX@Z 0041fce0 f i DiskCalculatorMainPage.obj
 0001:0001ed00       ?ResolutionToText@NM_DiskCalculator@@YA?AVQString@@H@Z 0041fd00 f   UiManager.obj
 0001:0001ed40       ??0AboutDialog@@QAE@PAVQObject@@@Z 0041fd40 f   AboutDialog.obj
 0001:0001ef10       ??1AboutDialog@@UAE@XZ     0041ff10 f   AboutDialog.obj
 0001:0001ef30       ?onGetHelp@AboutDialog@@AAE_NXZ 0041ff30 f   AboutDialog.obj
 0001:0001f2e0       ?tr@AboutDialog@@SA?AVQString@@PBD0@Z 004202e0 f i AboutDialog.obj
 0001:0001f320       ??_GAboutDialog@@UAEPAXI@Z 00420320 f i AboutDialog.obj
 0001:0001f320       ??_EAboutDialog@@UAEPAXI@Z 00420320 f i AboutDialog.obj
 0001:0001f360       ??H@YA?BVQString@@PBDABV0@@Z 00420360 f i AboutDialog.obj
 0001:0001f410       ??0DeviceEditor@@QAE@PAVQWidget@@@Z 00420410 f   DeviceEditor.obj
 0001:0001f840       ?initUi@DeviceEditor@@AAEXXZ 00420840 f   DeviceEditor.obj
 0001:0001fb40       ?setDeviceTypes@DeviceEditor@@QAEXABV?$QVector@USCENCE_ITEM@NM_DiskCalculator@@@@@Z 00420b40 f   DeviceEditor.obj
 0001:0001fb70       ?setDeviceResolutions@DeviceEditor@@QAEXABV?$QMap@HVQString@@@@@Z 00420b70 f   DeviceEditor.obj
 0001:0001fba0       ?selectFixedRate@DeviceEditor@@AAEXXZ 00420ba0 f   DeviceEditor.obj
 0001:0001fe60       ?OnRateSelected@DeviceEditor@@QAEXXZ 00420e60 f   DeviceEditor.obj
 0001:0001ff10       ?setScenceRecommandRateText@DeviceEditor@@QAEXABVQString@@@Z 00420f10 f   DeviceEditor.obj
 0001:0001ff30       ?getScenceSelector@DeviceEditor@@QAEPAVQObject@@XZ 00420f30 f   DeviceEditor.obj
 0001:0001ff50       ??1DeviceEditor@@UAE@XZ    00420f50 f   DeviceEditor.obj
 0001:0001ffe0       ?OnDeviceTypeChanged@DeviceEditor@@AAEXH@Z 00420fe0 f   DeviceEditor.obj
 0001:000201e0       ?OnResolutionChanged@DeviceEditor@@AAEXH@Z 004211e0 f   DeviceEditor.obj
 0001:00020220       ?OnFixedRateFrameRateChanged@DeviceEditor@@AAEXH@Z 00421220 f   DeviceEditor.obj
 0001:00020240       ?OnEncodingTypeChanged@DeviceEditor@@AAEXH@Z 00421240 f   DeviceEditor.obj
 0001:00020420       ?OnScenceChanged@DeviceEditor@@AAEXH@Z 00421420 f   DeviceEditor.obj
 0001:00020690       ?CalculateBitRate@DeviceEditor@@AAEXXZ 00421690 f   DeviceEditor.obj
 0001:000208c0       ?FreshPictureAndBitrateAndEncoding@DeviceEditor@@AAEXXZ 004218c0 f   DeviceEditor.obj
 0001:00020aa0       ?FreshPictureAndBitrate@DeviceEditor@@AAEXXZ 00421aa0 f   DeviceEditor.obj
 0001:00020be0       ?OnBtnAddDeviceClicked@DeviceEditor@@AAEXXZ 00421be0 f   DeviceEditor.obj
 0001:00021020       ?OnDeleteChannelGroupNumber@DeviceEditor@@AAEXH@Z 00422020 f   DeviceEditor.obj
 0001:00021040       ?OnSetFrameByStandard@DeviceEditor@@AAEXH@Z 00422040 f   DeviceEditor.obj
 0001:000210e0       ?OnSpreadChanged@DeviceEditor@@QAEX_N@Z 004220e0 f   DeviceEditor.obj
 0001:00021160       ?OnFrametareStandardPAL@DeviceEditor@@QAEXXZ 00422160 f   DeviceEditor.obj
 0001:00021210       ?OnFrametareStandardNTSC@DeviceEditor@@QAEXXZ 00422210 f   DeviceEditor.obj
 0001:00021a60       ?setupUi@Ui_DeviceEditor@@QAEXPAVQWidget@@@Z 00422a60 f i DeviceEditor.obj
 0001:00026550       ?retranslateUi@Ui_DeviceEditor@@QAEXPAVQWidget@@@Z 00427550 f i DeviceEditor.obj
 0001:00026da0       ??_GQCheckBox@@UAEPAXI@Z   00427da0 f i DeviceEditor.obj
 0001:00026da0       ??_EQCheckBox@@UAEPAXI@Z   00427da0 f i DeviceEditor.obj
 0001:00026de0       ??_EQLabel@@UAEPAXI@Z      00427de0 f i DeviceEditor.obj
 0001:00026de0       ??_GQLabel@@UAEPAXI@Z      00427de0 f i DeviceEditor.obj
 0001:00026e20       ??_ECLineEdit@iVMSGUIToolkit@@UAEPAXI@Z 00427e20 f i DeviceEditor.obj
 0001:00026e20       ??_GCLineEdit@iVMSGUIToolkit@@UAEPAXI@Z 00427e20 f i DeviceEditor.obj
 0001:00026e60       ??_GCComboBox@iVMSGUIToolkit@@UAEPAXI@Z 00427e60 f i DeviceEditor.obj
 0001:00026e60       ??_ECComboBox@iVMSGUIToolkit@@UAEPAXI@Z 00427e60 f i DeviceEditor.obj
 0001:00026ea0       ??_ECRadioButton@iVMSGUIToolkit@@UAEPAXI@Z 00427ea0 f i DeviceEditor.obj
 0001:00026ea0       ??_GCRadioButton@iVMSGUIToolkit@@UAEPAXI@Z 00427ea0 f i DeviceEditor.obj
 0001:00026ee0       ??_ECPushButton@iVMSGUIToolkit@@UAEPAXI@Z 00427ee0 f i DeviceEditor.obj
 0001:00026ee0       ??_GCPushButton@iVMSGUIToolkit@@UAEPAXI@Z 00427ee0 f i DeviceEditor.obj
 0001:00026f20       ??_EQFrame@@UAEPAXI@Z      00427f20 f i DeviceEditor.obj
 0001:00026f20       ??_GQFrame@@UAEPAXI@Z      00427f20 f i DeviceEditor.obj
 0001:00026f60       ??_GDeviceEditor@@UAEPAXI@Z 00427f60 f i DeviceEditor.obj
 0001:00026f60       ??_EDeviceEditor@@UAEPAXI@Z 00427f60 f i DeviceEditor.obj
 0001:00026fa0       ??_GCIntValidator@iVMSGUIToolkit@@UAEPAXI@Z 00427fa0 f i DeviceEditor.obj
 0001:00026fa0       ??_ECIntValidator@iVMSGUIToolkit@@UAEPAXI@Z 00427fa0 f i DeviceEditor.obj
 0001:00026fe0       ?tr@DeviceEditor@@SA?AVQString@@PBD0@Z 00427fe0 f i DeviceEditor.obj
 0001:00027020       ??0SCENCE_ITEM@NM_DiskCalculator@@QAE@XZ 00428020 f i DeviceEditor.obj
 0001:00027040       ??1SCENCE_ITEM@NM_DiskCalculator@@QAE@XZ 00428040 f i DeviceEditor.obj
 0001:00027060       ?setConstantEncodingMode@CCalculate@APT_DCS@@QAEXABVQString@@@Z 00428060 f i DeviceEditor.obj
 0001:00027090       ??0StructDeviceItem@NM_DiskCalculator@@QAE@XZ 00428090 f i DeviceEditor.obj
 0001:00027180       ?begin@?$QVector@VQString@@@@QAEPAVQString@@XZ 00428180 f i DeviceEditor.obj
 0001:000271b0       ?end@?$QVector@VQString@@@@QAEPAVQString@@XZ 004281b0 f i DeviceEditor.obj
 0001:000271e0       ??0?$QVector@USCENCE_ITEM@NM_DiskCalculator@@@@QAE@XZ 004281e0 f i DeviceEditor.obj
 0001:00027210       ??1?$QVector@USCENCE_ITEM@NM_DiskCalculator@@@@QAE@XZ 00428210 f i DeviceEditor.obj
 0001:00027260       ?size@?$QVector@USCENCE_ITEM@NM_DiskCalculator@@@@QBEHXZ 00428260 f i DeviceEditor.obj
 0001:00027280       ?removeAll@?$QList@VQString@@@@QAEHABVQString@@@Z 00428280 f i DeviceEditor.obj
 0001:00027400       ?append@?$QVector@USCENCE_ITEM@NM_DiskCalculator@@@@QAEXABUSCENCE_ITEM@NM_DiskCalculator@@@Z 00428400 f i DeviceEditor.obj
 0001:00027640       ?free@?$QVector@USCENCE_ITEM@NM_DiskCalculator@@@@AAEXPAU?$QVectorTypedData@USCENCE_ITEM@NM_DiskCalculator@@@@@Z 00428640 f i DeviceEditor.obj
 0001:000276d0       ??$insertComboxData@USCENCE_ITEM@NM_DiskCalculator@@@ShareFunction@@YAXABV?$QVector@USCENCE_ITEM@NM_DiskCalculator@@@@PAVQComboBox@@@Z 004286d0 f i DeviceEditor.obj
 0001:00027820       ??$insertComboxData@H@ShareFunction@@YAXABV?$QMap@HVQString@@@@PAVQComboBox@@@Z 00428820 f i DeviceEditor.obj
 0001:000279a0       ??$castToQObject@VScenceSelector@@@ShareFunction@@YAPAVQObject@@PAVScenceSelector@@@Z 004289a0 f i DeviceEditor.obj
 0001:000279c0       ??$DELETE_OBJECT@PAVCCalculate@APT_DCS@@@NM_SHARE_TOOL@@YAXAAPAVCCalculate@APT_DCS@@@Z 004289c0 f i DeviceEditor.obj
 0001:00027a20       ??$DELETE_OBJECT@PAVBitrateConfig@APT_DCS@@@NM_SHARE_TOOL@@YAXAAPAVBitrateConfig@APT_DCS@@@Z 00428a20 f i DeviceEditor.obj
 0001:00027a80       ??$DELETE_OBJECT@PAVDeviceEditor@Ui@@@NM_SHARE_TOOL@@YAXAAPAVDeviceEditor@Ui@@@Z 00428a80 f i DeviceEditor.obj
 0001:00027ac0       ??0SCENCE_ITEM@NM_DiskCalculator@@QAE@ABU01@@Z 00428ac0 f i DeviceEditor.obj
 0001:00027b10       ??4SCENCE_ITEM@NM_DiskCalculator@@QAEAAU01@ABU01@@Z 00428b10 f i DeviceEditor.obj
 0001:00027b60       ??_GSCENCE_ITEM@NM_DiskCalculator@@QAEPAXI@Z 00428b60 f i DeviceEditor.obj
 0001:00027ba0       ??1?$QMapIterator@HVQString@@@@QAE@XZ 00428ba0 f i DeviceEditor.obj
 0001:00027bc0       ??_GCCalculate@APT_DCS@@QAEPAXI@Z 00428bc0 f i DeviceEditor.obj
 0001:00027c00       ??_GBitrateConfig@APT_DCS@@QAEPAXI@Z 00428c00 f i DeviceEditor.obj
 0001:00027c40       ?count@?$QVector@USCENCE_ITEM@NM_DiskCalculator@@@@QBEHXZ 00428c40 f i DeviceEditor.obj
 0001:00027c60       ?sizeOfTypedData@?$QVector@USCENCE_ITEM@NM_DiskCalculator@@@@AAEHXZ 00428c60 f i DeviceEditor.obj
 0001:00027c80       ?alignOfTypedData@?$QVector@USCENCE_ITEM@NM_DiskCalculator@@@@ABEHXZ 00428c80 f i DeviceEditor.obj
 0001:00027cc0       ??1?$QMap@HVQString@@@@QAE@XZ 00428cc0 f i DeviceEditor.obj
 0001:00027d10       ?free@?$QVectorTypedData@USCENCE_ITEM@NM_DiskCalculator@@@@SAXPAU1@H@Z 00428d10 f i DeviceEditor.obj
 0001:00027d30       ??0?$QMapIterator@HVQString@@@@QAE@ABV?$QMap@HVQString@@@@@Z 00428d30 f i DeviceEditor.obj
 0001:00027dc0       ?hasNext@?$QMapIterator@HVQString@@@@QBE_NXZ 00428dc0 f i DeviceEditor.obj
 0001:00027df0       ?next@?$QMapIterator@HVQString@@@@QAE?AVconst_iterator@?$QMap@HVQString@@@@XZ 00428df0 f i DeviceEditor.obj
 0001:00027e40       ?value@?$QMapIterator@HVQString@@@@QBEABVQString@@XZ 00428e40 f i DeviceEditor.obj
 0001:00027e70       ?key@?$QMapIterator@HVQString@@@@QBEABHXZ 00428e70 f i DeviceEditor.obj
 0001:00027ea0       ??0?$QMap@HVQString@@@@QAE@ABV0@@Z 00428ea0 f i DeviceEditor.obj
 0001:00027ef0       ?constBegin@?$QMap@HVQString@@@@QBE?AVconst_iterator@1@XZ 00428ef0 f i DeviceEditor.obj
 0001:00027f20       ?constEnd@?$QMap@HVQString@@@@QBE?AVconst_iterator@1@XZ 00428f20 f i DeviceEditor.obj
 0001:00027f50       ?key@const_iterator@?$QMap@HVQString@@@@QBEABHXZ 00428f50 f i DeviceEditor.obj
 0001:00027f70       ??Dconst_iterator@?$QMap@HVQString@@@@QBEABVQString@@XZ 00428f70 f i DeviceEditor.obj
 0001:00027fa0       ??9const_iterator@?$QMap@HVQString@@@@QBE_NABV01@@Z 00428fa0 f i DeviceEditor.obj
 0001:00027fd0       ??Econst_iterator@?$QMap@HVQString@@@@QAE?AV01@H@Z 00428fd0 f i DeviceEditor.obj
 0001:00028010       ?concrete@?$QMap@HVQString@@@@CAPAU?$QMapNode@HVQString@@@@PAUNode@QMapData@@@Z 00429010 f i DeviceEditor.obj
 0001:00028030       ?detach@?$QMap@HVQString@@@@QAEXXZ 00429030 f i DeviceEditor.obj
 0001:00028070       ??0const_iterator@?$QMap@HVQString@@@@QAE@PAUNode@QMapData@@@Z 00429070 f i DeviceEditor.obj
 0001:00028090       ?payload@?$QMap@HVQString@@@@CAHXZ 00429090 f i DeviceEditor.obj
 0001:000280a0       ??A?$QVector@USCENCE_ITEM@NM_DiskCalculator@@@@QBEABUSCENCE_ITEM@NM_DiskCalculator@@H@Z 004290a0 f i DeviceEditor.obj
 0001:000280d0       ?realloc@?$QVector@USCENCE_ITEM@NM_DiskCalculator@@@@AAEXHH@Z 004290d0 f i DeviceEditor.obj
 0001:000286c0       ?detach_helper@?$QMap@HVQString@@@@AAEXXZ 004296c0 f i DeviceEditor.obj
 0001:00028840       ?freeData@?$QMap@HVQString@@@@AAEXPAUQMapData@@@Z 00429840 f i DeviceEditor.obj
 0001:000288d0       ?alignment@?$QMap@HVQString@@@@CAHXZ 004298d0 f i DeviceEditor.obj
 0001:00028910       ?malloc@?$QVector@USCENCE_ITEM@NM_DiskCalculator@@@@AAEPAUQVectorData@@H@Z 00429910 f i DeviceEditor.obj
 0001:00028970       ?node_create@?$QMap@HVQString@@@@AAEPAUNode@QMapData@@PAU3@QAPAU23@ABHABVQString@@@Z 00429970 f i DeviceEditor.obj
 0001:00028b20       ??_EQLabel@@W7AEPAXI@Z     00429b20 f i DeviceEditor.obj
 0001:00028b30       ??_EQFrame@@W7AEPAXI@Z     00429b30 f i DeviceEditor.obj
 0001:00028b40       ??_EDeviceEditor@@W7AEPAXI@Z 00429b40 f i DeviceEditor.obj
 0001:00028b50       ??_ECLineEdit@iVMSGUIToolkit@@W7AEPAXI@Z 00429b50 f i DeviceEditor.obj
 0001:00028b60       ??_EQCheckBox@@W7AEPAXI@Z  00429b60 f i DeviceEditor.obj
 0001:00028b70       ??_ECRadioButton@iVMSGUIToolkit@@W7AEPAXI@Z 00429b70 f i DeviceEditor.obj
 0001:00028b80       ??_ECComboBox@iVMSGUIToolkit@@W7AEPAXI@Z 00429b80 f i DeviceEditor.obj
 0001:00028b90       ??_ECPushButton@iVMSGUIToolkit@@W7AEPAXI@Z 00429b90 f i DeviceEditor.obj
 0001:00028ba0       ?sort@QStringList@@QAEXXZ  00429ba0 f i DeviceEditor.obj
 0001:00028bc0       ??_EQSpacerItem@@UAEPAXI@Z 00429bc0 f i DeviceEditor.obj
 0001:00028bc0       ??_GQSpacerItem@@UAEPAXI@Z 00429bc0 f i DeviceEditor.obj
 0001:00028c00       ??0DeviceInfoManager@@QAE@PAVQWidget@@@Z 00429c00 f   DeviceInfoManager.obj
 0001:00028d80       ??1DeviceInfoManager@@UAE@XZ 00429d80 f   DeviceInfoManager.obj
 0001:00028e90       ?getDeviceType@DeviceInfoManager@@QAE?AVQStringList@@XZ 00429e90 f   DeviceInfoManager.obj
 0001:00028ed0       ?getResolutionFixedRate@DeviceInfoManager@@QAE?AVQStringList@@H@Z 00429ed0 f   DeviceInfoManager.obj
 0001:00028f10       ?getResolutionFixedRate@DeviceInfoManager@@QAE?AVQStringList@@HVQString@@@Z 00429f10 f   DeviceInfoManager.obj
 0001:00029030       ?getSceneName@DeviceInfoManager@@QAE?AVQString@@H@Z 0042a030 f   DeviceInfoManager.obj
 0001:00029070       ?getSceneInfo@DeviceInfoManager@@QAE?AUSceneInfo@APT_DCS@@ABVQString@@@Z 0042a070 f   DeviceInfoManager.obj
 0001:000290b0       ?getAllScene@DeviceInfoManager@@QAE?AV?$QVector@VQString@@@@XZ 0042a0b0 f   DeviceInfoManager.obj
 0001:000290f0       ?getScenePicture@DeviceInfoManager@@QAE?AVQString@@ABV2@00@Z 0042a0f0 f   DeviceInfoManager.obj
 0001:00029180       ?getSceneBitrate@DeviceInfoManager@@QAEHABVQString@@00@Z 0042a180 f   DeviceInfoManager.obj
 0001:000291b0       ?initDevInfo@DeviceInfoManager@@QAEXXZ 0042a1b0 f   DeviceInfoManager.obj
 0001:00029360       ?getChanelGroupNumber@DeviceInfoManager@@QAEHXZ 0042a360 f   DeviceInfoManager.obj
 0001:000293c0       ?deleteChannelGroupNumber@DeviceInfoManager@@QAEXH@Z 0042a3c0 f   DeviceInfoManager.obj
 0001:00029450       ?upDateScence@DeviceInfoManager@@QAEXXZ 0042a450 f   DeviceInfoManager.obj
 0001:00029530       ?getFrameRate@DeviceInfoManager@@QAEXAAVQStringList@@H@Z 0042a530 f   DeviceInfoManager.obj
 0001:000297b0       ??_GDeviceInfoManager@@UAEPAXI@Z 0042a7b0 f i DeviceInfoManager.obj
 0001:000297b0       ??_EDeviceInfoManager@@UAEPAXI@Z 0042a7b0 f i DeviceInfoManager.obj
 0001:000297f0       ?tr@DeviceInfoManager@@SA?AVQString@@PBD0@Z 0042a7f0 f i DeviceInfoManager.obj
 0001:00029830       ??0?$QVector@VQStringList@@@@QAE@XZ 0042a830 f i DeviceInfoManager.obj
 0001:00029860       ??1?$QVector@VQStringList@@@@QAE@XZ 0042a860 f i DeviceInfoManager.obj
 0001:000298b0       ?push_back@?$QVector@VQStringList@@@@QAEXABVQStringList@@@Z 0042a8b0 f i DeviceInfoManager.obj
 0001:000298d0       ??0?$QVector@VQString@@@@QAE@ABV0@@Z 0042a8d0 f i DeviceInfoManager.obj
 0001:00029920       ??0?$QMap@VQString@@USceneInfo@APT_DCS@@@@QAE@XZ 0042a920 f i DeviceInfoManager.obj
 0001:00029950       ??1?$QMap@VQString@@USceneInfo@APT_DCS@@@@QAE@XZ 0042a950 f i DeviceInfoManager.obj
 0001:000299a0       ??0?$QVector@H@@QAE@XZ     0042a9a0 f i DeviceInfoManager.obj
 0001:000299d0       ??1?$QVector@H@@QAE@XZ     0042a9d0 f i DeviceInfoManager.obj
 0001:00029a20       ?begin@?$QVector@H@@QAEPAHXZ 0042aa20 f i DeviceInfoManager.obj
 0001:00029a50       ?end@?$QVector@H@@QAEPAHXZ 0042aa50 f i DeviceInfoManager.obj
 0001:00029a80       ?erase@?$QVector@H@@QAEPAHPAH@Z 0042aa80 f i DeviceInfoManager.obj
 0001:00029ab0       ?push_back@?$QVector@H@@QAEXABH@Z 0042aab0 f i DeviceInfoManager.obj
 0001:00029ad0       ?detach@?$QVector@H@@QAEXXZ 0042aad0 f i DeviceInfoManager.obj
 0001:00029b00       ?clear@?$QVector@VQStringList@@@@QAEXXZ 0042ab00 f i DeviceInfoManager.obj
 0001:00029b90       ??A?$QVector@VQStringList@@@@QAEAAVQStringList@@H@Z 0042ab90 f i DeviceInfoManager.obj
 0001:00029bc0       ?append@?$QVector@VQStringList@@@@QAEXABVQStringList@@@Z 0042abc0 f i DeviceInfoManager.obj
 0001:00029df0       ?free@?$QVector@VQStringList@@@@AAEXPAU?$QVectorTypedData@VQStringList@@@@@Z 0042adf0 f i DeviceInfoManager.obj
 0001:00029e80       ?clear@?$QVector@VQString@@@@QAEXXZ 0042ae80 f i DeviceInfoManager.obj
 0001:00029f10       ?clear@?$QMap@VQString@@USceneInfo@APT_DCS@@@@QAEXXZ 0042af10 f i DeviceInfoManager.obj
 0001:00029fa0       ?value@?$QMap@VQString@@USceneInfo@APT_DCS@@@@QBE?BUSceneInfo@APT_DCS@@ABVQString@@@Z 0042afa0 f i DeviceInfoManager.obj
 0001:0002a040       ?insert@?$QMap@VQString@@USceneInfo@APT_DCS@@@@QAE?AViterator@1@ABVQString@@ABUSceneInfo@APT_DCS@@@Z 0042b040 f i DeviceInfoManager.obj
 0001:0002a0e0       ?freeData@?$QMap@VQString@@USceneInfo@APT_DCS@@@@AAEXPAUQMapData@@@Z 0042b0e0 f i DeviceInfoManager.obj
 0001:0002a180       ?clear@?$QVector@H@@QAEXXZ 0042b180 f i DeviceInfoManager.obj
 0001:0002a210       ?append@?$QVector@H@@QAEXABH@Z 0042b210 f i DeviceInfoManager.obj
 0001:0002a3a0       ?contains@?$QVector@H@@QBE_NABH@Z 0042b3a0 f i DeviceInfoManager.obj
 0001:0002a410       ?erase@?$QVector@H@@QAEPAHPAH0@Z 0042b410 f i DeviceInfoManager.obj
 0001:0002a570       ?detach_helper@?$QVector@H@@AAEXXZ 0042b570 f i DeviceInfoManager.obj
 0001:0002a5a0       ?free@?$QVector@H@@AAEXPAU?$QVectorTypedData@H@@@Z 0042b5a0 f i DeviceInfoManager.obj
 0001:0002a620       ??_GQStringList@@QAEPAXI@Z 0042b620 f i DeviceInfoManager.obj
 0001:0002a660       ??0SceneInfo@APT_DCS@@QAE@ABU01@@Z 0042b660 f i DeviceInfoManager.obj
 0001:0002a700       ??4SceneInfo@APT_DCS@@QAEAAU01@ABU01@@Z 0042b700 f i DeviceInfoManager.obj
 0001:0002a760       ??_GSceneInfo@APT_DCS@@QAEPAXI@Z 0042b760 f i DeviceInfoManager.obj
 0001:0002a7a0       ?data@?$QVector@VQStringList@@@@QAEPAVQStringList@@XZ 0042b7a0 f i DeviceInfoManager.obj
 0001:0002a7d0       ?sizeOfTypedData@?$QVector@VQStringList@@@@AAEHXZ 0042b7d0 f i DeviceInfoManager.obj
 0001:0002a7f0       ?alignOfTypedData@?$QVector@VQStringList@@@@ABEHXZ 0042b7f0 f i DeviceInfoManager.obj
 0001:0002a830       ?payload@?$QMap@VQString@@USceneInfo@APT_DCS@@@@CAHXZ 0042b830 f i DeviceInfoManager.obj
 0001:0002a840       ?concrete@?$QMap@VQString@@USceneInfo@APT_DCS@@@@CAPAU?$QMapNode@VQString@@USceneInfo@APT_DCS@@@@PAUNode@QMapData@@@Z 0042b840 f i DeviceInfoManager.obj
 0001:0002a860       ?detach@?$QMap@VQString@@USceneInfo@APT_DCS@@@@QAEXXZ 0042b860 f i DeviceInfoManager.obj
 0001:0002a8a0       ?sizeOfTypedData@?$QVector@H@@AAEHXZ 0042b8a0 f i DeviceInfoManager.obj
 0001:0002a8c0       ?alignOfTypedData@?$QVector@H@@ABEHXZ 0042b8c0 f i DeviceInfoManager.obj
 0001:0002a900       ??0iterator@?$QMap@VQString@@USceneInfo@APT_DCS@@@@QAE@PAUNode@QMapData@@@Z 0042b900 f i DeviceInfoManager.obj
 0001:0002a920       ?free@?$QVectorTypedData@H@@SAXPAU1@H@Z 0042b920 f i DeviceInfoManager.obj
 0001:0002a940       ?free@?$QVectorTypedData@VQStringList@@@@SAXPAU1@H@Z 0042b940 f i DeviceInfoManager.obj
 0001:0002a960       ?detach@?$QVector@VQStringList@@@@QAEXXZ 0042b960 f i DeviceInfoManager.obj
 0001:0002a990       ??4?$QVector@VQStringList@@@@QAEAAV0@ABV0@@Z 0042b990 f i DeviceInfoManager.obj
 0001:0002aa10       ?detach_helper@?$QVector@VQStringList@@@@AAEXXZ 0042ba10 f i DeviceInfoManager.obj
 0001:0002aa40       ?realloc@?$QVector@VQStringList@@@@AAEXHH@Z 0042ba40 f i DeviceInfoManager.obj
 0001:0002b010       ??4?$QVector@VQString@@@@QAEAAV0@ABV0@@Z 0042c010 f i DeviceInfoManager.obj
 0001:0002b090       ??4?$QMap@VQString@@USceneInfo@APT_DCS@@@@QAEAAV0@ABV0@@Z 0042c090 f i DeviceInfoManager.obj
 0001:0002b130       ?detach_helper@?$QMap@VQString@@USceneInfo@APT_DCS@@@@AAEXXZ 0042c130 f i DeviceInfoManager.obj
 0001:0002b2b0       ?findNode@?$QMap@VQString@@USceneInfo@APT_DCS@@@@ABEPAUNode@QMapData@@ABVQString@@@Z 0042c2b0 f i DeviceInfoManager.obj
 0001:0002b390       ?mutableFindNode@?$QMap@VQString@@USceneInfo@APT_DCS@@@@ABEPAUNode@QMapData@@QAPAU23@ABVQString@@@Z 0042c390 f i DeviceInfoManager.obj
 0001:0002b480       ?node_create@?$QMap@VQString@@USceneInfo@APT_DCS@@@@AAEPAUNode@QMapData@@PAU3@QAPAU23@ABVQString@@ABUSceneInfo@APT_DCS@@@Z 0042c480 f i DeviceInfoManager.obj
 0001:0002b650       ??4?$QVector@H@@QAEAAV0@ABV0@@Z 0042c650 f i DeviceInfoManager.obj
 0001:0002b6d0       ?realloc@?$QVector@H@@AAEXHH@Z 0042c6d0 f i DeviceInfoManager.obj
 0001:0002bc00       ??$qCopy@PAHPAH@@YAPAHPAH00@Z 0042cc00 f i DeviceInfoManager.obj
 0001:0002bc40       ?alignment@?$QMap@VQString@@USceneInfo@APT_DCS@@@@CAHXZ 0042cc40 f i DeviceInfoManager.obj
 0001:0002bc80       ?malloc@?$QVector@VQStringList@@@@AAEPAUQVectorData@@H@Z 0042cc80 f i DeviceInfoManager.obj
 0001:0002bce0       ?malloc@?$QVector@H@@AAEPAUQVectorData@@H@Z 0042cce0 f i DeviceInfoManager.obj
 0001:0002bd40       ??0QStringList@@QAE@ABV0@@Z 0042cd40 f i DeviceInfoManager.obj
 0001:0002bd70       ??0?$QList@VQString@@@@QAE@ABV0@@Z 0042cd70 f i DeviceInfoManager.obj
 0001:0002bdc0       ??0ScenceSelector@@QAE@PAVQWidget@@@Z 0042cdc0 f   ScenceSelector.obj
 0001:0002bed0       ?setScenceData@ScenceSelector@@QAEXABV?$QVector@USCENCE_ITEM@NM_DiskCalculator@@@@@Z 0042ced0 f   ScenceSelector.obj
 0001:0002bf70       ?addScenceItem@ScenceSelector@@QAEXABUSCENCE_ITEM@NM_DiskCalculator@@@Z 0042cf70 f   ScenceSelector.obj
 0001:0002c110       ?OnScenceSelected@ScenceSelector@@QAEXH@Z 0042d110 f   ScenceSelector.obj
 0001:0002c310       ?setScenePicture@ScenceSelector@@QAEXABVQString@@@Z 0042d310 f   ScenceSelector.obj
 0001:0002c590       ?clearScenceRadioButtons@ScenceSelector@@AAEXXZ 0042d590 f   ScenceSelector.obj
 0001:0002c5c0       ?resizeEvent@ScenceSelector@@EAEXPAVQResizeEvent@@@Z 0042d5c0 f   ScenceSelector.obj
 0001:0002c5f0       ??1ScenceSelector@@UAE@XZ  0042d5f0 f   ScenceSelector.obj
 0001:0002c8c0       ?setupUi@Ui_ScenceSelector@@QAEXPAVQWidget@@@Z 0042d8c0 f i ScenceSelector.obj
 0001:0002d470       ?retranslateUi@Ui_ScenceSelector@@QAEXPAVQWidget@@@Z 0042e470 f i ScenceSelector.obj
 0001:0002d5d0       ??_EQListWidget@@UAEPAXI@Z 0042e5d0 f i ScenceSelector.obj
 0001:0002d5d0       ??_GQListWidget@@UAEPAXI@Z 0042e5d0 f i ScenceSelector.obj
 0001:0002d610       ??_EScenceSelector@@UAEPAXI@Z 0042e610 f i ScenceSelector.obj
 0001:0002d610       ??_GScenceSelector@@UAEPAXI@Z 0042e610 f i ScenceSelector.obj
 0001:0002d650       ??0ScenceQRaidoButton@ScenceSelector@@QAE@PAVQWidget@@HABVQString@@@Z 0042e650 f i ScenceSelector.obj
 0001:0002d720       ??_GScenceQRaidoButton@ScenceSelector@@UAEPAXI@Z 0042e720 f i ScenceSelector.obj
 0001:0002d720       ??_EScenceQRaidoButton@ScenceSelector@@UAEPAXI@Z 0042e720 f i ScenceSelector.obj
 0001:0002d760       ??1ScenceQRaidoButton@ScenceSelector@@UAE@XZ 0042e760 f i ScenceSelector.obj
 0001:0002d780       ??1?$QMapIterator@HPAVScenceQRaidoButton@ScenceSelector@@@@QAE@XZ 0042e780 f i ScenceSelector.obj
 0001:0002d7a0       ?tr@ScenceSelector@@SA?AVQString@@PBD0@Z 0042e7a0 f i ScenceSelector.obj
 0001:0002d7e0       ??0?$QMap@HPAVScenceQRaidoButton@ScenceSelector@@@@QAE@XZ 0042e7e0 f i ScenceSelector.obj
 0001:0002d810       ??1?$QMap@HPAVScenceQRaidoButton@ScenceSelector@@@@QAE@XZ 0042e810 f i ScenceSelector.obj
 0001:0002d860       ??0?$QMapIterator@HPAVScenceQRaidoButton@ScenceSelector@@@@QAE@ABV?$QMap@HPAVScenceQRaidoButton@ScenceSelector@@@@@Z 0042e860 f i ScenceSelector.obj
 0001:0002d8f0       ?hasNext@?$QMapIterator@HPAVScenceQRaidoButton@ScenceSelector@@@@QBE_NXZ 0042e8f0 f i ScenceSelector.obj
 0001:0002d920       ?next@?$QMapIterator@HPAVScenceQRaidoButton@ScenceSelector@@@@QAE?AVconst_iterator@?$QMap@HPAVScenceQRaidoButton@ScenceSelector@@@@XZ 0042e920 f i ScenceSelector.obj
 0001:0002d970       ?value@?$QMapIterator@HPAVScenceQRaidoButton@ScenceSelector@@@@QBEABQAVScenceQRaidoButton@ScenceSelector@@XZ 0042e970 f i ScenceSelector.obj
 0001:0002d9a0       ?key@?$QMapIterator@HPAVScenceQRaidoButton@ScenceSelector@@@@QBEABHXZ 0042e9a0 f i ScenceSelector.obj
 0001:0002d9d0       ??0?$QMap@HPAVScenceQRaidoButton@ScenceSelector@@@@QAE@ABV0@@Z 0042e9d0 f i ScenceSelector.obj
 0001:0002da20       ?constBegin@?$QMap@HPAVScenceQRaidoButton@ScenceSelector@@@@QBE?AVconst_iterator@1@XZ 0042ea20 f i ScenceSelector.obj
 0001:0002da50       ?constEnd@?$QMap@HPAVScenceQRaidoButton@ScenceSelector@@@@QBE?AVconst_iterator@1@XZ 0042ea50 f i ScenceSelector.obj
 0001:0002da80       ?key@const_iterator@?$QMap@HPAVScenceQRaidoButton@ScenceSelector@@@@QBEABHXZ 0042ea80 f i ScenceSelector.obj
 0001:0002daa0       ??Dconst_iterator@?$QMap@HPAVScenceQRaidoButton@ScenceSelector@@@@QBEABQAVScenceQRaidoButton@ScenceSelector@@XZ 0042eaa0 f i ScenceSelector.obj
 0001:0002dad0       ??9const_iterator@?$QMap@HPAVScenceQRaidoButton@ScenceSelector@@@@QBE_NABV01@@Z 0042ead0 f i ScenceSelector.obj
 0001:0002db00       ??Econst_iterator@?$QMap@HPAVScenceQRaidoButton@ScenceSelector@@@@QAE?AV01@H@Z 0042eb00 f i ScenceSelector.obj
 0001:0002db40       ?concrete@?$QMap@HPAVScenceQRaidoButton@ScenceSelector@@@@CAPAU?$QMapNode@HPAVScenceQRaidoButton@ScenceSelector@@@@PAUNode@QMapData@@@Z 0042eb40 f i ScenceSelector.obj
 0001:0002db60       ?detach@?$QMap@HPAVScenceQRaidoButton@ScenceSelector@@@@QAEXXZ 0042eb60 f i ScenceSelector.obj
 0001:0002dba0       ??0const_iterator@?$QMap@HPAVScenceQRaidoButton@ScenceSelector@@@@QAE@PAUNode@QMapData@@@Z 0042eba0 f i ScenceSelector.obj
 0001:0002dbc0       ?payload@?$QMap@HPAVScenceQRaidoButton@ScenceSelector@@@@CAHXZ 0042ebc0 f i ScenceSelector.obj
 0001:0002dbd0       ?contains@?$QMap@HPAVScenceQRaidoButton@ScenceSelector@@@@QBE_NABH@Z 0042ebd0 f i ScenceSelector.obj
 0001:0002dc00       ?value@?$QMap@HPAVScenceQRaidoButton@ScenceSelector@@@@QBEQAVScenceQRaidoButton@ScenceSelector@@ABH@Z 0042ec00 f i ScenceSelector.obj
 0001:0002dc60       ?insert@?$QMap@HPAVScenceQRaidoButton@ScenceSelector@@@@QAE?AViterator@1@ABHABQAVScenceQRaidoButton@ScenceSelector@@@Z 0042ec60 f i ScenceSelector.obj
 0001:0002dd00       ?detach_helper@?$QMap@HPAVScenceQRaidoButton@ScenceSelector@@@@AAEXXZ 0042ed00 f i ScenceSelector.obj
 0001:0002de80       ?freeData@?$QMap@HPAVScenceQRaidoButton@ScenceSelector@@@@AAEXPAUQMapData@@@Z 0042ee80 f i ScenceSelector.obj
 0001:0002def0       ??$clearListWidgetData@HVQListWidget@@VScenceQRaidoButton@ScenceSelector@@@ShareFunction@@YAXPAVQListWidget@@AAV?$QMap@HPAVScenceQRaidoButton@ScenceSelector@@@@@Z 0042eef0 f i ScenceSelector.obj
 0001:0002dfe0       ?alignment@?$QMap@HPAVScenceQRaidoButton@ScenceSelector@@@@CAHXZ 0042efe0 f i ScenceSelector.obj
 0001:0002e020       ??0iterator@?$QMap@HPAVScenceQRaidoButton@ScenceSelector@@@@QAE@PAUNode@QMapData@@@Z 0042f020 f i ScenceSelector.obj
 0001:0002e040       ?value@const_iterator@?$QMap@HPAVScenceQRaidoButton@ScenceSelector@@@@QBEABQAVScenceQRaidoButton@ScenceSelector@@XZ 0042f040 f i ScenceSelector.obj
 0001:0002e070       ?clear@?$QMap@HPAVScenceQRaidoButton@ScenceSelector@@@@QAEXXZ 0042f070 f i ScenceSelector.obj
 0001:0002e100       ?findNode@?$QMap@HPAVScenceQRaidoButton@ScenceSelector@@@@ABEPAUNode@QMapData@@ABH@Z 0042f100 f i ScenceSelector.obj
 0001:0002e1e0       ?mutableFindNode@?$QMap@HPAVScenceQRaidoButton@ScenceSelector@@@@ABEPAUNode@QMapData@@QAPAU23@ABH@Z 0042f1e0 f i ScenceSelector.obj
 0001:0002e2d0       ?node_create@?$QMap@HPAVScenceQRaidoButton@ScenceSelector@@@@AAEPAUNode@QMapData@@PAU3@QAPAU23@ABHABQAVScenceQRaidoButton@ScenceSelector@@@Z 0042f2d0 f i ScenceSelector.obj
 0001:0002e460       ??4?$QMap@HPAVScenceQRaidoButton@ScenceSelector@@@@QAEAAV0@ABV0@@Z 0042f460 f i ScenceSelector.obj
 0001:0002e500       ??$qMapLessThanKey@H@@YA_NABH0@Z 0042f500 f i ScenceSelector.obj
 0001:0002e520       ??_EScenceQRaidoButton@ScenceSelector@@W7AEPAXI@Z 0042f520 f i ScenceSelector.obj
 0001:0002e530       ??_EQListWidget@@W7AEPAXI@Z 0042f530 f i ScenceSelector.obj
 0001:0002e540       ??_EScenceSelector@@W7AEPAXI@Z 0042f540 f i ScenceSelector.obj
 0001:0002e550       ??0?$QFlags@W4ImageConversionFlag@Qt@@@@QAE@W4ImageConversionFlag@Qt@@@Z 0042f550 f i ScenceSelector.obj
 0001:0002e570       ??0CapacityCalculation@@QAE@PAVQWidget@@@Z 0042f570 f   CapacityCalculation.obj
 0001:0002e730       ?resizeLayout@CapacityCalculation@@QAEXHH@Z 0042f730 f   CapacityCalculation.obj
 0001:0002e740       ?showNullPage@CapacityCalculation@@QAEXXZ 0042f740 f   CapacityCalculation.obj
 0001:0002e7b0       ?showNormalPage@CapacityCalculation@@QAEXXZ 0042f7b0 f   CapacityCalculation.obj
 0001:0002e820       ?getDeviceAddPage@CapacityCalculation@@QAEPAVQObject@@XZ 0042f820 f   CapacityCalculation.obj
 0001:0002e840       ?getDataDisplayPageSize@CapacityCalculation@@QAEPAVQObject@@XZ 0042f840 f   CapacityCalculation.obj
 0001:0002e870       ?getDataDisplayPageTime@CapacityCalculation@@QAEPAVQObject@@XZ 0042f870 f   CapacityCalculation.obj
 0001:0002e8a0       ?getDataCalculatorPage@CapacityCalculation@@QAEPAVQObject@@XZ 0042f8a0 f   CapacityCalculation.obj
 0001:0002e8c0       ??1CapacityCalculation@@UAE@XZ 0042f8c0 f   CapacityCalculation.obj
 0001:0002e9f0       ?setupUi@Ui_CapacityCalculation@@QAEXPAVQWidget@@@Z 0042f9f0 f i CapacityCalculation.obj
 0001:00030220       ?retranslateUi@Ui_CapacityCalculation@@QAEXPAVQWidget@@@Z 00431220 f i CapacityCalculation.obj
 0001:00030430       ??_GQPushButton@@UAEPAXI@Z 00431430 f i CapacityCalculation.obj
 0001:00030430       ??_EQPushButton@@UAEPAXI@Z 00431430 f i CapacityCalculation.obj
 0001:00030470       ??_GCapacityCalculation@@UAEPAXI@Z 00431470 f i CapacityCalculation.obj
 0001:00030470       ??_ECapacityCalculation@@UAEPAXI@Z 00431470 f i CapacityCalculation.obj
 0001:000304b0       ??_EQPushButton@@W7AEPAXI@Z 004314b0 f i CapacityCalculation.obj
 0001:000304c0       ??_ECapacityCalculation@@W7AEPAXI@Z 004314c0 f i CapacityCalculation.obj
 0001:000304d0       ??0WidgetDeviceListBorder@@QAE@PAVQWidget@@@Z 004314d0 f   WidgetDeviceListBorder.obj
 0001:000305a0       ??1WidgetDeviceListBorder@@UAE@XZ 004315a0 f   WidgetDeviceListBorder.obj
 0001:00030630       ?setupUi@Ui_WidgetDeviceListBorder@@QAEXPAVQWidget@@@Z 00431630 f i WidgetDeviceListBorder.obj
 0001:00030f00       ?retranslateUi@Ui_WidgetDeviceListBorder@@QAEXPAVQWidget@@@Z 00431f00 f i WidgetDeviceListBorder.obj
 0001:00031050       ??_EWidgetDeviceListBorder@@UAEPAXI@Z 00432050 f i WidgetDeviceListBorder.obj
 0001:00031050       ??_GWidgetDeviceListBorder@@UAEPAXI@Z 00432050 f i WidgetDeviceListBorder.obj
 0001:00031090       ??_EWidgetDeviceListBorder@@W7AEPAXI@Z 00432090 f i WidgetDeviceListBorder.obj
 0001:000310a0       ??0BandWidthPage@@QAE@PAVQWidget@@@Z 004320a0 f   BandWidthPage.obj
 0001:00031340       ?setChannelCount@BandWidthPage@@QAEXABVQString@@@Z 00432340 f   BandWidthPage.obj
 0001:00031460       ?setIPCCount@BandWidthPage@@QAEXABVQString@@@Z 00432460 f   BandWidthPage.obj
 0001:00031470       ?setDVRCount@BandWidthPage@@QAEXABVQString@@@Z 00432470 f   BandWidthPage.obj
 0001:00031480       ?setBandWidthCount@BandWidthPage@@QAEXABVQString@@0@Z 00432480 f   BandWidthPage.obj
 0001:000315e0       ?onSetAllCount@BandWidthPage@@QAEXABVQString@@0000@Z 004325e0 f   BandWidthPage.obj
 0001:00031a40       ?channelCount@BandWidthPage@@QAE?AVQString@@ABV2@@Z 00432a40 f   BandWidthPage.obj
 0001:00031a80       ?IPCCount@BandWidthPage@@QAE?AVQString@@ABV2@@Z 00432a80 f   BandWidthPage.obj
 0001:00031ac0       ?DVRCount@BandWidthPage@@QAE?AVQString@@ABV2@@Z 00432ac0 f   BandWidthPage.obj
 0001:00031b00       ?bandWidthCount@BandWidthPage@@QAE?AVQString@@ABV2@@Z 00432b00 f   BandWidthPage.obj
 0001:00031b40       ??1BandWidthPage@@UAE@XZ   00432b40 f   BandWidthPage.obj
 0001:00031f00       ?setupUi@Ui_BandWidthPage@@QAEXPAVQWidget@@@Z 00432f00 f i BandWidthPage.obj
 0001:00032ce0       ?retranslateUi@Ui_BandWidthPage@@QAEXPAVQWidget@@@Z 00433ce0 f i BandWidthPage.obj
 0001:00032f20       ??_EBandWidthPage@@UAEPAXI@Z 00433f20 f i BandWidthPage.obj
 0001:00032f20       ??_GBandWidthPage@@UAEPAXI@Z 00433f20 f i BandWidthPage.obj
 0001:00032f60       ?tr@BandWidthPage@@SA?AVQString@@PBD0@Z 00433f60 f i BandWidthPage.obj
 0001:00032fa0       ??_EBandWidthPage@@W7AEPAXI@Z 00433fa0 f i BandWidthPage.obj
 0001:00032fb0       ??0DataCalculatorPage@@QAE@PAVQWidget@@@Z 00433fb0 f   DataCalculatorPage.obj
 0001:000334e0       ?getDataDisplayPageSize@DataCalculatorPage@@QAEPAVQObject@@XZ 004344e0 f   DataCalculatorPage.obj
 0001:00033500       ?getDataDisplayPageTime@DataCalculatorPage@@QAEPAVQObject@@XZ 00434500 f   DataCalculatorPage.obj
 0001:00033520       ?OnCalculateTypeSelectedChanged@DataCalculatorPage@@AAEXH@Z 00434520 f   DataCalculatorPage.obj
 0001:00033550       ?OnSwitchBarChanged@DataCalculatorPage@@QAEX_N@Z 00434550 f   DataCalculatorPage.obj
 0001:00033590       ??1DataCalculatorPage@@UAE@XZ 00434590 f   DataCalculatorPage.obj
 0001:00033700       ?initUi@DataCalculatorPage@@QAEXXZ 00434700 f   DataCalculatorPage.obj
 0001:000338d0       ?OnDeviceChanged@DataCalculatorPage@@QAEXN@Z 004348d0 f   DataCalculatorPage.obj
 0001:00033de0       ?OnCalculateTimeDataChanged@DataCalculatorPage@@AAEXXZ 00434de0 f   DataCalculatorPage.obj
 0001:00034d70       ?OnCalculateDiskSizeDataChanged@DataCalculatorPage@@AAEXXZ 00435d70 f   DataCalculatorPage.obj
 0001:00035760       ?getCurrentCalculateSection@DataCalculatorPage@@AAE?AW4CalculatorSection@1@XZ 00436760 f   DataCalculatorPage.obj
 0001:00035780       ?resizeEvent@DataCalculatorPage@@EAEXPAVQResizeEvent@@@Z 00436780 f   DataCalculatorPage.obj
 0001:000357a0       ?getDialogLocation@DataCalculatorPage@@AAE?AVQPoint@@XZ 004367a0 f   DataCalculatorPage.obj
 0001:00035860       ?onSwitchBtnChanged@DataCalculatorPage@@QAEXXZ 00436860 f   DataCalculatorPage.obj
 0001:00035b00       ?onDeviceChangedToBandWidth@DataCalculatorPage@@QAEXAAVQString@@0000@Z 00436b00 f   DataCalculatorPage.obj
 0001:00035be0       ?getCalResults@DataCalculatorPage@@QAEXAAUResult@@@Z 00436be0 f   DataCalculatorPage.obj
 0001:00035cc0       ?setResults@DataCalculatorPage@@AAEXXZ 00436cc0 f   DataCalculatorPage.obj
 0001:000382f0       ?setupUi@Ui_DataCalculatorPage@@QAEXPAVQWidget@@@Z 004392f0 f i DataCalculatorPage.obj
 0001:0003c4b0       ?retranslateUi@Ui_DataCalculatorPage@@QAEXPAVQWidget@@@Z 0043d4b0 f i DataCalculatorPage.obj
 0001:0003cb10       ??_EQStackedWidget@@UAEPAXI@Z 0043db10 f i DataCalculatorPage.obj
 0001:0003cb10       ??_GQStackedWidget@@UAEPAXI@Z 0043db10 f i DataCalculatorPage.obj
 0001:0003cb50       ??_ECSlider@iVMSGUIToolkit@@UAEPAXI@Z 0043db50 f i DataCalculatorPage.obj
 0001:0003cb50       ??_GCSlider@iVMSGUIToolkit@@UAEPAXI@Z 0043db50 f i DataCalculatorPage.obj
 0001:0003cb90       ??_EDataCalculatorPage@@UAEPAXI@Z 0043db90 f i DataCalculatorPage.obj
 0001:0003cb90       ??_GDataCalculatorPage@@UAEPAXI@Z 0043db90 f i DataCalculatorPage.obj
 0001:0003cbd0       ?tr@DataCalculatorPage@@SA?AVQString@@PBD0@Z 0043dbd0 f i DataCalculatorPage.obj
 0001:0003cc10       ??_EQStackedWidget@@W7AEPAXI@Z 0043dc10 f i DataCalculatorPage.obj
 0001:0003cc20       ??_EDataCalculatorPage@@W7AEPAXI@Z 0043dc20 f i DataCalculatorPage.obj
 0001:0003cc30       ??_ECSlider@iVMSGUIToolkit@@W7AEPAXI@Z 0043dc30 f i DataCalculatorPage.obj
 0001:0003cc40       ??0DataDisplayPage@@QAE@PAVQWidget@@@Z 0043dc40 f   DataDisplayPage.obj
 0001:0003cd40       ?displayTime@DataDisplayPage@@QAEXABVQString@@00@Z 0043dd40 f   DataDisplayPage.obj
 0001:0003ceb0       ??1DataDisplayPage@@UAE@XZ 0043deb0 f   DataDisplayPage.obj
 0001:0003d010       ?setupUi@Ui_DataDisplayPage@@QAEXPAVQWidget@@@Z 0043e010 f i DataDisplayPage.obj
 0001:00040a90       ??U@YA?AV?$QFlags@W4AlignmentFlag@Qt@@@@W4AlignmentFlag@Qt@@0@Z 00441a90 f i DataDisplayPage.obj
 0001:00040ac0       ?retranslateUi@Ui_DataDisplayPage@@QAEXPAVQWidget@@@Z 00441ac0 f i DataDisplayPage.obj
 0001:00040f40       ??_EDataDisplayPage@@UAEPAXI@Z 00441f40 f i DataDisplayPage.obj
 0001:00040f40       ??_GDataDisplayPage@@UAEPAXI@Z 00441f40 f i DataDisplayPage.obj
 0001:00040f80       ??_EDataDisplayPage@@W7AEPAXI@Z 00441f80 f i DataDisplayPage.obj
 0001:00040f90       ??0?$QFlags@W4AlignmentFlag@Qt@@@@QAE@W4AlignmentFlag@Qt@@@Z 00441f90 f i DataDisplayPage.obj
 0001:00040fb0       ??U?$QFlags@W4AlignmentFlag@Qt@@@@QBE?AV0@W4AlignmentFlag@Qt@@@Z 00441fb0 f i DataDisplayPage.obj
 0001:00040fe0       ??0SizeDisplayPage@@QAE@PAVQWidget@@@Z 00441fe0 f   SizeDisplayPage.obj
 0001:000410b0       ?displaySize@SizeDisplayPage@@QAEXABVQString@@0@Z 004420b0 f   SizeDisplayPage.obj
 0001:000411b0       ??1SizeDisplayPage@@UAE@XZ 004421b0 f   SizeDisplayPage.obj
 0001:00041280       ?setupUi@Ui_SizeDisplayPage@@QAEXPAVQWidget@@@Z 00442280 f i SizeDisplayPage.obj
 0001:00041c90       ?retranslateUi@Ui_SizeDisplayPage@@QAEXPAVQWidget@@@Z 00442c90 f i SizeDisplayPage.obj
 0001:00041df0       ??_GSizeDisplayPage@@UAEPAXI@Z 00442df0 f i SizeDisplayPage.obj
 0001:00041df0       ??_ESizeDisplayPage@@UAEPAXI@Z 00442df0 f i SizeDisplayPage.obj
 0001:00041e30       ??_ESizeDisplayPage@@W7AEPAXI@Z 00442e30 f i SizeDisplayPage.obj
 0001:00041e40       ??0DeviceAddPage@@QAE@PAVQWidget@@@Z 00442e40 f   DeviceAddPage.obj
 0001:00041fb0       ?getDeviceData@DeviceAddPage@@QBE?AV?$QMap@_JUStructDeviceItem@NM_DiskCalculator@@@@XZ 00442fb0 f   DeviceAddPage.obj
 0001:00041ff0       ?setDeviceTypeData@DeviceAddPage@@QAEXABV?$QVector@UStructDeviceItem@NM_DiskCalculator@@@@@Z 00442ff0 f   DeviceAddPage.obj
 0001:00042480       ?addDeviceTypeItem@DeviceAddPage@@QAEXABUStructDeviceItem@NM_DiskCalculator@@_N@Z 00443480 f   DeviceAddPage.obj
 0001:00042dd0       ?OnDeleteDeviceItem@DeviceAddPage@@QAEX_JH@Z 00443dd0 f   DeviceAddPage.obj
 0001:000432a0       ?onClearDeviceItems@DeviceAddPage@@QAEXXZ 004442a0 f   DeviceAddPage.obj
 0001:000433c0       ?clearDeviceItems@DeviceAddPage@@AAEXXZ 004443c0 f   DeviceAddPage.obj
 0001:00043850       ??1DeviceAddPage@@UAE@XZ   00444850 f   DeviceAddPage.obj
 0001:00043910       ?calculateBitrate@DeviceAddPage@@AAENXZ 00444910 f   DeviceAddPage.obj
 0001:000439a0       ?getFrameStandard@DeviceAddPage@@QAEHXZ 004449a0 f   DeviceAddPage.obj
 0001:000439c0       ?OnGetFramerateStandard@DeviceAddPage@@AAEXXZ 004449c0 f   DeviceAddPage.obj
 0001:00043a00       ?OnFrametareStandardChanged@DeviceAddPage@@AAEXH@Z 00444a00 f   DeviceAddPage.obj
 0001:00043a30       ?resizeEvent@DeviceAddPage@@EAEXPAVQResizeEvent@@@Z 00444a30 f   DeviceAddPage.obj
 0001:00043af0       ?setDeviceItemsPAL@DeviceAddPage@@AAEXXZ 00444af0 f   DeviceAddPage.obj
 0001:00044540       ?setDeviceItemsNTSC@DeviceAddPage@@AAEXXZ 00445540 f   DeviceAddPage.obj
 0001:00044f90       ?getAllDeviceCount@DeviceAddPage@@AAEHXZ 00445f90 f   DeviceAddPage.obj
 0001:00045010       ?getIPCCount@DeviceAddPage@@AAEHXZ 00446010 f   DeviceAddPage.obj
 0001:000450b0       ?getDVRCount@DeviceAddPage@@AAEHXZ 004460b0 f   DeviceAddPage.obj
 0001:00045150       ?onExportDeviceItems@DeviceAddPage@@QAEXUResult@@@Z 00446150 f   DeviceAddPage.obj
 0001:00048c40       ?setupUi@Ui_DeviceAddPage@@QAEXPAVQWidget@@@Z 00449c40 f i DeviceAddPage.obj
 0001:00048fa0       ?retranslateUi@Ui_DeviceAddPage@@QAEXPAVQWidget@@@Z 00449fa0 f i DeviceAddPage.obj
 0001:00049050       ??_EDeviceAddPage@@UAEPAXI@Z 0044a050 f i DeviceAddPage.obj
 0001:00049050       ??_GDeviceAddPage@@UAEPAXI@Z 0044a050 f i DeviceAddPage.obj
 0001:00049090       ?tr@DeviceAddPage@@SA?AVQString@@PBD0@Z 0044a090 f i DeviceAddPage.obj
 0001:000490d0       ?getId@DeviceItemWidget@NM_DiskCalculator@@QBEHXZ 0044a0d0 f i DeviceAddPage.obj
 0001:000490f0       ??1?$QMapIterator@_JPAVDeviceItemWidget@NM_DiskCalculator@@@@QAE@XZ 0044a0f0 f i DeviceAddPage.obj
 0001:00049110       ??0?$QFlags@W4Option@QFileDialog@@@@QAE@PAPAX@Z 0044a110 f i DeviceAddPage.obj
 0001:00049130       ??0?$QMap@_JPAVDeviceItemWidget@NM_DiskCalculator@@@@QAE@XZ 0044a130 f i DeviceAddPage.obj
 0001:00049160       ??1?$QMap@_JPAVDeviceItemWidget@NM_DiskCalculator@@@@QAE@XZ 0044a160 f i DeviceAddPage.obj
 0001:000491b0       ?size@?$QMap@_JPAVDeviceItemWidget@NM_DiskCalculator@@@@QBEHXZ 0044a1b0 f i DeviceAddPage.obj
 0001:000491d0       ??0?$QMap@_JUStructDeviceItem@NM_DiskCalculator@@@@QAE@XZ 0044a1d0 f i DeviceAddPage.obj
 0001:00049200       ??0?$QMap@_JUStructDeviceItem@NM_DiskCalculator@@@@QAE@ABV0@@Z 0044a200 f i DeviceAddPage.obj
 0001:00049250       ?begin@?$QMap@_JUStructDeviceItem@NM_DiskCalculator@@@@QAE?AViterator@1@XZ 0044a250 f i DeviceAddPage.obj
 0001:00049290       ?end@?$QMap@_JUStructDeviceItem@NM_DiskCalculator@@@@QAE?AViterator@1@XZ 0044a290 f i DeviceAddPage.obj
 0001:000492c0       ?count@?$QVector@UStructDeviceItem@NM_DiskCalculator@@@@QBEHXZ 0044a2c0 f i DeviceAddPage.obj
 0001:000492e0       ?key@iterator@?$QMap@_JUStructDeviceItem@NM_DiskCalculator@@@@QBEAB_JXZ 0044a2e0 f i DeviceAddPage.obj
 0001:00049300       ??Citerator@?$QMap@_JUStructDeviceItem@NM_DiskCalculator@@@@QBEPAUStructDeviceItem@NM_DiskCalculator@@XZ 0044a300 f i DeviceAddPage.obj
 0001:00049330       ??9iterator@?$QMap@_JUStructDeviceItem@NM_DiskCalculator@@@@QBE_NABV01@@Z 0044a330 f i DeviceAddPage.obj
 0001:00049360       ??Eiterator@?$QMap@_JUStructDeviceItem@NM_DiskCalculator@@@@QAEAAV01@XZ 0044a360 f i DeviceAddPage.obj
 0001:00049390       ??0?$QMapIterator@_JPAVDeviceItemWidget@NM_DiskCalculator@@@@QAE@ABV?$QMap@_JPAVDeviceItemWidget@NM_DiskCalculator@@@@@Z 0044a390 f i DeviceAddPage.obj
 0001:00049420       ?hasNext@?$QMapIterator@_JPAVDeviceItemWidget@NM_DiskCalculator@@@@QBE_NXZ 0044a420 f i DeviceAddPage.obj
 0001:00049450       ?next@?$QMapIterator@_JPAVDeviceItemWidget@NM_DiskCalculator@@@@QAE?AVconst_iterator@?$QMap@_JPAVDeviceItemWidget@NM_DiskCalculator@@@@XZ 0044a450 f i DeviceAddPage.obj
 0001:000494a0       ?value@const_iterator@?$QMap@_JPAVDeviceItemWidget@NM_DiskCalculator@@@@QBEABQAVDeviceItemWidget@NM_DiskCalculator@@XZ 0044a4a0 f i DeviceAddPage.obj
 0001:000494d0       ?concrete@?$QMap@_JPAVDeviceItemWidget@NM_DiskCalculator@@@@CAPAU?$QMapNode@_JPAVDeviceItemWidget@NM_DiskCalculator@@@@PAUNode@QMapData@@@Z 0044a4d0 f i DeviceAddPage.obj
 0001:000494f0       ??0?$QMap@_JPAVDeviceItemWidget@NM_DiskCalculator@@@@QAE@ABV0@@Z 0044a4f0 f i DeviceAddPage.obj
 0001:00049540       ?constBegin@?$QMap@_JPAVDeviceItemWidget@NM_DiskCalculator@@@@QBE?AVconst_iterator@1@XZ 0044a540 f i DeviceAddPage.obj
 0001:00049570       ?constEnd@?$QMap@_JPAVDeviceItemWidget@NM_DiskCalculator@@@@QBE?AVconst_iterator@1@XZ 0044a570 f i DeviceAddPage.obj
 0001:000495a0       ?detach@?$QMap@_JUStructDeviceItem@NM_DiskCalculator@@@@QAEXXZ 0044a5a0 f i DeviceAddPage.obj
 0001:000495e0       ??0iterator@?$QMap@_JUStructDeviceItem@NM_DiskCalculator@@@@QAE@PAUNode@QMapData@@@Z 0044a5e0 f i DeviceAddPage.obj
 0001:00049600       ??9const_iterator@?$QMap@_JPAVDeviceItemWidget@NM_DiskCalculator@@@@QBE_NABV01@@Z 0044a600 f i DeviceAddPage.obj
 0001:00049630       ??Econst_iterator@?$QMap@_JPAVDeviceItemWidget@NM_DiskCalculator@@@@QAE?AV01@H@Z 0044a630 f i DeviceAddPage.obj
 0001:00049670       ?payload@?$QMap@_JPAVDeviceItemWidget@NM_DiskCalculator@@@@CAHXZ 0044a670 f i DeviceAddPage.obj
 0001:00049680       ?detach@?$QMap@_JPAVDeviceItemWidget@NM_DiskCalculator@@@@QAEXXZ 0044a680 f i DeviceAddPage.obj
 0001:000496c0       ??0const_iterator@?$QMap@_JPAVDeviceItemWidget@NM_DiskCalculator@@@@QAE@PAUNode@QMapData@@@Z 0044a6c0 f i DeviceAddPage.obj
 0001:000496e0       ?clear@?$QMap@_JPAVDeviceItemWidget@NM_DiskCalculator@@@@QAEXXZ 0044a6e0 f i DeviceAddPage.obj
 0001:00049770       ?remove@?$QMap@_JPAVDeviceItemWidget@NM_DiskCalculator@@@@QAEHAB_J@Z 0044a770 f i DeviceAddPage.obj
 0001:00049940       ?contains@?$QMap@_JPAVDeviceItemWidget@NM_DiskCalculator@@@@QBE_NAB_J@Z 0044a940 f i DeviceAddPage.obj
 0001:00049970       ?value@?$QMap@_JPAVDeviceItemWidget@NM_DiskCalculator@@@@QBEQAVDeviceItemWidget@NM_DiskCalculator@@AB_J@Z 0044a970 f i DeviceAddPage.obj
 0001:000499d0       ?insert@?$QMap@_JPAVDeviceItemWidget@NM_DiskCalculator@@@@QAE?AViterator@1@AB_JABQAVDeviceItemWidget@NM_DiskCalculator@@@Z 0044a9d0 f i DeviceAddPage.obj
 0001:00049a70       ?detach_helper@?$QMap@_JPAVDeviceItemWidget@NM_DiskCalculator@@@@AAEXXZ 0044aa70 f i DeviceAddPage.obj
 0001:00049bf0       ?freeData@?$QMap@_JPAVDeviceItemWidget@NM_DiskCalculator@@@@AAEXPAUQMapData@@@Z 0044abf0 f i DeviceAddPage.obj
 0001:00049c60       ?clear@?$QMap@_JUStructDeviceItem@NM_DiskCalculator@@@@QAEXXZ 0044ac60 f i DeviceAddPage.obj
 0001:00049cf0       ?remove@?$QMap@_JUStructDeviceItem@NM_DiskCalculator@@@@QAEHAB_J@Z 0044acf0 f i DeviceAddPage.obj
 0001:00049ed0       ?insert@?$QMap@_JUStructDeviceItem@NM_DiskCalculator@@@@QAE?AViterator@1@AB_JABUStructDeviceItem@NM_DiskCalculator@@@Z 0044aed0 f i DeviceAddPage.obj
 0001:00049f70       ??A?$QVector@UStructDeviceItem@NM_DiskCalculator@@@@QBEABUStructDeviceItem@NM_DiskCalculator@@H@Z 0044af70 f i DeviceAddPage.obj
 0001:00049fa0       ??4StructDeviceItem@NM_DiskCalculator@@QAEAAU01@ABU01@@Z 0044afa0 f i DeviceAddPage.obj
 0001:0004a0a0       ?alignment@?$QMap@_JPAVDeviceItemWidget@NM_DiskCalculator@@@@CAHXZ 0044b0a0 f i DeviceAddPage.obj
 0001:0004a0e0       ??0iterator@?$QMap@_JPAVDeviceItemWidget@NM_DiskCalculator@@@@QAE@PAUNode@QMapData@@@Z 0044b0e0 f i DeviceAddPage.obj
 0001:0004a100       ??4?$QMap@_JPAVDeviceItemWidget@NM_DiskCalculator@@@@QAEAAV0@ABV0@@Z 0044b100 f i DeviceAddPage.obj
 0001:0004a1a0       ?findNode@?$QMap@_JPAVDeviceItemWidget@NM_DiskCalculator@@@@ABEPAUNode@QMapData@@AB_J@Z 0044b1a0 f i DeviceAddPage.obj
 0001:0004a280       ?mutableFindNode@?$QMap@_JPAVDeviceItemWidget@NM_DiskCalculator@@@@ABEPAUNode@QMapData@@QAPAU23@AB_J@Z 0044b280 f i DeviceAddPage.obj
 0001:0004a370       ?node_create@?$QMap@_JPAVDeviceItemWidget@NM_DiskCalculator@@@@AAEPAUNode@QMapData@@PAU3@QAPAU23@AB_JABQAVDeviceItemWidget@NM_DiskCalculator@@@Z 0044b370 f i DeviceAddPage.obj
 0001:0004a500       ??$qMapLessThanKey@_J@@YA_NAB_J0@Z 0044b500 f i DeviceAddPage.obj
 0001:0004a560       ?mutableFindNode@?$QMap@_JUStructDeviceItem@NM_DiskCalculator@@@@ABEPAUNode@QMapData@@QAPAU23@AB_J@Z 0044b560 f i DeviceAddPage.obj
 0001:0004a650       ??_EDeviceAddPage@@W7AEPAXI@Z 0044b650 f i DeviceAddPage.obj
 0001:0004a660       ??8@YA_NPBDABVQString@@@Z  0044b660 f i DeviceAddPage.obj
 0001:0004a680       ?qStringComparisonHelper@@YA_NABVQString@@PBD@Z 0044b680 f i DeviceAddPage.obj
 0001:0004a750       ?ceil@@YAMM@Z              0044b750 f i DeviceAddPage.obj
 0001:0004a770       _ceilf                     0044b770 f i DeviceAddPage.obj
 0001:0004a7a0       ??0DeviceItemWidget@NM_DiskCalculator@@QAE@PAVQWidget@@VQString@@11@Z 0044b7a0 f   DeviceItemWidget.obj
 0001:0004aad0       ?OnDeleteButtonClicked@DeviceItemWidget@NM_DiskCalculator@@AAEXXZ 0044bad0 f   DeviceItemWidget.obj
 0001:0004ab20       ?geteElidedText@DeviceItemWidget@NM_DiskCalculator@@AAE?AVQString@@VQFont@@V3@H@Z 0044bb20 f   DeviceItemWidget.obj
 0001:0004ac20       ?setData@DeviceItemWidget@NM_DiskCalculator@@QAEXHVQString@@0NHH00@Z 0044bc20 f   DeviceItemWidget.obj
 0001:0004bd50       ?setData@DeviceItemWidget@NM_DiskCalculator@@QAEXVQString@@@Z 0044cd50 f   DeviceItemWidget.obj
 0001:0004be30       ?setFrameRate@DeviceItemWidget@NM_DiskCalculator@@QAEXABVQString@@N@Z 0044ce30 f   DeviceItemWidget.obj
 0001:0004bfc0       ?relayoutUI@DeviceItemWidget@NM_DiskCalculator@@QAEXH@Z 0044cfc0 f   DeviceItemWidget.obj
 0001:0004c450       ?resizeEvent@DeviceItemWidget@NM_DiskCalculator@@EAEXPAVQResizeEvent@@@Z 0044d450 f   DeviceItemWidget.obj
 0001:0004c490       ??1DeviceItemWidget@NM_DiskCalculator@@UAE@XZ 0044d490 f   DeviceItemWidget.obj
 0001:0004ccc0       ?tr@DeviceItemWidget@NM_DiskCalculator@@SA?AVQString@@PBD0@Z 0044dcc0 f i DeviceItemWidget.obj
 0001:0004cd00       ?setupUi@Ui_DeviceItemWidget@@QAEXPAVQWidget@@@Z 0044dd00 f i DeviceItemWidget.obj
 0001:0004f690       ?retranslateUi@Ui_DeviceItemWidget@@QAEXPAVQWidget@@@Z 00450690 f i DeviceItemWidget.obj
 0001:0004faa0       ??_GQToolButton@@UAEPAXI@Z 00450aa0 f i DeviceItemWidget.obj
 0001:0004faa0       ??_EQToolButton@@UAEPAXI@Z 00450aa0 f i DeviceItemWidget.obj
 0001:0004fae0       ??_GDeviceItemWidget@NM_DiskCalculator@@UAEPAXI@Z 00450ae0 f i DeviceItemWidget.obj
 0001:0004fae0       ??_EDeviceItemWidget@NM_DiskCalculator@@UAEPAXI@Z 00450ae0 f i DeviceItemWidget.obj
 0001:0004fb20       ??_EDeviceItemWidget@NM_DiskCalculator@@W7AEPAXI@Z 00450b20 f i DeviceItemWidget.obj
 0001:0004fb30       ??_EQToolButton@@W7AEPAXI@Z 00450b30 f i DeviceItemWidget.obj
 0001:0004fb40       ??0ButtonRadio@aptui@@QAE@PAVQWidget@@@Z 00450b40 f   ButtonRadio.obj
 0001:0004fb70       ??1ButtonRadio@aptui@@UAE@XZ 00450b70 f   ButtonRadio.obj
 0001:0004fbb0       ??_GButtonRadio@aptui@@UAEPAXI@Z 00450bb0 f i ButtonRadio.obj
 0001:0004fbb0       ??_EButtonRadio@aptui@@UAEPAXI@Z 00450bb0 f i ButtonRadio.obj
 0001:0004fbf0       ??_EButtonRadio@aptui@@W7AEPAXI@Z 00450bf0 f i ButtonRadio.obj
 0001:0004fc00       ??0UpdateDialog@@QAE@PAVQWidget@@@Z 00450c00 f   UpdateDialog.obj
 0001:0004fe40       ?setMethodResultDisplay@UpdateDialog@@QAEXW4Methods@1@_N@Z 00450e40 f   UpdateDialog.obj
 0001:00050410       ??1UpdateDialog@@UAE@XZ    00451410 f   UpdateDialog.obj
 0001:00050490       ?onExportTemplate@UpdateDialog@@AAEXXZ 00451490 f   UpdateDialog.obj
 0001:00050740       ?onImportScene@UpdateDialog@@AAEXXZ 00451740 f   UpdateDialog.obj
 0001:000510a0       ?tr@UpdateDialog@@SA?AVQString@@PBD0@Z 004520a0 f i UpdateDialog.obj
 0001:000510e0       ?setupUi@Ui_UpdateDialog@@QAEXPAVQWidget@@@Z 004520e0 f i UpdateDialog.obj
 0001:00052930       ?retranslateUi@Ui_UpdateDialog@@QAEXPAVQWidget@@@Z 00453930 f i UpdateDialog.obj
 0001:00052bf0       ??_EUpdateDialog@@UAEPAXI@Z 00453bf0 f i UpdateDialog.obj
 0001:00052bf0       ??_GUpdateDialog@@UAEPAXI@Z 00453bf0 f i UpdateDialog.obj
 0001:00052c30       ??$DELETE_OBJECT@PAVUi_UpdateDialog@@@NM_SHARE_TOOL@@YAXAAPAVUi_UpdateDialog@@@Z 00453c30 f i UpdateDialog.obj
 0001:00052c70       ??$DELETE_OBJECT@PAVQWidget@@@NM_SHARE_TOOL@@YAXAAPAVQWidget@@@Z 00453c70 f i UpdateDialog.obj
 0001:00052cd0       ??_EUpdateDialog@@W7AEPAXI@Z 00453cd0 f i UpdateDialog.obj
 0001:00052ce0       ??0WarningDialog@NM_DiskCalculator@@QAE@XZ 00453ce0 f   WarningDialog.obj
 0001:00052dc0       ??0WarningDialog@NM_DiskCalculator@@QAE@W4PictureType@01@ABVQString@@@Z 00453dc0 f   WarningDialog.obj
 0001:00052eb0       ??1WarningDialog@NM_DiskCalculator@@UAE@XZ 00453eb0 f   WarningDialog.obj
 0001:00052ee0       ?onBtnClose@WarningDialog@NM_DiskCalculator@@AAEXXZ 00453ee0 f   WarningDialog.obj
 0001:00052f00       ?setText@WarningDialog@NM_DiskCalculator@@QAEXW4PictureType@12@ABVQString@@@Z 00453f00 f   WarningDialog.obj
 0001:00053200       ?showWarningDialog@WarningDialog@NM_DiskCalculator@@SAXABVQPoint@@W4PictureType@12@ABVQString@@@Z 00454200 f   WarningDialog.obj
 0001:00053270       ?showBigWarningDialog@WarningDialog@NM_DiskCalculator@@SAXABVQPoint@@W4PictureType@12@ABVQString@@@Z 00454270 f   WarningDialog.obj
 0001:00053300       ?timerEvent@WarningDialog@NM_DiskCalculator@@MAEXPAVQTimerEvent@@@Z 00454300 f   WarningDialog.obj
 0001:000534b0       ?setupUi@Ui_WarningDialog@@QAEXPAVQWidget@@@Z 004544b0 f i WarningDialog.obj
 0001:000544c0       ?retranslateUi@Ui_WarningDialog@@QAEXPAVQWidget@@@Z 004554c0 f i WarningDialog.obj
 0001:00054640       ??_EWarningDialog@NM_DiskCalculator@@UAEPAXI@Z 00455640 f i WarningDialog.obj
 0001:00054640       ??_GWarningDialog@NM_DiskCalculator@@UAEPAXI@Z 00455640 f i WarningDialog.obj
 0001:00054680       ??_EWarningDialog@NM_DiskCalculator@@W7AEPAXI@Z 00455680 f i WarningDialog.obj
 0001:00054690       ??0TipDialog@NM_DiskCalculator@@QAE@PAVQWidget@@@Z 00455690 f   TipDialog.obj
 0001:000547a0       ??1TipDialog@NM_DiskCalculator@@UAE@XZ 004557a0 f   TipDialog.obj
 0001:000547d0       ?setTip@TipDialog@NM_DiskCalculator@@QAEXABVQString@@@Z 004557d0 f   TipDialog.obj
 0001:00054850       ?setupUi@Ui_TipDialog@@QAEXPAVQWidget@@@Z 00455850 f i TipDialog.obj
 0001:00054c80       ?retranslateUi@Ui_TipDialog@@QAEXPAVQWidget@@@Z 00455c80 f i TipDialog.obj
 0001:00054d80       ??_GTipDialog@NM_DiskCalculator@@UAEPAXI@Z 00455d80 f i TipDialog.obj
 0001:00054d80       ??_ETipDialog@NM_DiskCalculator@@UAEPAXI@Z 00455d80 f i TipDialog.obj
 0001:00054dc0       ??_ETipDialog@NM_DiskCalculator@@W7AEPAXI@Z 00455dc0 f i TipDialog.obj
 0001:00054dd0       ??0BaseTitle@aptui@@QAE@_N0000PAVQWidget@@@Z 00455dd0 f   BaseTitle.obj
 0001:00055050       ?setAppButtonShow@BaseTitle@aptui@@QAEX_N@Z 00456050 f   BaseTitle.obj
 0001:00055090       ?setOptionButtonShow@BaseTitle@aptui@@QAEX_N@Z 00456090 f   BaseTitle.obj
 0001:000550d0       ?setMinButtonShow@BaseTitle@aptui@@QAEX_N@Z 004560d0 f   BaseTitle.obj
 0001:00055110       ?setMaxButtonShow@BaseTitle@aptui@@QAEX_N@Z 00456110 f   BaseTitle.obj
 0001:00055150       ?setCloseButtonShow@BaseTitle@aptui@@QAEX_N@Z 00456150 f   BaseTitle.obj
 0001:00055190       ?addCustomButton@BaseTitle@aptui@@QAEXPAVQAbstractButton@@@Z 00456190 f   BaseTitle.obj
 0001:000551c0       ?setTitle@BaseTitle@aptui@@QAEXABVQString@@@Z 004561c0 f   BaseTitle.obj
 0001:000551e0       ?setTitleIcon@BaseTitle@aptui@@QAEXABVQIcon@@@Z 004561e0 f   BaseTitle.obj
 0001:00055200       ?clearLayout@BaseTitle@aptui@@AAEXPAVQBoxLayout@@@Z 00456200 f   BaseTitle.obj
 0001:00055270       ??1BaseTitle@aptui@@UAE@XZ 00456270 f   BaseTitle.obj
 0001:00055450       ?setupUi@Ui_BaseTitle@@QAEXPAVQWidget@@@Z 00456450 f i BaseTitle.obj
 0001:00056210       ?retranslateUi@Ui_BaseTitle@@QAEXPAVQWidget@@@Z 00457210 f i BaseTitle.obj
 0001:00056460       ??_GBaseTitle@aptui@@UAEPAXI@Z 00457460 f i BaseTitle.obj
 0001:00056460       ??_EBaseTitle@aptui@@UAEPAXI@Z 00457460 f i BaseTitle.obj
 0001:000564a0       ??_EBaseTitle@aptui@@W7AEPAXI@Z 004574a0 f i BaseTitle.obj
 0001:000564b0       ??_EBaseTitle@aptui@@WBE@AEPAXI@Z 004574b0 f i BaseTitle.obj
 0001:000564c0       ??0WindowTitle@aptui@@QAE@PAVQWidget@@@Z 004574c0 f   WindowTitle.obj
 0001:000565f0       ??1WindowTitle@aptui@@UAE@XZ 004575f0 f   WindowTitle.obj
 0001:000567f0       ?setAppIcon@WindowTitle@aptui@@QAEXABVQIcon@@@Z 004577f0 f   WindowTitle.obj
 0001:00056810       ?setAppTitle@WindowTitle@aptui@@QAEXABVQString@@@Z 00457810 f   WindowTitle.obj
 0001:00056830       ?initTitle@WindowTitle@aptui@@AAEXXZ 00457830 f   WindowTitle.obj
 0001:000571c0       ?minimizeWindow@WindowTitle@aptui@@AAEXXZ 004581c0 f   WindowTitle.obj
 0001:000571f0       ?closeWindow@WindowTitle@aptui@@AAEXXZ 004581f0 f   WindowTitle.obj
 0001:00057230       ?maxOrRestoreWindow@WindowTitle@aptui@@AAEXXZ 00458230 f   WindowTitle.obj
 0001:00057380       ?mouseDoubleClickEvent@WindowTitle@aptui@@EAEXPAVQMouseEvent@@@Z 00458380 f   WindowTitle.obj
 0001:00057400       ?displaySyetemMenu@WindowTitle@aptui@@AAEXXZ 00458400 f   WindowTitle.obj
 0001:000577f0       ??_GWindowTitle@aptui@@UAEPAXI@Z 004587f0 f i WindowTitle.obj
 0001:000577f0       ??_EWindowTitle@aptui@@UAEPAXI@Z 004587f0 f i WindowTitle.obj
 0001:00057830       ??_GCHBoxLayout@iVMSGUIToolkit@@UAEPAXI@Z 00458830 f i WindowTitle.obj
 0001:00057830       ??_ECHBoxLayout@iVMSGUIToolkit@@UAEPAXI@Z 00458830 f i WindowTitle.obj
 0001:00057870       ??_ECWidgetItem@iVMSGUIToolkit@@UAEPAXI@Z 00458870 f i WindowTitle.obj
 0001:00057870       ??_GCWidgetItem@iVMSGUIToolkit@@UAEPAXI@Z 00458870 f i WindowTitle.obj
 0001:000578b0       ??_ECHBoxLayout@iVMSGUIToolkit@@W7AEPAXI@Z 004588b0 f i WindowTitle.obj
 0001:000578c0       ??_EWindowTitle@aptui@@W7AEPAXI@Z 004588c0 f i WindowTitle.obj
 0001:000578d0       ??_EWindowTitle@aptui@@WBE@AEPAXI@Z 004588d0 f i WindowTitle.obj
 0001:000578e0       ??0Menu@aptui@@QAE@ABVQString@@PAVQWidget@@@Z 004588e0 f   Menu.obj
 0001:00057960       ??0Menu@aptui@@QAE@PAVQWidget@@@Z 00458960 f   Menu.obj
 0001:000579d0       ??1Menu@aptui@@UAE@XZ      004589d0 f   Menu.obj
 0001:00057a00       ?event@Menu@aptui@@MAE_NPAVQEvent@@@Z 00458a00 f   Menu.obj
 0001:00057a90       ?addMenu@Menu@aptui@@QAEPAVQAction@@PAV12@@Z 00458a90 f   Menu.obj
 0001:00057ab0       ?addMenu@Menu@aptui@@QAEPAV12@ABVQString@@@Z 00458ab0 f   Menu.obj
 0001:00057b50       ?addMenu@Menu@aptui@@QAEPAV12@ABVQIcon@@ABVQString@@@Z 00458b50 f   Menu.obj
 0001:00057c00       ?Init@Menu@aptui@@AAEXXZ   00458c00 f   Menu.obj
 0001:00057ca0       ?_DrawNinePatch@aptui@@YA?BVQPixmap@@VQSize@@ABV2@@Z 00458ca0 f   Menu.obj
 0001:000582b0       ??0CCustomStyle@Menu@aptui@@QAE@PAVQStyle@@@Z 004592b0 f   Menu.obj
 0001:00058360       ?drawPrimitive@CCustomStyle@Menu@aptui@@UBEXW4PrimitiveElement@QStyle@@PBVQStyleOption@@PAVQPainter@@PBVQWidget@@@Z 00459360 f   Menu.obj
 0001:000584e0       ?pixelMetric@CCustomStyle@Menu@aptui@@UBEHW4PixelMetric@QStyle@@PBVQStyleOption@@PBVQWidget@@@Z 004594e0 f   Menu.obj
 0001:00058520       ?drawControl@CCustomStyle@Menu@aptui@@UBEXW4ControlElement@QStyle@@PBVQStyleOption@@PAVQPainter@@PBVQWidget@@@Z 00459520 f   Menu.obj
 0001:00058580       ?_DrawMenuItem@CCustomStyle@Menu@aptui@@EBEXPBVQStyleOption@@PAVQPainter@@PBVQWidget@@@Z 00459580 f   Menu.obj
 0001:00059f20       ??_GMenu@aptui@@UAEPAXI@Z  0045af20 f i Menu.obj
 0001:00059f20       ??_EMenu@aptui@@UAEPAXI@Z  0045af20 f i Menu.obj
 0001:00059f60       ??_GCCustomStyle@Menu@aptui@@UAEPAXI@Z 0045af60 f i Menu.obj
 0001:00059f60       ??_ECCustomStyle@Menu@aptui@@UAEPAXI@Z 0045af60 f i Menu.obj
 0001:00059fa0       ??1CCustomStyle@Menu@aptui@@UAE@XZ 0045afa0 f i Menu.obj
 0001:0005a010       ??4?$QFlags@W4StateFlag@QStyle@@@@QAEAAV0@ABV0@@Z 0045b010 f i Menu.obj
 0001:0005a030       ??_5?$QFlags@W4StateFlag@QStyle@@@@QAEAAV0@W4StateFlag@QStyle@@@Z 0045b030 f i Menu.obj
 0001:0005a060       ??B?$QFlags@W4StateFlag@QStyle@@@@QBEHXZ 0045b060 f i Menu.obj
 0001:0005a080       ??I?$QFlags@W4StateFlag@QStyle@@@@QBE?AV0@W4StateFlag@QStyle@@@Z 0045b080 f i Menu.obj
 0001:0005a0b0       ??7?$QFlags@W4StateFlag@QStyle@@@@QBE_NXZ 0045b0b0 f i Menu.obj
 0001:0005a0d0       ??$qstyleoption_cast@PBVQStyleOptionMenuItem@@@@YAPBVQStyleOptionMenuItem@@PBVQStyleOption@@@Z 0045b0d0 f i Menu.obj
 0001:0005a110       ??$qobject_cast@PBVQComboBox@@@@YAPBVQComboBox@@PBVQObject@@@Z 0045b110 f i Menu.obj
 0001:0005a140       ??$qt_check_for_QOBJECT_macro@VQComboBox@@@QComboBox@@QBEXABV0@@Z 0045b140 f i Menu.obj
 0001:0005a180       ??$qYouForgotTheQ_OBJECT_Macro@PBVQComboBox@@@@YAHPBVQComboBox@@0@Z 0045b180 f i Menu.obj
 0001:0005a190       ??_EMenu@aptui@@W7AEPAXI@Z 0045b190 f i Menu.obj
 0001:0005a1a0       ??U@YA?AVQIncompatibleFlag@@W4AlignmentFlag@Qt@@H@Z 0045b1a0 f i Menu.obj
 0001:0005a1c0       ??B?$QFlags@W4AlignmentFlag@Qt@@@@QBEHXZ 0045b1c0 f i Menu.obj
 0001:0005a1e0       ??0?$QFlags@W4StateFlag@QStyle@@@@QAE@W4StateFlag@QStyle@@@Z 0045b1e0 f i Menu.obj
 0001:0005a200       ??0SystemMenu@aptui@@QAE@PAVQWidget@@@Z 0045b200 f   TitleMenu.obj
 0001:0005a230       ??1SystemMenu@aptui@@UAE@XZ 0045b230 f   TitleMenu.obj
 0001:0005a260       ?openUserManual@SystemMenu@aptui@@AAEXXZ 0045b260 f   TitleMenu.obj
 0001:0005a270       ?updateData@SystemMenu@aptui@@AAEXXZ 0045b270 f   TitleMenu.obj
 0001:0005a280       ?settings@SystemMenu@aptui@@AAEXXZ 0045b280 f   TitleMenu.obj
 0001:0005a290       ?about@SystemMenu@aptui@@AAEXXZ 0045b290 f   TitleMenu.obj
 0001:0005a2a0       ?getHelp@SystemMenu@aptui@@AAE_NXZ 0045b2a0 f   TitleMenu.obj
 0001:0005a2e0       ??_ESystemMenu@aptui@@UAEPAXI@Z 0045b2e0 f i TitleMenu.obj
 0001:0005a2e0       ??_GSystemMenu@aptui@@UAEPAXI@Z 0045b2e0 f i TitleMenu.obj
 0001:0005a320       ??_ESystemMenu@aptui@@W7AEPAXI@Z 0045b320 f i TitleMenu.obj
 0001:0005a330       ??0LineEditInterger@aptui@@QAE@PAVQWidget@@@Z 0045b330 f   LineEditInterger.obj
 0001:0005a360       ??1LineEditInterger@aptui@@UAE@XZ 0045b360 f   LineEditInterger.obj
 0001:0005a3a0       ??_ELineEditInterger@aptui@@UAEPAXI@Z 0045b3a0 f i LineEditInterger.obj
 0001:0005a3a0       ??_GLineEditInterger@aptui@@UAEPAXI@Z 0045b3a0 f i LineEditInterger.obj
 0001:0005a3e0       ??_ELineEditInterger@aptui@@W7AEPAXI@Z 0045b3e0 f i LineEditInterger.obj
 0001:0005a3f0       ??0TabWidget@aptui@@QAE@PAVQWidget@@@Z 0045b3f0 f   TabWidget.obj
 0001:0005a4f0       ?setObjectName@TabWidget@aptui@@QAEXABVQString@@@Z 0045b4f0 f   TabWidget.obj
 0001:0005a580       ?resizeEvent@TabWidget@aptui@@EAEXPAVQResizeEvent@@@Z 0045b580 f   TabWidget.obj
 0001:0005a5a0       ??1TabWidget@aptui@@UAE@XZ 0045b5a0 f   TabWidget.obj
 0001:0005a640       ??_GTabWidget@aptui@@UAEPAXI@Z 0045b640 f i TabWidget.obj
 0001:0005a640       ??_ETabWidget@aptui@@UAEPAXI@Z 0045b640 f i TabWidget.obj
 0001:0005a680       ??_ETabWidget@aptui@@W7AEPAXI@Z 0045b680 f i TabWidget.obj
 0001:0005a690       ??0Line@aptui@@QAE@PAVQWidget@@V?$QFlags@W4WindowType@Qt@@@@@Z 0045b690 f   Line.obj
 0001:0005a6e0       ??1Line@aptui@@UAE@XZ      0045b6e0 f   Line.obj
 0001:0005a730       ??_GLine@aptui@@UAEPAXI@Z  0045b730 f i Line.obj
 0001:0005a730       ??_ELine@aptui@@UAEPAXI@Z  0045b730 f i Line.obj
 0001:0005a770       ??_ELine@aptui@@W7AEPAXI@Z 0045b770 f i Line.obj
 0001:0005a780       ??0?$QFlags@W4WindowType@Qt@@@@QAE@ABV0@@Z 0045b780 f i Line.obj
 0001:0005a7a0       ?GetBuildDate@aptui@@YAKXZ 0045b7a0 f   DlgAbout.obj
 0001:0005aac0       ??0CDlgAbout@aptui@@QAE@PAVQObject@@@Z 0045bac0 f   DlgAbout.obj
 0001:0005adc0       ?SetNameValue@CDlgAbout@aptui@@QAEXABVQString@@@Z 0045bdc0 f   DlgAbout.obj
 0001:0005ae70       ?SetVersionValue@CDlgAbout@aptui@@QAEXABVQString@@@Z 0045be70 f   DlgAbout.obj
 0001:0005af20       ?SetBtn1Text@CDlgAbout@aptui@@QAEXABVQString@@@Z 0045bf20 f   DlgAbout.obj
 0001:0005af40       ?SetBtn2Text@CDlgAbout@aptui@@QAEXABVQString@@@Z 0045bf40 f   DlgAbout.obj
 0001:0005af60       ?setConerText@CDlgAbout@aptui@@QAEXABVQString@@@Z 0045bf60 f   DlgAbout.obj
 0001:0005af80       ?setBtn1Visible@CDlgAbout@aptui@@QAEX_N@Z 0045bf80 f   DlgAbout.obj
 0001:0005b040       ?setBtn2Visible@CDlgAbout@aptui@@QAEX_N@Z 0045c040 f   DlgAbout.obj
 0001:0005b100       ?setConerBtnVisible@CDlgAbout@aptui@@QAEX_N@Z 0045c100 f   DlgAbout.obj
 0001:0005b130       ?setBottomBtnsVisible@CDlgAbout@aptui@@QAEX_N@Z 0045c130 f   DlgAbout.obj
 0001:0005b1c0       ?focusOutEvent@CDlgAbout@aptui@@EAEXPAVQFocusEvent@@@Z 0045c1c0 f   DlgAbout.obj
 0001:0005b1d0       ??1CDlgAbout@aptui@@UAE@XZ 0045c1d0 f   DlgAbout.obj
 0001:0005b550       ?tr@CDlgAbout@aptui@@SA?AVQString@@PBD0@Z 0045c550 f i DlgAbout.obj
 0001:0005b590       ?setupUi@Ui_AboutClass@@QAEXPAVQWidget@@@Z 0045c590 f i DlgAbout.obj
 0001:0005d5b0       ?retranslateUi@Ui_AboutClass@@QAEXPAVQWidget@@@Z 0045e5b0 f i DlgAbout.obj
 0001:0005d870       ??_GCDlgAbout@aptui@@UAEPAXI@Z 0045e870 f i DlgAbout.obj
 0001:0005d870       ??_ECDlgAbout@aptui@@UAEPAXI@Z 0045e870 f i DlgAbout.obj
 0001:0005d8b0       ??0Switch@aptui@@QAE@_NPAVQWidget@@@Z 0045e8b0 f   Switch.obj
 0001:0005d9c0       ?initUI@Switch@aptui@@AAEXXZ 0045e9c0 f   Switch.obj
 0001:0005dd50       ?retranslateUi@Switch@aptui@@AAEXXZ 0045ed50 f   Switch.obj
 0001:0005de00       ?setSwitch@Switch@aptui@@QAEX_N@Z 0045ee00 f   Switch.obj
 0001:0005e020       ?switchOn@Switch@aptui@@QAEXXZ 0045f020 f   Switch.obj
 0001:0005e040       ?switchOff@Switch@aptui@@QAEXXZ 0045f040 f   Switch.obj
 0001:0005e060       ?onBtnsToggled@Switch@aptui@@AAEX_N@Z 0045f060 f   Switch.obj
 0001:0005e0b0       ?setOnText@Switch@aptui@@QAEXABVQString@@@Z 0045f0b0 f   Switch.obj
 0001:0005e0d0       ?setOffText@Switch@aptui@@QAEXABVQString@@@Z 0045f0d0 f   Switch.obj
 0001:0005e0f0       ?setOnIcon@Switch@aptui@@QAEXABVQIcon@@H@Z 0045f0f0 f   Switch.obj
 0001:0005e130       ?setOffIcon@Switch@aptui@@QAEXABVQIcon@@H@Z 0045f130 f   Switch.obj
 0001:0005e170       ?checked@Switch@aptui@@AAE?AVQString@@XZ 0045f170 f   Switch.obj
 0001:0005e210       ?setChecked@Switch@aptui@@AAEXVQString@@@Z 0045f210 f   Switch.obj
 0001:0005e320       ?resizeEvent@Switch@aptui@@MAEXPAVQResizeEvent@@@Z 0045f320 f   Switch.obj
 0001:0005e380       ??1Switch@aptui@@UAE@XZ    0045f380 f   Switch.obj
 0001:0005e7b0       ??_GSwitch@aptui@@UAEPAXI@Z 0045f7b0 f i Switch.obj
 0001:0005e7b0       ??_ESwitch@aptui@@UAEPAXI@Z 0045f7b0 f i Switch.obj
 0001:0005e7f0       ??_ESwitch@aptui@@W7AEPAXI@Z 0045f7f0 f i Switch.obj
 0001:0005e800       ??0CoverWidget@aptui@@QAE@PAVQWidget@@@Z 0045f800 f   CoverWidget.obj
 0001:0005e9c0       ??1CoverWidget@aptui@@UAE@XZ 0045f9c0 f   CoverWidget.obj
 0001:0005eb50       ??_GCoverWidget@aptui@@UAEPAXI@Z 0045fb50 f i CoverWidget.obj
 0001:0005eb50       ??_ECoverWidget@aptui@@UAEPAXI@Z 0045fb50 f i CoverWidget.obj
 0001:0005eb90       ??_ECoverWidget@aptui@@W7AEPAXI@Z 0045fb90 f i CoverWidget.obj
 0001:0005eba0       ??0Widget@aptui@@QAE@PAVQWidget@@@Z 0045fba0 f   Widget.obj
 0001:0005ebe0       ?paintEvent@Widget@aptui@@MAEXPAVQPaintEvent@@@Z 0045fbe0 f   Widget.obj
 0001:0005ecc0       ?event@Widget@aptui@@MAE_NPAVQEvent@@@Z 0045fcc0 f   Widget.obj
 0001:0005ed50       ??1Widget@aptui@@UAE@XZ    0045fd50 f   Widget.obj
 0001:0005edf0       ??_GWidget@aptui@@UAEPAXI@Z 0045fdf0 f i Widget.obj
 0001:0005edf0       ??_EWidget@aptui@@UAEPAXI@Z 0045fdf0 f i Widget.obj
 0001:0005ee30       ??_EWidget@aptui@@W7AEPAXI@Z 0045fe30 f i Widget.obj
 0001:0005ee40       ??0MultiStatePushButton@aptui@@QAE@PAVQWidget@@@Z 0045fe40 f   MultiStatePushButton.obj
 0001:0005f040       ?setButtonState@MultiStatePushButton@aptui@@QAEXW4State@12@@Z 00460040 f   MultiStatePushButton.obj
 0001:0005f100       ?state@MultiStatePushButton@aptui@@AAE?AVQString@@XZ 00460100 f   MultiStatePushButton.obj
 0001:0005f140       ?setState@MultiStatePushButton@aptui@@AAEXVQString@@@Z 00460140 f   MultiStatePushButton.obj
 0001:0005f210       ?getStringFromEnum@MultiStatePushButton@aptui@@AAE?AVQString@@W4State@12@@Z 00460210 f   MultiStatePushButton.obj
 0001:0005f290       ?paintEvent@MultiStatePushButton@aptui@@MAEXPAVQPaintEvent@@@Z 00460290 f   MultiStatePushButton.obj
 0001:0005f2b0       ??1MultiStatePushButton@aptui@@UAE@XZ 004602b0 f   MultiStatePushButton.obj
 0001:0005f450       ??_GMultiStatePushButton@aptui@@UAEPAXI@Z 00460450 f i MultiStatePushButton.obj
 0001:0005f450       ??_EMultiStatePushButton@aptui@@UAEPAXI@Z 00460450 f i MultiStatePushButton.obj
 0001:0005f490       ??0?$QMap@VQString@@W4State@MultiStatePushButton@aptui@@@@QAE@XZ 00460490 f i MultiStatePushButton.obj
 0001:0005f4c0       ??1?$QMap@VQString@@W4State@MultiStatePushButton@aptui@@@@QAE@XZ 004604c0 f i MultiStatePushButton.obj
 0001:0005f510       ?contains@?$QMap@VQString@@W4State@MultiStatePushButton@aptui@@@@QBE_NABVQString@@@Z 00460510 f i MultiStatePushButton.obj
 0001:0005f540       ?value@?$QMap@VQString@@W4State@MultiStatePushButton@aptui@@@@QBE?BW4State@MultiStatePushButton@aptui@@ABVQString@@@Z 00460540 f i MultiStatePushButton.obj
 0001:0005f5a0       ?insert@?$QMap@VQString@@W4State@MultiStatePushButton@aptui@@@@QAE?AViterator@1@ABVQString@@ABW4State@MultiStatePushButton@aptui@@@Z 004605a0 f i MultiStatePushButton.obj
 0001:0005f640       ?freeData@?$QMap@VQString@@W4State@MultiStatePushButton@aptui@@@@AAEXPAUQMapData@@@Z 00460640 f i MultiStatePushButton.obj
 0001:0005f6d0       ??$qRegisterMetaType@W4State@MultiStatePushButton@aptui@@@@YAHPBDPAW4State@MultiStatePushButton@aptui@@@Z 004606d0 f i MultiStatePushButton.obj
 0001:0005f750       ?payload@?$QMap@VQString@@W4State@MultiStatePushButton@aptui@@@@CAHXZ 00460750 f i MultiStatePushButton.obj
 0001:0005f760       ?concrete@?$QMap@VQString@@W4State@MultiStatePushButton@aptui@@@@CAPAU?$QMapNode@VQString@@W4State@MultiStatePushButton@aptui@@@@PAUNode@QMapData@@@Z 00460760 f i MultiStatePushButton.obj
 0001:0005f780       ?detach@?$QMap@VQString@@W4State@MultiStatePushButton@aptui@@@@QAEXXZ 00460780 f i MultiStatePushButton.obj
 0001:0005f7c0       ??0iterator@?$QMap@VQString@@W4State@MultiStatePushButton@aptui@@@@QAE@PAUNode@QMapData@@@Z 004607c0 f i MultiStatePushButton.obj
 0001:0005f7e0       ?qt_metatype_id@?$QMetaTypeIdHelper@W4State@MultiStatePushButton@aptui@@$0A@@QtPrivate@@SAHXZ 004607e0 f i MultiStatePushButton.obj
 0001:0005f7f0       ?detach_helper@?$QMap@VQString@@W4State@MultiStatePushButton@aptui@@@@AAEXXZ 004607f0 f i MultiStatePushButton.obj
 0001:0005f970       ?findNode@?$QMap@VQString@@W4State@MultiStatePushButton@aptui@@@@ABEPAUNode@QMapData@@ABVQString@@@Z 00460970 f i MultiStatePushButton.obj
 0001:0005fa50       ?mutableFindNode@?$QMap@VQString@@W4State@MultiStatePushButton@aptui@@@@ABEPAUNode@QMapData@@QAPAU23@ABVQString@@@Z 00460a50 f i MultiStatePushButton.obj
 0001:0005fb40       ?node_create@?$QMap@VQString@@W4State@MultiStatePushButton@aptui@@@@AAEPAUNode@QMapData@@PAU3@QAPAU23@ABVQString@@ABW4State@MultiStatePushButton@aptui@@@Z 00460b40 f i MultiStatePushButton.obj
 0001:0005fcf0       ??$qMetaTypeConstructHelper@W4State@MultiStatePushButton@aptui@@@@YAPAXPBW4State@MultiStatePushButton@aptui@@@Z 00460cf0 f i MultiStatePushButton.obj
 0001:0005fd80       ??$qMetaTypeDeleteHelper@W4State@MultiStatePushButton@aptui@@@@YAXPAW4State@MultiStatePushButton@aptui@@@Z 00460d80 f i MultiStatePushButton.obj
 0001:0005fda0       ?alignment@?$QMap@VQString@@W4State@MultiStatePushButton@aptui@@@@CAHXZ 00460da0 f i MultiStatePushButton.obj
 0001:0005fde0       ??_EMultiStatePushButton@aptui@@W7AEPAXI@Z 00460de0 f i MultiStatePushButton.obj
 0001:0005fdf0       ??0BaseDialog@aptui@@QAE@_N000000PAVQWidget@@@Z 00460df0 f   BaseDialog.obj
 0001:0005ffd0       ?InitUI@BaseDialog@aptui@@AAEXXZ 00460fd0 f   BaseDialog.obj
 0001:00060150       ?restoreWindow@BaseDialog@aptui@@AAEXXZ 00461150 f   BaseDialog.obj
 0001:00060180       ?setConfirmBtnBehavior@BaseDialog@aptui@@QAEX_N@Z 00461180 f   BaseDialog.obj
 0001:000601a0       ?setCancelBtnBehavior@BaseDialog@aptui@@QAEX_N@Z 004611a0 f   BaseDialog.obj
 0001:000601c0       ?setMinBtnBehavior@BaseDialog@aptui@@QAEX_N@Z 004611c0 f   BaseDialog.obj
 0001:00060230       ?setMaxBtnBehavior@BaseDialog@aptui@@QAEX_N@Z 00461230 f   BaseDialog.obj
 0001:000602a0       ?setCloseBtnBehavior@BaseDialog@aptui@@QAEX_N@Z 004612a0 f   BaseDialog.obj
 0001:00060310       ?SetFixedSize@BaseDialog@aptui@@QAEXHH@Z 00461310 f   BaseDialog.obj
 0001:00060370       ?SetFixedSize@BaseDialog@aptui@@QAEXABVQSize@@@Z 00461370 f   BaseDialog.obj
 0001:000603a0       ?onConfirmBtnClicked@BaseDialog@aptui@@QAEXXZ 004613a0 f   BaseDialog.obj
 0001:000603d0       ?onCancelBtnClicked@BaseDialog@aptui@@QAEXXZ 004613d0 f   BaseDialog.obj
 0001:00060400       ?setEnableDefaultConnections@BaseDialog@aptui@@QAEX_N0000@Z 00461400 f   BaseDialog.obj
 0001:00060540       ?setTitle@BaseDialog@aptui@@QAEXABVQString@@@Z 00461540 f   BaseDialog.obj
 0001:00060570       ?setDefaultText@BaseDialog@aptui@@QAEXABVQString@@H_N@Z 00461570 f   BaseDialog.obj
 0001:000606d0       ?setDefaultText@BaseDialog@aptui@@QAEXABVQString@@@Z 004616d0 f   BaseDialog.obj
 0001:00060700       ?setConfirmButtonText@BaseDialog@aptui@@QAEXABVQString@@@Z 00461700 f   BaseDialog.obj
 0001:00060720       ?setCancelButtonText@BaseDialog@aptui@@QAEXABVQString@@@Z 00461720 f   BaseDialog.obj
 0001:00060740       ?setBottomBarHeight@BaseDialog@aptui@@QAEXH@Z 00461740 f   BaseDialog.obj
 0001:00060760       ?setBottomVisible@BaseDialog@aptui@@QAEX_N@Z 00461760 f   BaseDialog.obj
 0001:00060790       ?addTitleButton@BaseDialog@aptui@@QAEXPAVQAbstractButton@@@Z 00461790 f   BaseDialog.obj
 0001:000607b0       ?addBottomBarButton@BaseDialog@aptui@@QAEXPAVQAbstractButton@@@Z 004617b0 f   BaseDialog.obj
 0001:000607e0       ?setCenterWidget@BaseDialog@aptui@@QAEXPAVQWidget@@@Z 004617e0 f   BaseDialog.obj
 0001:00060870       ?clearLayout@BaseDialog@aptui@@AAEXPAVQBoxLayout@@@Z 00461870 f   BaseDialog.obj
 0001:000608e0       ??1BaseDialog@aptui@@UAE@XZ 004618e0 f   BaseDialog.obj
 0001:00060cb0       ?setupUi@Ui_BaseDialog@@QAEXPAVQWidget@@@Z 00461cb0 f i BaseDialog.obj
 0001:00061e40       ?retranslateUi@Ui_BaseDialog@@QAEXPAVQWidget@@@Z 00462e40 f i BaseDialog.obj
 0001:00062000       ??_GBaseDialog@aptui@@UAEPAXI@Z 00463000 f i BaseDialog.obj
 0001:00062000       ??_EBaseDialog@aptui@@UAEPAXI@Z 00463000 f i BaseDialog.obj
 0001:00062040       ??_EBaseDialog@aptui@@W7AEPAXI@Z 00463040 f i BaseDialog.obj
 0001:00062050       ??0Label@aptui@@QAE@PAVQWidget@@@Z 00463050 f   Label.obj
 0001:000620f0       ??0Label@aptui@@QAE@ABVQString@@PAVQWidget@@@Z 004630f0 f   Label.obj
 0001:00062190       ??1Label@aptui@@UAE@XZ     00463190 f   Label.obj
 0001:00062210       ?event@Label@aptui@@MAE_NPAVQEvent@@@Z 00463210 f   Label.obj
 0001:000622a0       ?GetText@Label@aptui@@QBE?AVQString@@XZ 004632a0 f   Label.obj
 0001:000622e0       ?SetText@Label@aptui@@QAEXABVQString@@@Z 004632e0 f   Label.obj
 0001:00062370       ?GetPunctuation@Label@aptui@@QBE?AVQString@@XZ 00463370 f   Label.obj
 0001:000623b0       ?SetPunctuation@Label@aptui@@QAEXABVQString@@@Z 004633b0 f   Label.obj
 0001:00062440       ??0EditableLabel@aptui@@QAE@PAVQWidget@@@Z 00463440 f   Label.obj
 0001:000624f0       ?mousePressEvent@EditableLabel@aptui@@MAEXPAVQMouseEvent@@@Z 004634f0 f   Label.obj
 0001:00062560       ?mouseReleaseEvent@EditableLabel@aptui@@MAEXPAVQMouseEvent@@@Z 00463560 f   Label.obj
 0001:000625a0       ?mouseMoveEvent@EditableLabel@aptui@@MAEXPAVQMouseEvent@@@Z 004635a0 f   Label.obj
 0001:00062610       ?paintEvent@EditableLabel@aptui@@MAEXPAVQPaintEvent@@@Z 00463610 f   Label.obj
 0001:00062730       ?enterEvent@EditableLabel@aptui@@MAEXPAVQEvent@@@Z 00463730 f   Label.obj
 0001:00062810       ?leaveEvent@EditableLabel@aptui@@MAEXPAVQEvent@@@Z 00463810 f   Label.obj
 0001:00062890       ?OnPreviewChanged@EditableLabel@aptui@@AAEXXZ 00463890 f   Label.obj
 0001:000628b0       ??0ColorLabel@aptui@@QAE@PAVQWidget@@@Z 004638b0 f   Label.obj
 0001:00062990       ??1ColorLabel@aptui@@UAE@XZ 00463990 f   Label.obj
 0001:00062a40       ?SetColor@ColorLabel@aptui@@QAEXHHH@Z 00463a40 f   Label.obj
 0001:00062a70       ?GetColor@ColorLabel@aptui@@QAEXAAH00@Z 00463a70 f   Label.obj
 0001:00062aa0       ?OnLabelClicked@ColorLabel@aptui@@AAEXXZ 00463aa0 f   Label.obj
 0001:00062bf0       ?SetLabelColor@ColorLabel@aptui@@AAEXXZ 00463bf0 f   Label.obj
 0001:000631b0       ??_ELabel@aptui@@UAEPAXI@Z 004641b0 f i Label.obj
 0001:000631b0       ??_GLabel@aptui@@UAEPAXI@Z 004641b0 f i Label.obj
 0001:000631f0       ??_GEditableLabel@aptui@@UAEPAXI@Z 004641f0 f i Label.obj
 0001:000631f0       ??_EEditableLabel@aptui@@UAEPAXI@Z 004641f0 f i Label.obj
 0001:00063230       ??1EditableLabel@aptui@@UAE@XZ 00464230 f i Label.obj
 0001:000632b0       ??_EColorLabel@aptui@@UAEPAXI@Z 004642b0 f i Label.obj
 0001:000632b0       ??_GColorLabel@aptui@@UAEPAXI@Z 004642b0 f i Label.obj
 0001:000632f0       ??_EQColorDialog@@UAEPAXI@Z 004642f0 f i Label.obj
 0001:000632f0       ??_GQColorDialog@@UAEPAXI@Z 004642f0 f i Label.obj
 0001:00063330       ??0?$QList@VQPolygon@@@@QAE@XZ 00464330 f i Label.obj
 0001:00063360       ?size@?$QList@VQPolygon@@@@QBEHXZ 00464360 f i Label.obj
 0001:00063380       ??1?$QList@VQPolygon@@@@QAE@XZ 00464380 f i Label.obj
 0001:000633c0       ?clear@?$QList@VQPolygon@@@@QAEXXZ 004643c0 f i Label.obj
 0001:00063450       ??A?$QList@VQPolygon@@@@QAEAAVQPolygon@@H@Z 00464450 f i Label.obj
 0001:00063490       ?append@?$QList@VQPolygon@@@@QAEXABVQPolygon@@@Z 00464490 f i Label.obj
 0001:00063660       ?detach@?$QList@VQPolygon@@@@QAEXXZ 00464660 f i Label.obj
 0001:00063690       ?t@Node@?$QList@VQPolygon@@@@QAEAAVQPolygon@@XZ 00464690 f i Label.obj
 0001:000636d0       ??4?$QList@VQPolygon@@@@QAEAAV0@ABV0@@Z 004646d0 f i Label.obj
 0001:00063760       ?detach_helper_grow@?$QList@VQPolygon@@@@AAEPAUNode@1@HH@Z 00464760 f i Label.obj
 0001:00063960       ?detach_helper@?$QList@VQPolygon@@@@AAEXXZ 00464960 f i Label.obj
 0001:00063990       ?free@?$QList@VQPolygon@@@@AAEXPAUData@QListData@@@Z 00464990 f i Label.obj
 0001:000639e0       ?node_construct@?$QList@VQPolygon@@@@AAEXPAUNode@1@ABVQPolygon@@@Z 004649e0 f i Label.obj
 0001:00063b10       ?node_destruct@?$QList@VQPolygon@@@@AAEXPAUNode@1@@Z 00464b10 f i Label.obj
 0001:00063b80       ??_GQPolygon@@QAEPAXI@Z    00464b80 f i Label.obj
 0001:00063bc0       ?detach_helper@?$QList@VQPolygon@@@@AAEXH@Z 00464bc0 f i Label.obj
 0001:00063ce0       ?node_destruct@?$QList@VQPolygon@@@@AAEXPAUNode@1@0@Z 00464ce0 f i Label.obj
 0001:00063d80       ?node_copy@?$QList@VQPolygon@@@@AAEXPAUNode@1@00@Z 00464d80 f i Label.obj
 0001:00064020       ??_EColorLabel@aptui@@W7AEPAXI@Z 00465020 f i Label.obj
 0001:00064030       ??_EEditableLabel@aptui@@W7AEPAXI@Z 00465030 f i Label.obj
 0001:00064040       ??_EQColorDialog@@W7AEPAXI@Z 00465040 f i Label.obj
 0001:00064050       ??_ELabel@aptui@@W7AEPAXI@Z 00465050 f i Label.obj
 0001:00064060       ??0QtLockedFile@SharedTools@@QAE@XZ 00465060 f   qtlockedfile.obj
 0001:000640a0       ??0QtLockedFile@SharedTools@@QAE@ABVQString@@@Z 004650a0 f   qtlockedfile.obj
 0001:000640f0       ?isLocked@QtLockedFile@SharedTools@@QBE_NXZ 004650f0 f   qtlockedfile.obj
 0001:00064110       ?lockMode@QtLockedFile@SharedTools@@QBE?AW4LockMode@12@XZ 00465110 f   qtlockedfile.obj
 0001:00064160       ??_GQtLockedFile@SharedTools@@UAEPAXI@Z 00465160 f i qtlockedfile.obj
 0001:00064160       ??_EQtLockedFile@SharedTools@@UAEPAXI@Z 00465160 f i qtlockedfile.obj
 0001:000641a0       ?lock@QtLockedFile@SharedTools@@QAE_NW4LockMode@12@_N@Z 004651a0 f   qtlockedfile_win.obj
 0001:000649a0       ?unlock@QtLockedFile@SharedTools@@QAE_NXZ 004659a0 f   qtlockedfile_win.obj
 0001:00064ad0       ??1QtLockedFile@SharedTools@@UAE@XZ 00465ad0 f   qtlockedfile_win.obj
 0001:00064f30       ??0QtLocalPeer@SharedTools@@QAE@PAVQObject@@ABVQString@@@Z 00465f30 f   qtlocalpeer.obj
 0001:00065450       ?isClient@QtLocalPeer@SharedTools@@QAE_NXZ 00466450 f   qtlocalpeer.obj
 0001:00065590       ?sendMessage@QtLocalPeer@SharedTools@@QAE_NABVQString@@H@Z 00466590 f   qtlocalpeer.obj
 0001:00065780       ?receiveConnection@QtLocalPeer@SharedTools@@IAEXXZ 00466780 f   qtlocalpeer.obj
 0001:00065cf0       ??_EQtLocalPeer@SharedTools@@UAEPAXI@Z 00466cf0 f i qtlocalpeer.obj
 0001:00065cf0       ??_GQtLocalPeer@SharedTools@@UAEPAXI@Z 00466cf0 f i qtlocalpeer.obj
 0001:00065d30       ??_GQLocalServer@@UAEPAXI@Z 00466d30 f i qtlocalpeer.obj
 0001:00065d30       ??_EQLocalServer@@UAEPAXI@Z 00466d30 f i qtlocalpeer.obj
 0001:00065d70       ??1QtLocalPeer@SharedTools@@UAE@XZ 00466d70 f i qtlocalpeer.obj
 0001:00065e10       ?qstrlen@@YAIPBD@Z         00466e10 f i qtlocalpeer.obj
 0001:00065e50       ??8@YA_NABVQByteArray@@PBD@Z 00466e50 f i qtlocalpeer.obj
 0001:00065ea0       ??H@YA?BVQString@@VQChar@@ABV0@@Z 00466ea0 f i qtlocalpeer.obj
 0001:00065f50       ?sysInit@QtSingleApplication@SharedTools@@AAEXABVQString@@@Z 00466f50 f   qtsingleapplication.obj
 0001:00066160       ??0QtSingleApplication@SharedTools@@QAE@AAHPAPAD_N@Z 00467160 f   qtsingleapplication.obj
 0001:00066210       ??0QtSingleApplication@SharedTools@@QAE@ABVQString@@AAHPAPAD@Z 00467210 f   qtsingleapplication.obj
 0001:000662b0       ?event@QtSingleApplication@SharedTools@@UAE_NPAVQEvent@@@Z 004672b0 f   qtsingleapplication.obj
 0001:00066350       ?isRunning@QtSingleApplication@SharedTools@@QAE_N_J@Z 00467350 f   qtsingleapplication.obj
 0001:00066480       ?initialize@QtSingleApplication@SharedTools@@QAEX_N@Z 00467480 f   qtsingleapplication.obj
 0001:000664b0       ?sendMessage@QtSingleApplication@SharedTools@@QAE_NABVQString@@H_J@Z 004674b0 f   qtsingleapplication.obj
 0001:000665f0       ?id@QtSingleApplication@SharedTools@@QBE?AVQString@@XZ 004675f0 f   qtsingleapplication.obj
 0001:00066630       ?applicationId@QtSingleApplication@SharedTools@@QBE?AVQString@@XZ 00467630 f   qtsingleapplication.obj
 0001:00066670       ?setActivationWindow@QtSingleApplication@SharedTools@@QAEXPAVQWidget@@_N@Z 00467670 f   qtsingleapplication.obj
 0001:00066710       ?activationWindow@QtSingleApplication@SharedTools@@QBEPAVQWidget@@XZ 00467710 f   qtsingleapplication.obj
 0001:00066730       ?activateWindow@QtSingleApplication@SharedTools@@QAEXXZ 00467730 f   qtsingleapplication.obj
 0001:000669a0       ??_EQtSingleApplication@SharedTools@@UAEPAXI@Z 004679a0 f i qtsingleapplication.obj
 0001:000669a0       ??_GQtSingleApplication@SharedTools@@UAEPAXI@Z 004679a0 f i qtsingleapplication.obj
 0001:000669e0       ?applicationId@QtLocalPeer@SharedTools@@QBE?AVQString@@XZ 004679e0 f i qtsingleapplication.obj
 0001:00066a20       ??I?$QFlags@W4WindowState@Qt@@@@QBE?AV0@H@Z 00467a20 f i qtsingleapplication.obj
 0001:00066a50       ??0?$QFlags@W4WindowState@Qt@@@@QAE@W4WindowState@Qt@@@Z 00467a50 f i qtsingleapplication.obj
 0001:00066a70       ??0QtSingleCoreApplication@SharedTools@@QAE@AAHPAPAD@Z 00467a70 f   qtsinglecoreapplication.obj
 0001:00066b80       ??0QtSingleCoreApplication@SharedTools@@QAE@ABVQString@@AAHPAPAD@Z 00467b80 f   qtsinglecoreapplication.obj
 0001:00066c50       ?isRunning@QtSingleCoreApplication@SharedTools@@QAE_NXZ 00467c50 f   qtsinglecoreapplication.obj
 0001:00066c70       ?sendMessage@QtSingleCoreApplication@SharedTools@@QAE_NABVQString@@H@Z 00467c70 f   qtsinglecoreapplication.obj
 0001:00066c90       ?id@QtSingleCoreApplication@SharedTools@@QBE?AVQString@@XZ 00467c90 f   qtsinglecoreapplication.obj
 0001:00066d60       ??_GQtSingleCoreApplication@SharedTools@@UAEPAXI@Z 00467d60 f i qtsinglecoreapplication.obj
 0001:00066d60       ??_EQtSingleCoreApplication@SharedTools@@UAEPAXI@Z 00467d60 f i qtsinglecoreapplication.obj
 0001:00066da0       ??1QtSingleCoreApplication@SharedTools@@UAE@XZ 00467da0 f i qtsinglecoreapplication.obj
 0001:00066dc0       ?clearLayout@NM_SHARE_TOOL@@YAXPAVQBoxLayout@@@Z 00467dc0 f   ShareToolFunction.obj
 0001:00066e30       ?addWidgetToListwidget@NM_SHARE_TOOL@@YAXPAVQListWidget@@PAVQWidget@@PAVQListWidgetItem@@@Z 00467e30 f   ShareToolFunction.obj
 0001:00066e60       ?getListitemFromWidget@NM_SHARE_TOOL@@YA_NPAVQListWidget@@PAVQWidget@@PAPAVQListWidgetItem@@@Z 00467e60 f   ShareToolFunction.obj
 0001:00066f20       ??$qobject_cast@PAVQWidget@@@@YAPAVQWidget@@PAVQObject@@@Z 00467f20 f i ShareToolFunction.obj
 0001:00066f4a       ?activate@QMetaObject@@SAXPAVQObject@@PBU1@HPAPAX@Z 00467f4a f   QtCore4:QtCore4.dll
 0001:00066f50       ??1QString@@QAE@XZ         00467f50 f   QtCore4:QtCore4.dll
 0001:00066f56       ??4QString@@QAEAAV0@ABV0@@Z 00467f56 f   QtCore4:QtCore4.dll
 0001:00066f5c       ??0QString@@QAE@ABV0@@Z    00467f5c f   QtCore4:QtCore4.dll
 0001:00066f62       ?deref@QBasicAtomicInt@@QAE_NXZ 00467f62 f   QtCore4:QtCore4.dll
 0001:00066f68       ?ref@QBasicAtomicInt@@QAE_NXZ 00467f68 f   QtCore4:QtCore4.dll
 0001:00066f6e       ?continueFreeData@QMapData@@QAEXH@Z 00467f6e f   QtCore4:QtCore4.dll
 0001:00066f74       ?createData@QMapData@@SAPAU1@H@Z 00467f74 f   QtCore4:QtCore4.dll
 0001:00066f7a       ?node_delete@QMapData@@QAEXQAPAUNode@1@HPAU21@@Z 00467f7a f   QtCore4:QtCore4.dll
 0001:00066f80       ?node_create@QMapData@@QAEPAUNode@1@QAPAU21@HH@Z 00467f80 f   QtCore4:QtCore4.dll
 0001:00066f86       ?qt_metacast@QObject@@UAEPAXPBD@Z 00467f86 f   QtCore4:QtCore4.dll
 0001:00066f8c       ?qt_metacall@QObject@@UAEHW4Call@QMetaObject@@HPAPAX@Z 00467f8c f   QtCore4:QtCore4.dll
 0001:00066f92       ?qt_metacast@QCoreApplication@@UAEPAXPBD@Z 00467f92 f   QtCore4:QtCore4.dll
 0001:00066f98       ?qt_metacall@QCoreApplication@@UAEHW4Call@QMetaObject@@HPAPAX@Z 00467f98 f   QtCore4:QtCore4.dll
 0001:00066f9e       ?height@QSize@@QBEHXZ      00467f9e f   QtCore4:QtCore4.dll
 0001:00066fa4       ?width@QSize@@QBEHXZ       00467fa4 f   QtCore4:QtCore4.dll
 0001:00066faa       ?size@QRect@@QBE?AVQSize@@XZ 00467faa f   QtCore4:QtCore4.dll
 0001:00066fb0       ?exit@QCoreApplication@@SAXH@Z 00467fb0 f   QtCore4:QtCore4.dll
 0001:00066fb6       ?addLibraryPath@QCoreApplication@@SAXABVQString@@@Z 00467fb6 f   QtCore4:QtCore4.dll
 0001:00066fbc       ?instance@QCoreApplication@@SAPAV1@XZ 00467fbc f   QtCore4:QtCore4.dll
 0001:00066fc2       ?toNativeSeparators@QDir@@SA?AVQString@@ABV2@@Z 00467fc2 f   QtCore4:QtCore4.dll
 0001:00066fc8       ?applicationDirPath@QCoreApplication@@SA?AVQString@@XZ 00467fc8 f   QtCore4:QtCore4.dll
 0001:00066fce       ?separator@QDir@@SA?AVQChar@@XZ 00467fce f   QtCore4:QtCore4.dll
 0001:00066fd4       ?setApplicationName@QCoreApplication@@SAXABVQString@@@Z 00467fd4 f   QtCore4:QtCore4.dll
 0001:00066fda       ?tr@QObject@@SA?AVQString@@PBD0@Z 00467fda f   QtCore4:QtCore4.dll
 0001:00066fe0       ??YQString@@QAEAAV0@VQChar@@@Z 00467fe0 f   QtCore4:QtCore4.dll
 0001:00066fe6       ??YQString@@QAEAAV0@ABV0@@Z 00467fe6 f   QtCore4:QtCore4.dll
 0001:00066fec       ?fromAscii@QString@@SA?AV1@PBDH@Z 00467fec f   QtCore4:QtCore4.dll
 0001:00066ff2       ??4QString@@QAEAAV0@PBD@Z  00467ff2 f   QtCore4:QtCore4.dll
 0001:00066ff8       ??0QString@@QAE@PBD@Z      00467ff8 f   QtCore4:QtCore4.dll
 0001:00066ffe       ??0QString@@QAE@XZ         00467ffe f   QtCore4:QtCore4.dll
 0001:00067004       ?close@QFile@@UAEXXZ       00468004 f   QtCore4:QtCore4.dll
 0001:0006700a       ??1QFile@@UAE@XZ           0046800a f   QtCore4:QtCore4.dll
 0001:00067010       ?open@QFile@@UAE_NV?$QFlags@W4OpenModeFlag@QIODevice@@@@@Z 00468010 f   QtCore4:QtCore4.dll
 0001:00067016       ??0QFile@@QAE@ABVQString@@@Z 00468016 f   QtCore4:QtCore4.dll
 0001:0006701c       ?isNull@QString@@QBE_NXZ   0046801c f   QtCore4:QtCore4.dll
 0001:00067022       ??1QTextStream@@UAE@XZ     00468022 f   QtCore4:QtCore4.dll
 0001:00067028       ?setCodec@QTextStream@@QAEXPAVQTextCodec@@@Z 00468028 f   QtCore4:QtCore4.dll
 0001:0006702e       ?codecForName@QTextCodec@@SAPAV1@PBD@Z 0046802e f   QtCore4:QtCore4.dll
 0001:00067034       ??0QTextStream@@QAE@PAVQIODevice@@@Z 00468034 f   QtCore4:QtCore4.dll
 0001:0006703a       ?number@QString@@SA?AV1@HH@Z 0046803a f   QtCore4:QtCore4.dll
 0001:00067040       ??8QString@@QBE_NABV0@@Z   00468040 f   QtCore4:QtCore4.dll
 0001:00067046       ??1QDir@@QAE@XZ            00468046 f   QtCore4:QtCore4.dll
 0001:0006704c       ?absoluteFilePath@QFileInfo@@QBE?AVQString@@XZ 0046804c f   QtCore4:QtCore4.dll
 0001:00067052       ?completeBaseName@QFileInfo@@QBE?AVQString@@XZ 00468052 f   QtCore4:QtCore4.dll
 0001:00067058       ?entryInfoList@QDir@@QBE?AV?$QList@VQFileInfo@@@@V?$QFlags@W4Filter@QDir@@@@V?$QFlags@W4SortFlag@QDir@@@@@Z 00468058 f   QtCore4:QtCore4.dll
 0001:0006705e       ??0QDir@@QAE@ABVQString@@@Z 0046805e f   QtCore4:QtCore4.dll
 0001:00067064       ?toInt@QString@@QBEHPA_NH@Z 00468064 f   QtCore4:QtCore4.dll
 0001:0006706a       ?isEmpty@QString@@QBE_NXZ  0046806a f   QtCore4:QtCore4.dll
 0001:00067070       ?toDouble@QString@@QBENPA_N@Z 00468070 f   QtCore4:QtCore4.dll
 0001:00067076       ??1QDebug@@QAE@XZ          00468076 f   QtCore4:QtCore4.dll
 0001:0006707c       ??6QDebug@@QAEAAV0@P6AAAVQTextStream@@AAV1@@Z@Z 0046807c f   QtCore4:QtCore4.dll
 0001:00067082       ??6QDebug@@QAEAAV0@ABVQString@@@Z 00468082 f   QtCore4:QtCore4.dll
 0001:00067088       ?qDebug@@YA?AVQDebug@@XZ   00468088 f   QtCore4:QtCore4.dll
 0001:0006708e       ?endl@@YAAAVQTextStream@@AAV1@@Z 0046808e f   QtCore4:QtCore4.dll
 0001:00067094       ?split@QString@@QBE?AVQStringList@@ABV1@W4SplitBehavior@1@W4CaseSensitivity@Qt@@@Z 00468094 f   QtCore4:QtCore4.dll
 0001:0006709a       ?readLine@QTextStream@@QAE?AVQString@@_J@Z 0046809a f   QtCore4:QtCore4.dll
 0001:000670a0       ?atEnd@QTextStream@@QBE_NXZ 004680a0 f   QtCore4:QtCore4.dll
 0001:000670a6       ?setFileName@QFile@@QAEXABVQString@@@Z 004680a6 f   QtCore4:QtCore4.dll
 0001:000670ac       ??0QFile@@QAE@XZ           004680ac f   QtCore4:QtCore4.dll
 0001:000670b2       ?size@QListData@@QBEHXZ    004680b2 f   QtCore4:QtCore4.dll
 0001:000670b8       ?at@QListData@@QBEPAPAXH@Z 004680b8 f   QtCore4:QtCore4.dll
 0001:000670be       ?grow@QVectorData@@SAHHHH_N@Z 004680be f   QtCore4:QtCore4.dll
 0001:000670c4       ??9QBasicAtomicInt@@QBE_NH@Z 004680c4 f   QtCore4:QtCore4.dll
 0001:000670ca       ?free@QVectorData@@SAXPAU1@H@Z 004680ca f   QtCore4:QtCore4.dll
 0001:000670d0       ?qMemSet@@YAPAXPAXHI@Z     004680d0 f   QtCore4:QtCore4.dll
 0001:000670d6       ??4QBasicAtomicInt@@QAEAAV0@H@Z 004680d6 f   QtCore4:QtCore4.dll
 0001:000670dc       ?reallocate@QVectorData@@SAPAU1@PAU1@HHH@Z 004680dc f   QtCore4:QtCore4.dll
 0001:000670e2       ?qBadAlloc@@YAXXZ          004680e2 f   QtCore4:QtCore4.dll
 0001:000670e8       ??8QBasicAtomicInt@@QBE_NH@Z 004680e8 f   QtCore4:QtCore4.dll
 0001:000670ee       ?qFree@@YAXPAX@Z           004680ee f   QtCore4:QtCore4.dll
 0001:000670f4       ?allocate@QVectorData@@SAPAU1@HH@Z 004680f4 f   QtCore4:QtCore4.dll
 0001:000670fa       ??MQString@@QBE_NABV0@@Z   004680fa f   QtCore4:QtCore4.dll
 0001:00067100       ??1QFileInfo@@QAE@XZ       00468100 f   QtCore4:QtCore4.dll
 0001:00067106       ?append@QListData@@QAEPAPAXXZ 00468106 f   QtCore4:QtCore4.dll
 0001:0006710c       ?end@QListData@@QBEPAPAXXZ 0046810c f   QtCore4:QtCore4.dll
 0001:00067112       ?detach_grow@QListData@@QAEPAUData@1@PAHH@Z 00468112 f   QtCore4:QtCore4.dll
 0001:00067118       ?begin@QListData@@QBEPAPAXXZ 00468118 f   QtCore4:QtCore4.dll
 0001:0006711e       ?detach@QListData@@QAEPAUData@1@H@Z 0046811e f   QtCore4:QtCore4.dll
 0001:00067124       ?flush@QTextStream@@QAEXXZ 00468124 f   QtCore4:QtCore4.dll
 0001:0006712a       ??6QTextStream@@QAEAAV0@ABVQString@@@Z 0046812a f   QtCore4:QtCore4.dll
 0001:00067130       ?remove@QFile@@SA_NABVQString@@@Z 00468130 f   QtCore4:QtCore4.dll
 0001:00067136       ?exists@QFileInfo@@QBE_NXZ 00468136 f   QtCore4:QtCore4.dll
 0001:0006713c       ??0QFileInfo@@QAE@ABVQString@@@Z 0046813c f   QtCore4:QtCore4.dll
 0001:00067142       ?fileName@QFile@@QBE?AVQString@@XZ 00468142 f   QtCore4:QtCore4.dll
 0001:00067148       ?fileName@QFileInfo@@QBE?AVQString@@XZ 00468148 f   QtCore4:QtCore4.dll
 0001:0006714e       ?append@QString@@QAEAAV1@PBD@Z 0046814e f   QtCore4:QtCore4.dll
 0001:00067154       ?QStringList_contains@QtPrivate@@YA?AVQBool@@PBVQStringList@@ABVQString@@W4CaseSensitivity@Qt@@@Z 00468154 f   QtCore4:QtCore4.dll
 0001:0006715a       ?toUInt@QString@@QBEIPA_NH@Z 0046815a f   QtCore4:QtCore4.dll
 0001:00067160       ??0QLocale@@QAE@XZ         00468160 f   QtCore4:QtCore4.dll
 0001:00067166       ?installTranslator@QCoreApplication@@SAXPAVQTranslator@@@Z 00468166 f   QtCore4:QtCore4.dll
 0001:0006716c       ?load@QTranslator@@QAE_NABVQString@@000@Z 0046816c f   QtCore4:QtCore4.dll
 0001:00067172       ??0QTranslator@@QAE@PAVQObject@@@Z 00468172 f   QtCore4:QtCore4.dll
 0001:00067178       ??4QLocale@@QAEAAV0@ABV0@@Z 00468178 f   QtCore4:QtCore4.dll
 0001:0006717e       ??0QLocale@@QAE@W4Language@0@W4Country@0@@Z 0046817e f   QtCore4:QtCore4.dll
 0001:00067184       ?metaObject@QTranslator@@UBEPBUQMetaObject@@XZ 00468184 f   QtCore4:QtCore4.dll
 0001:0006718a       ?qt_metacast@QTranslator@@UAEPAXPBD@Z 0046818a f   QtCore4:QtCore4.dll
 0001:00067190       ?qt_metacall@QTranslator@@UAEHW4Call@QMetaObject@@HPAPAX@Z 00468190 f   QtCore4:QtCore4.dll
 0001:00067196       ?event@QObject@@UAE_NPAVQEvent@@@Z 00468196 f   QtCore4:QtCore4.dll
 0001:0006719c       ?eventFilter@QObject@@UAE_NPAV1@PAVQEvent@@@Z 0046819c f   QtCore4:QtCore4.dll
 0001:000671a2       ?timerEvent@QObject@@MAEXPAVQTimerEvent@@@Z 004681a2 f   QtCore4:QtCore4.dll
 0001:000671a8       ?childEvent@QObject@@MAEXPAVQChildEvent@@@Z 004681a8 f   QtCore4:QtCore4.dll
 0001:000671ae       ?customEvent@QObject@@MAEXPAVQEvent@@@Z 004681ae f   QtCore4:QtCore4.dll
 0001:000671b4       ?connectNotify@QObject@@MAEXPBD@Z 004681b4 f   QtCore4:QtCore4.dll
 0001:000671ba       ?disconnectNotify@QObject@@MAEXPBD@Z 004681ba f   QtCore4:QtCore4.dll
 0001:000671c0       ?translate@QTranslator@@UBE?AVQString@@PBD00@Z 004681c0 f   QtCore4:QtCore4.dll
 0001:000671c6       ?isEmpty@QTranslator@@UBE_NXZ 004681c6 f   QtCore4:QtCore4.dll
 0001:000671cc       ??1QTranslator@@UAE@XZ     004681cc f   QtCore4:QtCore4.dll
 0001:000671d2       ??0QLocale@@QAE@ABV0@@Z    004681d2 f   QtCore4:QtCore4.dll
 0001:000671d8       ??1QMutexLocker@@QAE@XZ    004681d8 f   QtCore4:QtCore4.dll
 0001:000671de       ??0QMutexLocker@@QAE@PAVQMutex@@@Z 004681de f   QtCore4:QtCore4.dll
 0001:000671e4       ??0QMutex@@QAE@W4RecursionMode@0@@Z 004681e4 f   QtCore4:QtCore4.dll
 0001:000671ea       ??1QMutex@@QAE@XZ          004681ea f   QtCore4:QtCore4.dll
 0001:000671f0       ?winEventFilter@QCoreApplication@@UAE_NPAUtagMSG@@PAJ@Z 004681f0 f   QtCore4:QtCore4.dll
 0001:000671f6       ?toString@QVariant@@QBE?AVQString@@XZ 004681f6 f   QtCore4:QtCore4.dll
 0001:000671fc       ?inherits@QObject@@QBE_NPBD@Z 004681fc f   QtCore4:QtCore4.dll
 0001:00067202       ??1QVariant@@QAE@XZ        00468202 f   QtCore4:QtCore4.dll
 0001:00067208       ?isNull@QVariant@@QBE_NXZ  00468208 f   QtCore4:QtCore4.dll
 0001:0006720e       ?property@QObject@@QBE?AVQVariant@@PBD@Z 0046820e f   QtCore4:QtCore4.dll
 0001:00067214       ?type@QEvent@@QBE?AW4Type@1@XZ 00468214 f   QtCore4:QtCore4.dll
 0001:0006721a       ?setObjectName@QObject@@QAEXABVQString@@@Z 0046821a f   QtCore4:QtCore4.dll
 0001:00067220       ?tr@QMetaObject@@QBE?AVQString@@PBD0@Z 00468220 f   QtCore4:QtCore4.dll
 0001:00067226       ?qWarning@@YAXPBDZZ        00468226 f   QtCore4:QtCore4.dll
 0001:0006722c       ?toStdString@QString@@QBE?AV?$basic_string@DU?$char_traits@D@std@@V?$allocator@D@2@@std@@XZ 0046822c f   QtCore4:QtCore4.dll
 0001:00067232       ?fromUtf8@QString@@SA?AV1@PBDH@Z 00468232 f   QtCore4:QtCore4.dll
 0001:00067238       ?append@QString@@QAEAAV1@ABV1@@Z 00468238 f   QtCore4:QtCore4.dll
 0001:0006723e       ?entryList@QDir@@QBE?AVQStringList@@V?$QFlags@W4Filter@QDir@@@@V?$QFlags@W4SortFlag@QDir@@@@@Z 0046823e f   QtCore4:QtCore4.dll
 0001:00067244       ?qDebug@@YAXPBDZZ          00468244 f   QtCore4:QtCore4.dll
 0001:0006724a       ?codecForLocale@QTextCodec@@SAPAV1@XZ 0046824a f   QtCore4:QtCore4.dll
 0001:00067250       ?bottom@QRect@@QBEHXZ      00468250 f   QtCore4:QtCore4.dll
 0001:00067256       ?right@QRect@@QBEHXZ       00468256 f   QtCore4:QtCore4.dll
 0001:0006725c       ?load@QPluginLoader@@QAE_NXZ 0046825c f   QtCore4:QtCore4.dll
 0001:00067262       ??1QPluginLoader@@UAE@XZ   00468262 f   QtCore4:QtCore4.dll
 0001:00067268       ?instance@QPluginLoader@@QAEPAVQObject@@XZ 00468268 f   QtCore4:QtCore4.dll
 0001:0006726e       ?isLoaded@QPluginLoader@@QBE_NXZ 0046826e f   QtCore4:QtCore4.dll
 0001:00067274       ??0QPluginLoader@@QAE@ABVQString@@PAVQObject@@@Z 00468274 f   QtCore4:QtCore4.dll
 0001:0006727a       ?cleanPath@QDir@@SA?AVQString@@ABV2@@Z 0046827a f   QtCore4:QtCore4.dll
 0001:00067280       ??0QChar@@QAE@UQLatin1Char@@@Z 00468280 f   QtCore4:QtCore4.dll
 0001:00067286       ?remove@QListData@@QAEXH@Z 00468286 f   QtCore4:QtCore4.dll
 0001:0006728c       ?connectSlotsByName@QMetaObject@@SAXPAVQObject@@@Z 0046828c f   QtCore4:QtCore4.dll
 0001:00067292       ??0QRect@@QAE@HHHH@Z       00468292 f   QtCore4:QtCore4.dll
 0001:00067298       ??0QSize@@QAE@HH@Z         00468298 f   QtCore4:QtCore4.dll
 0001:0006729e       ?objectName@QObject@@QBE?AVQString@@XZ 0046829e f   QtCore4:QtCore4.dll
 0001:000672a4       ?translate@QCoreApplication@@SA?AVQString@@PBD00W4Encoding@1@@Z 004682a4 f   QtCore4:QtCore4.dll
 0001:000672aa       ?connect@QObject@@SA_NPBV1@PBD01W4ConnectionType@Qt@@@Z 004682aa f   QtCore4:QtCore4.dll
 0001:000672b0       ??0QPoint@@QAE@HH@Z        004682b0 f   QtCore4:QtCore4.dll
 0001:000672b6       ?x@QPoint@@QBEHXZ          004682b6 f   QtCore4:QtCore4.dll
 0001:000672bc       ?y@QPoint@@QBEHXZ          004682bc f   QtCore4:QtCore4.dll
 0001:000672c2       ?ignore@QEvent@@QAEXXZ     004682c2 f   QtCore4:QtCore4.dll
 0001:000672c8       ?accept@QEvent@@QAEXXZ     004682c8 f   QtCore4:QtCore4.dll
 0001:000672ce       ?setNum@QString@@QAEAAV1@KH@Z 004682ce f   QtCore4:QtCore4.dll
 0001:000672d4       ??1QUrl@@QAE@XZ            004682d4 f   QtCore4:QtCore4.dll
 0001:000672da       ??0QUrl@@QAE@ABVQString@@@Z 004682da f   QtCore4:QtCore4.dll
 0001:000672e0       ??YQString@@QAEAAV0@PBD@Z  004682e0 f   QtCore4:QtCore4.dll
 0001:000672e6       ?toUnicode@QTextCodec@@QBE?AVQString@@PBD@Z 004682e6 f   QtCore4:QtCore4.dll
 0001:000672ec       ?currentPath@QDir@@SA?AVQString@@XZ 004682ec f   QtCore4:QtCore4.dll
 0001:000672f2       ?disconnect@QObject@@SA_NPBV1@PBD01@Z 004682f2 f   QtCore4:QtCore4.dll
 0001:000672f8       ?sender@QObject@@IBEPAV1@XZ 004682f8 f   QtCore4:QtCore4.dll
 0001:000672fe       ??0QVariant@@QAE@H@Z       004682fe f   QtCore4:QtCore4.dll
 0001:00067304       ??0QVariant@@QAE@XZ        00468304 f   QtCore4:QtCore4.dll
 0001:0006730a       ?QStringList_sort@QtPrivate@@YAXPAVQStringList@@@Z 0046830a f   QtCore4:QtCore4.dll
 0001:00067310       ??1QObject@@UAE@XZ         00468310 f   QtCore4:QtCore4.dll
 0001:00067316       ??0QObject@@QAE@PAV0@@Z    00468316 f   QtCore4:QtCore4.dll
 0001:0006731c       ?arg@QString@@QBE?AV1@ABV1@HABVQChar@@@Z 0046831c f   QtCore4:QtCore4.dll
 0001:00067322       ?exists@QFile@@SA_NABVQString@@@Z 00468322 f   QtCore4:QtCore4.dll
 0001:00067328       ??6QDebug@@QAEAAV0@PBD@Z   00468328 f   QtCore4:QtCore4.dll
 0001:0006732e       ?number@QString@@SA?AV1@_JH@Z 0046832e f   QtCore4:QtCore4.dll
 0001:00067334       ?setY@QPoint@@QAEXH@Z      00468334 f   QtCore4:QtCore4.dll
 0001:0006733a       ?setX@QPoint@@QAEXH@Z      0046833a f   QtCore4:QtCore4.dll
 0001:00067340       ??0QPoint@@QAE@XZ          00468340 f   QtCore4:QtCore4.dll
 0001:00067346       ?parent@QObject@@QBEPAV1@XZ 00468346 f   QtCore4:QtCore4.dll
 0001:0006734c       ?sprintf@QString@@QAAAAV1@PBDZZ 0046834c f   QtCore4:QtCore4.dll
 0001:00067352       ?unlock@QMutex@@QAEXXZ     00468352 f   QtCore4:QtCore4.dll
 0001:00067358       ?lock@QMutex@@QAEXXZ       00468358 f   QtCore4:QtCore4.dll
 0001:0006735e       ?blockSignals@QObject@@QAE_N_N@Z 0046835e f   QtCore4:QtCore4.dll
 0001:00067364       ??8QString@@QBE_NPBD@Z     00468364 f   QtCore4:QtCore4.dll
 0001:0006736a       ??0QSizeF@@QAE@NN@Z        0046836a f   QtCore4:QtCore4.dll
 0001:00067370       ?number@QString@@SA?AV1@NDH@Z 00468370 f   QtCore4:QtCore4.dll
 0001:00067376       ??8QString@@QBE_NABVQLatin1String@@@Z 00468376 f   QtCore4:QtCore4.dll
 0001:0006737c       ??0QLatin1String@@QAE@PBD@Z 0046837c f   QtCore4:QtCore4.dll
 0001:00067382       ?toUpper@QString@@QBE?AV1@XZ 00468382 f   QtCore4:QtCore4.dll
 0001:00067388       ??6QDebug@@QAEAAV0@H@Z     00468388 f   QtCore4:QtCore4.dll
 0001:0006738e       ?copy@QFile@@SA_NABVQString@@0@Z 0046838e f   QtCore4:QtCore4.dll
 0001:00067394       ??0QSize@@QAE@XZ           00468394 f   QtCore4:QtCore4.dll
 0001:0006739a       ??9QString@@QBE_NPBD@Z     0046839a f   QtCore4:QtCore4.dll
 0001:000673a0       ?top@QRect@@QBEHXZ         004683a0 f   QtCore4:QtCore4.dll
 0001:000673a6       ?width@QRect@@QBEHXZ       004683a6 f   QtCore4:QtCore4.dll
 0001:000673ac       ?left@QString@@QBE?AV1@H@Z 004683ac f   QtCore4:QtCore4.dll
 0001:000673b2       ?mid@QString@@QBE?AV1@HH@Z 004683b2 f   QtCore4:QtCore4.dll
 0001:000673b8       ??0QRect@@QAE@ABVQPoint@@0@Z 004683b8 f   QtCore4:QtCore4.dll
 0001:000673be       ?topRight@QRect@@QBE?AVQPoint@@XZ 004683be f   QtCore4:QtCore4.dll
 0001:000673c4       ??BQIncompatibleFlag@@QBEHXZ 004683c4 f   QtCore4:QtCore4.dll
 0001:000673ca       ?indexOf@QString@@QBEHVQChar@@HW4CaseSensitivity@Qt@@@Z 004683ca f   QtCore4:QtCore4.dll
 0001:000673d0       ?getRect@QRect@@QBEXPAH000@Z 004683d0 f   QtCore4:QtCore4.dll
 0001:000673d6       ?topLeft@QRect@@QBE?AVQPoint@@XZ 004683d6 f   QtCore4:QtCore4.dll
 0001:000673dc       ?moveCenter@QRect@@QAEXABVQPoint@@@Z 004683dc f   QtCore4:QtCore4.dll
 0001:000673e2       ?x@QRect@@QBEHXZ           004683e2 f   QtCore4:QtCore4.dll
 0001:000673e8       ?y@QRect@@QBEHXZ           004683e8 f   QtCore4:QtCore4.dll
 0001:000673ee       ?height@QRect@@QBEHXZ      004683ee f   QtCore4:QtCore4.dll
 0001:000673f4       ?left@QRect@@QBEHXZ        004683f4 f   QtCore4:QtCore4.dll
 0001:000673fa       ?center@QRect@@QBE?AVQPoint@@XZ 004683fa f   QtCore4:QtCore4.dll
 0001:00067400       ?adjusted@QRect@@QBE?AV1@HHHH@Z 00468400 f   QtCore4:QtCore4.dll
 0001:00067406       ?cast@QMetaObject@@QBEPBVQObject@@PBV2@@Z 00468406 f   QtCore4:QtCore4.dll
 0001:0006740c       ??0QIncompatibleFlag@@QAE@H@Z 0046840c f   QtCore4:QtCore4.dll
 0001:00067412       ?setProperty@QObject@@QAE_NPBDABVQVariant@@@Z 00468412 f   QtCore4:QtCore4.dll
 0001:00067418       ??0QVariant@@QAE@ABVQString@@@Z 00468418 f   QtCore4:QtCore4.dll
 0001:0006741e       ?registerType@QMetaType@@SAHPBDP6AXPAX@ZP6APAXPBX@Z@Z 0046841e f   QtCore4:QtCore4.dll
 0001:00067424       ?registerTypedef@QMetaType@@SAHPBDH@Z 00468424 f   QtCore4:QtCore4.dll
 0001:0006742a       ?append@?$QVector@VQPoint@@@@QAEXABVQPoint@@@Z 0046842a f   QtCore4:QtCore4.dll
 0001:00067430       ?clear@?$QVector@VQPoint@@@@QAEXXZ 00468430 f   QtCore4:QtCore4.dll
 0001:00067436       ?arg@QString@@QBE?AV1@HHHABVQChar@@@Z 00468436 f   QtCore4:QtCore4.dll
 0001:0006743c       ?metaObject@QFile@@UBEPBUQMetaObject@@XZ 0046843c f   QtCore4:QtCore4.dll
 0001:00067442       ?qt_metacast@QFile@@UAEPAXPBD@Z 00468442 f   QtCore4:QtCore4.dll
 0001:00067448       ?qt_metacall@QFile@@UAEHW4Call@QMetaObject@@HPAPAX@Z 00468448 f   QtCore4:QtCore4.dll
 0001:0006744e       ?isSequential@QFile@@UBE_NXZ 0046844e f   QtCore4:QtCore4.dll
 0001:00067454       ?pos@QFile@@UBE_JXZ        00468454 f   QtCore4:QtCore4.dll
 0001:0006745a       ?size@QFile@@UBE_JXZ       0046845a f   QtCore4:QtCore4.dll
 0001:00067460       ?seek@QFile@@UAE_N_J@Z     00468460 f   QtCore4:QtCore4.dll
 0001:00067466       ?atEnd@QFile@@UBE_NXZ      00468466 f   QtCore4:QtCore4.dll
 0001:0006746c       ?reset@QIODevice@@UAE_NXZ  0046846c f   QtCore4:QtCore4.dll
 0001:00067472       ?bytesAvailable@QIODevice@@UBE_JXZ 00468472 f   QtCore4:QtCore4.dll
 0001:00067478       ?bytesToWrite@QIODevice@@UBE_JXZ 00468478 f   QtCore4:QtCore4.dll
 0001:0006747e       ?canReadLine@QIODevice@@UBE_NXZ 0046847e f   QtCore4:QtCore4.dll
 0001:00067484       ?waitForReadyRead@QIODevice@@UAE_NH@Z 00468484 f   QtCore4:QtCore4.dll
 0001:0006748a       ?waitForBytesWritten@QIODevice@@UAE_NH@Z 0046848a f   QtCore4:QtCore4.dll
 0001:00067490       ?readData@QFile@@MAE_JPAD_J@Z 00468490 f   QtCore4:QtCore4.dll
 0001:00067496       ?readLineData@QFile@@MAE_JPAD_J@Z 00468496 f   QtCore4:QtCore4.dll
 0001:0006749c       ?writeData@QFile@@MAE_JPBD_J@Z 0046849c f   QtCore4:QtCore4.dll
 0001:000674a2       ?fileEngine@QFile@@UBEPAVQAbstractFileEngine@@XZ 004684a2 f   QtCore4:QtCore4.dll
 0001:000674a8       ??1QByteArray@@QAE@XZ      004684a8 f   QtCore4:QtCore4.dll
 0001:000674ae       ?constData@QByteArray@@QBEPBDXZ 004684ae f   QtCore4:QtCore4.dll
 0001:000674b4       ?toLatin1@QString@@QBE?AVQByteArray@@XZ 004684b4 f   QtCore4:QtCore4.dll
 0001:000674ba       ?utf16@QString@@QBEPBGXZ   004684ba f   QtCore4:QtCore4.dll
 0001:000674c0       ?fromLatin1@QString@@SA?AV1@PBDH@Z 004684c0 f   QtCore4:QtCore4.dll
 0001:000674c6       ?toLower@QString@@QBE?AV1@XZ 004684c6 f   QtCore4:QtCore4.dll
 0001:000674cc       ??0QFileInfo@@QAE@ABVQFile@@@Z 004684cc f   QtCore4:QtCore4.dll
 0001:000674d2       ?isOpen@QIODevice@@QBE_NXZ 004684d2 f   QtCore4:QtCore4.dll
 0001:000674d8       ?truncate@QString@@QAEXH@Z 004684d8 f   QtCore4:QtCore4.dll
 0001:000674de       ?length@QString@@QBEHXZ    004684de f   QtCore4:QtCore4.dll
 0001:000674e4       ?endsWith@QString@@QBE_NABVQChar@@W4CaseSensitivity@Qt@@@Z 004684e4 f   QtCore4:QtCore4.dll
 0001:000674ea       ??0QChar@@QAE@D@Z          004684ea f   QtCore4:QtCore4.dll
 0001:000674f0       ?fromLocal8Bit@QString@@SA?AV1@PBDH@Z 004684f0 f   QtCore4:QtCore4.dll
 0001:000674f6       ?absolutePath@QDir@@QBE?AVQString@@XZ 004684f6 f   QtCore4:QtCore4.dll
 0001:000674fc       ?tempPath@QDir@@SA?AVQString@@XZ 004684fc f   QtCore4:QtCore4.dll
 0001:00067502       ?number@QString@@SA?AV1@KH@Z 00468502 f   QtCore4:QtCore4.dll
 0001:00067508       ??1QLibrary@@UAE@XZ        00468508 f   QtCore4:QtCore4.dll
 0001:0006750e       ?resolve@QLibrary@@QAEPAXPBD@Z 0046850e f   QtCore4:QtCore4.dll
 0001:00067514       ??0QLibrary@@QAE@ABVQString@@PAVQObject@@@Z 00468514 f   QtCore4:QtCore4.dll
 0001:0006751a       ??0QString@@QAE@ABVQLatin1String@@@Z 0046851a f   QtCore4:QtCore4.dll
 0001:00067520       ?qChecksum@@YAGPBDI@Z      00468520 f   QtCore4:QtCore4.dll
 0001:00067526       ?size@QByteArray@@QBEHXZ   00468526 f   QtCore4:QtCore4.dll
 0001:0006752c       ?toUtf8@QString@@QBE?AVQByteArray@@XZ 0046852c f   QtCore4:QtCore4.dll
 0001:00067532       ?applicationFilePath@QCoreApplication@@SA?AVQString@@XZ 00468532 f   QtCore4:QtCore4.dll
 0001:00067538       ?connect@QObject@@QBE_NPBV1@PBD1W4ConnectionType@Qt@@@Z 00468538 f   QtCore4:QtCore4.dll
 0001:0006753e       ?toLocal8Bit@QString@@QBE?AVQByteArray@@XZ 0046853e f   QtCore4:QtCore4.dll
 0001:00067544       ??1QDataStream@@UAE@XZ     00468544 f   QtCore4:QtCore4.dll
 0001:0006754a       ?read@QIODevice@@QAE?AVQByteArray@@_J@Z 0046854a f   QtCore4:QtCore4.dll
 0001:00067550       ?writeBytes@QDataStream@@QAEAAV1@PBDI@Z 00468550 f   QtCore4:QtCore4.dll
 0001:00067556       ??0QDataStream@@QAE@PAVQIODevice@@@Z 00468556 f   QtCore4:QtCore4.dll
 0001:0006755c       ?write@QIODevice@@QAE_JPBD_J@Z 0046855c f   QtCore4:QtCore4.dll
 0001:00067562       ?qWarning@@YA?AVQDebug@@XZ 00468562 f   QtCore4:QtCore4.dll
 0001:00067568       ?errorString@QIODevice@@QBE?AVQString@@XZ 00468568 f   QtCore4:QtCore4.dll
 0001:0006756e       ?readRawData@QDataStream@@QAEHPADH@Z 0046856e f   QtCore4:QtCore4.dll
 0001:00067574       ?data@QByteArray@@QAEPADXZ 00468574 f   QtCore4:QtCore4.dll
 0001:0006757a       ?resize@QByteArray@@QAEXH@Z 0046857a f   QtCore4:QtCore4.dll
 0001:00067580       ??5QDataStream@@QAEAAV0@AAI@Z 00468580 f   QtCore4:QtCore4.dll
 0001:00067586       ??0QByteArray@@QAE@XZ      00468586 f   QtCore4:QtCore4.dll
 0001:0006758c       ?isEmpty@QByteArray@@QBE_NXZ 0046858c f   QtCore4:QtCore4.dll
 0001:00067592       ?qstrcmp@@YAHABVQByteArray@@PBD@Z 00468592 f   QtCore4:QtCore4.dll
 0001:00067598       ??0QString@@QAE@VQChar@@@Z 00468598 f   QtCore4:QtCore4.dll
 0001:0006759e       ?applicationPid@QCoreApplication@@SA_JXZ 0046859e f   QtCore4:QtCore4.dll
 0001:000675a4       ??1QCoreApplication@@UAE@XZ 004685a4 f   QtCore4:QtCore4.dll
 0001:000675aa       ??0QCoreApplication@@QAE@AAHPAPADH@Z 004685aa f   QtCore4:QtCore4.dll
 0001:000675b0       ?event@QCoreApplication@@MAE_NPAVQEvent@@@Z 004685b0 f   QtCore4:QtCore4.dll
 0001:000675b6       ?notify@QCoreApplication@@UAE_NPAVQObject@@PAVQEvent@@@Z 004685b6 f   QtCore4:QtCore4.dll
 0001:000675bc       ?compressEvent@QCoreApplication@@MAE_NPAVQEvent@@PAVQObject@@PAVQPostEventList@@@Z 004685bc f   QtCore4:QtCore4.dll
 0001:000675c2       ?isWidgetType@QObject@@QBE_NXZ 004685c2 f   QtCore4:QtCore4.dll
 0001:000675c8       ?qt_metacast@QWidget@@UAEPAXPBD@Z 004685c8 f   QtGui4:QtGui4.dll
 0001:000675ce       ?qt_metacall@QWidget@@UAEHW4Call@QMetaObject@@HPAPAX@Z 004685ce f   QtGui4:QtGui4.dll
 0001:000675d4       ?qt_metacast@QDialog@@UAEPAXPBD@Z 004685d4 f   QtGui4:QtGui4.dll
 0001:000675da       ?qt_metacall@QDialog@@UAEHW4Call@QMetaObject@@HPAPAX@Z 004685da f   QtGui4:QtGui4.dll
 0001:000675e0       ?qt_metacast@QRadioButton@@UAEPAXPBD@Z 004685e0 f   QtGui4:QtGui4.dll
 0001:000675e6       ?qt_metacall@QRadioButton@@UAEHW4Call@QMetaObject@@HPAPAX@Z 004685e6 f   QtGui4:QtGui4.dll
 0001:000675ec       ?qt_metacast@QMainWindow@@UAEPAXPBD@Z 004685ec f   QtGui4:QtGui4.dll
 0001:000675f2       ?qt_metacall@QMainWindow@@UAEHW4Call@QMetaObject@@HPAPAX@Z 004685f2 f   QtGui4:QtGui4.dll
 0001:000675f8       ?qt_metacast@QWidgetAction@@UAEPAXPBD@Z 004685f8 f   QtGui4:QtGui4.dll
 0001:000675fe       ?qt_metacall@QWidgetAction@@UAEHW4Call@QMetaObject@@HPAPAX@Z 004685fe f   QtGui4:QtGui4.dll
 0001:00067604       ?qt_metacast@QLabel@@UAEPAXPBD@Z 00468604 f   QtGui4:QtGui4.dll
 0001:0006760a       ?qt_metacall@QLabel@@UAEHW4Call@QMetaObject@@HPAPAX@Z 0046860a f   QtGui4:QtGui4.dll
 0001:00067610       ?qt_metacast@QFrame@@UAEPAXPBD@Z 00468610 f   QtGui4:QtGui4.dll
 0001:00067616       ?qt_metacall@QFrame@@UAEHW4Call@QMetaObject@@HPAPAX@Z 00468616 f   QtGui4:QtGui4.dll
 0001:0006761c       ?qt_metacast@QSpinBox@@UAEPAXPBD@Z 0046861c f   QtGui4:QtGui4.dll
 0001:00067622       ?qt_metacall@QSpinBox@@UAEHW4Call@QMetaObject@@HPAPAX@Z 00468622 f   QtGui4:QtGui4.dll
 0001:00067628       ?qt_metacast@QMenu@@UAEPAXPBD@Z 00468628 f   QtGui4:QtGui4.dll
 0001:0006762e       ?qt_metacall@QMenu@@UAEHW4Call@QMetaObject@@HPAPAX@Z 0046862e f   QtGui4:QtGui4.dll
 0001:00067634       ?qt_metacast@QProxyStyle@@UAEPAXPBD@Z 00468634 f   QtGui4:QtGui4.dll
 0001:0006763a       ?qt_metacall@QProxyStyle@@UAEHW4Call@QMetaObject@@HPAPAX@Z 0046863a f   QtGui4:QtGui4.dll
 0001:00067640       ?qt_metacast@QPushButton@@UAEPAXPBD@Z 00468640 f   QtGui4:QtGui4.dll
 0001:00067646       ?qt_metacall@QPushButton@@UAEHW4Call@QMetaObject@@HPAPAX@Z 00468646 f   QtGui4:QtGui4.dll
 0001:0006764c       ?qt_metacast@QApplication@@UAEPAXPBD@Z 0046864c f   QtGui4:QtGui4.dll
 0001:00067652       ?qt_metacall@QApplication@@UAEHW4Call@QMetaObject@@HPAPAX@Z 00468652 f   QtGui4:QtGui4.dll
 0001:00067658       ?qt_metacast@QTabWidget@@UAEPAXPBD@Z 00468658 f   QtGui4:QtGui4.dll
 0001:0006765e       ?qt_metacall@QTabWidget@@UAEHW4Call@QMetaObject@@HPAPAX@Z 0046865e f   QtGui4:QtGui4.dll
 0001:00067664       ?exec@QApplication@@SAHXZ  00468664 f   QtGui4:QtGui4.dll
 0001:0006766a       ?show@QWidget@@QAEXXZ      0046866a f   QtGui4:QtGui4.dll
 0001:00067670       ?move@QWidget@@QAEXHH@Z    00468670 f   QtGui4:QtGui4.dll
 0001:00067676       ?resize@QWidget@@QAEXABVQSize@@@Z 00468676 f   QtGui4:QtGui4.dll
 0001:0006767c       ?resize@QWidget@@QAEXHH@Z  0046867c f   QtGui4:QtGui4.dll
 0001:00067682       ?availableGeometry@QDesktopWidget@@QBE?BVQRect@@H@Z 00468682 f   QtGui4:QtGui4.dll
 0001:00067688       ?desktop@QApplication@@SAPAVQDesktopWidget@@XZ 00468688 f   QtGui4:QtGui4.dll
 0001:0006768e       ?compressEvent@QApplication@@MAE_NPAVQEvent@@PAVQObject@@PAVQPostEventList@@@Z 0046868e f   QtGui4:QtGui4.dll
 0001:00067694       ?commitData@QApplication@@UAEXAAVQSessionManager@@@Z 00468694 f   QtGui4:QtGui4.dll
 0001:0006769a       ?saveState@QApplication@@UAEXAAVQSessionManager@@@Z 0046869a f   QtGui4:QtGui4.dll
 0001:000676a0       ??1QApplication@@UAE@XZ    004686a0 f   QtGui4:QtGui4.dll
 0001:000676a6       ?notify@QApplication@@UAE_NPAVQObject@@PAVQEvent@@@Z 004686a6 f   QtGui4:QtGui4.dll
 0001:000676ac       ?showText@QToolTip@@SAXABVQPoint@@ABVQString@@PAVQWidget@@@Z 004686ac f   QtGui4:QtGui4.dll
 0001:000676b2       ?globalPos@QHelpEvent@@QBEABVQPoint@@XZ 004686b2 f   QtGui4:QtGui4.dll
 0001:000676b8       ??1QIcon@@QAE@XZ           004686b8 f   QtGui4:QtGui4.dll
 0001:000676be       ?setWindowIcon@QApplication@@SAXABVQIcon@@@Z 004686be f   QtGui4:QtGui4.dll
 0001:000676c4       ??0QIcon@@QAE@ABVQString@@@Z 004686c4 f   QtGui4:QtGui4.dll
 0001:000676ca       ?exec@QDialog@@QAEHXZ      004686ca f   QtGui4:QtGui4.dll
 0001:000676d0       ?setFixedSize@QWidget@@QAEXHH@Z 004686d0 f   QtGui4:QtGui4.dll
 0001:000676d6       ??1QFont@@QAE@XZ           004686d6 f   QtGui4:QtGui4.dll
 0001:000676dc       ?setFont@QApplication@@SAXABVQFont@@PBD@Z 004686dc f   QtGui4:QtGui4.dll
 0001:000676e2       ?setStyleHint@QFont@@QAEXW4StyleHint@1@W4StyleStrategy@1@@Z 004686e2 f   QtGui4:QtGui4.dll
 0001:000676e8       ?setPointSize@QFont@@QAEXH@Z 004686e8 f   QtGui4:QtGui4.dll
 0001:000676ee       ?setFamily@QFont@@QAEXABVQString@@@Z 004686ee f   QtGui4:QtGui4.dll
 0001:000676f4       ??0QFont@@QAE@XZ           004686f4 f   QtGui4:QtGui4.dll
 0001:000676fa       ?setStyleSheet@QApplication@@QAEXABVQString@@@Z 004686fa f   QtGui4:QtGui4.dll
 0001:00067700       ?setStyle@QApplication@@SAXPAVQStyle@@@Z 00468700 f   QtGui4:QtGui4.dll
 0001:00067706       ?create@QStyleFactory@@SAPAVQStyle@@ABVQString@@@Z 00468706 f   QtGui4:QtGui4.dll
 0001:0006770c       ?screenGeometry@QDesktopWidget@@QBE?BVQRect@@H@Z 0046870c f   QtGui4:QtGui4.dll
 0001:00067712       ?screenCount@QDesktopWidget@@QBEHXZ 00468712 f   QtGui4:QtGui4.dll
 0001:00067718       ??1QMainWindow@@UAE@XZ     00468718 f   QtGui4:QtGui4.dll
 0001:0006771e       ??0QMainWindow@@QAE@PAVQWidget@@V?$QFlags@W4WindowType@Qt@@@@@Z 0046871e f   QtGui4:QtGui4.dll
 0001:00067724       ?event@QMainWindow@@MAE_NPAVQEvent@@@Z 00468724 f   QtGui4:QtGui4.dll
 0001:0006772a       ?setVisible@QWidget@@UAEX_N@Z 0046872a f   QtGui4:QtGui4.dll
 0001:00067730       ?sizeHint@QWidget@@UBE?AVQSize@@XZ 00468730 f   QtGui4:QtGui4.dll
 0001:00067736       ?minimumSizeHint@QWidget@@UBE?AVQSize@@XZ 00468736 f   QtGui4:QtGui4.dll
 0001:0006773c       ?heightForWidth@QWidget@@UBEHH@Z 0046873c f   QtGui4:QtGui4.dll
 0001:00067742       ?mousePressEvent@QWidget@@MAEXPAVQMouseEvent@@@Z 00468742 f   QtGui4:QtGui4.dll
 0001:00067748       ?mouseReleaseEvent@QWidget@@MAEXPAVQMouseEvent@@@Z 00468748 f   QtGui4:QtGui4.dll
 0001:0006774e       ?mouseDoubleClickEvent@QWidget@@MAEXPAVQMouseEvent@@@Z 0046874e f   QtGui4:QtGui4.dll
 0001:00067754       ?mouseMoveEvent@QWidget@@MAEXPAVQMouseEvent@@@Z 00468754 f   QtGui4:QtGui4.dll
 0001:0006775a       ?wheelEvent@QWidget@@MAEXPAVQWheelEvent@@@Z 0046875a f   QtGui4:QtGui4.dll
 0001:00067760       ?keyReleaseEvent@QWidget@@MAEXPAVQKeyEvent@@@Z 00468760 f   QtGui4:QtGui4.dll
 0001:00067766       ?focusInEvent@QWidget@@MAEXPAVQFocusEvent@@@Z 00468766 f   QtGui4:QtGui4.dll
 0001:0006776c       ?focusOutEvent@QWidget@@MAEXPAVQFocusEvent@@@Z 0046876c f   QtGui4:QtGui4.dll
 0001:00067772       ?enterEvent@QWidget@@MAEXPAVQEvent@@@Z 00468772 f   QtGui4:QtGui4.dll
 0001:00067778       ?leaveEvent@QWidget@@MAEXPAVQEvent@@@Z 00468778 f   QtGui4:QtGui4.dll
 0001:0006777e       ?paintEvent@QWidget@@MAEXPAVQPaintEvent@@@Z 0046877e f   QtGui4:QtGui4.dll
 0001:00067784       ?moveEvent@QWidget@@MAEXPAVQMoveEvent@@@Z 00468784 f   QtGui4:QtGui4.dll
 0001:0006778a       ?contextMenuEvent@QMainWindow@@MAEXPAVQContextMenuEvent@@@Z 0046878a f   QtGui4:QtGui4.dll
 0001:00067790       ?tabletEvent@QWidget@@MAEXPAVQTabletEvent@@@Z 00468790 f   QtGui4:QtGui4.dll
 0001:00067796       ?actionEvent@QWidget@@MAEXPAVQActionEvent@@@Z 00468796 f   QtGui4:QtGui4.dll
 0001:0006779c       ?dragEnterEvent@QWidget@@MAEXPAVQDragEnterEvent@@@Z 0046879c f   QtGui4:QtGui4.dll
 0001:000677a2       ?dragMoveEvent@QWidget@@MAEXPAVQDragMoveEvent@@@Z 004687a2 f   QtGui4:QtGui4.dll
 0001:000677a8       ?dragLeaveEvent@QWidget@@MAEXPAVQDragLeaveEvent@@@Z 004687a8 f   QtGui4:QtGui4.dll
 0001:000677ae       ?dropEvent@QWidget@@MAEXPAVQDropEvent@@@Z 004687ae f   QtGui4:QtGui4.dll
 0001:000677b4       ?showEvent@QWidget@@MAEXPAVQShowEvent@@@Z 004687b4 f   QtGui4:QtGui4.dll
 0001:000677ba       ?hideEvent@QWidget@@MAEXPAVQHideEvent@@@Z 004687ba f   QtGui4:QtGui4.dll
 0001:000677c0       ?winEvent@QWidget@@MAE_NPAUtagMSG@@PAJ@Z 004687c0 f   QtGui4:QtGui4.dll
 0001:000677c6       ?changeEvent@QWidget@@MAEXPAVQEvent@@@Z 004687c6 f   QtGui4:QtGui4.dll
 0001:000677cc       ?inputMethodEvent@QWidget@@MAEXPAVQInputMethodEvent@@@Z 004687cc f   QtGui4:QtGui4.dll
 0001:000677d2       ?inputMethodQuery@QWidget@@UBE?AVQVariant@@W4InputMethodQuery@Qt@@@Z 004687d2 f   QtGui4:QtGui4.dll
 0001:000677d8       ?focusNextPrevChild@QWidget@@MAE_N_N@Z 004687d8 f   QtGui4:QtGui4.dll
 0001:000677de       ?styleChange@QWidget@@MAEXAAVQStyle@@@Z 004687de f   QtGui4:QtGui4.dll
 0001:000677e4       ?enabledChange@QWidget@@MAEX_N@Z 004687e4 f   QtGui4:QtGui4.dll
 0001:000677ea       ?paletteChange@QWidget@@MAEXABVQPalette@@@Z 004687ea f   QtGui4:QtGui4.dll
 0001:000677f0       ?fontChange@QWidget@@MAEXABVQFont@@@Z 004687f0 f   QtGui4:QtGui4.dll
 0001:000677f6       ?windowActivationChange@QWidget@@MAEX_N@Z 004687f6 f   QtGui4:QtGui4.dll
 0001:000677fc       ?languageChange@QWidget@@MAEXXZ 004687fc f   QtGui4:QtGui4.dll
 0001:00067802       ?createPopupMenu@QMainWindow@@UAEPAVQMenu@@XZ 00468802 f   QtGui4:QtGui4.dll
 0001:00067808       ?devType@QWidget@@UBEHXZ   00468808 f   QtGui4:QtGui4.dll
 0001:0006780e       ?paintEngine@QWidget@@UBEPAVQPaintEngine@@XZ 0046880e f   QtGui4:QtGui4.dll
 0001:00067814       ?getDC@QWidget@@UBEPAUHDC__@@XZ 00468814 f   QtGui4:QtGui4.dll
 0001:0006781a       ?releaseDC@QWidget@@UBEXPAUHDC__@@@Z 0046881a f   QtGui4:QtGui4.dll
 0001:00067820       ?metric@QWidget@@MBEHW4PaintDeviceMetric@QPaintDevice@@@Z 00468820 f   QtGui4:QtGui4.dll
 0001:00067826       ?setCentralWidget@QMainWindow@@QAEXPAVQWidget@@@Z 00468826 f   QtGui4:QtGui4.dll
 0001:0006782c       ?addWidget@QGridLayout@@QAEXPAVQWidget@@HHHHV?$QFlags@W4AlignmentFlag@Qt@@@@@Z 0046882c f   QtGui4:QtGui4.dll
 0001:00067832       ?setWidget@QScrollArea@@QAEXPAVQWidget@@@Z 00468832 f   QtGui4:QtGui4.dll
 0001:00067838       ?addLayout@QGridLayout@@QAEXPAVQLayout@@HHHHV?$QFlags@W4AlignmentFlag@Qt@@@@@Z 00468838 f   QtGui4:QtGui4.dll
 0001:0006783e       ?setSpacing@QBoxLayout@@QAEXH@Z 0046883e f   QtGui4:QtGui4.dll
 0001:00067844       ??0QVBoxLayout@@QAE@XZ     00468844 f   QtGui4:QtGui4.dll
 0001:0006784a       ?setGeometry@QWidget@@QAEXABVQRect@@@Z 0046884a f   QtGui4:QtGui4.dll
 0001:00067850       ?setWidgetResizable@QScrollArea@@QAEX_N@Z 00468850 f   QtGui4:QtGui4.dll
 0001:00067856       ??0QScrollArea@@QAE@PAVQWidget@@@Z 00468856 f   QtGui4:QtGui4.dll
 0001:0006785c       ?setContentsMargins@QLayout@@QAEXHHHH@Z 0046885c f   QtGui4:QtGui4.dll
 0001:00067862       ?setSpacing@QGridLayout@@QAEXH@Z 00468862 f   QtGui4:QtGui4.dll
 0001:00067868       ??0QGridLayout@@QAE@PAVQWidget@@@Z 00468868 f   QtGui4:QtGui4.dll
 0001:0006786e       ??0QWidget@@QAE@PAV0@V?$QFlags@W4WindowType@Qt@@@@@Z 0046886e f   QtGui4:QtGui4.dll
 0001:00067874       ?setMaximumSize@QWidget@@QAEXABVQSize@@@Z 00468874 f   QtGui4:QtGui4.dll
 0001:0006787a       ?setWindowModality@QWidget@@QAEXW4WindowModality@Qt@@@Z 0046887a f   QtGui4:QtGui4.dll
 0001:00067880       ?metaObject@QWidget@@UBEPBUQMetaObject@@XZ 00468880 f   QtGui4:QtGui4.dll
 0001:00067886       ?event@QWidget@@MAE_NPAVQEvent@@@Z 00468886 f   QtGui4:QtGui4.dll
 0001:0006788c       ?keyPressEvent@QWidget@@MAEXPAVQKeyEvent@@@Z 0046888c f   QtGui4:QtGui4.dll
 0001:00067892       ?resizeEvent@QWidget@@MAEXPAVQResizeEvent@@@Z 00468892 f   QtGui4:QtGui4.dll
 0001:00067898       ?closeEvent@QWidget@@MAEXPAVQCloseEvent@@@Z 00468898 f   QtGui4:QtGui4.dll
 0001:0006789e       ?contextMenuEvent@QWidget@@MAEXPAVQContextMenuEvent@@@Z 0046889e f   QtGui4:QtGui4.dll
 0001:000678a4       ?metaObject@QGridLayout@@UBEPBUQMetaObject@@XZ 004688a4 f   QtGui4:QtGui4.dll
 0001:000678aa       ?qt_metacast@QGridLayout@@UAEPAXPBD@Z 004688aa f   QtGui4:QtGui4.dll
 0001:000678b0       ?qt_metacall@QGridLayout@@UAEHW4Call@QMetaObject@@HPAPAX@Z 004688b0 f   QtGui4:QtGui4.dll
 0001:000678b6       ?childEvent@QLayout@@MAEXPAVQChildEvent@@@Z 004688b6 f   QtGui4:QtGui4.dll
 0001:000678bc       ?addItem@QGridLayout@@MAEXPAVQLayoutItem@@@Z 004688bc f   QtGui4:QtGui4.dll
 0001:000678c2       ?itemAt@QGridLayout@@UBEPAVQLayoutItem@@H@Z 004688c2 f   QtGui4:QtGui4.dll
 0001:000678c8       ?takeAt@QGridLayout@@UAEPAVQLayoutItem@@H@Z 004688c8 f   QtGui4:QtGui4.dll
 0001:000678ce       ?indexOf@QLayout@@UBEHPAVQWidget@@@Z 004688ce f   QtGui4:QtGui4.dll
 0001:000678d4       ?count@QGridLayout@@UBEHXZ 004688d4 f   QtGui4:QtGui4.dll
 0001:000678da       ?sizeHint@QGridLayout@@UBE?AVQSize@@XZ 004688da f   QtGui4:QtGui4.dll
 0001:000678e0       ?minimumSize@QGridLayout@@UBE?AVQSize@@XZ 004688e0 f   QtGui4:QtGui4.dll
 0001:000678e6       ?maximumSize@QGridLayout@@UBE?AVQSize@@XZ 004688e6 f   QtGui4:QtGui4.dll
 0001:000678ec       ?expandingDirections@QGridLayout@@UBE?AV?$QFlags@W4Orientation@Qt@@@@XZ 004688ec f   QtGui4:QtGui4.dll
 0001:000678f2       ?setGeometry@QGridLayout@@UAEXABVQRect@@@Z 004688f2 f   QtGui4:QtGui4.dll
 0001:000678f8       ?geometry@QLayout@@UBE?AVQRect@@XZ 004688f8 f   QtGui4:QtGui4.dll
 0001:000678fe       ?isEmpty@QLayout@@UBE_NXZ  004688fe f   QtGui4:QtGui4.dll
 0001:00067904       ?hasHeightForWidth@QGridLayout@@UBE_NXZ 00468904 f   QtGui4:QtGui4.dll
 0001:0006790a       ?heightForWidth@QGridLayout@@UBEHH@Z 0046890a f   QtGui4:QtGui4.dll
 0001:00067910       ?minimumHeightForWidth@QGridLayout@@UBEHH@Z 00468910 f   QtGui4:QtGui4.dll
 0001:00067916       ?invalidate@QGridLayout@@UAEXXZ 00468916 f   QtGui4:QtGui4.dll
 0001:0006791c       ?widget@QLayoutItem@@UAEPAVQWidget@@XZ 0046891c f   QtGui4:QtGui4.dll
 0001:00067922       ?layout@QLayout@@UAEPAV1@XZ 00468922 f   QtGui4:QtGui4.dll
 0001:00067928       ?spacerItem@QLayoutItem@@UAEPAVQSpacerItem@@XZ 00468928 f   QtGui4:QtGui4.dll
 0001:0006792e       ?metaObject@QScrollArea@@UBEPBUQMetaObject@@XZ 0046892e f   QtGui4:QtGui4.dll
 0001:00067934       ?qt_metacast@QScrollArea@@UAEPAXPBD@Z 00468934 f   QtGui4:QtGui4.dll
 0001:0006793a       ?qt_metacall@QScrollArea@@UAEHW4Call@QMetaObject@@HPAPAX@Z 0046893a f   QtGui4:QtGui4.dll
 0001:00067940       ?event@QScrollArea@@MAE_NPAVQEvent@@@Z 00468940 f   QtGui4:QtGui4.dll
 0001:00067946       ?eventFilter@QScrollArea@@MAE_NPAVQObject@@PAVQEvent@@@Z 00468946 f   QtGui4:QtGui4.dll
 0001:0006794c       ?sizeHint@QScrollArea@@UBE?AVQSize@@XZ 0046894c f   QtGui4:QtGui4.dll
 0001:00067952       ?minimumSizeHint@QAbstractScrollArea@@UBE?AVQSize@@XZ 00468952 f   QtGui4:QtGui4.dll
 0001:00067958       ?mousePressEvent@QAbstractScrollArea@@MAEXPAVQMouseEvent@@@Z 00468958 f   QtGui4:QtGui4.dll
 0001:0006795e       ?mouseReleaseEvent@QAbstractScrollArea@@MAEXPAVQMouseEvent@@@Z 0046895e f   QtGui4:QtGui4.dll
 0001:00067964       ?mouseDoubleClickEvent@QAbstractScrollArea@@MAEXPAVQMouseEvent@@@Z 00468964 f   QtGui4:QtGui4.dll
 0001:0006796a       ?mouseMoveEvent@QAbstractScrollArea@@MAEXPAVQMouseEvent@@@Z 0046896a f   QtGui4:QtGui4.dll
 0001:00067970       ?wheelEvent@QAbstractScrollArea@@MAEXPAVQWheelEvent@@@Z 00468970 f   QtGui4:QtGui4.dll
 0001:00067976       ?keyPressEvent@QAbstractScrollArea@@MAEXPAVQKeyEvent@@@Z 00468976 f   QtGui4:QtGui4.dll
 0001:0006797c       ?paintEvent@QAbstractScrollArea@@MAEXPAVQPaintEvent@@@Z 0046897c f   QtGui4:QtGui4.dll
 0001:00067982       ?resizeEvent@QScrollArea@@MAEXPAVQResizeEvent@@@Z 00468982 f   QtGui4:QtGui4.dll
 0001:00067988       ?contextMenuEvent@QAbstractScrollArea@@MAEXPAVQContextMenuEvent@@@Z 00468988 f   QtGui4:QtGui4.dll
 0001:0006798e       ?dragEnterEvent@QAbstractScrollArea@@MAEXPAVQDragEnterEvent@@@Z 0046898e f   QtGui4:QtGui4.dll
 0001:00067994       ?dragMoveEvent@QAbstractScrollArea@@MAEXPAVQDragMoveEvent@@@Z 00468994 f   QtGui4:QtGui4.dll
 0001:0006799a       ?dragLeaveEvent@QAbstractScrollArea@@MAEXPAVQDragLeaveEvent@@@Z 0046899a f   QtGui4:QtGui4.dll
 0001:000679a0       ?dropEvent@QAbstractScrollArea@@MAEXPAVQDropEvent@@@Z 004689a0 f   QtGui4:QtGui4.dll
 0001:000679a6       ?changeEvent@QFrame@@MAEXPAVQEvent@@@Z 004689a6 f   QtGui4:QtGui4.dll
 0001:000679ac       ?focusNextPrevChild@QScrollArea@@UAE_N_N@Z 004689ac f   QtGui4:QtGui4.dll
 0001:000679b2       ?viewportEvent@QAbstractScrollArea@@MAE_NPAVQEvent@@@Z 004689b2 f   QtGui4:QtGui4.dll
 0001:000679b8       ?scrollContentsBy@QScrollArea@@MAEXHH@Z 004689b8 f   QtGui4:QtGui4.dll
 0001:000679be       ?metaObject@QVBoxLayout@@UBEPBUQMetaObject@@XZ 004689be f   QtGui4:QtGui4.dll
 0001:000679c4       ?qt_metacast@QVBoxLayout@@UAEPAXPBD@Z 004689c4 f   QtGui4:QtGui4.dll
 0001:000679ca       ?qt_metacall@QVBoxLayout@@UAEHW4Call@QMetaObject@@HPAPAX@Z 004689ca f   QtGui4:QtGui4.dll
 0001:000679d0       ?addItem@QBoxLayout@@UAEXPAVQLayoutItem@@@Z 004689d0 f   QtGui4:QtGui4.dll
 0001:000679d6       ?itemAt@QBoxLayout@@UBEPAVQLayoutItem@@H@Z 004689d6 f   QtGui4:QtGui4.dll
 0001:000679dc       ?takeAt@QBoxLayout@@UAEPAVQLayoutItem@@H@Z 004689dc f   QtGui4:QtGui4.dll
 0001:000679e2       ?count@QBoxLayout@@UBEHXZ  004689e2 f   QtGui4:QtGui4.dll
 0001:000679e8       ?sizeHint@QBoxLayout@@UBE?AVQSize@@XZ 004689e8 f   QtGui4:QtGui4.dll
 0001:000679ee       ?minimumSize@QBoxLayout@@UBE?AVQSize@@XZ 004689ee f   QtGui4:QtGui4.dll
 0001:000679f4       ?maximumSize@QBoxLayout@@UBE?AVQSize@@XZ 004689f4 f   QtGui4:QtGui4.dll
 0001:000679fa       ?expandingDirections@QBoxLayout@@UBE?AV?$QFlags@W4Orientation@Qt@@@@XZ 004689fa f   QtGui4:QtGui4.dll
 0001:00067a00       ?setGeometry@QBoxLayout@@UAEXABVQRect@@@Z 00468a00 f   QtGui4:QtGui4.dll
 0001:00067a06       ?hasHeightForWidth@QBoxLayout@@UBE_NXZ 00468a06 f   QtGui4:QtGui4.dll
 0001:00067a0c       ?heightForWidth@QBoxLayout@@UBEHH@Z 00468a0c f   QtGui4:QtGui4.dll
 0001:00067a12       ?minimumHeightForWidth@QBoxLayout@@UBEHH@Z 00468a12 f   QtGui4:QtGui4.dll
 0001:00067a18       ?invalidate@QBoxLayout@@UAEXXZ 00468a18 f   QtGui4:QtGui4.dll
 0001:00067a1e       ?setWindowTitle@QWidget@@QAEXABVQString@@@Z 00468a1e f   QtGui4:QtGui4.dll
 0001:00067a24       ??1QWidget@@UAE@XZ         00468a24 f   QtGui4:QtGui4.dll
 0001:00067a2a       ??1QGridLayout@@UAE@XZ     00468a2a f   QtGui4:QtGui4.dll
 0001:00067a30       ??1QScrollArea@@UAE@XZ     00468a30 f   QtGui4:QtGui4.dll
 0001:00067a36       ??1QVBoxLayout@@UAE@XZ     00468a36 f   QtGui4:QtGui4.dll
 0001:00067a3c       ?lower@QWidget@@QAEXXZ     00468a3c f   QtGui4:QtGui4.dll
 0001:00067a42       ?addLayout@QBoxLayout@@QAEXPAVQLayout@@H@Z 00468a42 f   QtGui4:QtGui4.dll
 0001:00067a48       ?addWidget@QBoxLayout@@QAEXPAVQWidget@@HV?$QFlags@W4AlignmentFlag@Qt@@@@@Z 00468a48 f   QtGui4:QtGui4.dll
 0001:00067a4e       ?setFocusPolicy@QWidget@@QAEXW4FocusPolicy@Qt@@@Z 00468a4e f   QtGui4:QtGui4.dll
 0001:00067a54       ?setAttribute@QWidget@@QAEXW4WidgetAttribute@Qt@@_N@Z 00468a54 f   QtGui4:QtGui4.dll
 0001:00067a5a       ?addAction@QWidget@@QAEXPAVQAction@@@Z 00468a5a f   QtGui4:QtGui4.dll
 0001:00067a60       ??0QHBoxLayout@@QAE@XZ     00468a60 f   QtGui4:QtGui4.dll
 0001:00067a66       ?setWindowFlags@QWidget@@QAEXV?$QFlags@W4WindowType@Qt@@@@@Z 00468a66 f   QtGui4:QtGui4.dll
 0001:00067a6c       ?metaObject@QHBoxLayout@@UBEPBUQMetaObject@@XZ 00468a6c f   QtGui4:QtGui4.dll
 0001:00067a72       ?qt_metacast@QHBoxLayout@@UAEPAXPBD@Z 00468a72 f   QtGui4:QtGui4.dll
 0001:00067a78       ?qt_metacall@QHBoxLayout@@UAEHW4Call@QMetaObject@@HPAPAX@Z 00468a78 f   QtGui4:QtGui4.dll
 0001:00067a7e       ??1QHBoxLayout@@UAE@XZ     00468a7e f   QtGui4:QtGui4.dll
 0001:00067a84       ?raise@QWidget@@QAEXXZ     00468a84 f   QtGui4:QtGui4.dll
 0001:00067a8a       ?size@QResizeEvent@@QBEABVQSize@@XZ 00468a8a f   QtGui4:QtGui4.dll
 0001:00067a90       ?popup@QMenu@@QAEXABVQPoint@@PAVQAction@@@Z 00468a90 f   QtGui4:QtGui4.dll
 0001:00067a96       ?pos@QCursor@@SA?AVQPoint@@XZ 00468a96 f   QtGui4:QtGui4.dll
 0001:00067a9c       ?close@QWidget@@QAE_NXZ    00468a9c f   QtGui4:QtGui4.dll
 0001:00067aa2       ?width@QWidget@@QBEHXZ     00468aa2 f   QtGui4:QtGui4.dll
 0001:00067aa8       ?height@QWidget@@QBEHXZ    00468aa8 f   QtGui4:QtGui4.dll
 0001:00067aae       ?pos@QWidget@@QBE?AVQPoint@@XZ 00468aae f   QtGui4:QtGui4.dll
 0001:00067ab4       ?key@QKeyEvent@@QBEHXZ     00468ab4 f   QtGui4:QtGui4.dll
 0001:00067aba       ?event@QWidgetAction@@MAE_NPAVQEvent@@@Z 00468aba f   QtGui4:QtGui4.dll
 0001:00067ac0       ?eventFilter@QWidgetAction@@MAE_NPAVQObject@@PAVQEvent@@@Z 00468ac0 f   QtGui4:QtGui4.dll
 0001:00067ac6       ?createWidget@QWidgetAction@@MAEPAVQWidget@@PAV2@@Z 00468ac6 f   QtGui4:QtGui4.dll
 0001:00067acc       ?deleteWidget@QWidgetAction@@MAEXPAVQWidget@@@Z 00468acc f   QtGui4:QtGui4.dll
 0001:00067ad2       ?openUrl@QDesktopServices@@SA_NABVQUrl@@@Z 00468ad2 f   QtGui4:QtGui4.dll
 0001:00067ad8       ?setMaxLength@QLineEdit@@QAEXH@Z 00468ad8 f   QtGui4:QtGui4.dll
 0001:00067ade       ?setValidator@QLineEdit@@QAEXPBVQValidator@@@Z 00468ade f   QtGui4:QtGui4.dll
 0001:00067ae4       ?setFixedWidth@QWidget@@QAEXH@Z 00468ae4 f   QtGui4:QtGui4.dll
 0001:00067aea       ?fixup@QIntValidator@@UBEXAAVQString@@@Z 00468aea f   QtGui4:QtGui4.dll
 0001:00067af0       ?setRange@QIntValidator@@UAEXHH@Z 00468af0 f   QtGui4:QtGui4.dll
 0001:00067af6       ?setTabOrder@QWidget@@SAXPAV1@0@Z 00468af6 f   QtGui4:QtGui4.dll
 0001:00067afc       ?setFrameShape@QFrame@@QAEXW4Shape@1@@Z 00468afc f   QtGui4:QtGui4.dll
 0001:00067b02       ??0QFrame@@QAE@PAVQWidget@@V?$QFlags@W4WindowType@Qt@@@@@Z 00468b02 f   QtGui4:QtGui4.dll
 0001:00067b08       ?setFrame@QComboBox@@QAEX_N@Z 00468b08 f   QtGui4:QtGui4.dll
 0001:00067b0e       ?setDuplicatesEnabled@QComboBox@@QAEX_N@Z 00468b0e f   QtGui4:QtGui4.dll
 0001:00067b14       ?setEditable@QComboBox@@QAEX_N@Z 00468b14 f   QtGui4:QtGui4.dll
 0001:00067b1a       ?setMinimumSize@QWidget@@QAEXABVQSize@@@Z 00468b1a f   QtGui4:QtGui4.dll
 0001:00067b20       ?setSizePolicy@QWidget@@QAEXVQSizePolicy@@@Z 00468b20 f   QtGui4:QtGui4.dll
 0001:00067b26       ?setHeightForWidth@QSizePolicy@@QAEX_N@Z 00468b26 f   QtGui4:QtGui4.dll
 0001:00067b2c       ?hasHeightForWidth@QSizePolicy@@QBE_NXZ 00468b2c f   QtGui4:QtGui4.dll
 0001:00067b32       ?sizePolicy@QWidget@@QBE?AVQSizePolicy@@XZ 00468b32 f   QtGui4:QtGui4.dll
 0001:00067b38       ?setVerticalStretch@QSizePolicy@@QAEXE@Z 00468b38 f   QtGui4:QtGui4.dll
 0001:00067b3e       ?setHorizontalStretch@QSizePolicy@@QAEXE@Z 00468b3e f   QtGui4:QtGui4.dll
 0001:00067b44       ??0QSizePolicy@@QAE@W4Policy@0@0@Z 00468b44 f   QtGui4:QtGui4.dll
 0001:00067b4a       ??0QLabel@@QAE@PAVQWidget@@V?$QFlags@W4WindowType@Qt@@@@@Z 00468b4a f   QtGui4:QtGui4.dll
 0001:00067b50       ?setVerticalSpacing@QGridLayout@@QAEXH@Z 00468b50 f   QtGui4:QtGui4.dll
 0001:00067b56       ?setHorizontalSpacing@QGridLayout@@QAEXH@Z 00468b56 f   QtGui4:QtGui4.dll
 0001:00067b5c       ?setChecked@QAbstractButton@@QAEX_N@Z 00468b5c f   QtGui4:QtGui4.dll
 0001:00067b62       ??0QCheckBox@@QAE@PAVQWidget@@@Z 00468b62 f   QtGui4:QtGui4.dll
 0001:00067b68       ??0QSpacerItem@@QAE@HHW4Policy@QSizePolicy@@0@Z 00468b68 f   QtGui4:QtGui4.dll
 0001:00067b6e       ??0QVBoxLayout@@QAE@PAVQWidget@@@Z 00468b6e f   QtGui4:QtGui4.dll
 0001:00067b74       ??0QGridLayout@@QAE@XZ     00468b74 f   QtGui4:QtGui4.dll
 0001:00067b7a       ?setStyleSheet@QWidget@@QAEXABVQString@@@Z 00468b7a f   QtGui4:QtGui4.dll
 0001:00067b80       ?sizeHint@QSpacerItem@@UBE?AVQSize@@XZ 00468b80 f   QtGui4:QtGui4.dll
 0001:00067b86       ?minimumSize@QSpacerItem@@UBE?AVQSize@@XZ 00468b86 f   QtGui4:QtGui4.dll
 0001:00067b8c       ?maximumSize@QSpacerItem@@UBE?AVQSize@@XZ 00468b8c f   QtGui4:QtGui4.dll
 0001:00067b92       ?expandingDirections@QSpacerItem@@UBE?AV?$QFlags@W4Orientation@Qt@@@@XZ 00468b92 f   QtGui4:QtGui4.dll
 0001:00067b98       ?setGeometry@QSpacerItem@@UAEXABVQRect@@@Z 00468b98 f   QtGui4:QtGui4.dll
 0001:00067b9e       ?geometry@QSpacerItem@@UBE?AVQRect@@XZ 00468b9e f   QtGui4:QtGui4.dll
 0001:00067ba4       ?isEmpty@QSpacerItem@@UBE_NXZ 00468ba4 f   QtGui4:QtGui4.dll
 0001:00067baa       ?hasHeightForWidth@QLayoutItem@@UBE_NXZ 00468baa f   QtGui4:QtGui4.dll
 0001:00067bb0       ?heightForWidth@QLayoutItem@@UBEHH@Z 00468bb0 f   QtGui4:QtGui4.dll
 0001:00067bb6       ?minimumHeightForWidth@QLayoutItem@@UBEHH@Z 00468bb6 f   QtGui4:QtGui4.dll
 0001:00067bbc       ?invalidate@QLayoutItem@@UAEXXZ 00468bbc f   QtGui4:QtGui4.dll
 0001:00067bc2       ?layout@QLayoutItem@@UAEPAVQLayout@@XZ 00468bc2 f   QtGui4:QtGui4.dll
 0001:00067bc8       ?spacerItem@QSpacerItem@@UAEPAV1@XZ 00468bc8 f   QtGui4:QtGui4.dll
 0001:00067bce       ?metaObject@QCheckBox@@UBEPBUQMetaObject@@XZ 00468bce f   QtGui4:QtGui4.dll
 0001:00067bd4       ?qt_metacast@QCheckBox@@UAEPAXPBD@Z 00468bd4 f   QtGui4:QtGui4.dll
 0001:00067bda       ?qt_metacall@QCheckBox@@UAEHW4Call@QMetaObject@@HPAPAX@Z 00468bda f   QtGui4:QtGui4.dll
 0001:00067be0       ?event@QCheckBox@@MAE_NPAVQEvent@@@Z 00468be0 f   QtGui4:QtGui4.dll
 0001:00067be6       ?timerEvent@QAbstractButton@@MAEXPAVQTimerEvent@@@Z 00468be6 f   QtGui4:QtGui4.dll
 0001:00067bec       ?sizeHint@QCheckBox@@UBE?AVQSize@@XZ 00468bec f   QtGui4:QtGui4.dll
 0001:00067bf2       ?minimumSizeHint@QCheckBox@@UBE?AVQSize@@XZ 00468bf2 f   QtGui4:QtGui4.dll
 0001:00067bf8       ?mousePressEvent@QAbstractButton@@MAEXPAVQMouseEvent@@@Z 00468bf8 f   QtGui4:QtGui4.dll
 0001:00067bfe       ?mouseReleaseEvent@QAbstractButton@@MAEXPAVQMouseEvent@@@Z 00468bfe f   QtGui4:QtGui4.dll
 0001:00067c04       ?mouseMoveEvent@QCheckBox@@MAEXPAVQMouseEvent@@@Z 00468c04 f   QtGui4:QtGui4.dll
 0001:00067c0a       ?keyPressEvent@QAbstractButton@@MAEXPAVQKeyEvent@@@Z 00468c0a f   QtGui4:QtGui4.dll
 0001:00067c10       ?keyReleaseEvent@QAbstractButton@@MAEXPAVQKeyEvent@@@Z 00468c10 f   QtGui4:QtGui4.dll
 0001:00067c16       ?focusInEvent@QAbstractButton@@MAEXPAVQFocusEvent@@@Z 00468c16 f   QtGui4:QtGui4.dll
 0001:00067c1c       ?focusOutEvent@QAbstractButton@@MAEXPAVQFocusEvent@@@Z 00468c1c f   QtGui4:QtGui4.dll
 0001:00067c22       ?paintEvent@QCheckBox@@MAEXPAVQPaintEvent@@@Z 00468c22 f   QtGui4:QtGui4.dll
 0001:00067c28       ?changeEvent@QAbstractButton@@MAEXPAVQEvent@@@Z 00468c28 f   QtGui4:QtGui4.dll
 0001:00067c2e       ?hitButton@QCheckBox@@MBE_NABVQPoint@@@Z 00468c2e f   QtGui4:QtGui4.dll
 0001:00067c34       ?checkStateSet@QCheckBox@@MAEXXZ 00468c34 f   QtGui4:QtGui4.dll
 0001:00067c3a       ?nextCheckState@QCheckBox@@MAEXXZ 00468c3a f   QtGui4:QtGui4.dll
 0001:00067c40       ?metaObject@QLabel@@UBEPBUQMetaObject@@XZ 00468c40 f   QtGui4:QtGui4.dll
 0001:00067c46       ?event@QLabel@@MAE_NPAVQEvent@@@Z 00468c46 f   QtGui4:QtGui4.dll
 0001:00067c4c       ?sizeHint@QLabel@@UBE?AVQSize@@XZ 00468c4c f   QtGui4:QtGui4.dll
 0001:00067c52       ?minimumSizeHint@QLabel@@UBE?AVQSize@@XZ 00468c52 f   QtGui4:QtGui4.dll
 0001:00067c58       ?heightForWidth@QLabel@@UBEHH@Z 00468c58 f   QtGui4:QtGui4.dll
 0001:00067c5e       ?mousePressEvent@QLabel@@MAEXPAVQMouseEvent@@@Z 00468c5e f   QtGui4:QtGui4.dll
 0001:00067c64       ?mouseReleaseEvent@QLabel@@MAEXPAVQMouseEvent@@@Z 00468c64 f   QtGui4:QtGui4.dll
 0001:00067c6a       ?mouseMoveEvent@QLabel@@MAEXPAVQMouseEvent@@@Z 00468c6a f   QtGui4:QtGui4.dll
 0001:00067c70       ?keyPressEvent@QLabel@@MAEXPAVQKeyEvent@@@Z 00468c70 f   QtGui4:QtGui4.dll
 0001:00067c76       ?focusInEvent@QLabel@@MAEXPAVQFocusEvent@@@Z 00468c76 f   QtGui4:QtGui4.dll
 0001:00067c7c       ?focusOutEvent@QLabel@@MAEXPAVQFocusEvent@@@Z 00468c7c f   QtGui4:QtGui4.dll
 0001:00067c82       ?paintEvent@QLabel@@MAEXPAVQPaintEvent@@@Z 00468c82 f   QtGui4:QtGui4.dll
 0001:00067c88       ?contextMenuEvent@QLabel@@MAEXPAVQContextMenuEvent@@@Z 00468c88 f   QtGui4:QtGui4.dll
 0001:00067c8e       ?changeEvent@QLabel@@MAEXPAVQEvent@@@Z 00468c8e f   QtGui4:QtGui4.dll
 0001:00067c94       ?focusNextPrevChild@QLabel@@MAE_N_N@Z 00468c94 f   QtGui4:QtGui4.dll
 0001:00067c9a       ?event@QLineEdit@@UAE_NPAVQEvent@@@Z 00468c9a f   QtGui4:QtGui4.dll
 0001:00067ca0       ?sizeHint@QLineEdit@@UBE?AVQSize@@XZ 00468ca0 f   QtGui4:QtGui4.dll
 0001:00067ca6       ?minimumSizeHint@QLineEdit@@UBE?AVQSize@@XZ 00468ca6 f   QtGui4:QtGui4.dll
 0001:00067cac       ?mouseReleaseEvent@QLineEdit@@MAEXPAVQMouseEvent@@@Z 00468cac f   QtGui4:QtGui4.dll
 0001:00067cb2       ?mouseDoubleClickEvent@QLineEdit@@MAEXPAVQMouseEvent@@@Z 00468cb2 f   QtGui4:QtGui4.dll
 0001:00067cb8       ?mouseMoveEvent@QLineEdit@@MAEXPAVQMouseEvent@@@Z 00468cb8 f   QtGui4:QtGui4.dll
 0001:00067cbe       ?keyPressEvent@QLineEdit@@MAEXPAVQKeyEvent@@@Z 00468cbe f   QtGui4:QtGui4.dll
 0001:00067cc4       ?focusOutEvent@QLineEdit@@MAEXPAVQFocusEvent@@@Z 00468cc4 f   QtGui4:QtGui4.dll
 0001:00067cca       ?paintEvent@QLineEdit@@MAEXPAVQPaintEvent@@@Z 00468cca f   QtGui4:QtGui4.dll
 0001:00067cd0       ?contextMenuEvent@QLineEdit@@MAEXPAVQContextMenuEvent@@@Z 00468cd0 f   QtGui4:QtGui4.dll
 0001:00067cd6       ?dragEnterEvent@QLineEdit@@MAEXPAVQDragEnterEvent@@@Z 00468cd6 f   QtGui4:QtGui4.dll
 0001:00067cdc       ?dragMoveEvent@QLineEdit@@MAEXPAVQDragMoveEvent@@@Z 00468cdc f   QtGui4:QtGui4.dll
 0001:00067ce2       ?dragLeaveEvent@QLineEdit@@MAEXPAVQDragLeaveEvent@@@Z 00468ce2 f   QtGui4:QtGui4.dll
 0001:00067ce8       ?dropEvent@QLineEdit@@MAEXPAVQDropEvent@@@Z 00468ce8 f   QtGui4:QtGui4.dll
 0001:00067cee       ?changeEvent@QLineEdit@@MAEXPAVQEvent@@@Z 00468cee f   QtGui4:QtGui4.dll
 0001:00067cf4       ?inputMethodEvent@QLineEdit@@MAEXPAVQInputMethodEvent@@@Z 00468cf4 f   QtGui4:QtGui4.dll
 0001:00067cfa       ?inputMethodQuery@QLineEdit@@UBE?AVQVariant@@W4InputMethodQuery@Qt@@@Z 00468cfa f   QtGui4:QtGui4.dll
 0001:00067d00       ?event@QComboBox@@UAE_NPAVQEvent@@@Z 00468d00 f   QtGui4:QtGui4.dll
 0001:00067d06       ?sizeHint@QComboBox@@UBE?AVQSize@@XZ 00468d06 f   QtGui4:QtGui4.dll
 0001:00067d0c       ?minimumSizeHint@QComboBox@@UBE?AVQSize@@XZ 00468d0c f   QtGui4:QtGui4.dll
 0001:00067d12       ?mousePressEvent@QComboBox@@MAEXPAVQMouseEvent@@@Z 00468d12 f   QtGui4:QtGui4.dll
 0001:00067d18       ?mouseReleaseEvent@QComboBox@@MAEXPAVQMouseEvent@@@Z 00468d18 f   QtGui4:QtGui4.dll
 0001:00067d1e       ?wheelEvent@QComboBox@@MAEXPAVQWheelEvent@@@Z 00468d1e f   QtGui4:QtGui4.dll
 0001:00067d24       ?keyPressEvent@QComboBox@@MAEXPAVQKeyEvent@@@Z 00468d24 f   QtGui4:QtGui4.dll
 0001:00067d2a       ?keyReleaseEvent@QComboBox@@MAEXPAVQKeyEvent@@@Z 00468d2a f   QtGui4:QtGui4.dll
 0001:00067d30       ?focusInEvent@QComboBox@@MAEXPAVQFocusEvent@@@Z 00468d30 f   QtGui4:QtGui4.dll
 0001:00067d36       ?focusOutEvent@QComboBox@@MAEXPAVQFocusEvent@@@Z 00468d36 f   QtGui4:QtGui4.dll
 0001:00067d3c       ?paintEvent@QComboBox@@MAEXPAVQPaintEvent@@@Z 00468d3c f   QtGui4:QtGui4.dll
 0001:00067d42       ?resizeEvent@QComboBox@@MAEXPAVQResizeEvent@@@Z 00468d42 f   QtGui4:QtGui4.dll
 0001:00067d48       ?contextMenuEvent@QComboBox@@MAEXPAVQContextMenuEvent@@@Z 00468d48 f   QtGui4:QtGui4.dll
 0001:00067d4e       ?showEvent@QComboBox@@MAEXPAVQShowEvent@@@Z 00468d4e f   QtGui4:QtGui4.dll
 0001:00067d54       ?hideEvent@QComboBox@@MAEXPAVQHideEvent@@@Z 00468d54 f   QtGui4:QtGui4.dll
 0001:00067d5a       ?changeEvent@QComboBox@@MAEXPAVQEvent@@@Z 00468d5a f   QtGui4:QtGui4.dll
 0001:00067d60       ?inputMethodEvent@QComboBox@@MAEXPAVQInputMethodEvent@@@Z 00468d60 f   QtGui4:QtGui4.dll
 0001:00067d66       ?inputMethodQuery@QComboBox@@MBE?AVQVariant@@W4InputMethodQuery@Qt@@@Z 00468d66 f   QtGui4:QtGui4.dll
 0001:00067d6c       ?showPopup@QComboBox@@UAEXXZ 00468d6c f   QtGui4:QtGui4.dll
 0001:00067d72       ?hidePopup@QComboBox@@UAEXXZ 00468d72 f   QtGui4:QtGui4.dll
 0001:00067d78       ?event@QRadioButton@@MAE_NPAVQEvent@@@Z 00468d78 f   QtGui4:QtGui4.dll
 0001:00067d7e       ?sizeHint@QRadioButton@@UBE?AVQSize@@XZ 00468d7e f   QtGui4:QtGui4.dll
 0001:00067d84       ?minimumSizeHint@QRadioButton@@UBE?AVQSize@@XZ 00468d84 f   QtGui4:QtGui4.dll
 0001:00067d8a       ?mouseMoveEvent@QRadioButton@@MAEXPAVQMouseEvent@@@Z 00468d8a f   QtGui4:QtGui4.dll
 0001:00067d90       ?paintEvent@QRadioButton@@MAEXPAVQPaintEvent@@@Z 00468d90 f   QtGui4:QtGui4.dll
 0001:00067d96       ?hitButton@QRadioButton@@MBE_NABVQPoint@@@Z 00468d96 f   QtGui4:QtGui4.dll
 0001:00067d9c       ?checkStateSet@QAbstractButton@@MAEXXZ 00468d9c f   QtGui4:QtGui4.dll
 0001:00067da2       ?nextCheckState@QAbstractButton@@MAEXXZ 00468da2 f   QtGui4:QtGui4.dll
 0001:00067da8       ?event@QPushButton@@MAE_NPAVQEvent@@@Z 00468da8 f   QtGui4:QtGui4.dll
 0001:00067dae       ?sizeHint@QPushButton@@UBE?AVQSize@@XZ 00468dae f   QtGui4:QtGui4.dll
 0001:00067db4       ?minimumSizeHint@QPushButton@@UBE?AVQSize@@XZ 00468db4 f   QtGui4:QtGui4.dll
 0001:00067dba       ?mouseMoveEvent@QAbstractButton@@MAEXPAVQMouseEvent@@@Z 00468dba f   QtGui4:QtGui4.dll
 0001:00067dc0       ?keyPressEvent@QPushButton@@MAEXPAVQKeyEvent@@@Z 00468dc0 f   QtGui4:QtGui4.dll
 0001:00067dc6       ?focusInEvent@QPushButton@@MAEXPAVQFocusEvent@@@Z 00468dc6 f   QtGui4:QtGui4.dll
 0001:00067dcc       ?focusOutEvent@QPushButton@@MAEXPAVQFocusEvent@@@Z 00468dcc f   QtGui4:QtGui4.dll
 0001:00067dd2       ?hitButton@QAbstractButton@@MBE_NABVQPoint@@@Z 00468dd2 f   QtGui4:QtGui4.dll
 0001:00067dd8       ?metaObject@QFrame@@UBEPBUQMetaObject@@XZ 00468dd8 f   QtGui4:QtGui4.dll
 0001:00067dde       ?event@QFrame@@MAE_NPAVQEvent@@@Z 00468dde f   QtGui4:QtGui4.dll
 0001:00067de4       ?sizeHint@QFrame@@UBE?AVQSize@@XZ 00468de4 f   QtGui4:QtGui4.dll
 0001:00067dea       ?paintEvent@QFrame@@MAEXPAVQPaintEvent@@@Z 00468dea f   QtGui4:QtGui4.dll
 0001:00067df0       ?insertItems@QComboBox@@QAEXHABVQStringList@@@Z 00468df0 f   QtGui4:QtGui4.dll
 0001:00067df6       ?clear@QComboBox@@QAEXXZ   00468df6 f   QtGui4:QtGui4.dll
 0001:00067dfc       ?setText@QLabel@@QAEXABVQString@@@Z 00468dfc f   QtGui4:QtGui4.dll
 0001:00067e02       ?setText@QAbstractButton@@QAEXABVQString@@@Z 00468e02 f   QtGui4:QtGui4.dll
 0001:00067e08       ??1QCheckBox@@UAE@XZ       00468e08 f   QtGui4:QtGui4.dll
 0001:00067e0e       ??1QLabel@@UAE@XZ          00468e0e f   QtGui4:QtGui4.dll
 0001:00067e14       ??1QFrame@@UAE@XZ          00468e14 f   QtGui4:QtGui4.dll
 0001:00067e1a       ?hide@QWidget@@QAEXXZ      00468e1a f   QtGui4:QtGui4.dll
 0001:00067e20       ?addItems@QComboBox@@QAEXABVQStringList@@@Z 00468e20 f   QtGui4:QtGui4.dll
 0001:00067e26       ?setText@QLineEdit@@QAEXABVQString@@@Z 00468e26 f   QtGui4:QtGui4.dll
 0001:00067e2c       ?currentIndex@QComboBox@@QBEHXZ 00468e2c f   QtGui4:QtGui4.dll
 0001:00067e32       ?isChecked@QAbstractButton@@QBE_NXZ 00468e32 f   QtGui4:QtGui4.dll
 0001:00067e38       ?currentText@QComboBox@@QBE?AVQString@@XZ 00468e38 f   QtGui4:QtGui4.dll
 0001:00067e3e       ?text@QLineEdit@@QBE?AVQString@@XZ 00468e3e f   QtGui4:QtGui4.dll
 0001:00067e44       ?setCurrentIndex@QComboBox@@QAEXH@Z 00468e44 f   QtGui4:QtGui4.dll
 0001:00067e4a       ?setItemData@QComboBox@@QAEXHABVQVariant@@H@Z 00468e4a f   QtGui4:QtGui4.dll
 0001:00067e50       ?count@QComboBox@@QBEHXZ   00468e50 f   QtGui4:QtGui4.dll
 0001:00067e56       ?addItem@QComboBox@@QAEXABVQString@@ABVQVariant@@@Z 00468e56 f   QtGui4:QtGui4.dll
 0001:00067e5c       ??1QSpacerItem@@UAE@XZ     00468e5c f   QtGui4:QtGui4.dll
 0001:00067e62       ?setSpacing@QListView@@QAEXH@Z 00468e62 f   QtGui4:QtGui4.dll
 0001:00067e68       ?addItem@QGridLayout@@QAEXPAVQLayoutItem@@HHHHV?$QFlags@W4AlignmentFlag@Qt@@@@@Z 00468e68 f   QtGui4:QtGui4.dll
 0001:00067e6e       ?setStretch@QBoxLayout@@QAEXHH@Z 00468e6e f   QtGui4:QtGui4.dll
 0001:00067e74       ?setFrameShadow@QFrame@@QAEXW4Shadow@1@@Z 00468e74 f   QtGui4:QtGui4.dll
 0001:00067e7a       ??0QListWidget@@QAE@PAVQWidget@@@Z 00468e7a f   QtGui4:QtGui4.dll
 0001:00067e80       ?setMargin@QLabel@@QAEXH@Z 00468e80 f   QtGui4:QtGui4.dll
 0001:00067e86       ?metaObject@QListWidget@@UBEPBUQMetaObject@@XZ 00468e86 f   QtGui4:QtGui4.dll
 0001:00067e8c       ?qt_metacast@QListWidget@@UAEPAXPBD@Z 00468e8c f   QtGui4:QtGui4.dll
 0001:00067e92       ?qt_metacall@QListWidget@@UAEHW4Call@QMetaObject@@HPAPAX@Z 00468e92 f   QtGui4:QtGui4.dll
 0001:00067e98       ?event@QListWidget@@MAE_NPAVQEvent@@@Z 00468e98 f   QtGui4:QtGui4.dll
 0001:00067e9e       ?timerEvent@QListView@@MAEXPAVQTimerEvent@@@Z 00468e9e f   QtGui4:QtGui4.dll
 0001:00067ea4       ?sizeHint@QAbstractScrollArea@@UBE?AVQSize@@XZ 00468ea4 f   QtGui4:QtGui4.dll
 0001:00067eaa       ?mousePressEvent@QAbstractItemView@@MAEXPAVQMouseEvent@@@Z 00468eaa f   QtGui4:QtGui4.dll
 0001:00067eb0       ?mouseReleaseEvent@QListView@@MAEXPAVQMouseEvent@@@Z 00468eb0 f   QtGui4:QtGui4.dll
 0001:00067eb6       ?mouseDoubleClickEvent@QAbstractItemView@@MAEXPAVQMouseEvent@@@Z 00468eb6 f   QtGui4:QtGui4.dll
 0001:00067ebc       ?mouseMoveEvent@QListView@@MAEXPAVQMouseEvent@@@Z 00468ebc f   QtGui4:QtGui4.dll
 0001:00067ec2       ?keyPressEvent@QAbstractItemView@@MAEXPAVQKeyEvent@@@Z 00468ec2 f   QtGui4:QtGui4.dll
 0001:00067ec8       ?focusInEvent@QAbstractItemView@@MAEXPAVQFocusEvent@@@Z 00468ec8 f   QtGui4:QtGui4.dll
 0001:00067ece       ?focusOutEvent@QAbstractItemView@@MAEXPAVQFocusEvent@@@Z 00468ece f   QtGui4:QtGui4.dll
 0001:00067ed4       ?paintEvent@QListView@@MAEXPAVQPaintEvent@@@Z 00468ed4 f   QtGui4:QtGui4.dll
 0001:00067eda       ?resizeEvent@QListView@@MAEXPAVQResizeEvent@@@Z 00468eda f   QtGui4:QtGui4.dll
 0001:00067ee0       ?dragEnterEvent@QAbstractItemView@@MAEXPAVQDragEnterEvent@@@Z 00468ee0 f   QtGui4:QtGui4.dll
 0001:00067ee6       ?dragMoveEvent@QListView@@MAEXPAVQDragMoveEvent@@@Z 00468ee6 f   QtGui4:QtGui4.dll
 0001:00067eec       ?dragLeaveEvent@QListView@@MAEXPAVQDragLeaveEvent@@@Z 00468eec f   QtGui4:QtGui4.dll
 0001:00067ef2       ?dropEvent@QListWidget@@UAEXPAVQDropEvent@@@Z 00468ef2 f   QtGui4:QtGui4.dll
 0001:00067ef8       ?inputMethodEvent@QAbstractItemView@@MAEXPAVQInputMethodEvent@@@Z 00468ef8 f   QtGui4:QtGui4.dll
 0001:00067efe       ?inputMethodQuery@QAbstractItemView@@UBE?AVQVariant@@W4InputMethodQuery@Qt@@@Z 00468efe f   QtGui4:QtGui4.dll
 0001:00067f04       ?focusNextPrevChild@QAbstractItemView@@MAE_N_N@Z 00468f04 f   QtGui4:QtGui4.dll
 0001:00067f0a       ?viewportEvent@QAbstractItemView@@MAE_NPAVQEvent@@@Z 00468f0a f   QtGui4:QtGui4.dll
 0001:00067f10       ?scrollContentsBy@QListView@@MAEXHH@Z 00468f10 f   QtGui4:QtGui4.dll
 0001:00067f16       ?setModel@QListWidget@@EAEXPAVQAbstractItemModel@@@Z 00468f16 f   QtGui4:QtGui4.dll
 0001:00067f1c       ?setSelectionModel@QAbstractItemView@@UAEXPAVQItemSelectionModel@@@Z 00468f1c f   QtGui4:QtGui4.dll
 0001:00067f22       ?keyboardSearch@QAbstractItemView@@UAEXABVQString@@@Z 00468f22 f   QtGui4:QtGui4.dll
 0001:00067f28       ?visualRect@QListView@@UBE?AVQRect@@ABVQModelIndex@@@Z 00468f28 f   QtGui4:QtGui4.dll
 0001:00067f2e       ?scrollTo@QListView@@UAEXABVQModelIndex@@W4ScrollHint@QAbstractItemView@@@Z 00468f2e f   QtGui4:QtGui4.dll
 0001:00067f34       ?indexAt@QListView@@UBE?AVQModelIndex@@ABVQPoint@@@Z 00468f34 f   QtGui4:QtGui4.dll
 0001:00067f3a       ?sizeHintForRow@QAbstractItemView@@UBEHH@Z 00468f3a f   QtGui4:QtGui4.dll
 0001:00067f40       ?sizeHintForColumn@QAbstractItemView@@UBEHH@Z 00468f40 f   QtGui4:QtGui4.dll
 0001:00067f46       ?reset@QListView@@UAEXXZ   00468f46 f   QtGui4:QtGui4.dll
 0001:00067f4c       ?setRootIndex@QListView@@UAEXABVQModelIndex@@@Z 00468f4c f   QtGui4:QtGui4.dll
 0001:00067f52       ?doItemsLayout@QListView@@UAEXXZ 00468f52 f   QtGui4:QtGui4.dll
 0001:00067f58       ?selectAll@QAbstractItemView@@UAEXXZ 00468f58 f   QtGui4:QtGui4.dll
 0001:00067f5e       ?edit@QAbstractItemView@@MAE_NABVQModelIndex@@W4EditTrigger@1@PAVQEvent@@@Z 00468f5e f   QtGui4:QtGui4.dll
 0001:00067f64       ?dataChanged@QListView@@MAEXABVQModelIndex@@0@Z 00468f64 f   QtGui4:QtGui4.dll
 0001:00067f6a       ?rowsInserted@QListView@@MAEXABVQModelIndex@@HH@Z 00468f6a f   QtGui4:QtGui4.dll
 0001:00067f70       ?rowsAboutToBeRemoved@QListView@@MAEXABVQModelIndex@@HH@Z 00468f70 f   QtGui4:QtGui4.dll
 0001:00067f76       ?selectionChanged@QListView@@MAEXABVQItemSelection@@0@Z 00468f76 f   QtGui4:QtGui4.dll
 0001:00067f7c       ?currentChanged@QListView@@MAEXABVQModelIndex@@0@Z 00468f7c f   QtGui4:QtGui4.dll
 0001:00067f82       ?updateEditorData@QAbstractItemView@@MAEXXZ 00468f82 f   QtGui4:QtGui4.dll
 0001:00067f88       ?updateEditorGeometries@QAbstractItemView@@MAEXXZ 00468f88 f   QtGui4:QtGui4.dll
 0001:00067f8e       ?updateGeometries@QListView@@MAEXXZ 00468f8e f   QtGui4:QtGui4.dll
 0001:00067f94       ?verticalScrollbarAction@QAbstractItemView@@MAEXH@Z 00468f94 f   QtGui4:QtGui4.dll
 0001:00067f9a       ?horizontalScrollbarAction@QAbstractItemView@@MAEXH@Z 00468f9a f   QtGui4:QtGui4.dll
 0001:00067fa0       ?verticalScrollbarValueChanged@QAbstractItemView@@MAEXH@Z 00468fa0 f   QtGui4:QtGui4.dll
 0001:00067fa6       ?horizontalScrollbarValueChanged@QAbstractItemView@@MAEXH@Z 00468fa6 f   QtGui4:QtGui4.dll
 0001:00067fac       ?closeEditor@QAbstractItemView@@MAEXPAVQWidget@@W4EndEditHint@QAbstractItemDelegate@@@Z 00468fac f   QtGui4:QtGui4.dll
 0001:00067fb2       ?commitData@QAbstractItemView@@MAEXPAVQWidget@@@Z 00468fb2 f   QtGui4:QtGui4.dll
 0001:00067fb8       ?editorDestroyed@QAbstractItemView@@MAEXPAVQObject@@@Z 00468fb8 f   QtGui4:QtGui4.dll
 0001:00067fbe       ?moveCursor@QListView@@MAE?AVQModelIndex@@W4CursorAction@QAbstractItemView@@V?$QFlags@W4KeyboardModifier@Qt@@@@@Z 00468fbe f   QtGui4:QtGui4.dll
 0001:00067fc4       ?horizontalOffset@QListView@@MBEHXZ 00468fc4 f   QtGui4:QtGui4.dll
 0001:00067fca       ?verticalOffset@QListView@@MBEHXZ 00468fca f   QtGui4:QtGui4.dll
 0001:00067fd0       ?isIndexHidden@QListView@@MBE_NABVQModelIndex@@@Z 00468fd0 f   QtGui4:QtGui4.dll
 0001:00067fd6       ?setSelection@QListView@@MAEXABVQRect@@V?$QFlags@W4SelectionFlag@QItemSelectionModel@@@@@Z 00468fd6 f   QtGui4:QtGui4.dll
 0001:00067fdc       ?visualRegionForSelection@QListView@@MBE?AVQRegion@@ABVQItemSelection@@@Z 00468fdc f   QtGui4:QtGui4.dll
 0001:00067fe2       ?selectedIndexes@QListView@@MBE?AV?$QList@VQModelIndex@@@@XZ 00468fe2 f   QtGui4:QtGui4.dll
 0001:00067fe8       ?selectionCommand@QAbstractItemView@@MBE?AV?$QFlags@W4SelectionFlag@QItemSelectionModel@@@@ABVQModelIndex@@PBVQEvent@@@Z 00468fe8 f   QtGui4:QtGui4.dll
 0001:00067fee       ?startDrag@QListView@@MAEXV?$QFlags@W4DropAction@Qt@@@@@Z 00468fee f   QtGui4:QtGui4.dll
 0001:00067ff4       ?viewOptions@QListView@@MBE?AVQStyleOptionViewItem@@XZ 00468ff4 f   QtGui4:QtGui4.dll
 0001:00067ffa       ?mimeTypes@QListWidget@@MBE?AVQStringList@@XZ 00468ffa f   QtGui4:QtGui4.dll
 0001:00068000       ?mimeData@QListWidget@@MBEPAVQMimeData@@V?$QList@PAVQListWidgetItem@@@@@Z 00469000 f   QtGui4:QtGui4.dll
 0001:00068006       ?dropMimeData@QListWidget@@MAE_NHPBVQMimeData@@W4DropAction@Qt@@@Z 00469006 f   QtGui4:QtGui4.dll
 0001:0006800c       ?supportedDropActions@QListWidget@@MBE?AV?$QFlags@W4DropAction@Qt@@@@XZ 0046900c f   QtGui4:QtGui4.dll
 0001:00068012       ??1QListWidget@@UAE@XZ     00469012 f   QtGui4:QtGui4.dll
 0001:00068018       ?setCheckable@QAbstractButton@@QAEX_N@Z 00469018 f   QtGui4:QtGui4.dll
 0001:0006801e       ?setItemWidget@QListWidget@@QAEXPAVQListWidgetItem@@PAVQWidget@@@Z 0046901e f   QtGui4:QtGui4.dll
 0001:00068024       ?setSizeHint@QListWidgetItem@@QAEXABVQSize@@@Z 00469024 f   QtGui4:QtGui4.dll
 0001:0006802a       ?item@QListWidget@@QBEPAVQListWidgetItem@@H@Z 0046902a f   QtGui4:QtGui4.dll
 0001:00068030       ?count@QListWidget@@QBEHXZ 00469030 f   QtGui4:QtGui4.dll
 0001:00068036       ?setToolTip@QWidget@@QAEXABVQString@@@Z 00469036 f   QtGui4:QtGui4.dll
 0001:0006803c       ?addItem@QListWidget@@QAEXABVQString@@@Z 0046903c f   QtGui4:QtGui4.dll
 0001:00068042       ??1QPushButton@@UAE@XZ     00469042 f   QtGui4:QtGui4.dll
 0001:00068048       ??0QPushButton@@QAE@PAVQWidget@@@Z 00469048 f   QtGui4:QtGui4.dll
 0001:0006804e       ?paintEvent@QPushButton@@MAEXPAVQPaintEvent@@@Z 0046904e f   QtGui4:QtGui4.dll
 0001:00068054       ?update@QWidget@@QAEXXZ    00469054 f   QtGui4:QtGui4.dll
 0001:0006805a       ?style@QWidget@@QBEPAVQStyle@@XZ 0046905a f   QtGui4:QtGui4.dll
 0001:00068060       ??1QImage@@UAE@XZ          00469060 f   QtGui4:QtGui4.dll
 0001:00068066       ??1QPixmap@@UAE@XZ         00469066 f   QtGui4:QtGui4.dll
 0001:0006806c       ?setPixmap@QLabel@@QAEXABVQPixmap@@@Z 0046906c f   QtGui4:QtGui4.dll
 0001:00068072       ?fromImage@QPixmap@@SA?AV1@ABVQImage@@V?$QFlags@W4ImageConversionFlag@Qt@@@@@Z 00469072 f   QtGui4:QtGui4.dll
 0001:00068078       ?scaled@QImage@@QBE?AV1@ABVQSize@@W4AspectRatioMode@Qt@@W4TransformationMode@4@@Z 00469078 f   QtGui4:QtGui4.dll
 0001:0006807e       ??0QImage@@QAE@ABVQString@@PBD@Z 0046907e f   QtGui4:QtGui4.dll
 0001:00068084       ?size@QWidget@@QBE?AVQSize@@XZ 00469084 f   QtGui4:QtGui4.dll
 0001:0006808a       ?clear@QLabel@@QAEXXZ      0046908a f   QtGui4:QtGui4.dll
 0001:00068090       ?clear@QListWidget@@QAEXXZ 00469090 f   QtGui4:QtGui4.dll
 0001:00068096       ?setLayout@QWidget@@QAEXPAVQLayout@@@Z 00469096 f   QtGui4:QtGui4.dll
 0001:0006809c       ??0QHBoxLayout@@QAE@PAVQWidget@@@Z 0046909c f   QtGui4:QtGui4.dll
 0001:000680a2       ?metaObject@QPushButton@@UBEPBUQMetaObject@@XZ 004690a2 f   QtGui4:QtGui4.dll
 0001:000680a8       ?setCurrentIndex@QStackedWidget@@QAEXH@Z 004690a8 f   QtGui4:QtGui4.dll
 0001:000680ae       ?addWidget@QStackedWidget@@QAEHPAVQWidget@@@Z 004690ae f   QtGui4:QtGui4.dll
 0001:000680b4       ?setMaximum@QSpinBox@@QAEXH@Z 004690b4 f   QtGui4:QtGui4.dll
 0001:000680ba       ?setOrientation@QAbstractSlider@@QAEXW4Orientation@Qt@@@Z 004690ba f   QtGui4:QtGui4.dll
 0001:000680c0       ?setPageStep@QAbstractSlider@@QAEXH@Z 004690c0 f   QtGui4:QtGui4.dll
 0001:000680c6       ?setMaximum@QAbstractSlider@@QAEXH@Z 004690c6 f   QtGui4:QtGui4.dll
 0001:000680cc       ?setLayoutDirection@QWidget@@QAEXW4LayoutDirection@Qt@@@Z 004690cc f   QtGui4:QtGui4.dll
 0001:000680d2       ??0QStackedWidget@@QAE@PAVQWidget@@@Z 004690d2 f   QtGui4:QtGui4.dll
 0001:000680d8       ?setAutoFillBackground@QWidget@@QAEX_N@Z 004690d8 f   QtGui4:QtGui4.dll
 0001:000680de       ?metaObject@QStackedWidget@@UBEPBUQMetaObject@@XZ 004690de f   QtGui4:QtGui4.dll
 0001:000680e4       ?qt_metacast@QStackedWidget@@UAEPAXPBD@Z 004690e4 f   QtGui4:QtGui4.dll
 0001:000680ea       ?qt_metacall@QStackedWidget@@UAEHW4Call@QMetaObject@@HPAPAX@Z 004690ea f   QtGui4:QtGui4.dll
 0001:000680f0       ?event@QStackedWidget@@MAE_NPAVQEvent@@@Z 004690f0 f   QtGui4:QtGui4.dll
 0001:000680f6       ?event@QSlider@@UAE_NPAVQEvent@@@Z 004690f6 f   QtGui4:QtGui4.dll
 0001:000680fc       ?timerEvent@QAbstractSlider@@MAEXPAVQTimerEvent@@@Z 004690fc f   QtGui4:QtGui4.dll
 0001:00068102       ?sizeHint@QSlider@@UBE?AVQSize@@XZ 00469102 f   QtGui4:QtGui4.dll
 0001:00068108       ?minimumSizeHint@QSlider@@UBE?AVQSize@@XZ 00469108 f   QtGui4:QtGui4.dll
 0001:0006810e       ?mouseMoveEvent@QSlider@@MAEXPAVQMouseEvent@@@Z 0046910e f   QtGui4:QtGui4.dll
 0001:00068114       ?wheelEvent@QAbstractSlider@@MAEXPAVQWheelEvent@@@Z 00469114 f   QtGui4:QtGui4.dll
 0001:0006811a       ?keyPressEvent@QAbstractSlider@@MAEXPAVQKeyEvent@@@Z 0046911a f   QtGui4:QtGui4.dll
 0001:00068120       ?paintEvent@QSlider@@MAEXPAVQPaintEvent@@@Z 00469120 f   QtGui4:QtGui4.dll
 0001:00068126       ?changeEvent@QAbstractSlider@@MAEXPAVQEvent@@@Z 00469126 f   QtGui4:QtGui4.dll
 0001:0006812c       ?sliderChange@QAbstractSlider@@MAEXW4SliderChange@1@@Z 0046912c f   QtGui4:QtGui4.dll
 0001:00068132       ??1QStackedWidget@@UAE@XZ  00469132 f   QtGui4:QtGui4.dll
 0001:00068138       ?setValue@QAbstractSlider@@QAEXH@Z 00469138 f   QtGui4:QtGui4.dll
 0001:0006813e       ?setValue@QSpinBox@@QAEXH@Z 0046913e f   QtGui4:QtGui4.dll
 0001:00068144       ?text@QAbstractSpinBox@@QBE?AVQString@@XZ 00469144 f   QtGui4:QtGui4.dll
 0001:0006814a       ?currentIndex@QStackedWidget@@QBEHXZ 0046914a f   QtGui4:QtGui4.dll
 0001:00068150       ?mapToGlobal@QWidget@@QBE?AVQPoint@@ABV2@@Z 00469150 f   QtGui4:QtGui4.dll
 0001:00068156       ?setAlignment@QLabel@@QAEXV?$QFlags@W4AlignmentFlag@Qt@@@@@Z 00469156 f   QtGui4:QtGui4.dll
 0001:0006815c       ?setSizeIncrement@QWidget@@QAEXABVQSize@@@Z 0046915c f   QtGui4:QtGui4.dll
 0001:00068162       ?setFlow@QListView@@QAEXW4Flow@1@@Z 00469162 f   QtGui4:QtGui4.dll
 0001:00068168       ?setAutoScrollMargin@QAbstractItemView@@QAEXH@Z 00469168 f   QtGui4:QtGui4.dll
 0001:0006816e       ?setLineWidth@QFrame@@QAEXH@Z 0046916e f   QtGui4:QtGui4.dll
 0001:00068174       ?takeItem@QListWidget@@QAEPAVQListWidgetItem@@H@Z 00469174 f   QtGui4:QtGui4.dll
 0001:0006817a       ?itemWidget@QListWidget@@QBEPAVQWidget@@PAVQListWidgetItem@@@Z 0046917a f   QtGui4:QtGui4.dll
 0001:00068180       ??1QTextEdit@@UAE@XZ       00469180 f   QtGui4:QtGui4.dll
 0001:00068186       ??1QPrinter@@UAE@XZ        00469186 f   QtGui4:QtGui4.dll
 0001:0006818c       ??1QPrintDialog@@UAE@XZ    0046918c f   QtGui4:QtGui4.dll
 0001:00068192       ?print@QTextDocument@@QBEXPAVQPrinter@@@Z 00469192 f   QtGui4:QtGui4.dll
 0001:00068198       ?document@QTextEdit@@QBEPAVQTextDocument@@XZ 00469198 f   QtGui4:QtGui4.dll
 0001:0006819e       ?setOutputFileName@QPrinter@@QAEXABVQString@@@Z 0046919e f   QtGui4:QtGui4.dll
 0001:000681a4       ?setOutputFormat@QPrinter@@QAEXW4OutputFormat@1@@Z 004691a4 f   QtGui4:QtGui4.dll
 0001:000681aa       ??0QPrintDialog@@QAE@PAVQPrinter@@PAVQWidget@@@Z 004691aa f   QtGui4:QtGui4.dll
 0001:000681b0       ?setPaperSize@QPrinter@@QAEXABVQSizeF@@W4Unit@1@@Z 004691b0 f   QtGui4:QtGui4.dll
 0001:000681b6       ?setPageSize@QPrinter@@QAEXW4PageSize@1@@Z 004691b6 f   QtGui4:QtGui4.dll
 0001:000681bc       ?setFullPage@QPrinter@@QAEX_N@Z 004691bc f   QtGui4:QtGui4.dll
 0001:000681c2       ??0QPrinter@@QAE@W4PrinterMode@0@@Z 004691c2 f   QtGui4:QtGui4.dll
 0001:000681c8       ?insertHtml@QTextEdit@@QAEXABVQString@@@Z 004691c8 f   QtGui4:QtGui4.dll
 0001:000681ce       ??0QTextEdit@@QAE@PAVQWidget@@@Z 004691ce f   QtGui4:QtGui4.dll
 0001:000681d4       ?getSaveFileName@QFileDialog@@SA?AVQString@@PAVQWidget@@ABV2@11PAV2@V?$QFlags@W4Option@QFileDialog@@@@@Z 004691d4 f   QtGui4:QtGui4.dll
 0001:000681da       ??0QLabel@@QAE@ABVQString@@PAVQWidget@@V?$QFlags@W4WindowType@Qt@@@@@Z 004691da f   QtGui4:QtGui4.dll
 0001:000681e0       ?setScaledContents@QLabel@@QAEX_N@Z 004691e0 f   QtGui4:QtGui4.dll
 0001:000681e6       ?setContextMenuPolicy@QWidget@@QAEXW4ContextMenuPolicy@Qt@@@Z 004691e6 f   QtGui4:QtGui4.dll
 0001:000681ec       ?setSizeConstraint@QLayout@@QAEXW4SizeConstraint@1@@Z 004691ec f   QtGui4:QtGui4.dll
 0001:000681f2       ??0QToolButton@@QAE@PAVQWidget@@@Z 004691f2 f   QtGui4:QtGui4.dll
 0001:000681f8       ?metaObject@QToolButton@@UBEPBUQMetaObject@@XZ 004691f8 f   QtGui4:QtGui4.dll
 0001:000681fe       ?qt_metacast@QToolButton@@UAEPAXPBD@Z 004691fe f   QtGui4:QtGui4.dll
 0001:00068204       ?qt_metacall@QToolButton@@UAEHW4Call@QMetaObject@@HPAPAX@Z 00469204 f   QtGui4:QtGui4.dll
 0001:0006820a       ?event@QToolButton@@MAE_NPAVQEvent@@@Z 0046920a f   QtGui4:QtGui4.dll
 0001:00068210       ?timerEvent@QToolButton@@MAEXPAVQTimerEvent@@@Z 00469210 f   QtGui4:QtGui4.dll
 0001:00068216       ?sizeHint@QToolButton@@UBE?AVQSize@@XZ 00469216 f   QtGui4:QtGui4.dll
 0001:0006821c       ?minimumSizeHint@QToolButton@@UBE?AVQSize@@XZ 0046921c f   QtGui4:QtGui4.dll
 0001:00068222       ?mousePressEvent@QToolButton@@MAEXPAVQMouseEvent@@@Z 00469222 f   QtGui4:QtGui4.dll
 0001:00068228       ?mouseReleaseEvent@QToolButton@@MAEXPAVQMouseEvent@@@Z 00469228 f   QtGui4:QtGui4.dll
 0001:0006822e       ?enterEvent@QToolButton@@MAEXPAVQEvent@@@Z 0046922e f   QtGui4:QtGui4.dll
 0001:00068234       ?leaveEvent@QToolButton@@MAEXPAVQEvent@@@Z 00469234 f   QtGui4:QtGui4.dll
 0001:0006823a       ?paintEvent@QToolButton@@MAEXPAVQPaintEvent@@@Z 0046923a f   QtGui4:QtGui4.dll
 0001:00068240       ?actionEvent@QToolButton@@MAEXPAVQActionEvent@@@Z 00469240 f   QtGui4:QtGui4.dll
 0001:00068246       ?changeEvent@QToolButton@@MAEXPAVQEvent@@@Z 00469246 f   QtGui4:QtGui4.dll
 0001:0006824c       ?hitButton@QToolButton@@MBE_NABVQPoint@@@Z 0046924c f   QtGui4:QtGui4.dll
 0001:00068252       ?nextCheckState@QToolButton@@MAEXXZ 00469252 f   QtGui4:QtGui4.dll
 0001:00068258       ??1QToolButton@@UAE@XZ     00469258 f   QtGui4:QtGui4.dll
 0001:0006825e       ?setFocus@QWidget@@QAEXW4FocusReason@Qt@@@Z 0046925e f   QtGui4:QtGui4.dll
 0001:00068264       ??1QFontMetrics@@QAE@XZ    00469264 f   QtGui4:QtGui4.dll
 0001:0006826a       ?elidedText@QFontMetrics@@QBE?AVQString@@ABV2@W4TextElideMode@Qt@@HH@Z 0046926a f   QtGui4:QtGui4.dll
 0001:00068270       ?width@QFontMetrics@@QBEHABVQString@@H@Z 00469270 f   QtGui4:QtGui4.dll
 0001:00068276       ??0QFontMetrics@@QAE@ABVQFont@@@Z 00469276 f   QtGui4:QtGui4.dll
 0001:0006827c       ??0QRadioButton@@QAE@PAVQWidget@@@Z 0046927c f   QtGui4:QtGui4.dll
 0001:00068282       ??1QRadioButton@@UAE@XZ    00469282 f   QtGui4:QtGui4.dll
 0001:00068288       ?eventFilter@QDialog@@MAE_NPAVQObject@@PAVQEvent@@@Z 00469288 f   QtGui4:QtGui4.dll
 0001:0006828e       ?setVisible@QDialog@@UAEX_N@Z 0046928e f   QtGui4:QtGui4.dll
 0001:00068294       ?sizeHint@QDialog@@UBE?AVQSize@@XZ 00469294 f   QtGui4:QtGui4.dll
 0001:0006829a       ?minimumSizeHint@QDialog@@UBE?AVQSize@@XZ 0046929a f   QtGui4:QtGui4.dll
 0001:000682a0       ?keyPressEvent@QDialog@@MAEXPAVQKeyEvent@@@Z 004692a0 f   QtGui4:QtGui4.dll
 0001:000682a6       ?resizeEvent@QDialog@@MAEXPAVQResizeEvent@@@Z 004692a6 f   QtGui4:QtGui4.dll
 0001:000682ac       ?closeEvent@QDialog@@MAEXPAVQCloseEvent@@@Z 004692ac f   QtGui4:QtGui4.dll
 0001:000682b2       ?contextMenuEvent@QDialog@@MAEXPAVQContextMenuEvent@@@Z 004692b2 f   QtGui4:QtGui4.dll
 0001:000682b8       ?showEvent@QDialog@@MAEXPAVQShowEvent@@@Z 004692b8 f   QtGui4:QtGui4.dll
 0001:000682be       ?done@QDialog@@UAEXH@Z     004692be f   QtGui4:QtGui4.dll
 0001:000682c4       ?accept@QDialog@@UAEXXZ    004692c4 f   QtGui4:QtGui4.dll
 0001:000682ca       ?reject@QDialog@@UAEXXZ    004692ca f   QtGui4:QtGui4.dll
 0001:000682d0       ?setWordWrap@QLabel@@QAEX_N@Z 004692d0 f   QtGui4:QtGui4.dll
 0001:000682d6       ??0QImage@@QAE@PBD0@Z      004692d6 f   QtGui4:QtGui4.dll
 0001:000682dc       ??0QPixmap@@QAE@XZ         004692dc f   QtGui4:QtGui4.dll
 0001:000682e2       ?getOpenFileName@QFileDialog@@SA?AVQString@@PAVQWidget@@ABV2@11PAV2@V?$QFlags@W4Option@QFileDialog@@@@@Z 004692e2 f   QtGui4:QtGui4.dll
 0001:000682e8       ??1QDialog@@UAE@XZ         004692e8 f   QtGui4:QtGui4.dll
 0001:000682ee       ??0QDialog@@QAE@PAVQWidget@@V?$QFlags@W4WindowType@Qt@@@@@Z 004692ee f   QtGui4:QtGui4.dll
 0001:000682f4       ?scaled@QImage@@QBE?AV1@HHW4AspectRatioMode@Qt@@W4TransformationMode@3@@Z 004692f4 f   QtGui4:QtGui4.dll
 0001:000682fa       ?move@QWidget@@QAEXABVQPoint@@@Z 004692fa f   QtGui4:QtGui4.dll
 0001:00068300       ?setEnabled@QWidget@@QAEX_N@Z 00469300 f   QtGui4:QtGui4.dll
 0001:00068306       ?setIcon@QAbstractButton@@QAEXABVQIcon@@@Z 00469306 f   QtGui4:QtGui4.dll
 0001:0006830c       ?addSpacerItem@QBoxLayout@@QAEXPAVQSpacerItem@@@Z 0046930c f   QtGui4:QtGui4.dll
 0001:00068312       ?addStretch@QBoxLayout@@QAEXH@Z 00469312 f   QtGui4:QtGui4.dll
 0001:00068318       ??1QKeySequence@@QAE@XZ    00469318 f   QtGui4:QtGui4.dll
 0001:0006831e       ?setShortcut@QAbstractButton@@QAEXABVQKeySequence@@@Z 0046931e f   QtGui4:QtGui4.dll
 0001:00068324       ??0QKeySequence@@QAE@HHHH@Z 00469324 f   QtGui4:QtGui4.dll
 0001:0006832a       ?setFixedHeight@QWidget@@QAEXH@Z 0046932a f   QtGui4:QtGui4.dll
 0001:00068330       ?metaObject@QBoxLayout@@UBEPBUQMetaObject@@XZ 00469330 f   QtGui4:QtGui4.dll
 0001:00068336       ?qt_metacast@QBoxLayout@@UAEPAXPBD@Z 00469336 f   QtGui4:QtGui4.dll
 0001:0006833c       ?qt_metacall@QBoxLayout@@UAEHW4Call@QMetaObject@@HPAPAX@Z 0046933c f   QtGui4:QtGui4.dll
 0001:00068342       ?sizeHint@QWidgetItem@@UBE?AVQSize@@XZ 00469342 f   QtGui4:QtGui4.dll
 0001:00068348       ?minimumSize@QWidgetItem@@UBE?AVQSize@@XZ 00469348 f   QtGui4:QtGui4.dll
 0001:0006834e       ?maximumSize@QWidgetItem@@UBE?AVQSize@@XZ 0046934e f   QtGui4:QtGui4.dll
 0001:00068354       ?expandingDirections@QWidgetItem@@UBE?AV?$QFlags@W4Orientation@Qt@@@@XZ 00469354 f   QtGui4:QtGui4.dll
 0001:0006835a       ?geometry@QWidgetItem@@UBE?AVQRect@@XZ 0046935a f   QtGui4:QtGui4.dll
 0001:00068360       ?isEmpty@QWidgetItem@@UBE_NXZ 00469360 f   QtGui4:QtGui4.dll
 0001:00068366       ?hasHeightForWidth@QWidgetItem@@UBE_NXZ 00469366 f   QtGui4:QtGui4.dll
 0001:0006836c       ?heightForWidth@QWidgetItem@@UBEHH@Z 0046936c f   QtGui4:QtGui4.dll
 0001:00068372       ?widget@QWidgetItem@@UAEPAVQWidget@@XZ 00469372 f   QtGui4:QtGui4.dll
 0001:00068378       ?showMinimized@QWidget@@QAEXXZ 00469378 f   QtGui4:QtGui4.dll
 0001:0006837e       ?button@QMouseEvent@@QBE?AW4MouseButton@Qt@@XZ 0046937e f   QtGui4:QtGui4.dll
 0001:00068384       ??1QMenu@@UAE@XZ           00469384 f   QtGui4:QtGui4.dll
 0001:0006838a       ??0QMenu@@QAE@ABVQString@@PAVQWidget@@@Z 0046938a f   QtGui4:QtGui4.dll
 0001:00068390       ?timerEvent@QMenu@@MAEXPAVQTimerEvent@@@Z 00469390 f   QtGui4:QtGui4.dll
 0001:00068396       ?sizeHint@QMenu@@UBE?AVQSize@@XZ 00469396 f   QtGui4:QtGui4.dll
 0001:0006839c       ?mousePressEvent@QMenu@@MAEXPAVQMouseEvent@@@Z 0046939c f   QtGui4:QtGui4.dll
 0001:000683a2       ?mouseReleaseEvent@QMenu@@MAEXPAVQMouseEvent@@@Z 004693a2 f   QtGui4:QtGui4.dll
 0001:000683a8       ?mouseMoveEvent@QMenu@@MAEXPAVQMouseEvent@@@Z 004693a8 f   QtGui4:QtGui4.dll
 0001:000683ae       ?wheelEvent@QMenu@@MAEXPAVQWheelEvent@@@Z 004693ae f   QtGui4:QtGui4.dll
 0001:000683b4       ?keyPressEvent@QMenu@@MAEXPAVQKeyEvent@@@Z 004693b4 f   QtGui4:QtGui4.dll
 0001:000683ba       ?enterEvent@QMenu@@MAEXPAVQEvent@@@Z 004693ba f   QtGui4:QtGui4.dll
 0001:000683c0       ?leaveEvent@QMenu@@MAEXPAVQEvent@@@Z 004693c0 f   QtGui4:QtGui4.dll
 0001:000683c6       ?paintEvent@QMenu@@MAEXPAVQPaintEvent@@@Z 004693c6 f   QtGui4:QtGui4.dll
 0001:000683cc       ?actionEvent@QMenu@@MAEXPAVQActionEvent@@@Z 004693cc f   QtGui4:QtGui4.dll
 0001:000683d2       ?hideEvent@QMenu@@MAEXPAVQHideEvent@@@Z 004693d2 f   QtGui4:QtGui4.dll
 0001:000683d8       ?changeEvent@QMenu@@MAEXPAVQEvent@@@Z 004693d8 f   QtGui4:QtGui4.dll
 0001:000683de       ?focusNextPrevChild@QMenu@@MAE_N_N@Z 004693de f   QtGui4:QtGui4.dll
 0001:000683e4       ??0QMenu@@QAE@PAVQWidget@@@Z 004693e4 f   QtGui4:QtGui4.dll
 0001:000683ea       ?event@QMenu@@MAE_NPAVQEvent@@@Z 004693ea f   QtGui4:QtGui4.dll
 0001:000683f0       ?winId@QWidget@@QBEPAUHWND__@@XZ 004693f0 f   QtGui4:QtGui4.dll
 0001:000683f6       ?addMenu@QMenu@@QAEPAVQAction@@PAV1@@Z 004693f6 f   QtGui4:QtGui4.dll
 0001:000683fc       ?menuAction@QMenu@@QBEPAVQAction@@XZ 004693fc f   QtGui4:QtGui4.dll
 0001:00068402       ?setIcon@QMenu@@QAEXABVQIcon@@@Z 00469402 f   QtGui4:QtGui4.dll
 0001:00068408       ??1QPainter@@QAE@XZ        00469408 f   QtGui4:QtGui4.dll
 0001:0006840e       ??0QPixmap@@QAE@ABV0@@Z    0046940e f   QtGui4:QtGui4.dll
 0001:00068414       ?end@QPainter@@QAE_NXZ     00469414 f   QtGui4:QtGui4.dll
 0001:0006841a       ?drawPixmap@QPainter@@QAEXABVQRect@@ABVQPixmap@@0@Z 0046941a f   QtGui4:QtGui4.dll
 0001:00068420       ?height@QPixmap@@QBEHXZ    00469420 f   QtGui4:QtGui4.dll
 0001:00068426       ?width@QPixmap@@QBEHXZ     00469426 f   QtGui4:QtGui4.dll
 0001:0006842c       ?begin@QPainter@@QAE_NPAVQPaintDevice@@@Z 0046942c f   QtGui4:QtGui4.dll
 0001:00068432       ??0QPainter@@QAE@XZ        00469432 f   QtGui4:QtGui4.dll
 0001:00068438       ?fill@QPixmap@@QAEXABVQColor@@@Z 00469438 f   QtGui4:QtGui4.dll
 0001:0006843e       ??0QColor@@QAE@HHHH@Z      0046943e f   QtGui4:QtGui4.dll
 0001:00068444       ??0QPixmap@@QAE@ABVQSize@@@Z 00469444 f   QtGui4:QtGui4.dll
 0001:0006844a       ??1QProxyStyle@@UAE@XZ     0046944a f   QtGui4:QtGui4.dll
 0001:00068450       ?load@QPixmap@@QAE_NABVQString@@PBDV?$QFlags@W4ImageConversionFlag@Qt@@@@@Z 00469450 f   QtGui4:QtGui4.dll
 0001:00068456       ??0QProxyStyle@@QAE@PAVQStyle@@@Z 00469456 f   QtGui4:QtGui4.dll
 0001:0006845c       ?event@QProxyStyle@@MAE_NPAVQEvent@@@Z 0046945c f   QtGui4:QtGui4.dll
 0001:00068462       ?polish@QProxyStyle@@UAEXAAVQPalette@@@Z 00469462 f   QtGui4:QtGui4.dll
 0001:00068468       ?polish@QProxyStyle@@UAEXPAVQApplication@@@Z 00469468 f   QtGui4:QtGui4.dll
 0001:0006846e       ?polish@QProxyStyle@@UAEXPAVQWidget@@@Z 0046946e f   QtGui4:QtGui4.dll
 0001:00068474       ?unpolish@QProxyStyle@@UAEXPAVQApplication@@@Z 00469474 f   QtGui4:QtGui4.dll
 0001:0006847a       ?unpolish@QProxyStyle@@UAEXPAVQWidget@@@Z 0046947a f   QtGui4:QtGui4.dll
 0001:00068480       ?itemTextRect@QProxyStyle@@UBE?AVQRect@@ABVQFontMetrics@@ABV2@H_NABVQString@@@Z 00469480 f   QtGui4:QtGui4.dll
 0001:00068486       ?itemPixmapRect@QProxyStyle@@UBE?AVQRect@@ABV2@HABVQPixmap@@@Z 00469486 f   QtGui4:QtGui4.dll
 0001:0006848c       ?drawItemText@QProxyStyle@@UBEXPAVQPainter@@ABVQRect@@HABVQPalette@@_NABVQString@@W4ColorRole@4@@Z 0046948c f   QtGui4:QtGui4.dll
 0001:00068492       ?drawItemPixmap@QProxyStyle@@UBEXPAVQPainter@@ABVQRect@@HABVQPixmap@@@Z 00469492 f   QtGui4:QtGui4.dll
 0001:00068498       ?standardPalette@QProxyStyle@@UBE?AVQPalette@@XZ 00469498 f   QtGui4:QtGui4.dll
 0001:0006849e       ?subElementRect@QProxyStyle@@UBE?AVQRect@@W4SubElement@QStyle@@PBVQStyleOption@@PBVQWidget@@@Z 0046949e f   QtGui4:QtGui4.dll
 0001:000684a4       ?drawComplexControl@QProxyStyle@@UBEXW4ComplexControl@QStyle@@PBVQStyleOptionComplex@@PAVQPainter@@PBVQWidget@@@Z 004694a4 f   QtGui4:QtGui4.dll
 0001:000684aa       ?hitTestComplexControl@QProxyStyle@@UBE?AW4SubControl@QStyle@@W4ComplexControl@3@PBVQStyleOptionComplex@@ABVQPoint@@PBVQWidget@@@Z 004694aa f   QtGui4:QtGui4.dll
 0001:000684b0       ?subControlRect@QProxyStyle@@UBE?AVQRect@@W4ComplexControl@QStyle@@PBVQStyleOptionComplex@@W4SubControl@4@PBVQWidget@@@Z 004694b0 f   QtGui4:QtGui4.dll
 0001:000684b6       ?sizeFromContents@QProxyStyle@@UBE?AVQSize@@W4ContentsType@QStyle@@PBVQStyleOption@@ABV2@PBVQWidget@@@Z 004694b6 f   QtGui4:QtGui4.dll
 0001:000684bc       ?styleHint@QProxyStyle@@UBEHW4StyleHint@QStyle@@PBVQStyleOption@@PBVQWidget@@PAVQStyleHintReturn@@@Z 004694bc f   QtGui4:QtGui4.dll
 0001:000684c2       ?standardPixmap@QProxyStyle@@UBE?AVQPixmap@@W4StandardPixmap@QStyle@@PBVQStyleOption@@PBVQWidget@@@Z 004694c2 f   QtGui4:QtGui4.dll
 0001:000684c8       ?generatedIconPixmap@QProxyStyle@@UBE?AVQPixmap@@W4Mode@QIcon@@ABV2@PBVQStyleOption@@@Z 004694c8 f   QtGui4:QtGui4.dll
 0001:000684ce       ?drawPixmap@QPainter@@QAEXABVQRect@@ABVQPixmap@@@Z 004694ce f   QtGui4:QtGui4.dll
 0001:000684d4       ?drawPrimitive@QProxyStyle@@UBEXW4PrimitiveElement@QStyle@@PBVQStyleOption@@PAVQPainter@@PBVQWidget@@@Z 004694d4 f   QtGui4:QtGui4.dll
 0001:000684da       ?restore@QPainter@@QAEXXZ  004694da f   QtGui4:QtGui4.dll
 0001:000684e0       ?isNull@QPixmap@@QBE_NXZ   004694e0 f   QtGui4:QtGui4.dll
 0001:000684e6       ?save@QPainter@@QAEXXZ     004694e6 f   QtGui4:QtGui4.dll
 0001:000684ec       ?pixelMetric@QProxyStyle@@UBEHW4PixelMetric@QStyle@@PBVQStyleOption@@PBVQWidget@@@Z 004694ec f   QtGui4:QtGui4.dll
 0001:000684f2       ?drawControl@QProxyStyle@@UBEXW4ControlElement@QStyle@@PBVQStyleOption@@PAVQPainter@@PBVQWidget@@@Z 004694f2 f   QtGui4:QtGui4.dll
 0001:000684f8       ??1QStyleOptionMenuItem@@QAE@XZ 004694f8 f   QtGui4:QtGui4.dll
 0001:000684fe       ?setColor@QPalette@@QAEXW4ColorRole@1@ABVQColor@@@Z 004694fe f   QtGui4:QtGui4.dll
 0001:00068504       ??0QStyleOptionMenuItem@@QAE@ABV0@@Z 00469504 f   QtGui4:QtGui4.dll
 0001:0006850a       ?color@QBrush@@QBEABVQColor@@XZ 0046950a f   QtGui4:QtGui4.dll
 0001:00068510       ?light@QPalette@@QBEABVQBrush@@XZ 00469510 f   QtGui4:QtGui4.dll
 0001:00068516       ?setBold@QFont@@QAEX_N@Z   00469516 f   QtGui4:QtGui4.dll
 0001:0006851c       ??1QFontInfo@@QAE@XZ       0046951c f   QtGui4:QtGui4.dll
 0001:00068522       ?setPointSizeF@QFont@@QAEXN@Z 00469522 f   QtGui4:QtGui4.dll
 0001:00068528       ?pointSizeF@QFontInfo@@QBENXZ 00469528 f   QtGui4:QtGui4.dll
 0001:0006852e       ??0QFontInfo@@QAE@ABVQFont@@@Z 0046952e f   QtGui4:QtGui4.dll
 0001:00068534       ??0QFont@@QAE@ABV0@@Z      00469534 f   QtGui4:QtGui4.dll
 0001:0006853a       ?drawText@QPainter@@QAEXABVQRect@@HABVQString@@PAV2@@Z 0046953a f   QtGui4:QtGui4.dll
 0001:00068540       ??4QColor@@QAEAAV0@ABV0@@Z 00469540 f   QtGui4:QtGui4.dll
 0001:00068546       ??0QColor@@QAE@XZ          00469546 f   QtGui4:QtGui4.dll
 0001:0006854c       ?drawPixmap@QPainter@@QAEXABVQPoint@@ABVQPixmap@@@Z 0046954c f   QtGui4:QtGui4.dll
 0001:00068552       ??1QStyleOption@@QAE@XZ    00469552 f   QtGui4:QtGui4.dll
 0001:00068558       ?setBrush@QPalette@@QAEXW4ColorRole@1@ABVQBrush@@@Z 00469558 f   QtGui4:QtGui4.dll
 0001:0006855e       ??0QStyleOption@@QAE@ABV0@@Z 0046955e f   QtGui4:QtGui4.dll
 0001:00068564       ??4QPixmap@@QAEAAV0@ABV0@@Z 00469564 f   QtGui4:QtGui4.dll
 0001:0006856a       ?pixmap@QIcon@@QBE?AVQPixmap@@ABVQSize@@W4Mode@1@W4State@1@@Z 0046956a f   QtGui4:QtGui4.dll
 0001:00068570       ?iconSize@QComboBox@@QBE?AVQSize@@XZ 00469570 f   QtGui4:QtGui4.dll
 0001:00068576       ??1QStyleOptionButton@@QAE@XZ 00469576 f   QtGui4:QtGui4.dll
 0001:0006857c       ??4QStyleOption@@QAEAAV0@ABV0@@Z 0046957c f   QtGui4:QtGui4.dll
 0001:00068582       ??0QStyleOptionButton@@QAE@XZ 00469582 f   QtGui4:QtGui4.dll
 0001:00068588       ?isNull@QIcon@@QBE_NXZ     00469588 f   QtGui4:QtGui4.dll
 0001:0006858e       ?visualRect@QStyle@@SA?AVQRect@@W4LayoutDirection@Qt@@ABV2@1@Z 0046958e f   QtGui4:QtGui4.dll
 0001:00068594       ?fillRect@QPainter@@QAEXABVQRect@@ABVQColor@@@Z 00469594 f   QtGui4:QtGui4.dll
 0001:0006859a       ?drawLine@QPainter@@QAEXHHHH@Z 0046959a f   QtGui4:QtGui4.dll
 0001:000685a0       ?proxy@QStyle@@QBEPBV1@XZ  004695a0 f   QtGui4:QtGui4.dll
 0001:000685a6       ?setFont@QPainter@@QAEXABVQFont@@@Z 004695a6 f   QtGui4:QtGui4.dll
 0001:000685ac       ?drawRect@QPainter@@QAEXABVQRect@@@Z 004695ac f   QtGui4:QtGui4.dll
 0001:000685b2       ??1QBrush@@QAE@XZ          004695b2 f   QtGui4:QtGui4.dll
 0001:000685b8       ?setBrush@QPainter@@QAEXABVQBrush@@@Z 004695b8 f   QtGui4:QtGui4.dll
 0001:000685be       ??0QBrush@@QAE@ABVQColor@@W4BrushStyle@Qt@@@Z 004695be f   QtGui4:QtGui4.dll
 0001:000685c4       ?setPen@QPainter@@QAEXABVQColor@@@Z 004695c4 f   QtGui4:QtGui4.dll
 0001:000685ca       ?setBlue@QColor@@QAEXH@Z   004695ca f   QtGui4:QtGui4.dll
 0001:000685d0       ?blue@QColor@@QBEHXZ       004695d0 f   QtGui4:QtGui4.dll
 0001:000685d6       ?setGreen@QColor@@QAEXH@Z  004695d6 f   QtGui4:QtGui4.dll
 0001:000685dc       ?green@QColor@@QBEHXZ      004695dc f   QtGui4:QtGui4.dll
 0001:000685e2       ?setRed@QColor@@QAEXH@Z    004695e2 f   QtGui4:QtGui4.dll
 0001:000685e8       ?red@QColor@@QBEHXZ        004695e8 f   QtGui4:QtGui4.dll
 0001:000685ee       ??0QColor@@QAE@ABV0@@Z     004695ee f   QtGui4:QtGui4.dll
 0001:000685f4       ??0QSpinBox@@QAE@PAVQWidget@@@Z 004695f4 f   QtGui4:QtGui4.dll
 0001:000685fa       ?event@QSpinBox@@MAE_NPAVQEvent@@@Z 004695fa f   QtGui4:QtGui4.dll
 0001:00068600       ?timerEvent@QAbstractSpinBox@@MAEXPAVQTimerEvent@@@Z 00469600 f   QtGui4:QtGui4.dll
 0001:00068606       ?sizeHint@QAbstractSpinBox@@UBE?AVQSize@@XZ 00469606 f   QtGui4:QtGui4.dll
 0001:0006860c       ?minimumSizeHint@QAbstractSpinBox@@UBE?AVQSize@@XZ 0046960c f   QtGui4:QtGui4.dll
 0001:00068612       ?mousePressEvent@QAbstractSpinBox@@MAEXPAVQMouseEvent@@@Z 00469612 f   QtGui4:QtGui4.dll
 0001:00068618       ?mouseReleaseEvent@QAbstractSpinBox@@MAEXPAVQMouseEvent@@@Z 00469618 f   QtGui4:QtGui4.dll
 0001:0006861e       ?mouseMoveEvent@QAbstractSpinBox@@MAEXPAVQMouseEvent@@@Z 0046961e f   QtGui4:QtGui4.dll
 0001:00068624       ?wheelEvent@QAbstractSpinBox@@MAEXPAVQWheelEvent@@@Z 00469624 f   QtGui4:QtGui4.dll
 0001:0006862a       ?keyPressEvent@QAbstractSpinBox@@MAEXPAVQKeyEvent@@@Z 0046962a f   QtGui4:QtGui4.dll
 0001:00068630       ?keyReleaseEvent@QAbstractSpinBox@@MAEXPAVQKeyEvent@@@Z 00469630 f   QtGui4:QtGui4.dll
 0001:00068636       ?focusInEvent@QAbstractSpinBox@@MAEXPAVQFocusEvent@@@Z 00469636 f   QtGui4:QtGui4.dll
 0001:0006863c       ?focusOutEvent@QAbstractSpinBox@@MAEXPAVQFocusEvent@@@Z 0046963c f   QtGui4:QtGui4.dll
 0001:00068642       ?paintEvent@QAbstractSpinBox@@MAEXPAVQPaintEvent@@@Z 00469642 f   QtGui4:QtGui4.dll
 0001:00068648       ?resizeEvent@QAbstractSpinBox@@MAEXPAVQResizeEvent@@@Z 00469648 f   QtGui4:QtGui4.dll
 0001:0006864e       ?closeEvent@QAbstractSpinBox@@MAEXPAVQCloseEvent@@@Z 0046964e f   QtGui4:QtGui4.dll
 0001:00068654       ?contextMenuEvent@QAbstractSpinBox@@MAEXPAVQContextMenuEvent@@@Z 00469654 f   QtGui4:QtGui4.dll
 0001:0006865a       ?showEvent@QAbstractSpinBox@@MAEXPAVQShowEvent@@@Z 0046965a f   QtGui4:QtGui4.dll
 0001:00068660       ?hideEvent@QAbstractSpinBox@@MAEXPAVQHideEvent@@@Z 00469660 f   QtGui4:QtGui4.dll
 0001:00068666       ?changeEvent@QAbstractSpinBox@@MAEXPAVQEvent@@@Z 00469666 f   QtGui4:QtGui4.dll
 0001:0006866c       ?inputMethodQuery@QAbstractSpinBox@@UBE?AVQVariant@@W4InputMethodQuery@Qt@@@Z 0046966c f   QtGui4:QtGui4.dll
 0001:00068672       ?validate@QSpinBox@@MBE?AW4State@QValidator@@AAVQString@@AAH@Z 00469672 f   QtGui4:QtGui4.dll
 0001:00068678       ?fixup@QSpinBox@@MBEXAAVQString@@@Z 00469678 f   QtGui4:QtGui4.dll
 0001:0006867e       ?stepBy@QAbstractSpinBox@@UAEXH@Z 0046967e f   QtGui4:QtGui4.dll
 0001:00068684       ?clear@QAbstractSpinBox@@UAEXXZ 00469684 f   QtGui4:QtGui4.dll
 0001:0006868a       ?stepEnabled@QAbstractSpinBox@@MBE?AV?$QFlags@W4StepEnabledFlag@QAbstractSpinBox@@@@XZ 0046968a f   QtGui4:QtGui4.dll
 0001:00068690       ?valueFromText@QSpinBox@@MBEHABVQString@@@Z 00469690 f   QtGui4:QtGui4.dll
 0001:00068696       ?textFromValue@QSpinBox@@MBE?AVQString@@H@Z 00469696 f   QtGui4:QtGui4.dll
 0001:0006869c       ??1QSpinBox@@UAE@XZ        0046969c f   QtGui4:QtGui4.dll
 0001:000686a2       ?setExpanding@QTabBar@@QAEX_N@Z 004696a2 f   QtGui4:QtGui4.dll
 0001:000686a8       ?tabBar@QTabWidget@@IBEPAVQTabBar@@XZ 004696a8 f   QtGui4:QtGui4.dll
 0001:000686ae       ??1QTabWidget@@UAE@XZ      004696ae f   QtGui4:QtGui4.dll
 0001:000686b4       ??0QTabWidget@@QAE@PAVQWidget@@@Z 004696b4 f   QtGui4:QtGui4.dll
 0001:000686ba       ?event@QTabWidget@@MAE_NPAVQEvent@@@Z 004696ba f   QtGui4:QtGui4.dll
 0001:000686c0       ?sizeHint@QTabWidget@@UBE?AVQSize@@XZ 004696c0 f   QtGui4:QtGui4.dll
 0001:000686c6       ?minimumSizeHint@QTabWidget@@UBE?AVQSize@@XZ 004696c6 f   QtGui4:QtGui4.dll
 0001:000686cc       ?heightForWidth@QTabWidget@@UBEHH@Z 004696cc f   QtGui4:QtGui4.dll
 0001:000686d2       ?keyPressEvent@QTabWidget@@MAEXPAVQKeyEvent@@@Z 004696d2 f   QtGui4:QtGui4.dll
 0001:000686d8       ?paintEvent@QTabWidget@@MAEXPAVQPaintEvent@@@Z 004696d8 f   QtGui4:QtGui4.dll
 0001:000686de       ?showEvent@QTabWidget@@MAEXPAVQShowEvent@@@Z 004696de f   QtGui4:QtGui4.dll
 0001:000686e4       ?changeEvent@QTabWidget@@MAEXPAVQEvent@@@Z 004696e4 f   QtGui4:QtGui4.dll
 0001:000686ea       ?tabInserted@QTabWidget@@MAEXH@Z 004696ea f   QtGui4:QtGui4.dll
 0001:000686f0       ?tabRemoved@QTabWidget@@MAEXH@Z 004696f0 f   QtGui4:QtGui4.dll
 0001:000686f6       ?resizeEvent@QTabWidget@@MAEXPAVQResizeEvent@@@Z 004696f6 f   QtGui4:QtGui4.dll
 0001:000686fc       ??1QWidgetAction@@UAE@XZ   004696fc f   QtGui4:QtGui4.dll
 0001:00068702       ?setDefaultWidget@QWidgetAction@@QAEXPAVQWidget@@@Z 00469702 f   QtGui4:QtGui4.dll
 0001:00068708       ??0QWidgetAction@@QAE@PAVQObject@@@Z 00469708 f   QtGui4:QtGui4.dll
 0001:0006870e       ?setFont@QWidget@@QAEXABVQFont@@@Z 0046970e f   QtGui4:QtGui4.dll
 0001:00068714       ?isVisible@QWidget@@QBE_NXZ 00469714 f   QtGui4:QtGui4.dll
 0001:0006871a       ?fill@QImage@@QAEXI@Z      0046971a f   QtGui4:QtGui4.dll
 0001:00068720       ?rgb@QColor@@QBEIXZ        00469720 f   QtGui4:QtGui4.dll
 0001:00068726       ??0QColor@@QAE@W4GlobalColor@Qt@@@Z 00469726 f   QtGui4:QtGui4.dll
 0001:0006872c       ??0QImage@@QAE@HHW4Format@0@@Z 0046972c f   QtGui4:QtGui4.dll
 0001:00068732       ?setIconSize@QAbstractButton@@QAEXABVQSize@@@Z 00469732 f   QtGui4:QtGui4.dll
 0001:00068738       ?setMargin@QLayout@@QAEXH@Z 00469738 f   QtGui4:QtGui4.dll
 0001:0006873e       ??0QPainter@@QAE@PAVQPaintDevice@@@Z 0046973e f   QtGui4:QtGui4.dll
 0001:00068744       ?init@QStyleOption@@QAEXPBVQWidget@@@Z 00469744 f   QtGui4:QtGui4.dll
 0001:0006874a       ??0QStyleOption@@QAE@HH@Z  0046974a f   QtGui4:QtGui4.dll
 0001:00068750       ?showMaximized@QWidget@@QAEXXZ 00469750 f   QtGui4:QtGui4.dll
 0001:00068756       ?showNormal@QWidget@@QAEXXZ 00469756 f   QtGui4:QtGui4.dll
 0001:0006875c       ?isMaximized@QWidget@@QBE_NXZ 0046975c f   QtGui4:QtGui4.dll
 0001:00068762       ??1QPolygon@@QAE@XZ        00469762 f   QtGui4:QtGui4.dll
 0001:00068768       ??0QPolygon@@QAE@XZ        00469768 f   QtGui4:QtGui4.dll
 0001:0006876e       ?pos@QMouseEvent@@QBEABVQPoint@@XZ 0046976e f   QtGui4:QtGui4.dll
 0001:00068774       ?drawPolyline@QPainter@@QAEXABVQPolygon@@@Z 00469774 f   QtGui4:QtGui4.dll
 0001:0006877a       ??1QPen@@QAE@XZ            0046977a f   QtGui4:QtGui4.dll
 0001:00068780       ?setPen@QPainter@@QAEXABVQPen@@@Z 00469780 f   QtGui4:QtGui4.dll
 0001:00068786       ??0QPen@@QAE@ABVQColor@@@Z 00469786 f   QtGui4:QtGui4.dll
 0001:0006878c       ??1QCursor@@QAE@XZ         0046978c f   QtGui4:QtGui4.dll
 0001:00068792       ?setCursor@QWidget@@QAEXABVQCursor@@@Z 00469792 f   QtGui4:QtGui4.dll
 0001:00068798       ??0QCursor@@QAE@ABVQPixmap@@HH@Z 00469798 f   QtGui4:QtGui4.dll
 0001:0006879e       ??0QPixmap@@QAE@ABVQString@@PBDV?$QFlags@W4ImageConversionFlag@Qt@@@@@Z 0046979e f   QtGui4:QtGui4.dll
 0001:000687a4       ??0QCursor@@QAE@W4CursorShape@Qt@@@Z 004697a4 f   QtGui4:QtGui4.dll
 0001:000687aa       ?currentColor@QColorDialog@@QBE?AVQColor@@XZ 004697aa f   QtGui4:QtGui4.dll
 0001:000687b0       ?setCurrentColor@QColorDialog@@QAEXABVQColor@@@Z 004697b0 f   QtGui4:QtGui4.dll
 0001:000687b6       ??0QColorDialog@@QAE@PAVQWidget@@@Z 004697b6 f   QtGui4:QtGui4.dll
 0001:000687bc       ?isEnabled@QWidget@@QBE_NXZ 004697bc f   QtGui4:QtGui4.dll
 0001:000687c2       ?metaObject@QColorDialog@@UBEPBUQMetaObject@@XZ 004697c2 f   QtGui4:QtGui4.dll
 0001:000687c8       ?qt_metacast@QColorDialog@@UAEPAXPBD@Z 004697c8 f   QtGui4:QtGui4.dll
 0001:000687ce       ?qt_metacall@QColorDialog@@UAEHW4Call@QMetaObject@@HPAPAX@Z 004697ce f   QtGui4:QtGui4.dll
 0001:000687d4       ?setVisible@QColorDialog@@UAEX_N@Z 004697d4 f   QtGui4:QtGui4.dll
 0001:000687da       ?changeEvent@QColorDialog@@MAEXPAVQEvent@@@Z 004697da f   QtGui4:QtGui4.dll
 0001:000687e0       ?done@QColorDialog@@MAEXH@Z 004697e0 f   QtGui4:QtGui4.dll
 0001:000687e6       ??1QColorDialog@@UAE@XZ    004697e6 f   QtGui4:QtGui4.dll
 0001:000687ec       ??0QPolygon@@QAE@ABV0@@Z   004697ec f   QtGui4:QtGui4.dll
 0001:000687f2       ??0QApplication@@QAE@AAHPAPAD_NH@Z 004697f2 f   QtGui4:QtGui4.dll
 0001:000687f8       ??0QApplication@@QAE@AAHPAPADH@Z 004697f8 f   QtGui4:QtGui4.dll
 0001:000687fe       ?event@QApplication@@MAE_NPAVQEvent@@@Z 004697fe f   QtGui4:QtGui4.dll
 0001:00068804       ?file@QFileOpenEvent@@QBE?AVQString@@XZ 00469804 f   QtGui4:QtGui4.dll
 0001:0006880a       ?activateWindow@QWidget@@QAEXXZ 0046980a f   QtGui4:QtGui4.dll
 0001:00068810       ?setWindowState@QWidget@@QAEXV?$QFlags@W4WindowState@Qt@@@@@Z 00469810 f   QtGui4:QtGui4.dll
 0001:00068816       ?windowState@QWidget@@QBE?AV?$QFlags@W4WindowState@Qt@@@@XZ 00469816 f   QtGui4:QtGui4.dll
 0001:0006881c       ?addItem@QListWidget@@QAEXPAVQListWidgetItem@@@Z 0046981c f   QtGui4:QtGui4.dll
 0001:00068822       ??1QDomElement@@QAE@XZ     00469822 f   QtXml4:QtXml4.dll
 0001:00068828       ??0QDomDocument@@QAE@XZ    00469828 f   QtXml4:QtXml4.dll
 0001:0006882e       ??0QDomElement@@QAE@XZ     0046982e f   QtXml4:QtXml4.dll
 0001:00068834       ??1QDomDocument@@QAE@XZ    00469834 f   QtXml4:QtXml4.dll
 0001:0006883a       ??4QDomElement@@QAEAAV0@ABV0@@Z 0046983a f   QtXml4:QtXml4.dll
 0001:00068840       ?documentElement@QDomDocument@@QBE?AVQDomElement@@XZ 00469840 f   QtXml4:QtXml4.dll
 0001:00068846       ?setContent@QDomDocument@@QAE_NPAVQIODevice@@PAVQString@@PAH2@Z 00469846 f   QtXml4:QtXml4.dll
 0001:0006884c       ?save@QDomNode@@QBEXAAVQTextStream@@H@Z 0046984c f   QtXml4:QtXml4.dll
 0001:00068852       ?isElement@QDomNode@@QBE_NXZ 00469852 f   QtXml4:QtXml4.dll
 0001:00068858       ??1QDomNode@@QAE@XZ        00469858 f   QtXml4:QtXml4.dll
 0001:0006885e       ??4QDomNode@@QAEAAV0@ABV0@@Z 0046985e f   QtXml4:QtXml4.dll
 0001:00068864       ?nextSibling@QDomNode@@QBE?AV1@XZ 00469864 f   QtXml4:QtXml4.dll
 0001:0006886a       ?firstChild@QDomNode@@QBE?AV1@XZ 0046986a f   QtXml4:QtXml4.dll
 0001:00068870       ?hasChildNodes@QDomNode@@QBE_NXZ 00469870 f   QtXml4:QtXml4.dll
 0001:00068876       ?isNull@QDomNode@@QBE_NXZ  00469876 f   QtXml4:QtXml4.dll
 0001:0006887c       ??4QDomDocument@@QAEAAV0@ABV0@@Z 0046987c f   QtXml4:QtXml4.dll
 0001:00068882       ?toElement@QDomNode@@QBE?AVQDomElement@@XZ 00469882 f   QtXml4:QtXml4.dll
 0001:00068888       ??0QDomDocument@@QAE@ABV0@@Z 00469888 f   QtXml4:QtXml4.dll
 0001:0006888e       ??0QDomElement@@QAE@ABV0@@Z 0046988e f   QtXml4:QtXml4.dll
 0001:00068894       ??1QDomNodeList@@QAE@XZ    00469894 f   QtXml4:QtXml4.dll
 0001:0006889a       ?item@QDomNodeList@@QBE?AVQDomNode@@H@Z 0046989a f   QtXml4:QtXml4.dll
 0001:000688a0       ?count@QDomNodeList@@QBEHXZ 004698a0 f   QtXml4:QtXml4.dll
 0001:000688a6       ?elementsByTagName@QDomElement@@QBE?AVQDomNodeList@@ABVQString@@@Z 004698a6 f   QtXml4:QtXml4.dll
 0001:000688ac       ?nodeName@QDomNode@@QBE?AVQString@@XZ 004698ac f   QtXml4:QtXml4.dll
 0001:000688b2       ?createElement@QDomDocument@@QAE?AVQDomElement@@ABVQString@@@Z 004698b2 f   QtXml4:QtXml4.dll
 0001:000688b8       ??1QDomProcessingInstruction@@QAE@XZ 004698b8 f   QtXml4:QtXml4.dll
 0001:000688be       ?appendChild@QDomNode@@QAE?AV1@ABV1@@Z 004698be f   QtXml4:QtXml4.dll
 0001:000688c4       ?createProcessingInstruction@QDomDocument@@QAE?AVQDomProcessingInstruction@@ABVQString@@0@Z 004698c4 f   QtXml4:QtXml4.dll
 0001:000688ca       ??0QDomNode@@QAE@ABV0@@Z   004698ca f   QtXml4:QtXml4.dll
 0001:000688d0       ?createTextNode@QDomDocument@@QAE?AVQDomText@@ABVQString@@@Z 004698d0 f   QtXml4:QtXml4.dll
 0001:000688d6       ??1QDomText@@QAE@XZ        004698d6 f   QtXml4:QtXml4.dll
 0001:000688dc       ?setData@QDomCharacterData@@QAEXABVQString@@@Z 004698dc f   QtXml4:QtXml4.dll
 0001:000688e2       ?toText@QDomNode@@QBE?AVQDomText@@XZ 004698e2 f   QtXml4:QtXml4.dll
 0001:000688e8       ?isText@QDomNode@@QBE_NXZ  004698e8 f   QtXml4:QtXml4.dll
 0001:000688ee       ?setAttribute@QDomElement@@QAEXABVQString@@0@Z 004698ee f   QtXml4:QtXml4.dll
 0001:000688f4       ?data@QDomCharacterData@@QBE?AVQString@@XZ 004698f4 f   QtXml4:QtXml4.dll
 0001:000688fa       ?attribute@QDomElement@@QBE?AVQString@@ABV2@0@Z 004698fa f   QtXml4:QtXml4.dll
 0001:00068900       ?removeChild@QDomNode@@QAE?AV1@ABV1@@Z 00469900 f   QtXml4:QtXml4.dll
 0001:00068906       ?tagName@QDomElement@@QBE?AVQString@@XZ 00469906 f   QtXml4:QtXml4.dll
 0001:0006890c       ?qt_metacast@CFancyTitle@iVMSGUIToolkit@@UAEPAXPBD@Z 0046990c f   iVMSGUIToolkit:iVMSGUIToolkit.dll
 0001:00068912       ?qt_metacall@CFancyTitle@iVMSGUIToolkit@@UAEHW4Call@QMetaObject@@HPAPAX@Z 00469912 f   iVMSGUIToolkit:iVMSGUIToolkit.dll
 0001:00068918       ?qt_metacast@CMenu@iVMSGUIToolkit@@UAEPAXPBD@Z 00469918 f   iVMSGUIToolkit:iVMSGUIToolkit.dll
 0001:0006891e       ?qt_metacall@CMenu@iVMSGUIToolkit@@UAEHW4Call@QMetaObject@@HPAPAX@Z 0046991e f   iVMSGUIToolkit:iVMSGUIToolkit.dll
 0001:00068924       ?GetTargetPathFile@iVMSGUIToolkit@@YA?AVQString@@ABV2@@Z 00469924 f   iVMSGUIToolkit:iVMSGUIToolkit.dll
 0001:0006892a       ?GetValue@CGenericDS@iVMSGUIToolkit@@QBE?AVQString@@XZ 0046992a f   iVMSGUIToolkit:iVMSGUIToolkit.dll
 0001:00068930       ??4CGenericDS@iVMSGUIToolkit@@QAEAAV01@ABV01@@Z 00469930 f   iVMSGUIToolkit:iVMSGUIToolkit.dll
 0001:00068936       ?GetChildByName@CGenericDS@iVMSGUIToolkit@@QBE?AV12@ABVQString@@@Z 00469936 f   iVMSGUIToolkit:iVMSGUIToolkit.dll
 0001:0006893c       ?GetName@CGenericDS@iVMSGUIToolkit@@QBE?AVQString@@XZ 0046993c f   iVMSGUIToolkit:iVMSGUIToolkit.dll
 0001:00068942       ?GetChild@CGenericDS@iVMSGUIToolkit@@QBE?AV12@H@Z 00469942 f   iVMSGUIToolkit:iVMSGUIToolkit.dll
 0001:00068948       ?GetChildrenCount@CGenericDS@iVMSGUIToolkit@@QBEHXZ 00469948 f   iVMSGUIToolkit:iVMSGUIToolkit.dll
 0001:0006894e       ??1CGenericDS@iVMSGUIToolkit@@QAE@XZ 0046994e f   iVMSGUIToolkit:iVMSGUIToolkit.dll
 0001:00068954       ?LoadXML@CGenericDS@iVMSGUIToolkit@@QAE_NABVQString@@@Z 00469954 f   iVMSGUIToolkit:iVMSGUIToolkit.dll
 0001:0006895a       ??0CGenericDS@iVMSGUIToolkit@@QAE@XZ 0046995a f   iVMSGUIToolkit:iVMSGUIToolkit.dll
 0001:00068960       ?SaveXML@CGenericDS@iVMSGUIToolkit@@QAE_NABVQString@@@Z 00469960 f   iVMSGUIToolkit:iVMSGUIToolkit.dll
 0001:00068966       ?SetValue@CGenericDS@iVMSGUIToolkit@@QAE_NABVQString@@@Z 00469966 f   iVMSGUIToolkit:iVMSGUIToolkit.dll
 0001:0006896c       ?GetTargetPath@iVMSGUIToolkit@@YA?AVQString@@XZ 0046996c f   iVMSGUIToolkit:iVMSGUIToolkit.dll
 0001:00068972       ?ReadAll@CFile@iVMSGUIToolkit@@SA?AVQString@@ABV3@@Z 00469972 f   iVMSGUIToolkit:iVMSGUIToolkit.dll
 0001:00068978       ?ReadAll@CFile@iVMSGUIToolkit@@SA?AVQString@@ABVQStringList@@ABV3@@Z 00469978 f   iVMSGUIToolkit:iVMSGUIToolkit.dll
 0001:0006897e       ?InitGuiLocale@iVMSGUIToolkit@@YAXABVQLocale@@@Z 0046997e f   iVMSGUIToolkit:iVMSGUIToolkit.dll
 0001:00068984       ?InitGuiTextCodec@iVMSGUIToolkit@@YAXPAVQTextCodec@@@Z 00469984 f   iVMSGUIToolkit:iVMSGUIToolkit.dll
 0001:0006898a       ??0CIntValidator@iVMSGUIToolkit@@QAE@HHPAVQObject@@@Z 0046998a f   iVMSGUIToolkit:iVMSGUIToolkit.dll
 0001:00068990       ?metaObject@CIntValidator@iVMSGUIToolkit@@UBEPBUQMetaObject@@XZ 00469990 f   iVMSGUIToolkit:iVMSGUIToolkit.dll
 0001:00068996       ?qt_metacast@CIntValidator@iVMSGUIToolkit@@UAEPAXPBD@Z 00469996 f   iVMSGUIToolkit:iVMSGUIToolkit.dll
 0001:0006899c       ?qt_metacall@CIntValidator@iVMSGUIToolkit@@UAEHW4Call@QMetaObject@@HPAPAX@Z 0046999c f   iVMSGUIToolkit:iVMSGUIToolkit.dll
 0001:000689a2       ?validate@CIntValidator@iVMSGUIToolkit@@UBE?AW4State@QValidator@@AAVQString@@AAH@Z 004699a2 f   iVMSGUIToolkit:iVMSGUIToolkit.dll
 0001:000689a8       ??0CPushButton@iVMSGUIToolkit@@QAE@PAVQWidget@@@Z 004699a8 f   iVMSGUIToolkit:iVMSGUIToolkit.dll
 0001:000689ae       ??0CRadioButton@iVMSGUIToolkit@@QAE@PAVQWidget@@@Z 004699ae f   iVMSGUIToolkit:iVMSGUIToolkit.dll
 0001:000689b4       ??0CComboBox@iVMSGUIToolkit@@QAE@PAVQWidget@@@Z 004699b4 f   iVMSGUIToolkit:iVMSGUIToolkit.dll
 0001:000689ba       ??0CLineEdit@iVMSGUIToolkit@@QAE@PAVQWidget@@@Z 004699ba f   iVMSGUIToolkit:iVMSGUIToolkit.dll
 0001:000689c0       ?metaObject@CLineEdit@iVMSGUIToolkit@@UBEPBUQMetaObject@@XZ 004699c0 f   iVMSGUIToolkit:iVMSGUIToolkit.dll
 0001:000689c6       ?qt_metacast@CLineEdit@iVMSGUIToolkit@@UAEPAXPBD@Z 004699c6 f   iVMSGUIToolkit:iVMSGUIToolkit.dll
 0001:000689cc       ?qt_metacall@CLineEdit@iVMSGUIToolkit@@UAEHW4Call@QMetaObject@@HPAPAX@Z 004699cc f   iVMSGUIToolkit:iVMSGUIToolkit.dll
 0001:000689d2       ?mousePressEvent@CLineEdit@iVMSGUIToolkit@@MAEXPAVQMouseEvent@@@Z 004699d2 f   iVMSGUIToolkit:iVMSGUIToolkit.dll
 0001:000689d8       ?focusInEvent@CLineEdit@iVMSGUIToolkit@@MAEXPAVQFocusEvent@@@Z 004699d8 f   iVMSGUIToolkit:iVMSGUIToolkit.dll
 0001:000689de       ?metaObject@CComboBox@iVMSGUIToolkit@@UBEPBUQMetaObject@@XZ 004699de f   iVMSGUIToolkit:iVMSGUIToolkit.dll
 0001:000689e4       ?qt_metacast@CComboBox@iVMSGUIToolkit@@UAEPAXPBD@Z 004699e4 f   iVMSGUIToolkit:iVMSGUIToolkit.dll
 0001:000689ea       ?qt_metacall@CComboBox@iVMSGUIToolkit@@UAEHW4Call@QMetaObject@@HPAPAX@Z 004699ea f   iVMSGUIToolkit:iVMSGUIToolkit.dll
 0001:000689f0       ?metaObject@CRadioButton@iVMSGUIToolkit@@UBEPBUQMetaObject@@XZ 004699f0 f   iVMSGUIToolkit:iVMSGUIToolkit.dll
 0001:000689f6       ?qt_metacast@CRadioButton@iVMSGUIToolkit@@UAEPAXPBD@Z 004699f6 f   iVMSGUIToolkit:iVMSGUIToolkit.dll
 0001:000689fc       ?qt_metacall@CRadioButton@iVMSGUIToolkit@@UAEHW4Call@QMetaObject@@HPAPAX@Z 004699fc f   iVMSGUIToolkit:iVMSGUIToolkit.dll
 0001:00068a02       ?metaObject@CPushButton@iVMSGUIToolkit@@UBEPBUQMetaObject@@XZ 00469a02 f   iVMSGUIToolkit:iVMSGUIToolkit.dll
 0001:00068a08       ?qt_metacast@CPushButton@iVMSGUIToolkit@@UAEPAXPBD@Z 00469a08 f   iVMSGUIToolkit:iVMSGUIToolkit.dll
 0001:00068a0e       ?qt_metacall@CPushButton@iVMSGUIToolkit@@UAEHW4Call@QMetaObject@@HPAPAX@Z 00469a0e f   iVMSGUIToolkit:iVMSGUIToolkit.dll
 0001:00068a14       ?enterEvent@CPushButton@iVMSGUIToolkit@@MAEXPAVQEvent@@@Z 00469a14 f   iVMSGUIToolkit:iVMSGUIToolkit.dll
 0001:00068a1a       ?leaveEvent@CPushButton@iVMSGUIToolkit@@MAEXPAVQEvent@@@Z 00469a1a f   iVMSGUIToolkit:iVMSGUIToolkit.dll
 0001:00068a20       ?paintEvent@CPushButton@iVMSGUIToolkit@@MAEXPAVQPaintEvent@@@Z 00469a20 f   iVMSGUIToolkit:iVMSGUIToolkit.dll
 0001:00068a26       ??1CLineEdit@iVMSGUIToolkit@@UAE@XZ 00469a26 f   iVMSGUIToolkit:iVMSGUIToolkit.dll
 0001:00068a2c       ??1CComboBox@iVMSGUIToolkit@@UAE@XZ 00469a2c f   iVMSGUIToolkit:iVMSGUIToolkit.dll
 0001:00068a32       ??1CRadioButton@iVMSGUIToolkit@@UAE@XZ 00469a32 f   iVMSGUIToolkit:iVMSGUIToolkit.dll
 0001:00068a38       ??1CPushButton@iVMSGUIToolkit@@UAE@XZ 00469a38 f   iVMSGUIToolkit:iVMSGUIToolkit.dll
 0001:00068a3e       ??1CIntValidator@iVMSGUIToolkit@@UAE@XZ 00469a3e f   iVMSGUIToolkit:iVMSGUIToolkit.dll
 0001:00068a44       ??0CSlider@iVMSGUIToolkit@@QAE@PAVQWidget@@@Z 00469a44 f   iVMSGUIToolkit:iVMSGUIToolkit.dll
 0001:00068a4a       ?metaObject@CSlider@iVMSGUIToolkit@@UBEPBUQMetaObject@@XZ 00469a4a f   iVMSGUIToolkit:iVMSGUIToolkit.dll
 0001:00068a50       ?qt_metacast@CSlider@iVMSGUIToolkit@@UAEPAXPBD@Z 00469a50 f   iVMSGUIToolkit:iVMSGUIToolkit.dll
 0001:00068a56       ?qt_metacall@CSlider@iVMSGUIToolkit@@UAEHW4Call@QMetaObject@@HPAPAX@Z 00469a56 f   iVMSGUIToolkit:iVMSGUIToolkit.dll
 0001:00068a5c       ?mousePressEvent@CSlider@iVMSGUIToolkit@@MAEXPAVQMouseEvent@@@Z 00469a5c f   iVMSGUIToolkit:iVMSGUIToolkit.dll
 0001:00068a62       ?mouseReleaseEvent@CSlider@iVMSGUIToolkit@@MAEXPAVQMouseEvent@@@Z 00469a62 f   iVMSGUIToolkit:iVMSGUIToolkit.dll
 0001:00068a68       ?enterEvent@CSlider@iVMSGUIToolkit@@MAEXPAVQEvent@@@Z 00469a68 f   iVMSGUIToolkit:iVMSGUIToolkit.dll
 0001:00068a6e       ?OnShowToolTip@CSlider@iVMSGUIToolkit@@MAEXH@Z 00469a6e f   iVMSGUIToolkit:iVMSGUIToolkit.dll
 0001:00068a74       ??1CSlider@iVMSGUIToolkit@@UAE@XZ 00469a74 f   iVMSGUIToolkit:iVMSGUIToolkit.dll
 0001:00068a7a       ??1CFancyTitle@iVMSGUIToolkit@@UAE@XZ 00469a7a f   iVMSGUIToolkit:iVMSGUIToolkit.dll
 0001:00068a80       ??0CFancyTitle@iVMSGUIToolkit@@QAE@PAVQWidget@@@Z 00469a80 f   iVMSGUIToolkit:iVMSGUIToolkit.dll
 0001:00068a86       ?mousePressEvent@CFancyTitle@iVMSGUIToolkit@@EAEXPAVQMouseEvent@@@Z 00469a86 f   iVMSGUIToolkit:iVMSGUIToolkit.dll
 0001:00068a8c       ?mouseReleaseEvent@CFancyTitle@iVMSGUIToolkit@@EAEXPAVQMouseEvent@@@Z 00469a8c f   iVMSGUIToolkit:iVMSGUIToolkit.dll
 0001:00068a92       ?mouseDoubleClickEvent@CFancyTitle@iVMSGUIToolkit@@EAEXPAVQMouseEvent@@@Z 00469a92 f   iVMSGUIToolkit:iVMSGUIToolkit.dll
 0001:00068a98       ?mouseMoveEvent@CFancyTitle@iVMSGUIToolkit@@EAEXPAVQMouseEvent@@@Z 00469a98 f   iVMSGUIToolkit:iVMSGUIToolkit.dll
 0001:00068a9e       ?resizeEvent@CFancyTitle@iVMSGUIToolkit@@EAEXPAVQResizeEvent@@@Z 00469a9e f   iVMSGUIToolkit:iVMSGUIToolkit.dll
 0001:00068aa4       ?SetOpenDoubleClickEnable@CFancyTitle@iVMSGUIToolkit@@QAEX_N@Z 00469aa4 f   iVMSGUIToolkit:iVMSGUIToolkit.dll
 0001:00068aaa       ?AddItem@CHBoxLayout@iVMSGUIToolkit@@QAEXPAVQLayoutItem@@H@Z 00469aaa f   iVMSGUIToolkit:iVMSGUIToolkit.dll
 0001:00068ab0       ??0CWidgetItem@iVMSGUIToolkit@@QAE@PAVQWidget@@V?$QFlags@W4AlignmentFlag@Qt@@@@@Z 00469ab0 f   iVMSGUIToolkit:iVMSGUIToolkit.dll
 0001:00068ab6       ?AddWidget@CHBoxLayout@iVMSGUIToolkit@@QAEXPAVQWidget@@@Z 00469ab6 f   iVMSGUIToolkit:iVMSGUIToolkit.dll
 0001:00068abc       ?SetLayoutSpacing@CHBoxLayout@iVMSGUIToolkit@@QAEXH@Z 00469abc f   iVMSGUIToolkit:iVMSGUIToolkit.dll
 0001:00068ac2       ?SetLayoutContentsMargins@CHBoxLayout@iVMSGUIToolkit@@QAEXHHHH@Z 00469ac2 f   iVMSGUIToolkit:iVMSGUIToolkit.dll
 0001:00068ac8       ??0CHBoxLayout@iVMSGUIToolkit@@QAE@PAVQWidget@@@Z 00469ac8 f   iVMSGUIToolkit:iVMSGUIToolkit.dll
 0001:00068ace       ?setGeometry@CWidgetItem@iVMSGUIToolkit@@UAEXABVQRect@@@Z 00469ace f   iVMSGUIToolkit:iVMSGUIToolkit.dll
 0001:00068ad4       ??1CHBoxLayout@iVMSGUIToolkit@@UAE@XZ 00469ad4 f   iVMSGUIToolkit:iVMSGUIToolkit.dll
 0001:00068ada       ??1CWidgetItem@iVMSGUIToolkit@@UAE@XZ 00469ada f   iVMSGUIToolkit:iVMSGUIToolkit.dll
 0001:00068ae0       ?GetIndependentWindow@iVMSGUIToolkit@@YAPAVQWidget@@PAV2@PBD@Z 00469ae0 f   iVMSGUIToolkit:iVMSGUIToolkit.dll
 0001:00068ae6       ?ShowMaximized@CWidgetSizeFactory@iVMSGUIToolkit@@QAEXPAVQWidget@@@Z 00469ae6 f   iVMSGUIToolkit:iVMSGUIToolkit.dll
 0001:00068aec       ?ShowNormal@CWidgetSizeFactory@iVMSGUIToolkit@@QAEXPAVQWidget@@ABVQSize@@@Z 00469aec f   iVMSGUIToolkit:iVMSGUIToolkit.dll
 0001:00068af2       ?IsMaximized@CWidgetSizeFactory@iVMSGUIToolkit@@QBE_NPAVQWidget@@@Z 00469af2 f   iVMSGUIToolkit:iVMSGUIToolkit.dll
 0001:00068af8       ?SignalWndSizeStatusChanged@CFancyTitle@iVMSGUIToolkit@@IAEXXZ 00469af8 f   iVMSGUIToolkit:iVMSGUIToolkit.dll
 0001:00068afe       ?IsFullScreen@CWidgetSizeFactory@iVMSGUIToolkit@@QBE_NPAVQWidget@@@Z 00469afe f   iVMSGUIToolkit:iVMSGUIToolkit.dll
 0001:00068b04       ??0CMenu@iVMSGUIToolkit@@QAE@PAVQWidget@@@Z 00469b04 f   iVMSGUIToolkit:iVMSGUIToolkit.dll
 0001:00068b0a       ??1CMenu@iVMSGUIToolkit@@UAE@XZ 00469b0a f   iVMSGUIToolkit:iVMSGUIToolkit.dll
 0001:00068b10       ??0QLocalServer@@QAE@PAVQObject@@@Z 00469b10 f   QtNetwork4:QtNetwork4.dll
 0001:00068b16       ?metaObject@QLocalServer@@UBEPBUQMetaObject@@XZ 00469b16 f   QtNetwork4:QtNetwork4.dll
 0001:00068b1c       ?qt_metacast@QLocalServer@@UAEPAXPBD@Z 00469b1c f   QtNetwork4:QtNetwork4.dll
 0001:00068b22       ?qt_metacall@QLocalServer@@UAEHW4Call@QMetaObject@@HPAPAX@Z 00469b22 f   QtNetwork4:QtNetwork4.dll
 0001:00068b28       ?hasPendingConnections@QLocalServer@@UBE_NXZ 00469b28 f   QtNetwork4:QtNetwork4.dll
 0001:00068b2e       ?nextPendingConnection@QLocalServer@@UAEPAVQLocalSocket@@XZ 00469b2e f   QtNetwork4:QtNetwork4.dll
 0001:00068b34       ?incomingConnection@QLocalServer@@MAEXI@Z 00469b34 f   QtNetwork4:QtNetwork4.dll
 0001:00068b3a       ??1QLocalServer@@UAE@XZ    00469b3a f   QtNetwork4:QtNetwork4.dll
 0001:00068b40       ?errorString@QLocalServer@@QBE?AVQString@@XZ 00469b40 f   QtNetwork4:QtNetwork4.dll
 0001:00068b46       ?listen@QLocalServer@@QAE_NABVQString@@@Z 00469b46 f   QtNetwork4:QtNetwork4.dll
 0001:00068b4c       ?removeServer@QLocalServer@@SA_NABVQString@@@Z 00469b4c f   QtNetwork4:QtNetwork4.dll
 0001:00068b52       ?waitForReadyRead@QLocalSocket@@UAE_NH@Z 00469b52 f   QtNetwork4:QtNetwork4.dll
 0001:00068b58       ?waitForBytesWritten@QLocalSocket@@UAE_NH@Z 00469b58 f   QtNetwork4:QtNetwork4.dll
 0001:00068b5e       ??1QLocalSocket@@UAE@XZ    00469b5e f   QtNetwork4:QtNetwork4.dll
 0001:00068b64       ?waitForConnected@QLocalSocket@@QAE_NH@Z 00469b64 f   QtNetwork4:QtNetwork4.dll
 0001:00068b6a       ?connectToServer@QLocalSocket@@QAEXABVQString@@V?$QFlags@W4OpenModeFlag@QIODevice@@@@@Z 00469b6a f   QtNetwork4:QtNetwork4.dll
 0001:00068b70       ??0QLocalSocket@@QAE@PAVQObject@@@Z 00469b70 f   QtNetwork4:QtNetwork4.dll
 0001:00068b76       ??1GenericDS@aptui@@UAE@XZ 00469b76 f   ToolGuiToolkit:ToolGuiToolkit.dll
 0001:00068b7c       ??0GenericDS@aptui@@QAE@XZ 00469b7c f   ToolGuiToolkit:ToolGuiToolkit.dll
 0001:00068b82       _ReleaseMutex@4            00469b82 f   kernel32:KERNEL32.dll
 0001:00068b88       _ReleaseSemaphore@12       00469b88 f   kernel32:KERNEL32.dll
 0001:00068b8e       _WaitForSingleObject@8     00469b8e f   kernel32:KERNEL32.dll
 0001:00068b94       _CreateMutexW@12           00469b94 f   kernel32:KERNEL32.dll
 0001:00068b9a       _GetLastError@0            00469b9a f   kernel32:KERNEL32.dll
 0001:00068ba0       _CreateSemaphoreW@16       00469ba0 f   kernel32:KERNEL32.dll
 0001:00068ba6       _LocalFree@4               00469ba6 f   kernel32:KERNEL32.dll
 0001:00068bac       _FormatMessageA@28         00469bac f   kernel32:KERNEL32.dll
 0001:00068bb2       _CloseHandle@4             00469bb2 f   kernel32:KERNEL32.dll
 0001:00068bb8       _GetCurrentProcessId@0     00469bb8 f   kernel32:KERNEL32.dll
 0001:00068bbe       _Sleep@4                   00469bbe f   kernel32:KERNEL32.dll
 0001:00068bc4       _SetClassLongW@12          00469bc4 f   user32:USER32.dll
 0001:00068bca       _GetClassLongW@8           00469bca f   user32:USER32.dll
 0001:00068bd0       ??1?$basic_string@DU?$char_traits@D@std@@V?$allocator@D@2@@std@@QAE@XZ 00469bd0 f   msvcprt:MSVCP90.dll
 0001:00068bd6       ?c_str@?$basic_string@DU?$char_traits@D@std@@V?$allocator@D@2@@std@@QBEPBDXZ 00469bd6 f   msvcprt:MSVCP90.dll
 0001:00068bdc       ??4_Init_locks@std@@QAEAAV01@ABV01@@Z 00469bdc f i msvcprt:nothrow.obj
 0001:00068be2       _strcmp                    00469be2 f   MSVCRT:MSVCR90.dll
 0001:00068be8       ___CxxFrameHandler3        00469be8 f   MSVCRT:MSVCR90.dll
 0001:00068bee       @__security_check_cookie@4 00469bee f   MSVCRT:secchk.obj
 0001:00068c00       ??3@YAXPAX@Z               00469c00 f   MSVCRT:MSVCR90.dll
 0001:00068c06       __CxxThrowException@8      00469c06 f   MSVCRT:MSVCR90.dll
 0001:00068c0c       ??2@YAPAXI@Z               00469c0c f   MSVCRT:MSVCR90.dll
 0001:00068c20       __ftol2_sse                00469c20 f   MSVCRT:ftol2.obj
 0001:00068c29       __ftol2_pentium4           00469c29 f   MSVCRT:ftol2.obj
 0001:00068c3c       __ftol2_sse_excpt          00469c3c f   MSVCRT:ftol2.obj
 0001:00068c56       __ftol2                    00469c56 f   MSVCRT:ftol2.obj
 0001:00068ccc       _pow                       00469ccc f   MSVCRT:MSVCR90.dll
 0001:00068cd2       _memcpy                    00469cd2 f   MSVCRT:MSVCR90.dll
 0001:00068cd8       ??0type_info@@AAE@ABV0@@Z  00469cd8 f   MSVCRT:ti_inst.obj
 0001:00068ce3       ??_Etype_info@@UAEPAXI@Z   00469ce3 f i MSVCRT:ti_inst.obj
 0001:00068d2f       ??4type_info@@AAEAAV0@ABV0@@Z 00469d2f f   MSVCRT:ti_inst.obj
 0001:00068d34       __onexit                   00469d34 f   MSVCRT:atonexit.obj
 0001:00068dd9       _atexit                    00469dd9 f   MSVCRT:atonexit.obj
 0001:00068df0       ??2@YAPAXIABUnothrow_t@std@@@Z 00469df0 f   MSVCRT:newopnt.obj
 0001:00068e20       _memset                    00469e20 f   MSVCRT:MSVCR90.dll
 0001:00068e26       ??3@YAXPAXABUnothrow_t@std@@@Z 00469e26 f   MSVCRT:delopnt.obj
 0001:00068e36       _memmove                   00469e36 f   MSVCRT:MSVCR90.dll
 0001:00068e3c       _ceil                      00469e3c f   MSVCRT:MSVCR90.dll
 0001:00068e42       ___RTDynamicCast           00469e42 f   MSVCRT:MSVCR90.dll
 0001:00068e48       _strlen                    00469e48 f   MSVCRT:MSVCR90.dll
 0001:00068e4e       _NtCurrentTeb              00469e4e f i MSVCRT:crtexew.obj
 0001:000691bf       _WinMainCRTStartup         0046a1bf f   MSVCRT:crtexew.obj
 0001:000691c9       ___report_gsfailure        0046a1c9 f   MSVCRT:gs_report.obj
 0001:0006931f       __get_sse2_info            0046a31f f   MSVCRT:cpu_disp.obj
 0001:00069381       ___sse2_available_init     0046a381 f   MSVCRT:cpu_disp.obj
 0001:000693a0       ?__ArrayUnwind@@YGXPAXIHP6EX0@Z@Z 0046a3a0 f   MSVCRT:ehvecdtr.obj
 0001:000693fe       ??_M@YGXPAXIHP6EX0@Z@Z     0046a3fe f   MSVCRT:ehvecdtr.obj
 0001:00069462       __unlock                   0046a462 f   MSVCRT:MSVCR90.dll
 0001:00069468       ___dllonexit               0046a468 f   MSVCRT:MSVCR90.dll
 0001:0006946e       __encode_pointer           0046a46e f   MSVCRT:MSVCR90.dll
 0001:00069474       __lock                     0046a474 f   MSVCRT:MSVCR90.dll
 0001:0006947a       __decode_pointer           0046a47a f   MSVCRT:MSVCR90.dll
 0001:00069480       __SEH_prolog4              0046a480 f   MSVCRT:sehprolg4.obj
 0001:000694c5       __SEH_epilog4              0046a4c5 f   MSVCRT:sehprolg4.obj
 0001:000694d9       __except_handler4          0046a4d9 f   MSVCRT:chandler4gs.obj
 0001:000694fe       __EH_prolog3               0046a4fe f   MSVCRT:ehprolg3.obj
 0001:00069531       __EH_prolog3_catch         0046a531 f   MSVCRT:ehprolg3.obj
 0001:00069567       __EH_prolog3_GS            0046a567 f   MSVCRT:ehprolg3.obj
 0001:0006959d       __EH_prolog3_catch_GS      0046a59d f   MSVCRT:ehprolg3.obj
 0001:000695d6       __EH_epilog3               0046a5d6 f   MSVCRT:ehprolg3.obj
 0001:000695ea       __EH_epilog3_GS            0046a5ea f   MSVCRT:ehprolg3.obj
 0001:000695f9       __EH_epilog3_catch_GS      0046a5f9 f   MSVCRT:ehprolg3.obj
 0001:00069608       ?__CxxUnhandledExceptionFilter@@YGJPAU_EXCEPTION_POINTERS@@@Z 0046a608 f   MSVCRT:unhandld.obj
 0001:0006964a       ___CxxSetUnhandledExceptionFilter 0046a64a f   MSVCRT:unhandld.obj
 0001:00069658       __amsg_exit                0046a658 f   MSVCRT:MSVCR90.dll
 0001:0006965e       ___getmainargs             0046a65e f   MSVCRT:MSVCR90.dll
 0001:00069664       __RTC_Initialize           0046a664 f   MSVCRT:_initsect_.obj
 0001:0006968a       __RTC_Terminate            0046a68a f   MSVCRT:_initsect_.obj
 0001:000696b0       __cexit                    0046a6b0 f   MSVCRT:MSVCR90.dll
 0001:000696b6       __exit                     0046a6b6 f   MSVCRT:MSVCR90.dll
 0001:000696bc       __XcptFilter               0046a6bc f   MSVCRT:MSVCR90.dll
 0001:000696c2       __ismbblead                0046a6c2 f   MSVCRT:MSVCR90.dll
 0001:000696c8       _exit                      0046a6c8 f   MSVCRT:MSVCR90.dll
 0001:000696d0       __ValidateImageBase        0046a6d0 f   MSVCRT:pesect.obj
 0001:00069710       __FindPESection            0046a710 f   MSVCRT:pesect.obj
 0001:00069760       __IsNonwritableInCurrentImage 0046a760 f   MSVCRT:pesect.obj
 0001:0006981e       __initterm                 0046a81e f   MSVCRT:MSVCR90.dll
 0001:00069824       __initterm_e               0046a824 f   MSVCRT:MSVCR90.dll
 0001:0006982a       __configthreadlocale       0046a82a f   MSVCRT:MSVCR90.dll
 0001:00069830       __invoke_watson_if_error   0046a830 f i MSVCRT:fp8.obj
 0001:00069854       __setdefaultprecision      0046a854 f   MSVCRT:fp8.obj
 0001:00069880       ___setusermatherr          0046a880 f   MSVCRT:MSVCR90.dll
 0001:00069886       __matherr                  0046a886 f   MSVCRT:merr.obj
 0001:00069889       __setargv                  0046a889 f   MSVCRT:dllargv.obj
 0001:0006988c       ___p__commode              0046a88c f   MSVCRT:MSVCR90.dll
 0001:00069892       ___p__fmode                0046a892 f   MSVCRT:MSVCR90.dll
 0001:00069898       ___set_app_type            0046a898 f   MSVCRT:MSVCR90.dll
 0001:0006989e       ___security_init_cookie    0046a89e f   MSVCRT:gs_support.obj
 0001:00069934       __crt_debugger_hook        0046a934 f   MSVCRT:MSVCR90.dll
 0001:0006993a       ?terminate@@YAXXZ          0046a93a f   MSVCRT:MSVCR90.dll
 0001:00069940       ?_type_info_dtor_internal_method@type_info@@QAEXXZ 0046a940 f   MSVCRT:MSVCR90.dll
 0001:00069940       ??1type_info@@UAE@XZ       0046a940 f   MSVCRT:MSVCR90.dll
 0001:00069946       __except_handler4_common   0046a946 f   MSVCRT:MSVCR90.dll
 0001:0006994c       __invoke_watson            0046a94c f   MSVCRT:MSVCR90.dll
 0001:00069952       __controlfp_s              0046a952 f   MSVCRT:MSVCR90.dll
 0001:00069960       ?alignOfTypedData@?$QVector@PAD@@ABEHXZ 0046a960 f i qtmain:qtmain_win.obj
 0001:00069970       ?free@?$QVectorTypedData@PAD@@SAXPAU1@H@Z 0046a970 f i qtmain:qtmain_win.obj
 0001:00069980       ?sizeOfTypedData@?$QVector@PAD@@AAEHXZ 0046a980 f i qtmain:qtmain_win.obj
 0001:00069990       ?free@?$QVector@PAD@@AAEXPAU?$QVectorTypedData@PAD@@@Z 0046a990 f i qtmain:qtmain_win.obj
 0001:000699b0       ?malloc@?$QVector@PAD@@AAEPAUQVectorData@@H@Z 0046a9b0 f i qtmain:qtmain_win.obj
 0001:000699e0       ?realloc@?$QVector@PAD@@AAEXHH@Z 0046a9e0 f i qtmain:qtmain_win.obj
 0001:00069b90       ??1?$QVector@PAD@@QAE@XZ   0046ab90 f i qtmain:qtmain_win.obj
 0001:00069bb0       ??0?$QVector@PAD@@QAE@H@Z  0046abb0 f i qtmain:qtmain_win.obj
 0001:00069c30       ?detach_helper@?$QVector@PAD@@AAEXXZ 0046ac30 f i qtmain:qtmain_win.obj
 0001:00069c40       ?detach@?$QVector@PAD@@QAEXXZ 0046ac40 f i qtmain:qtmain_win.obj
 0001:00069c60       ?data@?$QVector@PAD@@QAEPAPADXZ 0046ac60 f i qtmain:qtmain_win.obj
 0001:00069c90       _WinMain@16                0046ac90 f   qtmain:qtmain_win.obj
 0001:00069d92       ?qWinMain@@YAXPAUHINSTANCE__@@0PADHAAHAAV?$QVector@PAD@@@Z 0046ad92 f   QtCore4:QtCore4.dll
 0001:00069d98       ?detach@QByteArray@@QAEXXZ 0046ad98 f   QtCore4:QtCore4.dll
 0001:00069d9e       ?free@QString@@CAXPAUData@1@@Z 0046ad9e f   QtCore4:QtCore4.dll
 0001:00069da4       ?fromWCharArray@QString@@SA?AV1@PBGH@Z 0046ada4 f   QtCore4:QtCore4.dll
 0001:00069daa       _InterlockedExchange@8     0046adaa f   kernel32:KERNEL32.dll
 0001:00069db0       _InterlockedCompareExchange@12 0046adb0 f   kernel32:KERNEL32.dll
 0001:00069db6       _GetStartupInfoA@4         0046adb6 f   kernel32:KERNEL32.dll
 0001:00069dbc       _TerminateProcess@8        0046adbc f   kernel32:KERNEL32.dll
 0001:00069dc2       _GetCurrentProcess@0       0046adc2 f   kernel32:KERNEL32.dll
 0001:00069dc8       _UnhandledExceptionFilter@4 0046adc8 f   kernel32:KERNEL32.dll
 0001:00069dce       _SetUnhandledExceptionFilter@4 0046adce f   kernel32:KERNEL32.dll
 0001:00069dd4       _IsDebuggerPresent@0       0046add4 f   kernel32:KERNEL32.dll
 0001:00069dda       _QueryPerformanceCounter@4 0046adda f   kernel32:KERNEL32.dll
 0001:00069de0       _GetTickCount@0            0046ade0 f   kernel32:KERNEL32.dll
 0001:00069de6       _GetCurrentThreadId@0      0046ade6 f   kernel32:KERNEL32.dll
 0001:00069dec       _GetSystemTimeAsFileTime@4 0046adec f   kernel32:KERNEL32.dll
 0001:00069df2       _GetCommandLineW@0         0046adf2 f   kernel32:KERNEL32.dll
 0001:00078240       ??__Fm_mutex@?1??Instance@?$CUiSingleton@VConfigureManager@apt@@@iVMSGUIToolkit@@SAAAVConfigureManager@apt@@XZ@YAXXZ 00479240 f i ConfigManager.obj
 0001:00078260       ??__Fs_instance@?1??Instance@?$CUiSingleton@VConfigureManager@apt@@@iVMSGUIToolkit@@SAAAVConfigureManager@apt@@XZ@YAXXZ 00479260 f i ConfigManager.obj
 0001:000782a0       ??__Fm_mutex@?1??Instance@?$CUiSingleton@VLanaguageManager@apt@@@iVMSGUIToolkit@@SAAAVLanaguageManager@apt@@XZ@YAXXZ 004792a0 f i ToolsApplication.obj
 0001:000782c0       ??__Fs_instance@?1??Instance@?$CUiSingleton@VLanaguageManager@apt@@@iVMSGUIToolkit@@SAAAVLanaguageManager@apt@@XZ@YAXXZ 004792c0 f i ToolsApplication.obj
 0002:00000000       ___xc_a                    0047b000     MSVCRT:cinitexe.obj
 0002:000003cc       ___xc_z                    0047b3cc     MSVCRT:cinitexe.obj
 0002:000004d0       ___xi_a                    0047b4d0     MSVCRT:cinitexe.obj
 0002:000008e0       ___xi_z                    0047b8e0     MSVCRT:cinitexe.obj
 0002:00000ac8       ?staticMetaObjectExtraData@AboutDialog@@0UQMetaObjectExtraData@@B 0047bac8     moc_AboutDialog.obj
 0002:00000ad0       ?staticMetaObject@AboutDialog@@2UQMetaObject@@B 0047bad0     moc_AboutDialog.obj
 0002:00000d48       ?staticMetaObjectExtraData@BandWidthPage@@0UQMetaObjectExtraData@@B 0047bd48     moc_BandWidthPage.obj
 0002:00001208       ?staticMetaObjectExtraData@BaseDialog@aptui@@0UQMetaObjectExtraData@@B 0047c208     moc_BaseDialog.obj
 0002:0000159c       ?staticMetaObjectExtraData@BaseTitle@aptui@@0UQMetaObjectExtraData@@B 0047c59c     moc_BaseTitle.obj
 0002:00001680       ?staticMetaObjectExtraData@ButtonRadio@aptui@@0UQMetaObjectExtraData@@B 0047c680     moc_ButtonRadio.obj
 0002:00001784       ?staticMetaObjectExtraData@CapacityCalculation@@0UQMetaObjectExtraData@@B 0047c784     moc_CapacityCalculation.obj
 0002:0000180c       ?staticMetaObjectExtraData@CoverWidget@aptui@@0UQMetaObjectExtraData@@B 0047c80c     moc_CoverWidget.obj
 0002:00001814       ?staticMetaObject@CoverWidget@aptui@@2UQMetaObject@@B 0047c814     moc_CoverWidget.obj
 0002:00001b30       ?staticMetaObjectExtraData@DataCalculatorPage@@0UQMetaObjectExtraData@@B 0047cb30     moc_DataCalculatorPage.obj
 0002:00001c70       ?staticMetaObjectExtraData@DataDisplayPage@@0UQMetaObjectExtraData@@B 0047cc70     moc_DataDisplayPage.obj
 0002:000020a4       ?staticMetaObjectExtraData@DeviceAddPage@@0UQMetaObjectExtraData@@B 0047d0a4     moc_DeviceAddPage.obj
 0002:000025d0       ?staticMetaObjectExtraData@DeviceEditor@@0UQMetaObjectExtraData@@B 0047d5d0     moc_DeviceEditor.obj
 0002:00002708       ?staticMetaObjectExtraData@DeviceInfoManager@@0UQMetaObjectExtraData@@B 0047d708     moc_DeviceInfoManager.obj
 0002:000027f4       ?staticMetaObjectExtraData@DeviceItemWidget@NM_DiskCalculator@@0UQMetaObjectExtraData@@B 0047d7f4     moc_DeviceItemWidget.obj
 0002:00002b3c       ?staticMetaObjectExtraData@DiskCalculatorMainPage@@0UQMetaObjectExtraData@@B 0047db3c     moc_DiskCalculatorMainPage.obj
 0002:00002cb4       ?staticMetaObjectExtraData@CDlgAbout@aptui@@0UQMetaObjectExtraData@@B 0047dcb4     moc_DlgAbout.obj
 0002:00002e38       ?staticMetaObjectExtraData@Label@aptui@@0UQMetaObjectExtraData@@B 0047de38     moc_Label.obj
 0002:00002e90       ?staticMetaObjectExtraData@EditableLabel@aptui@@0UQMetaObjectExtraData@@B 0047de90     moc_Label.obj
 0002:00002e98       ?staticMetaObject@EditableLabel@aptui@@2UQMetaObject@@B 0047de98     moc_Label.obj
 0002:00002f20       ?staticMetaObjectExtraData@ColorLabel@aptui@@0UQMetaObjectExtraData@@B 0047df20     moc_Label.obj
 0002:00002f28       ?staticMetaObject@ColorLabel@aptui@@2UQMetaObject@@B 0047df28     moc_Label.obj
 0002:00002ffc       ?staticMetaObjectExtraData@Line@aptui@@0UQMetaObjectExtraData@@B 0047dffc     moc_Line.obj
 0002:0000306c       ?staticMetaObjectExtraData@LineEditInterger@aptui@@0UQMetaObjectExtraData@@B 0047e06c     moc_LineEditInterger.obj
 0002:000030d4       ?staticMetaObjectExtraData@Menu@aptui@@0UQMetaObjectExtraData@@B 0047e0d4     moc_Menu.obj
 0002:00003134       ?staticMetaObjectExtraData@CCustomStyle@Menu@aptui@@0UQMetaObjectExtraData@@B 0047e134     moc_Menu.obj
 0002:00003254       ?staticMetaObjectExtraData@MultiStatePushButton@aptui@@0UQMetaObjectExtraData@@B 0047e254     moc_MultiStatePushButton.obj
 0002:00003348       ?staticMetaObjectExtraData@QtLocalPeer@SharedTools@@0UQMetaObjectExtraData@@B 0047e348     moc_qtlocalpeer.obj
 0002:0000351c       ?staticMetaObjectExtraData@QtSingleApplication@SharedTools@@0UQMetaObjectExtraData@@B 0047e51c     moc_qtsingleapplication.obj
 0002:00003684       ?staticMetaObjectExtraData@QtSingleCoreApplication@SharedTools@@0UQMetaObjectExtraData@@B 0047e684     moc_qtsinglecoreapplication.obj
 0002:00003804       ?staticMetaObjectExtraData@ScenceSelector@@0UQMetaObjectExtraData@@B 0047e804     moc_ScenceSelector.obj
 0002:000038e0       ?staticMetaObjectExtraData@ScenceQRaidoButton@ScenceSelector@@0UQMetaObjectExtraData@@B 0047e8e0     moc_ScenceSelector.obj
 0002:000039e4       ?staticMetaObjectExtraData@SizeDisplayPage@@0UQMetaObjectExtraData@@B 0047e9e4     moc_SizeDisplayPage.obj
 0002:00003bb0       ?staticMetaObjectExtraData@Switch@aptui@@0UQMetaObjectExtraData@@B 0047ebb0     moc_Switch.obj
 0002:00003c5c       ?staticMetaObjectExtraData@TabWidget@aptui@@0UQMetaObjectExtraData@@B 0047ec5c     moc_TabWidget.obj
 0002:00003d50       ?staticMetaObjectExtraData@SystemMenu@aptui@@0UQMetaObjectExtraData@@B 0047ed50     moc_TitleMenu.obj
 0002:00003dd8       ?staticMetaObjectExtraData@ToolsApplication@apt@@0UQMetaObjectExtraData@@B 0047edd8     moc_ToolsApplication.obj
 0002:00003de0       ?staticMetaObject@ToolsApplication@apt@@2UQMetaObject@@B 0047ede0     moc_ToolsApplication.obj
 0002:00003ea0       ?staticMetaObjectExtraData@UpdateDialog@@0UQMetaObjectExtraData@@B 0047eea0     moc_UpdateDialog.obj
 0002:00003ea8       ?staticMetaObject@UpdateDialog@@2UQMetaObject@@B 0047eea8     moc_UpdateDialog.obj
 0002:00003f8c       ?staticMetaObjectExtraData@WarningDialog@NM_DiskCalculator@@0UQMetaObjectExtraData@@B 0047ef8c     moc_WarningDialog.obj
 0002:000040ac       ?staticMetaObjectExtraData@Widget@aptui@@0UQMetaObjectExtraData@@B 0047f0ac     moc_Widget.obj
 0002:0000413c       ?staticMetaObjectExtraData@WidgetDeviceListBorder@@0UQMetaObjectExtraData@@B 0047f13c     moc_WidgetDeviceListBorder.obj
 0002:00004294       ?staticMetaObjectExtraData@WindowTitle@aptui@@0UQMetaObjectExtraData@@B 0047f294     moc_WindowTitle.obj
 0002:0000431e       ?_Value@?$_Is_swap_move@U_Swap_move_tag@std@@@std@@2_NB 0047f31e     stdafx.obj
 0002:0000431f       ?value@?$integral_constant@_N$0A@@tr1@std@@2_NB 0047f31f     stdafx.obj
 0002:00004320       ?value@?$integral_constant@_N$00@tr1@std@@2_NB 0047f320     stdafx.obj
 0002:00004324       ?collate@?$_Locbase@H@std@@2HB 0047f324     stdafx.obj
 0002:00004328       ?ctype@?$_Locbase@H@std@@2HB 0047f328     stdafx.obj
 0002:0000432c       ?monetary@?$_Locbase@H@std@@2HB 0047f32c     stdafx.obj
 0002:00004330       ?numeric@?$_Locbase@H@std@@2HB 0047f330     stdafx.obj
 0002:00004334       ?time@?$_Locbase@H@std@@2HB 0047f334     stdafx.obj
 0002:00004338       ?messages@?$_Locbase@H@std@@2HB 0047f338     stdafx.obj
 0002:0000433c       ?all@?$_Locbase@H@std@@2HB 0047f33c     stdafx.obj
 0002:00004340       ?none@?$_Locbase@H@std@@2HB 0047f340     stdafx.obj
 0002:00004344       ?skipws@?$_Iosb@H@std@@2W4_Fmtflags@12@B 0047f344     stdafx.obj
 0002:00004348       ?unitbuf@?$_Iosb@H@std@@2W4_Fmtflags@12@B 0047f348     stdafx.obj
 0002:0000434c       ?uppercase@?$_Iosb@H@std@@2W4_Fmtflags@12@B 0047f34c     stdafx.obj
 0002:00004350       ?showbase@?$_Iosb@H@std@@2W4_Fmtflags@12@B 0047f350     stdafx.obj
 0002:00004354       ?showpoint@?$_Iosb@H@std@@2W4_Fmtflags@12@B 0047f354     stdafx.obj
 0002:00004358       ?showpos@?$_Iosb@H@std@@2W4_Fmtflags@12@B 0047f358     stdafx.obj
 0002:0000435c       ?left@?$_Iosb@H@std@@2W4_Fmtflags@12@B 0047f35c     stdafx.obj
 0002:00004360       ?right@?$_Iosb@H@std@@2W4_Fmtflags@12@B 0047f360     stdafx.obj
 0002:00004364       ?internal@?$_Iosb@H@std@@2W4_Fmtflags@12@B 0047f364     stdafx.obj
 0002:00004368       ?dec@?$_Iosb@H@std@@2W4_Fmtflags@12@B 0047f368     stdafx.obj
 0002:0000436c       ?oct@?$_Iosb@H@std@@2W4_Fmtflags@12@B 0047f36c     stdafx.obj
 0002:00004370       ?hex@?$_Iosb@H@std@@2W4_Fmtflags@12@B 0047f370     stdafx.obj
 0002:00004374       ?scientific@?$_Iosb@H@std@@2W4_Fmtflags@12@B 0047f374     stdafx.obj
 0002:00004378       ?fixed@?$_Iosb@H@std@@2W4_Fmtflags@12@B 0047f378     stdafx.obj
 0002:0000437c       ?hexfloat@?$_Iosb@H@std@@2W4_Fmtflags@12@B 0047f37c     stdafx.obj
 0002:00004380       ?boolalpha@?$_Iosb@H@std@@2W4_Fmtflags@12@B 0047f380     stdafx.obj
 0002:00004384       ?_Stdio@?$_Iosb@H@std@@2W4_Fmtflags@12@B 0047f384     stdafx.obj
 0002:00004388       ?adjustfield@?$_Iosb@H@std@@2W4_Fmtflags@12@B 0047f388     stdafx.obj
 0002:0000438c       ?basefield@?$_Iosb@H@std@@2W4_Fmtflags@12@B 0047f38c     stdafx.obj
 0002:00004390       ?floatfield@?$_Iosb@H@std@@2W4_Fmtflags@12@B 0047f390     stdafx.obj
 0002:00004394       ?goodbit@?$_Iosb@H@std@@2W4_Iostate@12@B 0047f394     stdafx.obj
 0002:00004398       ?eofbit@?$_Iosb@H@std@@2W4_Iostate@12@B 0047f398     stdafx.obj
 0002:0000439c       ?failbit@?$_Iosb@H@std@@2W4_Iostate@12@B 0047f39c     stdafx.obj
 0002:000043a0       ?badbit@?$_Iosb@H@std@@2W4_Iostate@12@B 0047f3a0     stdafx.obj
 0002:000043a4       ?_Hardfail@?$_Iosb@H@std@@2W4_Iostate@12@B 0047f3a4     stdafx.obj
 0002:000043a8       ?in@?$_Iosb@H@std@@2W4_Openmode@12@B 0047f3a8     stdafx.obj
 0002:000043ac       ?out@?$_Iosb@H@std@@2W4_Openmode@12@B 0047f3ac     stdafx.obj
 0002:000043b0       ?ate@?$_Iosb@H@std@@2W4_Openmode@12@B 0047f3b0     stdafx.obj
 0002:000043b4       ?app@?$_Iosb@H@std@@2W4_Openmode@12@B 0047f3b4     stdafx.obj
 0002:000043b8       ?trunc@?$_Iosb@H@std@@2W4_Openmode@12@B 0047f3b8     stdafx.obj
 0002:000043bc       ?_Nocreate@?$_Iosb@H@std@@2W4_Openmode@12@B 0047f3bc     stdafx.obj
 0002:000043c0       ?_Noreplace@?$_Iosb@H@std@@2W4_Openmode@12@B 0047f3c0     stdafx.obj
 0002:000043c4       ?binary@?$_Iosb@H@std@@2W4_Openmode@12@B 0047f3c4     stdafx.obj
 0002:000043c8       ?beg@?$_Iosb@H@std@@2W4_Seekdir@12@B 0047f3c8     stdafx.obj
 0002:000043cc       ?cur@?$_Iosb@H@std@@2W4_Seekdir@12@B 0047f3cc     stdafx.obj
 0002:000043d0       ?end@?$_Iosb@H@std@@2W4_Seekdir@12@B 0047f3d0     stdafx.obj
 0002:000046f0       __real@4022000000000000    0047f6f0     Calculate.obj
 0002:00004700       __real@3feccccccccccccd    0047f700     Calculate.obj
 0002:00004710       __real@3ff0000000000000    0047f710     Calculate.obj
 0002:00004720       __real@4024000000000000    0047f720     Calculate.obj
 0002:00004730       __real@0000000000000000    0047f730     Calculate.obj
 0002:00004740       __real@3ff0624dd2f1a9fc    0047f740     Calculate.obj
 0002:00004750       __real@3ff00c53318e81ed    0047f750     Calculate.obj
 0002:00004760       __real@415e848000000000    0047f760     Calculate.obj
 0002:00004770       __real@40ac200000000000    0047f770     Calculate.obj
 0002:00004780       __real@402e000000000000    0047f780     Calculate.obj
 0002:00004790       __real@3fb0000000000000    0047f790     Calculate.obj
 0002:000047a0       __real@402c000000000000    0047f7a0     Calculate.obj
 0002:000047b0       __real@3fc0000000000000    0047f7b0     Calculate.obj
 0002:000047c0       __real@402a000000000000    0047f7c0     Calculate.obj
 0002:000047d0       __real@3fd0000000000000    0047f7d0     Calculate.obj
 0002:000047e0       __real@4028000000000000    0047f7e0     Calculate.obj
 0002:000047f0       __real@3fe0000000000000    0047f7f0     Calculate.obj
 0002:00004800       __real@4014000000000000    0047f800     Calculate.obj
 0002:00004810       __real@4029000000000000    0047f810     Calculate.obj
 0002:00004820       __real@4026000000000000    0047f820     Calculate.obj
 0002:00004830       __real@4020000000000000    0047f830     Calculate.obj
 0002:00004840       __real@401c000000000000    0047f840     Calculate.obj
 0002:00004850       __real@4018000000000000    0047f850     Calculate.obj
 0002:00004860       __real@4010000000000000    0047f860     Calculate.obj
 0002:00004870       __real@4008000000000000    0047f870     Calculate.obj
 0002:00004880       __real@4000000000000000    0047f880     Calculate.obj
 0002:000048ed       ??_C@_00CNPNBAHC@?$AA@     0047f8ed     BitrateCalculate.obj
 0002:00004ba8       ??_7Configure@apt@@6B@     0047fba8     ConfigManager.obj
 0002:00004bb4       ??_7ConfigureManager@apt@@6B@ 0047fbb4     ConfigManager.obj
 0002:00004bc0       ??_7LanaguageManager@apt@@6B@ 0047fbc0     ConfigManager.obj
 0002:00004bcc       ??_SQTranslator@@6B@       0047fbcc     ConfigManager.obj
 0002:00004c10       ??_7?$CUiSingleton@VConfigureManager@apt@@@iVMSGUIToolkit@@6B@ 0047fc10     ConfigManager.obj
 0002:00004c1c       ??_7?$CUiSingleton@VLanaguageManager@apt@@@iVMSGUIToolkit@@6B@ 0047fc1c     ConfigManager.obj
 0002:00004f1c       ??_7ToolsApplication@apt@@6B@ 0047ff1c     ToolsApplication.obj
 0002:00004f6c       ??_C@_0BE@MEFFIPDM@com?4ISkinPlugin?11?41?$AA@ 0047ff6c     ToolsApplication.obj
 0002:000055ac       ??_7DiskCalculatorMainPage@@6BQPaintDevice@@@ 004805ac     DiskCalculatorMainPage.obj
 0002:000055d4       ??_7DiskCalculatorMainPage@@6BQObject@@@ 004805d4     DiskCalculatorMainPage.obj
 0002:000056cc       ??_C@_09CLANNNO@topLayout?$AA@ 004806cc     DiskCalculatorMainPage.obj
 0002:000056d8       ??_C@_0O@EGOAJBGL@m_boardLayout?$AA@ 004806d8     DiskCalculatorMainPage.obj
 0002:000056ec       ??_SQVBoxLayout@@6BQLayoutItem@@@ 004806ec     DiskCalculatorMainPage.obj
 0002:0000573c       ??_SQVBoxLayout@@6BQObject@@@ 0048073c     DiskCalculatorMainPage.obj
 0002:0000578c       ??_C@_0L@HFKHLBOD@gridLayout?$AA@ 0048078c     DiskCalculatorMainPage.obj
 0002:0000579c       ??_C@_0BJ@GIOELLGD@scrollAreaWidgetContents?$AA@ 0048079c     DiskCalculatorMainPage.obj
 0002:000057bc       ??_C@_0L@LLIJDPKF@scrollArea?$AA@ 004807bc     DiskCalculatorMainPage.obj
 0002:000057d0       ??_SQScrollArea@@6BQPaintDevice@@@ 004807d0     DiskCalculatorMainPage.obj
 0002:000057f4       ??_SQScrollArea@@6BQObject@@@ 004807f4     DiskCalculatorMainPage.obj
 0002:000058f0       ??_C@_0N@EDKFGLGO@gridLayout_2?$AA@ 004808f0     DiskCalculatorMainPage.obj
 0002:00005904       ??_SQGridLayout@@6BQLayoutItem@@@ 00480904     DiskCalculatorMainPage.obj
 0002:00005954       ??_SQGridLayout@@6BQObject@@@ 00480954     DiskCalculatorMainPage.obj
 0002:000059a4       ??_C@_0O@HKNJIMPD@centralWidget?$AA@ 004809a4     DiskCalculatorMainPage.obj
 0002:000059b8       ??_SQWidget@@6BQPaintDevice@@@ 004809b8     DiskCalculatorMainPage.obj
 0002:000059dc       ??_SQWidget@@6BQObject@@@  004809dc     DiskCalculatorMainPage.obj
 0002:00005acc       ??_C@_0BH@JNPINLCO@DiskCalculatorMainPage?$AA@ 00480acc     DiskCalculatorMainPage.obj
 0002:00005aec       ??_SQHBoxLayout@@6BQLayoutItem@@@ 00480aec     DiskCalculatorMainPage.obj
 0002:00005b3c       ??_SQHBoxLayout@@6BQObject@@@ 00480b3c     DiskCalculatorMainPage.obj
 0002:00005ca4       ??_7AboutDialog@@6B@       00480ca4     AboutDialog.obj
 0002:0000635c       ??_SCIntValidator@iVMSGUIToolkit@@6B@ 0048135c     DeviceEditor.obj
 0002:000063a4       ??_7DeviceEditor@@6BQPaintDevice@@@ 004813a4     DeviceEditor.obj
 0002:000063cc       ??_7DeviceEditor@@6BQObject@@@ 004813cc     DeviceEditor.obj
 0002:000064bc       ??_C@_0P@OKOIOHML@verticalLayout?$AA@ 004814bc     DeviceEditor.obj
 0002:000064d0       ??_C@_0O@DAPIDANK@verticalFrame?$AA@ 004814d0     DeviceEditor.obj
 0002:000064e4       ??_SQFrame@@6BQPaintDevice@@@ 004814e4     DeviceEditor.obj
 0002:0000650c       ??_SQFrame@@6BQObject@@@   0048150c     DeviceEditor.obj
 0002:000065fc       ??_C@_0P@CEOEGLF@m_btnAddDevice?$AA@ 004815fc     DeviceEditor.obj
 0002:00006614       ??_SCPushButton@iVMSGUIToolkit@@6BQPaintDevice@@@ 00481614     DeviceEditor.obj
 0002:0000663c       ??_SCPushButton@iVMSGUIToolkit@@6BQObject@@@ 0048163c     DeviceEditor.obj
 0002:0000673c       ??_C@_0BF@PCINLKC@m_comboBoxDeviceType?$AA@ 0048173c     DeviceEditor.obj
 0002:00006758       ??_C@_0BC@EEEGBGIA@m_lableDeviceType?$AA@ 00481758     DeviceEditor.obj
 0002:00006770       ??_C@_0BC@GALIIDEJ@verticalLayout_13?$AA@ 00481770     DeviceEditor.obj
 0002:00006788       ??_C@_0BG@LIEFLAID@m_lineEditChannelName?$AA@ 00481788     DeviceEditor.obj
 0002:000067a4       ??_C@_0BD@NCEPHBHC@horizontalLayout_3?$AA@ 004817a4     DeviceEditor.obj
 0002:000067bc       ??_C@_0BD@EEDBGJGJ@m_labelChannelName?$AA@ 004817bc     DeviceEditor.obj
 0002:000067d4       ??_C@_0BC@FCIOOBML@verticalLayout_11?$AA@ 004817d4     DeviceEditor.obj
 0002:000067ec       ??_C@_0BF@ICIPCLAP@m_radioButtonVarRate?$AA@ 004817ec     DeviceEditor.obj
 0002:00006808       ??_C@_0BH@JBAKEAMK@m_radioButtonFixedRate?$AA@ 00481808     DeviceEditor.obj
 0002:00006828       ??_SCRadioButton@iVMSGUIToolkit@@6BQPaintDevice@@@ 00481828     DeviceEditor.obj
 0002:0000684c       ??_SCRadioButton@iVMSGUIToolkit@@6BQObject@@@ 0048184c     DeviceEditor.obj
 0002:0000694c       ??_C@_05IDCCNNGI@label?$AA@ 0048194c     DeviceEditor.obj
 0002:00006954       ??_C@_0BD@MLFEEADD@horizontalLayout_2?$AA@ 00481954     DeviceEditor.obj
 0002:0000696c       ??_C@_0BE@IGEBCJEH@viewOrRecordingCmbx?$AA@ 0048196c     DeviceEditor.obj
 0002:00006984       ??_C@_07NPNGPBBI@label_2?$AA@ 00481984     DeviceEditor.obj
 0002:00006990       ??_C@_0BF@KGBIAOD@m_comboxEncodingType?$AA@ 00481990     DeviceEditor.obj
 0002:000069ac       ??_C@_0BH@DBGAIKKM@m_labelEncodeTypeLabel?$AA@ 004819ac     DeviceEditor.obj
 0002:000069c8       ??_C@_0BB@OBIHFKAP@verticalLayout_7?$AA@ 004819c8     DeviceEditor.obj
 0002:000069dc       ??_C@_0BF@FFFLKOIN@m_comboBoxResolution?$AA@ 004819dc     DeviceEditor.obj
 0002:000069f8       ??_C@_0BC@BODFGDKP@m_lableResolution?$AA@ 004819f8     DeviceEditor.obj
 0002:00006a10       ??_C@_0BB@NDLBDIIN@verticalLayout_5?$AA@ 00481a10     DeviceEditor.obj
 0002:00006a24       ??_C@_0BB@HJJEGAFK@m_scenceSelector?$AA@ 00481a24     DeviceEditor.obj
 0002:00006a38       ??_C@_0BO@CKPANNIM@m_lineEditScenceRecommandRate?$AA@ 00481a38     DeviceEditor.obj
 0002:00006a5c       ??_C@_0BL@BLMMFADI@m_labelScenceRecommandRate?$AA@ 00481a5c     DeviceEditor.obj
 0002:00006a7c       ??_C@_0BC@ELJFNAIK@verticalLayout_10?$AA@ 00481a7c     DeviceEditor.obj
 0002:00006a94       ??_C@_0BC@CEFCELAI@m_comboxFrameRate?$AA@ 00481a94     DeviceEditor.obj
 0002:00006ab0       ??_SCComboBox@iVMSGUIToolkit@@6BQPaintDevice@@@ 00481ab0     DeviceEditor.obj
 0002:00006ad4       ??_SCComboBox@iVMSGUIToolkit@@6BQObject@@@ 00481ad4     DeviceEditor.obj
 0002:00006bd0       ??_C@_0BB@OKKCHLFE@m_labelFrameRate?$AA@ 00481bd0     DeviceEditor.obj
 0002:00006be4       ??_C@_0BB@PIJMGLEO@verticalLayout_6?$AA@ 00481be4     DeviceEditor.obj
 0002:00006bf8       ??_C@_0N@MOEPNKJ@gridLayout_5?$AA@ 00481bf8     DeviceEditor.obj
 0002:00006c08       ??_C@_0O@IIHEFIMG@PalNtscSwitch?$AA@ 00481c08     DeviceEditor.obj
 0002:00006c18       ??_C@_0BC@HDEKIIDK@m_label_AddDevice?$AA@ 00481c18     DeviceEditor.obj
 0002:00006c30       ??_C@_0O@CJOIMKJI@m_labelStrech?$AA@ 00481c30     DeviceEditor.obj
 0002:00006c40       ??_C@_0BB@LNMDAGHP@horizontalLayout?$AA@ 00481c40     DeviceEditor.obj
 0002:00006c54       ??_C@_0BI@FAGJHBAK@m_lineEditChannelCounts?$AA@ 00481c54     DeviceEditor.obj
 0002:00006c74       ??_SCLineEdit@iVMSGUIToolkit@@6BQPaintDevice@@@ 00481c74     DeviceEditor.obj
 0002:00006c9c       ??_SCLineEdit@iVMSGUIToolkit@@6BQObject@@@ 00481c9c     DeviceEditor.obj
 0002:00006d8c       ??_C@_0BF@LPHPMGI@m_labelChannelCounts?$AA@ 00481d8c     DeviceEditor.obj
 0002:00006dac       ??_SQLabel@@6BQPaintDevice@@@ 00481dac     DeviceEditor.obj
 0002:00006dd4       ??_SQLabel@@6BQObject@@@   00481dd4     DeviceEditor.obj
 0002:00006ec4       ??_C@_0BC@HJKDLCAI@verticalLayout_12?$AA@ 00481ec4     DeviceEditor.obj
 0002:00006edc       ??_C@_0N@BFPPMMOI@gridLayout_4?$AA@ 00481edc     DeviceEditor.obj
 0002:00006eec       ??_C@_0BB@MKKKAJMM@verticalLayout_4?$AA@ 00481eec     DeviceEditor.obj
 0002:00006f00       ??_C@_0BK@HEPBKNGK@m_verticalWidgetAddBorder?$AA@ 00481f00     DeviceEditor.obj
 0002:00006f20       ??_C@_0N@FKLOFKCP@gridLayout_3?$AA@ 00481f20     DeviceEditor.obj
 0002:00006f30       ??_C@_0BB@HKILHLEA@m_checkBoxSpread?$AA@ 00481f30     DeviceEditor.obj
 0002:00006f48       ??_SQCheckBox@@6BQPaintDevice@@@ 00481f48     DeviceEditor.obj
 0002:00006f6c       ??_SQCheckBox@@6BQObject@@@ 00481f6c     DeviceEditor.obj
 0002:00007074       ??_SQSpacerItem@@6B@       00482074     DeviceEditor.obj
 0002:000070bc       ??_C@_0BB@JMPAKOEK@verticalLayout_2?$AA@ 004820bc     DeviceEditor.obj
 0002:000070d0       ??_C@_0P@LNFOBKHD@m_widgetShadow?$AA@ 004820d0     DeviceEditor.obj
 0002:000070e4       ??_C@_0BA@KNHDOGOF@m_TopGridLayout?$AA@ 004820e4     DeviceEditor.obj
 0002:000070f8       ??_C@_0DA@EFAHCELJ@QWideget?$CDDeviceEditor?$HL?6backgroun@ 004820f8     DeviceEditor.obj
 0002:00007134       ??_C@_0N@FAGFFPOA@DeviceEditor?$AA@ 00482134     DeviceEditor.obj
 0002:00007144       ??_C@_05IPHAHGKK@?$CL?5Add?$AA@ 00482144     DeviceEditor.obj
 0002:0000714c       ??_C@_0O@EDEIOMDC@Device?5Type?5?3?$AA@ 0048214c     DeviceEditor.obj
 0002:0000715c       ??_C@_0P@IPEHFMKN@Channel?5Name?5?3?$AA@ 0048215c     DeviceEditor.obj
 0002:00007170       ??_C@_07OIIEGCOP@VarRate?$AA@ 00482170     DeviceEditor.obj
 0002:0000717c       ??_C@_0L@KGGJEDHE@Fixed?5Rate?$AA@ 0048217c     DeviceEditor.obj
 0002:0000718c       ??_C@_0BJ@NMIKMKDP@Encode?5Section?5?3?5?5?5?5?5?5?5?5?$AA@ 0048218c     DeviceEditor.obj
 0002:000071ac       ??_C@_09MCPAPCCH@Live?5view?$AA@ 004821ac     DeviceEditor.obj
 0002:000071b8       ??_C@_09JAHJEAMH@Recording?$AA@ 004821b8     DeviceEditor.obj
 0002:000071c4       ??_C@_0BG@HFJJCGPJ@Live?5view?5?$CG?5Recording?$AA@ 004821c4     DeviceEditor.obj
 0002:000071e0       ??_C@_0P@HMKCBBNI@View?1Recording?$AA@ 004821e0     DeviceEditor.obj
 0002:000071f4       ??_C@_0BA@CMPPMMLB@Encoding?5Type?5?3?$AA@ 004821f4     DeviceEditor.obj
 0002:00007208       ??_C@_0BE@INGFDEJG@Device?5Resolution?5?3?$AA@ 00482208     DeviceEditor.obj
 0002:00007220       ??_C@_0BB@OBPDLAJP@Recommend?5Rate?5?3?$AA@ 00482220     DeviceEditor.obj
 0002:00007234       ??_C@_0BC@JIDLDAMN@Frame?5Rate?5?3?5?5?5?5?5?$AA@ 00482234     DeviceEditor.obj
 0002:0000724c       ??_C@_0L@CJJBBGDG@Add?5Device?$AA@ 0048224c     DeviceEditor.obj
 0002:0000725c       ??_C@_0BB@JFCMGBBG@Channel?5Counts?5?3?$AA@ 0048225c     DeviceEditor.obj
 0002:00007280       ??_7DeviceInfoManager@@6B@ 00482280     DeviceInfoManager.obj
 0002:00007408       ??_7ScenceSelector@@6BQPaintDevice@@@ 00482408     ScenceSelector.obj
 0002:0000742c       ??_7ScenceSelector@@6BQObject@@@ 0048242c     ScenceSelector.obj
 0002:0000751c       ??_C@_0O@IHFEEKGF@m_labelScence?$AA@ 0048251c     ScenceSelector.obj
 0002:0000752c       ??_C@_0BE@JIIOLPMC@m_listWidgetScences?$AA@ 0048252c     ScenceSelector.obj
 0002:00007548       ??_SQListWidget@@6BQPaintDevice@@@ 00482548     ScenceSelector.obj
 0002:0000756c       ??_SQListWidget@@6BQObject@@@ 0048256c     ScenceSelector.obj
 0002:00007730       ??_C@_0BD@CFHBPCPN@m_labelScenceImage?$AA@ 00482730     ScenceSelector.obj
 0002:00007748       ??_C@_0P@MIIFPHNM@ScenceSelector?$AA@ 00482748     ScenceSelector.obj
 0002:0000775c       ??_C@_07MHDHFKFB@Scence?3?$AA@ 0048275c     ScenceSelector.obj
 0002:00007768       ??_C@_0IB@CJHEJJPJ@?$DMhtml?$DO?$DMhead?1?$DO?$DMbody?$DO?$DMp?5align?$DN?$CCcen@ 00482768     ScenceSelector.obj
 0002:00007804       ??_C@_0L@OELOHDKG@2clicked?$CI?$CJ?$AA@ 00482804     ScenceSelector.obj
 0002:00007814       ??_C@_0BJ@EFOKOOFN@1OnScenceButtonClicked?$CI?$CJ?$AA@ 00482814     ScenceSelector.obj
 0002:00007838       ??_7ScenceQRaidoButton@ScenceSelector@@6BQPaintDevice@@@ 00482838     ScenceSelector.obj
 0002:0000785c       ??_7ScenceQRaidoButton@ScenceSelector@@6BQObject@@@ 0048285c     ScenceSelector.obj
 0002:000079a4       ??_7CapacityCalculation@@6BQPaintDevice@@@ 004829a4     CapacityCalculation.obj
 0002:000079cc       ??_7CapacityCalculation@@6BQObject@@@ 004829cc     CapacityCalculation.obj
 0002:00007abc       ??_C@_0BF@CFLIIEDB@m_dataCalculatorPage?$AA@ 00482abc     CapacityCalculation.obj
 0002:00007ad8       ??_C@_0N@JPIDGNDP@m_boardVline?$AA@ 00482ad8     CapacityCalculation.obj
 0002:00007ae8       ??_C@_0BA@FEAJDILG@m_deviceAddPage?$AA@ 00482ae8     CapacityCalculation.obj
 0002:00007afc       ??_C@_0BD@JHDDFIHA@m_widgetDeviceList?$AA@ 00482afc     CapacityCalculation.obj
 0002:00007b14       ??_C@_0N@KGFPAONE@m_boardHline?$AA@ 00482b14     CapacityCalculation.obj
 0002:00007b24       ??_C@_0L@ELMLBGMF@m_btnClear?$AA@ 00482b24     CapacityCalculation.obj
 0002:00007b34       ??_C@_09GCENGIDK@exportBtn?$AA@ 00482b34     CapacityCalculation.obj
 0002:00007b44       ??_SQPushButton@@6BQPaintDevice@@@ 00482b44     CapacityCalculation.obj
 0002:00007b6c       ??_SQPushButton@@6BQObject@@@ 00482b6c     CapacityCalculation.obj
 0002:00007c6c       ??_C@_0CA@HPJNKJP@m_labelCapacityCalculationTitle?$AA@ 00482c6c     CapacityCalculation.obj
 0002:00007c94       ??_C@_0CC@OBNKFCGH@m_labelCapacityCalculationSectio@ 00482c94     CapacityCalculation.obj
 0002:00007cbc       ??_C@_0BB@COLOJDPM@m_CapacityWidget?$AA@ 00482cbc     CapacityCalculation.obj
 0002:00007cd0       ??_C@_0P@JLMEIFJO@m_borderLayout?$AA@ 00482cd0     CapacityCalculation.obj
 0002:00007ce4       ??_C@_0BE@OAEMJOEL@CapacityCalculation?$AA@ 00482ce4     CapacityCalculation.obj
 0002:00007cfc       ??_C@_05MDNHABIA@Clear?$AA@ 00482cfc     CapacityCalculation.obj
 0002:00007d04       ??_C@_06BFGAPCKF@Export?$AA@ 00482d04     CapacityCalculation.obj
 0002:00007d0c       ??_C@_0BH@NFFHPHLG@Capacity?5Calculation?5?3?$AA@ 00482d0c     CapacityCalculation.obj
 0002:00007d2c       ??_7WidgetDeviceListBorder@@6BQPaintDevice@@@ 00482d2c     WidgetDeviceListBorder.obj
 0002:00007d54       ??_7WidgetDeviceListBorder@@6BQObject@@@ 00482d54     WidgetDeviceListBorder.obj
 0002:00007e44       ??_C@_0O@MJJIIIEL@m_labeNullTip?$AA@ 00482e44     WidgetDeviceListBorder.obj
 0002:00007e54       ??_C@_0P@CGHENIHE@m_labelNullPic?$AA@ 00482e54     WidgetDeviceListBorder.obj
 0002:00007e68       ??_C@_0BH@NOAFMBP@WidgetDeviceListBorder?$AA@ 00482e68     WidgetDeviceListBorder.obj
 0002:00007e88       ??_C@_0MB@KCEIACNG@?$DMhtml?$DO?$DMhead?1?$DO?$DMbody?$DO?$DMp?$DO?$DMspan?5styl@ 00482e88     WidgetDeviceListBorder.obj
 0002:000085e0       ??_7BandWidthPage@@6BQPaintDevice@@@ 004835e0     BandWidthPage.obj
 0002:00008604       ??_7BandWidthPage@@6BQObject@@@ 00483604     BandWidthPage.obj
 0002:000086f4       ??_C@_08FGBMEDGO@picLabel?$AA@ 004836f4     BandWidthPage.obj
 0002:00008700       ??_C@_0P@CLAPMLPD@bandWidthLabel?$AA@ 00483700     BandWidthPage.obj
 0002:00008714       ??_C@_08HHDIDNIH@DVRLabel?$AA@ 00483714     BandWidthPage.obj
 0002:00008720       ??_C@_08IBLBEECN@IPCLabel?$AA@ 00483720     BandWidthPage.obj
 0002:0000872c       ??_C@_0N@LJJHDMFK@channelLabel?$AA@ 0048372c     BandWidthPage.obj
 0002:0000873c       ??_C@_0O@JBCKIMHJ@BandWidthPage?$AA@ 0048373c     BandWidthPage.obj
 0002:00008750       ??_C@_0BDP@BMJMBCC@?$DMhtml?$DO?$DMhead?1?$DO?$DMbody?$DO?$DMp?5align?$DN?$CCcen@ 00483750     BandWidthPage.obj
 0002:000088d0       ??_C@_0PN@LMLHKMHC@?$DMhtml?$DO?$DMhead?1?$DO?$DMbody?$DO?$DMp?5align?$DN?$CCcen@ 004838d0     BandWidthPage.obj
 0002:00009518       ??_7DataCalculatorPage@@6BQPaintDevice@@@ 00484518     DataCalculatorPage.obj
 0002:0000953c       ??_7DataCalculatorPage@@6BQObject@@@ 0048453c     DataCalculatorPage.obj
 0002:0000962c       ??_C@_06KLKLDLLI@widget?$AA@ 0048462c     DataCalculatorPage.obj
 0002:00009634       ??_C@_0BB@IFOLJPAL@verticalLayout_3?$AA@ 00484634     DataCalculatorPage.obj
 0002:00009648       ??_C@_0BJ@KLDCOIIE@m_tabWidgetSectionsPage3?$AA@ 00484648     DataCalculatorPage.obj
 0002:00009668       ??_C@_0BC@EDMDDFMH@m_displayPageSize?$AA@ 00484668     DataCalculatorPage.obj
 0002:00009680       ??_C@_0BB@LEFCBBIN@m_labelDailyHour?$AA@ 00484680     DataCalculatorPage.obj
 0002:00009694       ??_C@_0BD@ODFLJLEB@m_spinBoxDailyTime?$AA@ 00484694     DataCalculatorPage.obj
 0002:000096ac       ??_C@_0BD@DCDOOJCP@m_hSliderDailyTime?$AA@ 004846ac     DataCalculatorPage.obj
 0002:000096c4       ??_C@_0BJ@OCIBEOGD@m_hlayoutDailyRecordTime?$AA@ 004846c4     DataCalculatorPage.obj
 0002:000096e4       ??_C@_0BI@IBLCGNPL@m_widgetDailyRecordTime?$AA@ 004846e4     DataCalculatorPage.obj
 0002:00009700       ??_C@_0BH@EEIKBAL@m_labelDailyRecordTime?$AA@ 00484700     DataCalculatorPage.obj
 0002:0000971c       ??_C@_0N@FBIEENFF@m_radioMonth?$AA@ 0048471c     DataCalculatorPage.obj
 0002:0000972c       ??_C@_0P@MPEGCJIO@m_radioBtnWeek?$AA@ 0048472c     DataCalculatorPage.obj
 0002:00009740       ??_C@_0O@IFAOKCBG@m_radioBtnDay?$AA@ 00484740     DataCalculatorPage.obj
 0002:00009750       ??_C@_0BD@LCBPPMLK@m_lineEditSaveTime?$AA@ 00484750     DataCalculatorPage.obj
 0002:00009768       ??_C@_0BC@BIANIGPO@m_hlayoutSaveTime?$AA@ 00484768     DataCalculatorPage.obj
 0002:00009780       ??_C@_0BB@LBKIGKHF@m_widgetSaveTime?$AA@ 00484780     DataCalculatorPage.obj
 0002:00009794       ??_C@_0BA@PBAFNNGK@m_labelSaveTime?$AA@ 00484794     DataCalculatorPage.obj
 0002:000097a8       ??_C@_0BJ@LCCJNJMF@m_tabWidgetSectionsPage2?$AA@ 004847a8     DataCalculatorPage.obj
 0002:000097c8       ??_C@_0BC@OIIKFMCC@m_displayPageTime?$AA@ 004847c8     DataCalculatorPage.obj
 0002:000097e0       ??_C@_0M@CJNBECDK@m_labelHour?$AA@ 004847e0     DataCalculatorPage.obj
 0002:000097f0       ??_C@_0O@NDDIPFG@m_spinBoxTime?$AA@ 004847f0     DataCalculatorPage.obj
 0002:00009800       ??_C@_0BH@CJANIGFO@m_horizontalSliderTime?$AA@ 00484800     DataCalculatorPage.obj
 0002:00009820       ??_SCSlider@iVMSGUIToolkit@@6BQPaintDevice@@@ 00484820     DataCalculatorPage.obj
 0002:00009844       ??_SCSlider@iVMSGUIToolkit@@6BQObject@@@ 00484844     DataCalculatorPage.obj
 0002:00009940       ??_C@_0BE@JPIHCLMB@m_hlayoutRecordTime?$AA@ 00484940     DataCalculatorPage.obj
 0002:00009958       ??_C@_0BD@OOEMGNLH@m_widgetRecordTime?$AA@ 00484958     DataCalculatorPage.obj
 0002:00009970       ??_C@_0BB@PCJMKOJH@m_labelRecordTim?$AA@ 00484970     DataCalculatorPage.obj
 0002:00009984       ??_C@_0N@POKEMOPC@m_radioBtnGB?$AA@ 00484984     DataCalculatorPage.obj
 0002:00009994       ??_C@_0N@OAMENDNL@m_radioBtnTB?$AA@ 00484994     DataCalculatorPage.obj
 0002:000099a4       ??_C@_0N@NCAGCPPM@m_lineEditGT?$AA@ 004849a4     DataCalculatorPage.obj
 0002:000099b4       ??_C@_0BC@MADCJFMB@m_hlayoutDiskSize?$AA@ 004849b4     DataCalculatorPage.obj
 0002:000099cc       ??_C@_0BB@GJJHHJEK@m_widgetDiskSize?$AA@ 004849cc     DataCalculatorPage.obj
 0002:000099e0       ??_C@_0BA@CJDKMOFF@m_labelDiskSize?$AA@ 004849e0     DataCalculatorPage.obj
 0002:000099f4       ??_C@_0BJ@JJAEIKAG@m_tabWidgetSectionsPage1?$AA@ 004849f4     DataCalculatorPage.obj
 0002:00009a14       ??_C@_0BE@MPHPOBOK@m_tabWidgetSections?$AA@ 00484a14     DataCalculatorPage.obj
 0002:00009a30       ??_SQStackedWidget@@6BQPaintDevice@@@ 00484a30     DataCalculatorPage.obj
 0002:00009a54       ??_SQStackedWidget@@6BQObject@@@ 00484a54     DataCalculatorPage.obj
 0002:00009b44       ??_C@_0P@JMPAMMCF@calBandWithBtn?$AA@ 00484b44     DataCalculatorPage.obj
 0002:00009b58       ??_C@_0L@JAAKEJNF@calDiskBtn?$AA@ 00484b58     DataCalculatorPage.obj
 0002:00009b68       ??_C@_0L@GKFNKFHE@calTimeBtn?$AA@ 00484b68     DataCalculatorPage.obj
 0002:00009b78       ??_C@_0BD@PKGJGDKJ@DataCalculatorPage?$AA@ 00484b78     DataCalculatorPage.obj
 0002:00009b90       ??_C@_0BH@GPBENDMD@record?5time?5each?5day?5?3?$AA@ 00484b90     DataCalculatorPage.obj
 0002:00009bac       ??_C@_05PIGOEBJ@MONTH?$AA@ 00484bac     DataCalculatorPage.obj
 0002:00009bb4       ??_C@_04HKPIGKND@WEEK?$AA@ 00484bb4     DataCalculatorPage.obj
 0002:00009bbc       ??_C@_03NAOMOOGD@DAY?$AA@  00484bbc     DataCalculatorPage.obj
 0002:00009bc0       ??_C@_0P@HOINLEEE@set?5save?5time?3?$AA@ 00484bc0     DataCalculatorPage.obj
 0002:00009bd4       ??_C@_01BDACAMKP@h?$AA@    00484bd4     DataCalculatorPage.obj
 0002:00009bd8       ??_C@_0O@OHFOCFDO@record?5time?5?3?$AA@ 00484bd8     DataCalculatorPage.obj
 0002:00009be8       ??_C@_02LHCEJACP@GB?$AA@   00484be8     DataCalculatorPage.obj
 0002:00009bec       ??_C@_02KJEEINAG@TB?$AA@   00484bec     DataCalculatorPage.obj
 0002:00009bf0       ??_C@_0BB@GPDFABLB@set?5disk?5size?5?3?5?$AA@ 00484bf0     DataCalculatorPage.obj
 0002:00009c04       ??_C@_0M@PFOIKLH@CalBandWith?$AA@ 00484c04     DataCalculatorPage.obj
 0002:00009c14       ??_C@_07FENLEPIN@CalDisk?$AA@ 00484c14     DataCalculatorPage.obj
 0002:00009c20       ??_C@_07LMAAHLPL@CalTime?$AA@ 00484c20     DataCalculatorPage.obj
 0002:00009c30       __real@beb0c6f7a0b5ed8d    00484c30     DataCalculatorPage.obj
 0002:00009c40       __real@3eb0c6f7a0b5ed8d    00484c40     DataCalculatorPage.obj
 0002:00009c50       __real@403e000000000000    00484c50     DataCalculatorPage.obj
 0002:00009c60       __real@408f400000000000    00484c60     DataCalculatorPage.obj
 0002:00009da4       ??_7DataDisplayPage@@6BQPaintDevice@@@ 00484da4     DataDisplayPage.obj
 0002:00009dcc       ??_7DataDisplayPage@@6BQObject@@@ 00484dcc     DataDisplayPage.obj
 0002:00009ebc       ??_C@_0O@IENNIHFD@diskplayLine1?$AA@ 00484ebc     DataDisplayPage.obj
 0002:00009ecc       ??_C@_0BI@CGLOABAA@m_labelDiskplayMonthTip?$AA@ 00484ecc     DataDisplayPage.obj
 0002:00009ee8       ??_C@_0BD@IEBFNGPE@horizontalLayout_5?$AA@ 00484ee8     DataDisplayPage.obj
 0002:00009f00       ??_C@_0P@NKNFGNHG@m_labelByMonth?$AA@ 00484f00     DataDisplayPage.obj
 0002:00009f14       ??_C@_0BL@PJEOONBI@m_labelDiskplayMonthMethod?$AA@ 00484f14     DataDisplayPage.obj
 0002:00009f34       ??_C@_0BD@DBLLKILJ@horizontalLayout_8?$AA@ 00484f34     DataDisplayPage.obj
 0002:00009f4c       ??_C@_0BI@PNNFFDNC@m_widgetDiskplayByMonth?$AA@ 00484f4c     DataDisplayPage.obj
 0002:00009f68       ??_C@_0O@LGOLOFNB@diskplayLine3?$AA@ 00484f68     DataDisplayPage.obj
 0002:00009f78       ??_C@_0BH@PLAGMHPD@m_labelDiskplayWeekTip?$AA@ 00484f78     DataDisplayPage.obj
 0002:00009f94       ??_C@_0BD@JNAOOHLF@horizontalLayout_4?$AA@ 00484f94     DataDisplayPage.obj
 0002:00009fac       ??_C@_0O@HCFOMBDJ@m_labelByWeek?$AA@ 00484fac     DataDisplayPage.obj
 0002:00009fbc       ??_C@_0BN@JJPGKNJM@m_labelDiskplayWeekTipMethod?$AA@ 00484fbc     DataDisplayPage.obj
 0002:00009fe0       ??_C@_0BD@LGCDLEHG@horizontalLayout_7?$AA@ 00484fe0     DataDisplayPage.obj
 0002:00009ff8       ??_C@_0BH@HACBMPEI@m_widgetDiskplayByWeek?$AA@ 00484ff8     DataDisplayPage.obj
 0002:0000a014       ??_C@_0O@KPPANEJA@diskplayLine2?$AA@ 00485014     DataDisplayPage.obj
 0002:0000a024       ??_C@_0BG@PFMCGOIJ@m_labelDiskplayDayTip?$AA@ 00485024     DataDisplayPage.obj
 0002:0000a040       ??_C@_0N@CABEAJOG@m_labelByDay?$AA@ 00485040     DataDisplayPage.obj
 0002:0000a050       ??_C@_0BJ@KMHMIHLL@m_labelDiskplayDayMethod?$AA@ 00485050     DataDisplayPage.obj
 0002:0000a070       ??_C@_0BD@KPDIIFDH@horizontalLayout_6?$AA@ 00485070     DataDisplayPage.obj
 0002:0000a088       ??_C@_0BG@DCIJHCCF@m_widgetDiskplayByDay?$AA@ 00485088     DataDisplayPage.obj
 0002:0000a0a4       ??_C@_0BI@DIHCFMFP@m_labelDiskplayTimeNeed?$AA@ 004850a4     DataDisplayPage.obj
 0002:0000a0c0       ??_C@_0BA@KPHKMFGD@DataDisplayPage?$AA@ 004850c0     DataDisplayPage.obj
 0002:0000a0d4       ??_C@_08KKOPDHMG@Month?$CIs?$CJ?$AA@ 004850d4     DataDisplayPage.obj
 0002:0000a0e0       ??_C@_0KG@BAGDKPLH@?$DMhtml?$DO?$DMhead?1?$DO?$DMbody?$DO?$DMp?5align?$DN?$CCcen@ 004850e0     DataDisplayPage.obj
 0002:0000a1a8       ??_C@_08BILBCLMK@By?5Month?$AA@ 004851a8     DataDisplayPage.obj
 0002:0000a1b4       ??_C@_07NNBMKPIN@Week?$CIs?$CJ?$AA@ 004851b4     DataDisplayPage.obj
 0002:0000a1c0       ??_C@_0KG@DEPHDPA@?$DMhtml?$DO?$DMhead?1?$DO?$DMbody?$DO?$DMp?5align?$DN?$CCcen@ 004851c0     DataDisplayPage.obj
 0002:0000a288       ??_C@_07MBOHNKIF@By?5Week?$AA@ 00485288     DataDisplayPage.obj
 0002:0000a294       ??_C@_06JCMKOBJJ@Day?$CIs?$CJ?$AA@ 00485294     DataDisplayPage.obj
 0002:0000a2a0       ??_C@_0KG@HOEODNFF@?$DMhtml?$DO?$DMhead?1?$DO?$DMbody?$DO?$DMp?5align?$DN?$CCcen@ 004852a0     DataDisplayPage.obj
 0002:0000a368       ??_C@_06PPHFJLBO@By?5Day?$AA@ 00485368     DataDisplayPage.obj
 0002:0000a370       ??_C@_0BE@BADNNHAI@Video?5can?5be?5saved?3?$AA@ 00485370     DataDisplayPage.obj
 0002:0000a4ac       ??_7SizeDisplayPage@@6BQPaintDevice@@@ 004854ac     SizeDisplayPage.obj
 0002:0000a4d4       ??_7SizeDisplayPage@@6BQObject@@@ 004854d4     SizeDisplayPage.obj
 0002:0000a5c4       ??_C@_0CL@OAKMEKGH@?1?$CKbackground?9color?3blue?$CK?1?6font?9s@ 004855c4     SizeDisplayPage.obj
 0002:0000a5f8       ??_C@_0BD@BHKCOJHP@m_labelDisplaySize?$AA@ 004855f8     SizeDisplayPage.obj
 0002:0000a610       ??_C@_0CO@DPBDJIJL@?1?$CKborder?9radius?3160?$DL?6background?9@ 00485610     SizeDisplayPage.obj
 0002:0000a648       ??_C@_0BB@JDCBGPGD@m_WidgetSizeBack?$AA@ 00485648     SizeDisplayPage.obj
 0002:0000a65c       ??_C@_0BI@LBKNLBIE@m_labelDisplaySizeTitle?$AA@ 0048565c     SizeDisplayPage.obj
 0002:0000a678       ??_C@_0BA@HAAPPABJ@SizeDisplayPage?$AA@ 00485678     SizeDisplayPage.obj
 0002:0000a690       ??_C@_0KF@PIPBIMCF@?$DMhtml?$DO?$DMhead?1?$DO?$DMbody?$DO?$DMp?5align?$DN?$CCcen@ 00485690     SizeDisplayPage.obj
 0002:0000a758       ??_C@_0CH@DHOBMFFA@Calculate?5the?5required?5disk?5capa@ 00485758     SizeDisplayPage.obj
 0002:0000bd64       ??_7DeviceAddPage@@6BQPaintDevice@@@ 00486d64     DeviceAddPage.obj
 0002:0000bd8c       ??_7DeviceAddPage@@6BQObject@@@ 00486d8c     DeviceAddPage.obj
 0002:0000be7c       ??_C@_0BF@PNHKAODE@m_listWidgetDiskData?$AA@ 00486e7c     DeviceAddPage.obj
 0002:0000be98       ??_C@_0O@EOHHJKIN@DeviceAddPage?$AA@ 00486e98     DeviceAddPage.obj
 0002:0000bea8       __real@408f3f3333333333    00486ea8     DeviceAddPage.obj
 0002:0000beb8       __real@4090000000000000    00486eb8     DeviceAddPage.obj
 0002:0000bec8       __real@4130000000000000    00486ec8     DeviceAddPage.obj
 0002:0000bed8       __real@4049000000000000    00486ed8     DeviceAddPage.obj
 0002:0000bee8       __real@404e000000000000    00486ee8     DeviceAddPage.obj
 0002:0000bef8       __real@4039000000000000    00486ef8     DeviceAddPage.obj
 0002:0000bf08       __real@4072900000000000    00486f08     DeviceAddPage.obj
 0002:0000bf18       __real@406a400000000000    00486f18     DeviceAddPage.obj
 0002:0000c150       ??_7DeviceItemWidget@NM_DiskCalculator@@6BQPaintDevice@@@ 00487150     DeviceItemWidget.obj
 0002:0000c174       ??_7DeviceItemWidget@NM_DiskCalculator@@6BQObject@@@ 00487174     DeviceItemWidget.obj
 0002:0000c264       ??_C@_05JCPNMPAM@line5?$AA@ 00487264     DeviceItemWidget.obj
 0002:0000c26c       ??_C@_0BC@OACCDACL@m_labelScenceName?$AA@ 0048726c     DeviceItemWidget.obj
 0002:0000c284       ??_C@_05ILOGPOEN@line4?$AA@ 00487284     DeviceItemWidget.obj
 0002:0000c28c       ??_C@_0BC@ICILDCPJ@m_labelEncodeType?$AA@ 0048728c     DeviceItemWidget.obj
 0002:0000c2a4       ??_C@_05MEKHGIIK@line3?$AA@ 004872a4     DeviceItemWidget.obj
 0002:0000c2ac       ??_C@_0BI@IGKGNEEO@m_labelDeviceResolution?$AA@ 004872ac     DeviceItemWidget.obj
 0002:0000c2c8       ??_C@_05NNLMFJML@line2?$AA@ 004872c8     DeviceItemWidget.obj
 0002:0000c2d0       ??_C@_0BF@FEGJBOON@m_labelDeviceBitRate?$AA@ 004872d0     DeviceItemWidget.obj
 0002:0000c2ec       ??_C@_05PGJBAKAI@line1?$AA@ 004872ec     DeviceItemWidget.obj
 0002:0000c2f4       ??_C@_0BE@CIIOCAHN@m_labelDeviceCounts?$AA@ 004872f4     DeviceItemWidget.obj
 0002:0000c30c       ??_C@_0L@MGCENAHH@m_hlayout3?$AA@ 0048730c     DeviceItemWidget.obj
 0002:0000c31c       ??_C@_0BA@HOFOBFKM@m_itemContainer?$AA@ 0048731c     DeviceItemWidget.obj
 0002:0000c330       ??_C@_04HJPCFDOP@line?$AA@ 00487330     DeviceItemWidget.obj
 0002:0000c338       ??_C@_0L@NPDPOBDG@m_hlayout2?$AA@ 00487338     DeviceItemWidget.obj
 0002:0000c348       ??_C@_0M@FFIOFBJA@m_hlayoutxx?$AA@ 00487348     DeviceItemWidget.obj
 0002:0000c358       ??_C@_0M@JHJIIEBJ@m_btnDelete?$AA@ 00487358     DeviceItemWidget.obj
 0002:0000c36c       ??_SQToolButton@@6BQPaintDevice@@@ 0048736c     DeviceItemWidget.obj
 0002:0000c394       ??_SQToolButton@@6BQObject@@@ 00487394     DeviceItemWidget.obj
 0002:0000c494       ??_C@_0BI@BIONNKMA@m_labelChannelGroupName?$AA@ 00487494     DeviceItemWidget.obj
 0002:0000c4b0       ??_C@_0BJ@LKHLMHAC@m_labelDeviceTypeIconIPC?$AA@ 004874b0     DeviceItemWidget.obj
 0002:0000c4d0       ??_C@_0BJ@BPEFEAHN@m_labelDeviceTypeIconDVR?$AA@ 004874d0     DeviceItemWidget.obj
 0002:0000c4f0       ??_C@_0P@MEEHJLIF@m_hlayoutTitle?$AA@ 004874f0     DeviceItemWidget.obj
 0002:0000c504       ??_C@_0BB@FHJLJOPL@DeviceItemWidget?$AA@ 00487504     DeviceItemWidget.obj
 0002:0000c518       ??_C@_0N@PEALLFCM@Scence?5Name?3?$AA@ 00487518     DeviceItemWidget.obj
 0002:0000c528       ??_C@_0N@ENPOHDIN@Encode?5Type?3?$AA@ 00487528     DeviceItemWidget.obj
 0002:0000c538       ??_C@_0M@NCGNHIAC@Resolution?3?$AA@ 00487538     DeviceItemWidget.obj
 0002:0000c548       ??_C@_09PLKBMGGF@Bit?5Rate?3?$AA@ 00487548     DeviceItemWidget.obj
 0002:0000c554       ??_C@_07KKJPLDHB@Counts?3?$AA@ 00487554     DeviceItemWidget.obj
 0002:0000c564       ??_7ButtonRadio@aptui@@6BQPaintDevice@@@ 00487564     ButtonRadio.obj
 0002:0000c58c       ??_7ButtonRadio@aptui@@6BQObject@@@ 0048758c     ButtonRadio.obj
 0002:0000ca60       ??_7UpdateDialog@@6BQPaintDevice@@@ 00487a60     UpdateDialog.obj
 0002:0000ca84       ??_7UpdateDialog@@6BQObject@@@ 00487a84     UpdateDialog.obj
 0002:0000cb84       ??_C@_0L@NFLFNCLJ@m_labelTip?$AA@ 00487b84     UpdateDialog.obj
 0002:0000cb94       ??_C@_0M@IHOFKCPB@m_btnImport?$AA@ 00487b94     UpdateDialog.obj
 0002:0000cba4       ??_C@_0M@BDFOFLKN@m_btnExport?$AA@ 00487ba4     UpdateDialog.obj
 0002:0000cbb4       ??_C@_09HIELOGFD@m_tipText?$AA@ 00487bb4     UpdateDialog.obj
 0002:0000cbc0       ??_C@_09GMBEKFJC@m_tipIcon?$AA@ 00487bc0     UpdateDialog.obj
 0002:0000cbcc       ??_C@_0N@ICCGCNK@UpdateDialog?$AA@ 00487bcc     UpdateDialog.obj
 0002:0000cbdc       ??_C@_0BF@GOMBHNAB@Tip?3?5Need?5to?5Restart?$AA@ 00487bdc     UpdateDialog.obj
 0002:0000cbf8       ??_C@_0BA@BJPEKGNH@Import?5Templete?$AA@ 00487bf8     UpdateDialog.obj
 0002:0000cc0c       ??_C@_0M@ONJBBCEN@Export?5Data?$AA@ 00487c0c     UpdateDialog.obj
 0002:0000cc1c       ??_C@_08IBMCNDCB@tip?5text?$AA@ 00487c1c     UpdateDialog.obj
 0002:0000cc28       ??_C@_09BHFPINEP@TextLabel?$AA@ 00487c28     UpdateDialog.obj
 0002:0000cd90       ??_7WarningDialog@NM_DiskCalculator@@6BQPaintDevice@@@ 00487d90     WarningDialog.obj
 0002:0000cdb4       ??_7WarningDialog@NM_DiskCalculator@@6BQObject@@@ 00487db4     WarningDialog.obj
 0002:0000ceb4       ??_C@_0BA@DBIDKFIF@m_labelWarnText?$AA@ 00487eb4     WarningDialog.obj
 0002:0000cec8       ??_C@_0BD@HJNKKGMI@m_labelWarnPicture?$AA@ 00487ec8     WarningDialog.obj
 0002:0000cee0       ??_C@_0L@DOFHAFCJ@m_btnClose?$AA@ 00487ee0     WarningDialog.obj
 0002:0000cef0       ??_C@_0P@FDKMBHGL@m_borderWidget?$AA@ 00487ef0     WarningDialog.obj
 0002:0000cf04       ??_C@_0O@DFGDPCAG@WarningDialog?$AA@ 00487f04     WarningDialog.obj
 0002:0000cf14       ??_C@_04KANOLIK@Form?$AA@  00487f14     WarningDialog.obj
 0002:0000cf20       ??_7TipDialog@NM_DiskCalculator@@6BQPaintDevice@@@ 00487f20     TipDialog.obj
 0002:0000cf44       ??_7TipDialog@NM_DiskCalculator@@6BQObject@@@ 00487f44     TipDialog.obj
 0002:0000d044       ??_C@_09NDDAHPBH@TipDialog?$AA@ 00488044     TipDialog.obj
 0002:0000d050       ??_C@_04JELBOBIP@sure?$AA@ 00488050     TipDialog.obj
 0002:0000d168       ??_7BaseTitle@aptui@@6B@   00488168     BaseTitle.obj
 0002:0000d174       ??_7BaseTitle@aptui@@6BQPaintDevice@@@ 00488174     BaseTitle.obj
 0002:0000d19c       ??_7BaseTitle@aptui@@6BQObject@@@ 0048819c     BaseTitle.obj
 0002:0000d28c       ??_C@_08GAIGKGJB@btnClose?$AA@ 0048828c     BaseTitle.obj
 0002:0000d298       ??_C@_06PIGCJLP@btnMax?$AA@ 00488298     BaseTitle.obj
 0002:0000d2a0       ??_C@_06BNANMNNA@btnMin?$AA@ 004882a0     BaseTitle.obj
 0002:0000d2a8       ??_C@_09OKKBFPHH@btnOption?$AA@ 004882a8     BaseTitle.obj
 0002:0000d2b4       ??_C@_0BH@GDKKHGIP@m_hlayoutCustomButtons?$AA@ 004882b4     BaseTitle.obj
 0002:0000d2d0       ??_C@_0L@OIDMMBHO@labelTitle?$AA@ 004882d0     BaseTitle.obj
 0002:0000d2e0       ??_C@_06JAGNNFEI@btnApp?$AA@ 004882e0     BaseTitle.obj
 0002:0000d2e8       ??_C@_09IIFEOFHC@BaseTitle?$AA@ 004882e8     BaseTitle.obj
 0002:0000d424       ??_7WindowTitle@aptui@@6B@ 00488424     WindowTitle.obj
 0002:0000d430       ??_7WindowTitle@aptui@@6BQPaintDevice@@@ 00488430     WindowTitle.obj
 0002:0000d454       ??_7WindowTitle@aptui@@6BQObject@@@ 00488454     WindowTitle.obj
 0002:0000d54c       ??_SCWidgetItem@iVMSGUIToolkit@@6B@ 0048854c     WindowTitle.obj
 0002:0000d59c       ??_SCHBoxLayout@iVMSGUIToolkit@@6BQLayoutItem@@@ 0048859c     WindowTitle.obj
 0002:0000d5ec       ??_SCHBoxLayout@iVMSGUIToolkit@@6BQObject@@@ 004885ec     WindowTitle.obj
 0002:0000d66c       ??_7Menu@aptui@@6BQPaintDevice@@@ 0048866c     Menu.obj
 0002:0000d694       ??_7Menu@aptui@@6BQObject@@@ 00488694     Menu.obj
 0002:0000d78c       ??_7CCustomStyle@Menu@aptui@@6B@ 0048878c     Menu.obj
 0002:0000d830       ??_7SystemMenu@aptui@@6BQPaintDevice@@@ 00488830     TitleMenu.obj
 0002:0000d854       ??_7SystemMenu@aptui@@6BQObject@@@ 00488854     TitleMenu.obj
 0002:0000d948       ??_7LineEditInterger@aptui@@6BQPaintDevice@@@ 00488948     LineEditInterger.obj
 0002:0000d96c       ??_7LineEditInterger@aptui@@6BQObject@@@ 0048896c     LineEditInterger.obj
 0002:0000da98       ??_7TabWidget@aptui@@6BQPaintDevice@@@ 00488a98     TabWidget.obj
 0002:0000dabc       ??_7TabWidget@aptui@@6BQObject@@@ 00488abc     TabWidget.obj
 0002:0000dbbc       ??_7Line@aptui@@6BQPaintDevice@@@ 00488bbc     Line.obj
 0002:0000dbe4       ??_7Line@aptui@@6BQObject@@@ 00488be4     Line.obj
 0002:0000de4c       ??_7CDlgAbout@aptui@@6B@   00488e4c     DlgAbout.obj
 0002:0000de90       ??_C@_09NPHLPCBE@aboutbtn2?$AA@ 00488e90     DlgAbout.obj
 0002:0000de9c       ??_C@_0L@DLFAPELO@aboutLine2?$AA@ 00488e9c     DlgAbout.obj
 0002:0000deac       ??_C@_09PEFGKBNH@aboutbtn1?$AA@ 00488eac     DlgAbout.obj
 0002:0000deb8       ??_C@_0L@BAHNKHHN@aboutLine1?$AA@ 00488eb8     DlgAbout.obj
 0002:0000dec8       ??_C@_0BC@MNONCPCN@m_labVersionValue?$AA@ 00488ec8     DlgAbout.obj
 0002:0000dee0       ??_C@_0P@NEELGEIO@m_labNameValue?$AA@ 00488ee0     DlgAbout.obj
 0002:0000def4       ??_C@_08OHLCLKBM@SoftIcon?$AA@ 00488ef4     DlgAbout.obj
 0002:0000df00       ??_C@_0L@LCDLELHC@m_conerBtn?$AA@ 00488f00     DlgAbout.obj
 0002:0000df10       ??_C@_09ENONNOAO@TopLayout?$AA@ 00488f10     DlgAbout.obj
 0002:0000df1c       ??_C@_0M@JDBDIJFO@AboutWidget?$AA@ 00488f1c     DlgAbout.obj
 0002:0000df2c       ??_C@_0L@CNNAPHBM@AboutClass?$AA@ 00488f2c     DlgAbout.obj
 0002:0000df3c       ??_C@_0L@OOAHNKCH@PushButton?$AA@ 00488f3c     DlgAbout.obj
 0002:0000df4c       ??_C@_05BDOHFCKE@About?$AA@ 00488f4c     DlgAbout.obj
 0002:0000e02c       ??_7Switch@aptui@@6BQPaintDevice@@@ 0048902c     Switch.obj
 0002:0000e054       ??_7Switch@aptui@@6BQObject@@@ 00489054     Switch.obj
 0002:0000e154       ??_7CoverWidget@aptui@@6BQPaintDevice@@@ 00489154     CoverWidget.obj
 0002:0000e17c       ??_7CoverWidget@aptui@@6BQObject@@@ 0048917c     CoverWidget.obj
 0002:0000e270       ??_7Widget@aptui@@6BQPaintDevice@@@ 00489270     Widget.obj
 0002:0000e294       ??_7Widget@aptui@@6BQObject@@@ 00489294     Widget.obj
 0002:0000e3f4       ??_7MultiStatePushButton@aptui@@6BQPaintDevice@@@ 004893f4     MultiStatePushButton.obj
 0002:0000e41c       ??_7MultiStatePushButton@aptui@@6BQObject@@@ 0048941c     MultiStatePushButton.obj
 0002:0000eb08       ??_7BaseDialog@aptui@@6BQPaintDevice@@@ 00489b08     BaseDialog.obj
 0002:0000eb2c       ??_7BaseDialog@aptui@@6BQObject@@@ 00489b2c     BaseDialog.obj
 0002:0000ec2c       ??_C@_09JPMHGMCO@btnCancel?$AA@ 00489c2c     BaseDialog.obj
 0002:0000ec38       ??_C@_0L@MIKLBKKG@btnConfirm?$AA@ 00489c38     BaseDialog.obj
 0002:0000ec48       ??_C@_09GPKENDME@btnLayout?$AA@ 00489c48     BaseDialog.obj
 0002:0000ec54       ??_C@_0N@GJFMGIIJ@layoutMyBtns?$AA@ 00489c54     BaseDialog.obj
 0002:0000ec64       ??_C@_0BD@IAFGNKKO@m_BaseDialogBottom?$AA@ 00489c64     BaseDialog.obj
 0002:0000ec7c       ??_C@_0M@FDHIGKDN@m_labelNULL?$AA@ 00489c7c     BaseDialog.obj
 0002:0000ec8c       ??_C@_0N@DPLCMDIK@BorderLayout?$AA@ 00489c8c     BaseDialog.obj
 0002:0000ec9c       ??_C@_0L@EKMJGHIP@mainBorder?$AA@ 00489c9c     BaseDialog.obj
 0002:0000ecac       ??_C@_0M@JLOMGCHL@titleLayout?$AA@ 00489cac     BaseDialog.obj
 0002:0000ecbc       ??_C@_0L@FGHGLIHP@BaseDialog?$AA@ 00489cbc     BaseDialog.obj
 0002:0000eccc       ??_C@_06FMBNCPDL@Cancel?$AA@ 00489ccc     BaseDialog.obj
 0002:0000ecd4       ??_C@_07KFLFCEAO@Confirm?$AA@ 00489cd4     BaseDialog.obj
 0002:0000ece0       ??_C@_0N@LDEHBFEN@null?5content?$AA@ 00489ce0     BaseDialog.obj
 0002:0000ede8       ??_7Label@aptui@@6BQPaintDevice@@@ 00489de8     Label.obj
 0002:0000ee0c       ??_7Label@aptui@@6BQObject@@@ 00489e0c     Label.obj
 0002:0000ef00       ??_7EditableLabel@aptui@@6BQPaintDevice@@@ 00489f00     Label.obj
 0002:0000ef24       ??_7EditableLabel@aptui@@6BQObject@@@ 00489f24     Label.obj
 0002:0000f018       ??_7ColorLabel@aptui@@6BQPaintDevice@@@ 0048a018     Label.obj
 0002:0000f03c       ??_7ColorLabel@aptui@@6BQObject@@@ 0048a03c     Label.obj
 0002:0000f130       ??_SQColorDialog@@6BQPaintDevice@@@ 0048a130     Label.obj
 0002:0000f154       ??_SQColorDialog@@6BQObject@@@ 0048a154     Label.obj
 0002:0000f25c       ??_7QtLockedFile@SharedTools@@6B@ 0048a25c     qtlockedfile.obj
 0002:0000f6b8       ??_SQLocalServer@@6B@      0048a6b8     qtlocalpeer.obj
 0002:0000f700       ??_7QtLocalPeer@SharedTools@@6B@ 0048a700     qtlocalpeer.obj
 0002:0000f8ac       ??_7QtSingleApplication@SharedTools@@6B@ 0048a8ac     qtsingleapplication.obj
 0002:0000f984       ??_7QtSingleCoreApplication@SharedTools@@6B@ 0048a984     qtsinglecoreapplication.obj
 0002:0000f9c8       ??_C@_0P@GHFPNOJB@bad?5allocation?$AA@ 0048a9c8     msvcprt:nothrow.obj
 0002:0000f9dc       ??_7type_info@@6B@         0048a9dc     MSVCRT:ti_inst.obj
 0002:0000f9e8       ?ProcessDetach@NativeDll@<CrtImplementationDetails>@@0IB 0048a9e8     MSVCRT:unhandld.obj
 0002:0000f9ec       ?ProcessAttach@NativeDll@<CrtImplementationDetails>@@0IB 0048a9ec     MSVCRT:unhandld.obj
 0002:0000f9f0       ?ThreadAttach@NativeDll@<CrtImplementationDetails>@@0IB 0048a9f0     MSVCRT:unhandld.obj
 0002:0000f9f4       ?ThreadDetach@NativeDll@<CrtImplementationDetails>@@0IB 0048a9f4     MSVCRT:unhandld.obj
 0002:0000f9f8       ?ProcessVerifier@NativeDll@<CrtImplementationDetails>@@0IB 0048a9f8     MSVCRT:unhandld.obj
 0002:0000fa00       __load_config_used         0048aa00     MSVCRT:loadcfg.obj
 0002:0000ff00       ??_R4Configure@apt@@6B@    0048af00     ConfigManager.obj
 0002:0000ff18       ??_R3Configure@apt@@8      0048af18     ConfigManager.obj
 0002:0000ff2c       ??_R2Configure@apt@@8      0048af2c     ConfigManager.obj
 0002:0000ff34       ??_R1A@?0A@EA@Configure@apt@@8 0048af34     ConfigManager.obj
 0002:0000ff58       ??_R4ConfigureManager@apt@@6B@ 0048af58     ConfigManager.obj
 0002:0000ff70       ??_R3ConfigureManager@apt@@8 0048af70     ConfigManager.obj
 0002:0000ff84       ??_R2ConfigureManager@apt@@8 0048af84     ConfigManager.obj
 0002:0000ff90       ??_R1A@?0A@EA@ConfigureManager@apt@@8 0048af90     ConfigManager.obj
 0002:0000ffb4       ??_R1A@?0A@EA@?$CUiSingleton@VConfigureManager@apt@@@iVMSGUIToolkit@@8 0048afb4     ConfigManager.obj
 0002:0000ffd8       ??_R3?$CUiSingleton@VConfigureManager@apt@@@iVMSGUIToolkit@@8 0048afd8     ConfigManager.obj
 0002:0000ffec       ??_R2?$CUiSingleton@VConfigureManager@apt@@@iVMSGUIToolkit@@8 0048afec     ConfigManager.obj
 0002:0000fff4       ??_R4LanaguageManager@apt@@6B@ 0048aff4     ConfigManager.obj
 0002:0001000c       ??_R3LanaguageManager@apt@@8 0048b00c     ConfigManager.obj
 0002:00010020       ??_R2LanaguageManager@apt@@8 0048b020     ConfigManager.obj
 0002:0001002c       ??_R1A@?0A@EA@LanaguageManager@apt@@8 0048b02c     ConfigManager.obj
 0002:00010050       ??_R1A@?0A@EA@?$CUiSingleton@VLanaguageManager@apt@@@iVMSGUIToolkit@@8 0048b050     ConfigManager.obj
 0002:00010074       ??_R3?$CUiSingleton@VLanaguageManager@apt@@@iVMSGUIToolkit@@8 0048b074     ConfigManager.obj
 0002:00010088       ??_R2?$CUiSingleton@VLanaguageManager@apt@@@iVMSGUIToolkit@@8 0048b088     ConfigManager.obj
 0002:00010090       ??_R4QTranslator@@6B@      0048b090     ConfigManager.obj
 0002:000100a8       ??_R3QTranslator@@8        0048b0a8     ConfigManager.obj
 0002:000100bc       ??_R2QTranslator@@8        0048b0bc     ConfigManager.obj
 0002:000100c8       ??_R1A@?0A@EA@QTranslator@@8 0048b0c8     ConfigManager.obj
 0002:000100ec       ??_R1A@?0A@EA@QObject@@8   0048b0ec     ConfigManager.obj
 0002:00010110       ??_R3QObject@@8            0048b110     ConfigManager.obj
 0002:00010124       ??_R2QObject@@8            0048b124     ConfigManager.obj
 0002:0001012c       ??_R4?$CUiSingleton@VConfigureManager@apt@@@iVMSGUIToolkit@@6B@ 0048b12c     ConfigManager.obj
 0002:00010144       ??_R4?$CUiSingleton@VLanaguageManager@apt@@@iVMSGUIToolkit@@6B@ 0048b144     ConfigManager.obj
 0002:0001015c       ??_R4ToolsApplication@apt@@6B@ 0048b15c     ToolsApplication.obj
 0002:00010174       ??_R3ToolsApplication@apt@@8 0048b174     ToolsApplication.obj
 0002:00010188       ??_R2ToolsApplication@apt@@8 0048b188     ToolsApplication.obj
 0002:000101a4       ??_R1A@?0A@EA@ToolsApplication@apt@@8 0048b1a4     ToolsApplication.obj
 0002:000101c8       ??_R1A@?0A@EA@QtSingleApplication@SharedTools@@8 0048b1c8     ToolsApplication.obj
 0002:000101ec       ??_R3QtSingleApplication@SharedTools@@8 0048b1ec     ToolsApplication.obj
 0002:00010200       ??_R2QtSingleApplication@SharedTools@@8 0048b200     ToolsApplication.obj
 0002:00010214       ??_R1A@?0A@EA@QApplication@@8 0048b214     ToolsApplication.obj
 0002:00010238       ??_R3QApplication@@8       0048b238     ToolsApplication.obj
 0002:0001024c       ??_R2QApplication@@8       0048b24c     ToolsApplication.obj
 0002:0001025c       ??_R1A@?0A@EA@QCoreApplication@@8 0048b25c     ToolsApplication.obj
 0002:00010280       ??_R3QCoreApplication@@8   0048b280     ToolsApplication.obj
 0002:00010294       ??_R2QCoreApplication@@8   0048b294     ToolsApplication.obj
 0002:000102a0       ??_R4DiskCalculatorMainPage@@6BQObject@@@ 0048b2a0     DiskCalculatorMainPage.obj
 0002:000102b8       ??_R3DiskCalculatorMainPage@@8 0048b2b8     DiskCalculatorMainPage.obj
 0002:000102cc       ??_R2DiskCalculatorMainPage@@8 0048b2cc     DiskCalculatorMainPage.obj
 0002:000102e8       ??_R1A@?0A@EA@DiskCalculatorMainPage@@8 0048b2e8     DiskCalculatorMainPage.obj
 0002:0001030c       ??_R1A@?0A@EA@QMainWindow@@8 0048b30c     DiskCalculatorMainPage.obj
 0002:00010330       ??_R3QMainWindow@@8        0048b330     DiskCalculatorMainPage.obj
 0002:00010344       ??_R2QMainWindow@@8        0048b344     DiskCalculatorMainPage.obj
 0002:00010358       ??_R1A@?0A@EA@QWidget@@8   0048b358     DiskCalculatorMainPage.obj
 0002:0001037c       ??_R3QWidget@@8            0048b37c     DiskCalculatorMainPage.obj
 0002:00010390       ??_R2QWidget@@8            0048b390     DiskCalculatorMainPage.obj
 0002:000103a0       ??_R17?0A@EA@QPaintDevice@@8 0048b3a0     DiskCalculatorMainPage.obj
 0002:000103c4       ??_R3QPaintDevice@@8       0048b3c4     DiskCalculatorMainPage.obj
 0002:000103d8       ??_R2QPaintDevice@@8       0048b3d8     DiskCalculatorMainPage.obj
 0002:000103e0       ??_R1A@?0A@EA@QPaintDevice@@8 0048b3e0     DiskCalculatorMainPage.obj
 0002:00010404       ??_R4DiskCalculatorMainPage@@6BQPaintDevice@@@ 0048b404     DiskCalculatorMainPage.obj
 0002:0001041c       ??_R4QWidget@@6BQObject@@@ 0048b41c     DiskCalculatorMainPage.obj
 0002:00010434       ??_R4QWidget@@6BQPaintDevice@@@ 0048b434     DiskCalculatorMainPage.obj
 0002:0001044c       ??_R4QGridLayout@@6BQObject@@@ 0048b44c     DiskCalculatorMainPage.obj
 0002:00010464       ??_R3QGridLayout@@8        0048b464     DiskCalculatorMainPage.obj
 0002:00010478       ??_R2QGridLayout@@8        0048b478     DiskCalculatorMainPage.obj
 0002:0001048c       ??_R1A@?0A@EA@QGridLayout@@8 0048b48c     DiskCalculatorMainPage.obj
 0002:000104b0       ??_R1A@?0A@EA@QLayout@@8   0048b4b0     DiskCalculatorMainPage.obj
 0002:000104d4       ??_R3QLayout@@8            0048b4d4     DiskCalculatorMainPage.obj
 0002:000104e8       ??_R2QLayout@@8            0048b4e8     DiskCalculatorMainPage.obj
 0002:000104f8       ??_R17?0A@EA@QLayoutItem@@8 0048b4f8     DiskCalculatorMainPage.obj
 0002:0001051c       ??_R3QLayoutItem@@8        0048b51c     DiskCalculatorMainPage.obj
 0002:00010530       ??_R2QLayoutItem@@8        0048b530     DiskCalculatorMainPage.obj
 0002:00010538       ??_R1A@?0A@EA@QLayoutItem@@8 0048b538     DiskCalculatorMainPage.obj
 0002:0001055c       ??_R4QGridLayout@@6BQLayoutItem@@@ 0048b55c     DiskCalculatorMainPage.obj
 0002:00010574       ??_R4QScrollArea@@6BQObject@@@ 0048b574     DiskCalculatorMainPage.obj
 0002:0001058c       ??_R3QScrollArea@@8        0048b58c     DiskCalculatorMainPage.obj
 0002:000105a0       ??_R2QScrollArea@@8        0048b5a0     DiskCalculatorMainPage.obj
 0002:000105c0       ??_R1A@?0A@EA@QScrollArea@@8 0048b5c0     DiskCalculatorMainPage.obj
 0002:000105e4       ??_R1A@?0A@EA@QAbstractScrollArea@@8 0048b5e4     DiskCalculatorMainPage.obj
 0002:00010608       ??_R3QAbstractScrollArea@@8 0048b608     DiskCalculatorMainPage.obj
 0002:0001061c       ??_R2QAbstractScrollArea@@8 0048b61c     DiskCalculatorMainPage.obj
 0002:00010638       ??_R1A@?0A@EA@QFrame@@8    0048b638     DiskCalculatorMainPage.obj
 0002:0001065c       ??_R3QFrame@@8             0048b65c     DiskCalculatorMainPage.obj
 0002:00010670       ??_R2QFrame@@8             0048b670     DiskCalculatorMainPage.obj
 0002:00010684       ??_R4QScrollArea@@6BQPaintDevice@@@ 0048b684     DiskCalculatorMainPage.obj
 0002:0001069c       ??_R4QVBoxLayout@@6BQObject@@@ 0048b69c     DiskCalculatorMainPage.obj
 0002:000106b4       ??_R3QVBoxLayout@@8        0048b6b4     DiskCalculatorMainPage.obj
 0002:000106c8       ??_R2QVBoxLayout@@8        0048b6c8     DiskCalculatorMainPage.obj
 0002:000106e4       ??_R1A@?0A@EA@QVBoxLayout@@8 0048b6e4     DiskCalculatorMainPage.obj
 0002:00010708       ??_R1A@?0A@EA@QBoxLayout@@8 0048b708     DiskCalculatorMainPage.obj
 0002:0001072c       ??_R3QBoxLayout@@8         0048b72c     DiskCalculatorMainPage.obj
 0002:00010740       ??_R2QBoxLayout@@8         0048b740     DiskCalculatorMainPage.obj
 0002:00010754       ??_R4QVBoxLayout@@6BQLayoutItem@@@ 0048b754     DiskCalculatorMainPage.obj
 0002:0001076c       ??_R4QHBoxLayout@@6BQObject@@@ 0048b76c     DiskCalculatorMainPage.obj
 0002:00010784       ??_R3QHBoxLayout@@8        0048b784     DiskCalculatorMainPage.obj
 0002:00010798       ??_R2QHBoxLayout@@8        0048b798     DiskCalculatorMainPage.obj
 0002:000107b4       ??_R1A@?0A@EA@QHBoxLayout@@8 0048b7b4     DiskCalculatorMainPage.obj
 0002:000107d8       ??_R4QHBoxLayout@@6BQLayoutItem@@@ 0048b7d8     DiskCalculatorMainPage.obj
 0002:000107f0       ??_R4AboutDialog@@6B@      0048b7f0     AboutDialog.obj
 0002:00010808       ??_R3AboutDialog@@8        0048b808     AboutDialog.obj
 0002:0001081c       ??_R2AboutDialog@@8        0048b81c     AboutDialog.obj
 0002:00010838       ??_R1A@?0A@EA@AboutDialog@@8 0048b838     AboutDialog.obj
 0002:0001085c       ??_R1A@?0A@EA@CDlgAbout@aptui@@8 0048b85c     AboutDialog.obj
 0002:00010880       ??_R3CDlgAbout@aptui@@8    0048b880     AboutDialog.obj
 0002:00010894       ??_R2CDlgAbout@aptui@@8    0048b894     AboutDialog.obj
 0002:000108a8       ??_R1A@?0A@EA@QWidgetAction@@8 0048b8a8     AboutDialog.obj
 0002:000108cc       ??_R3QWidgetAction@@8      0048b8cc     AboutDialog.obj
 0002:000108e0       ??_R2QWidgetAction@@8      0048b8e0     AboutDialog.obj
 0002:000108f0       ??_R1A@?0A@EA@QAction@@8   0048b8f0     AboutDialog.obj
 0002:00010914       ??_R3QAction@@8            0048b914     AboutDialog.obj
 0002:00010928       ??_R2QAction@@8            0048b928     AboutDialog.obj
 0002:00010934       ??_R4DeviceEditor@@6BQObject@@@ 0048b934     DeviceEditor.obj
 0002:0001094c       ??_R3DeviceEditor@@8       0048b94c     DeviceEditor.obj
 0002:00010960       ??_R2DeviceEditor@@8       0048b960     DeviceEditor.obj
 0002:00010974       ??_R1A@?0A@EA@DeviceEditor@@8 0048b974     DeviceEditor.obj
 0002:00010998       ??_R4DeviceEditor@@6BQPaintDevice@@@ 0048b998     DeviceEditor.obj
 0002:000109b0       ??_R4CIntValidator@iVMSGUIToolkit@@6B@ 0048b9b0     DeviceEditor.obj
 0002:000109c8       ??_R3CIntValidator@iVMSGUIToolkit@@8 0048b9c8     DeviceEditor.obj
 0002:000109dc       ??_R2CIntValidator@iVMSGUIToolkit@@8 0048b9dc     DeviceEditor.obj
 0002:000109f0       ??_R1A@?0A@EA@CIntValidator@iVMSGUIToolkit@@8 0048b9f0     DeviceEditor.obj
 0002:00010a14       ??_R1A@?0A@EA@QIntValidator@@8 0048ba14     DeviceEditor.obj
 0002:00010a38       ??_R3QIntValidator@@8      0048ba38     DeviceEditor.obj
 0002:00010a4c       ??_R2QIntValidator@@8      0048ba4c     DeviceEditor.obj
 0002:00010a5c       ??_R1A@?0A@EA@QValidator@@8 0048ba5c     DeviceEditor.obj
 0002:00010a80       ??_R3QValidator@@8         0048ba80     DeviceEditor.obj
 0002:00010a94       ??_R2QValidator@@8         0048ba94     DeviceEditor.obj
 0002:00010aa0       ??_R4QSpacerItem@@6B@      0048baa0     DeviceEditor.obj
 0002:00010ab8       ??_R3QSpacerItem@@8        0048bab8     DeviceEditor.obj
 0002:00010acc       ??_R2QSpacerItem@@8        0048bacc     DeviceEditor.obj
 0002:00010ad8       ??_R1A@?0A@EA@QSpacerItem@@8 0048bad8     DeviceEditor.obj
 0002:00010afc       ??_R4QCheckBox@@6BQObject@@@ 0048bafc     DeviceEditor.obj
 0002:00010b14       ??_R3QCheckBox@@8          0048bb14     DeviceEditor.obj
 0002:00010b28       ??_R2QCheckBox@@8          0048bb28     DeviceEditor.obj
 0002:00010b44       ??_R1A@?0A@EA@QCheckBox@@8 0048bb44     DeviceEditor.obj
 0002:00010b68       ??_R1A@?0A@EA@QAbstractButton@@8 0048bb68     DeviceEditor.obj
 0002:00010b8c       ??_R3QAbstractButton@@8    0048bb8c     DeviceEditor.obj
 0002:00010ba0       ??_R2QAbstractButton@@8    0048bba0     DeviceEditor.obj
 0002:00010bb4       ??_R4QCheckBox@@6BQPaintDevice@@@ 0048bbb4     DeviceEditor.obj
 0002:00010bcc       ??_R4QLabel@@6BQObject@@@  0048bbcc     DeviceEditor.obj
 0002:00010be4       ??_R3QLabel@@8             0048bbe4     DeviceEditor.obj
 0002:00010bf8       ??_R2QLabel@@8             0048bbf8     DeviceEditor.obj
 0002:00010c14       ??_R1A@?0A@EA@QLabel@@8    0048bc14     DeviceEditor.obj
 0002:00010c38       ??_R4QLabel@@6BQPaintDevice@@@ 0048bc38     DeviceEditor.obj
 0002:00010c50       ??_R4CLineEdit@iVMSGUIToolkit@@6BQObject@@@ 0048bc50     DeviceEditor.obj
 0002:00010c68       ??_R3CLineEdit@iVMSGUIToolkit@@8 0048bc68     DeviceEditor.obj
 0002:00010c7c       ??_R2CLineEdit@iVMSGUIToolkit@@8 0048bc7c     DeviceEditor.obj
 0002:00010c98       ??_R1A@?0A@EA@CLineEdit@iVMSGUIToolkit@@8 0048bc98     DeviceEditor.obj
 0002:00010cbc       ??_R1A@?0A@EA@QLineEdit@@8 0048bcbc     DeviceEditor.obj
 0002:00010ce0       ??_R3QLineEdit@@8          0048bce0     DeviceEditor.obj
 0002:00010cf4       ??_R2QLineEdit@@8          0048bcf4     DeviceEditor.obj
 0002:00010d08       ??_R4CLineEdit@iVMSGUIToolkit@@6BQPaintDevice@@@ 0048bd08     DeviceEditor.obj
 0002:00010d20       ??_R4CComboBox@iVMSGUIToolkit@@6BQObject@@@ 0048bd20     DeviceEditor.obj
 0002:00010d38       ??_R3CComboBox@iVMSGUIToolkit@@8 0048bd38     DeviceEditor.obj
 0002:00010d4c       ??_R2CComboBox@iVMSGUIToolkit@@8 0048bd4c     DeviceEditor.obj
 0002:00010d68       ??_R1A@?0A@EA@CComboBox@iVMSGUIToolkit@@8 0048bd68     DeviceEditor.obj
 0002:00010d8c       ??_R1A@?0A@EA@QComboBox@@8 0048bd8c     DeviceEditor.obj
 0002:00010db0       ??_R3QComboBox@@8          0048bdb0     DeviceEditor.obj
 0002:00010dc4       ??_R2QComboBox@@8          0048bdc4     DeviceEditor.obj
 0002:00010dd8       ??_R4CComboBox@iVMSGUIToolkit@@6BQPaintDevice@@@ 0048bdd8     DeviceEditor.obj
 0002:00010df0       ??_R4CRadioButton@iVMSGUIToolkit@@6BQObject@@@ 0048bdf0     DeviceEditor.obj
 0002:00010e08       ??_R3CRadioButton@iVMSGUIToolkit@@8 0048be08     DeviceEditor.obj
 0002:00010e1c       ??_R2CRadioButton@iVMSGUIToolkit@@8 0048be1c     DeviceEditor.obj
 0002:00010e3c       ??_R1A@?0A@EA@CRadioButton@iVMSGUIToolkit@@8 0048be3c     DeviceEditor.obj
 0002:00010e60       ??_R1A@?0A@EA@QRadioButton@@8 0048be60     DeviceEditor.obj
 0002:00010e84       ??_R3QRadioButton@@8       0048be84     DeviceEditor.obj
 0002:00010e98       ??_R2QRadioButton@@8       0048be98     DeviceEditor.obj
 0002:00010eb4       ??_R4CRadioButton@iVMSGUIToolkit@@6BQPaintDevice@@@ 0048beb4     DeviceEditor.obj
 0002:00010ecc       ??_R4CPushButton@iVMSGUIToolkit@@6BQObject@@@ 0048becc     DeviceEditor.obj
 0002:00010ee4       ??_R3CPushButton@iVMSGUIToolkit@@8 0048bee4     DeviceEditor.obj
 0002:00010ef8       ??_R2CPushButton@iVMSGUIToolkit@@8 0048bef8     DeviceEditor.obj
 0002:00010f18       ??_R1A@?0A@EA@CPushButton@iVMSGUIToolkit@@8 0048bf18     DeviceEditor.obj
 0002:00010f3c       ??_R1A@?0A@EA@QPushButton@@8 0048bf3c     DeviceEditor.obj
 0002:00010f60       ??_R3QPushButton@@8        0048bf60     DeviceEditor.obj
 0002:00010f74       ??_R2QPushButton@@8        0048bf74     DeviceEditor.obj
 0002:00010f90       ??_R4CPushButton@iVMSGUIToolkit@@6BQPaintDevice@@@ 0048bf90     DeviceEditor.obj
 0002:00010fa8       ??_R4QFrame@@6BQObject@@@  0048bfa8     DeviceEditor.obj
 0002:00010fc0       ??_R4QFrame@@6BQPaintDevice@@@ 0048bfc0     DeviceEditor.obj
 0002:00010fd8       ??_R4DeviceInfoManager@@6B@ 0048bfd8     DeviceInfoManager.obj
 0002:00010ff0       ??_R3DeviceInfoManager@@8  0048bff0     DeviceInfoManager.obj
 0002:00011004       ??_R2DeviceInfoManager@@8  0048c004     DeviceInfoManager.obj
 0002:00011010       ??_R1A@?0A@EA@DeviceInfoManager@@8 0048c010     DeviceInfoManager.obj
 0002:00011034       ??_R4ScenceSelector@@6BQObject@@@ 0048c034     ScenceSelector.obj
 0002:0001104c       ??_R3ScenceSelector@@8     0048c04c     ScenceSelector.obj
 0002:00011060       ??_R2ScenceSelector@@8     0048c060     ScenceSelector.obj
 0002:00011074       ??_R1A@?0A@EA@ScenceSelector@@8 0048c074     ScenceSelector.obj
 0002:00011098       ??_R4ScenceSelector@@6BQPaintDevice@@@ 0048c098     ScenceSelector.obj
 0002:000110b0       ??_R4QListWidget@@6BQObject@@@ 0048c0b0     ScenceSelector.obj
 0002:000110c8       ??_R3QListWidget@@8        0048c0c8     ScenceSelector.obj
 0002:000110dc       ??_R2QListWidget@@8        0048c0dc     ScenceSelector.obj
 0002:00011104       ??_R1A@?0A@EA@QListWidget@@8 0048c104     ScenceSelector.obj
 0002:00011128       ??_R1A@?0A@EA@QListView@@8 0048c128     ScenceSelector.obj
 0002:0001114c       ??_R3QListView@@8          0048c14c     ScenceSelector.obj
 0002:00011160       ??_R2QListView@@8          0048c160     ScenceSelector.obj
 0002:00011184       ??_R1A@?0A@EA@QAbstractItemView@@8 0048c184     ScenceSelector.obj
 0002:000111a8       ??_R3QAbstractItemView@@8  0048c1a8     ScenceSelector.obj
 0002:000111bc       ??_R2QAbstractItemView@@8  0048c1bc     ScenceSelector.obj
 0002:000111dc       ??_R4QListWidget@@6BQPaintDevice@@@ 0048c1dc     ScenceSelector.obj
 0002:000111f4       ??_R4ScenceQRaidoButton@ScenceSelector@@6BQObject@@@ 0048c1f4     ScenceSelector.obj
 0002:0001120c       ??_R3ScenceQRaidoButton@ScenceSelector@@8 0048c20c     ScenceSelector.obj
 0002:00011220       ??_R2ScenceQRaidoButton@ScenceSelector@@8 0048c220     ScenceSelector.obj
 0002:00011240       ??_R1A@?0A@EA@ScenceQRaidoButton@ScenceSelector@@8 0048c240     ScenceSelector.obj
 0002:00011264       ??_R4ScenceQRaidoButton@ScenceSelector@@6BQPaintDevice@@@ 0048c264     ScenceSelector.obj
 0002:0001127c       ??_R4CapacityCalculation@@6BQObject@@@ 0048c27c     CapacityCalculation.obj
 0002:00011294       ??_R3CapacityCalculation@@8 0048c294     CapacityCalculation.obj
 0002:000112a8       ??_R2CapacityCalculation@@8 0048c2a8     CapacityCalculation.obj
 0002:000112bc       ??_R1A@?0A@EA@CapacityCalculation@@8 0048c2bc     CapacityCalculation.obj
 0002:000112e0       ??_R4CapacityCalculation@@6BQPaintDevice@@@ 0048c2e0     CapacityCalculation.obj
 0002:000112f8       ??_R4QPushButton@@6BQObject@@@ 0048c2f8     CapacityCalculation.obj
 0002:00011310       ??_R4QPushButton@@6BQPaintDevice@@@ 0048c310     CapacityCalculation.obj
 0002:00011328       ??_R4WidgetDeviceListBorder@@6BQObject@@@ 0048c328     WidgetDeviceListBorder.obj
 0002:00011340       ??_R3WidgetDeviceListBorder@@8 0048c340     WidgetDeviceListBorder.obj
 0002:00011354       ??_R2WidgetDeviceListBorder@@8 0048c354     WidgetDeviceListBorder.obj
 0002:00011368       ??_R1A@?0A@EA@WidgetDeviceListBorder@@8 0048c368     WidgetDeviceListBorder.obj
 0002:0001138c       ??_R4WidgetDeviceListBorder@@6BQPaintDevice@@@ 0048c38c     WidgetDeviceListBorder.obj
 0002:000113a4       ??_R4BandWidthPage@@6BQObject@@@ 0048c3a4     BandWidthPage.obj
 0002:000113bc       ??_R3BandWidthPage@@8      0048c3bc     BandWidthPage.obj
 0002:000113d0       ??_R2BandWidthPage@@8      0048c3d0     BandWidthPage.obj
 0002:000113e4       ??_R1A@?0A@EA@BandWidthPage@@8 0048c3e4     BandWidthPage.obj
 0002:00011408       ??_R4BandWidthPage@@6BQPaintDevice@@@ 0048c408     BandWidthPage.obj
 0002:00011420       ??_R4DataCalculatorPage@@6BQObject@@@ 0048c420     DataCalculatorPage.obj
 0002:00011438       ??_R3DataCalculatorPage@@8 0048c438     DataCalculatorPage.obj
 0002:0001144c       ??_R2DataCalculatorPage@@8 0048c44c     DataCalculatorPage.obj
 0002:00011460       ??_R1A@?0A@EA@DataCalculatorPage@@8 0048c460     DataCalculatorPage.obj
 0002:00011484       ??_R4DataCalculatorPage@@6BQPaintDevice@@@ 0048c484     DataCalculatorPage.obj
 0002:0001149c       ??_R4QStackedWidget@@6BQObject@@@ 0048c49c     DataCalculatorPage.obj
 0002:000114b4       ??_R3QStackedWidget@@8     0048c4b4     DataCalculatorPage.obj
 0002:000114c8       ??_R2QStackedWidget@@8     0048c4c8     DataCalculatorPage.obj
 0002:000114e4       ??_R1A@?0A@EA@QStackedWidget@@8 0048c4e4     DataCalculatorPage.obj
 0002:00011508       ??_R4QStackedWidget@@6BQPaintDevice@@@ 0048c508     DataCalculatorPage.obj
 0002:00011520       ??_R4CSlider@iVMSGUIToolkit@@6BQObject@@@ 0048c520     DataCalculatorPage.obj
 0002:00011538       ??_R3CSlider@iVMSGUIToolkit@@8 0048c538     DataCalculatorPage.obj
 0002:0001154c       ??_R2CSlider@iVMSGUIToolkit@@8 0048c54c     DataCalculatorPage.obj
 0002:0001156c       ??_R1A@?0A@EA@CSlider@iVMSGUIToolkit@@8 0048c56c     DataCalculatorPage.obj
 0002:00011590       ??_R1A@?0A@EA@QSlider@@8   0048c590     DataCalculatorPage.obj
 0002:000115b4       ??_R3QSlider@@8            0048c5b4     DataCalculatorPage.obj
 0002:000115c8       ??_R2QSlider@@8            0048c5c8     DataCalculatorPage.obj
 0002:000115e4       ??_R1A@?0A@EA@QAbstractSlider@@8 0048c5e4     DataCalculatorPage.obj
 0002:00011608       ??_R3QAbstractSlider@@8    0048c608     DataCalculatorPage.obj
 0002:0001161c       ??_R2QAbstractSlider@@8    0048c61c     DataCalculatorPage.obj
 0002:00011630       ??_R4CSlider@iVMSGUIToolkit@@6BQPaintDevice@@@ 0048c630     DataCalculatorPage.obj
 0002:00011648       ??_R4DataDisplayPage@@6BQObject@@@ 0048c648     DataDisplayPage.obj
 0002:00011660       ??_R3DataDisplayPage@@8    0048c660     DataDisplayPage.obj
 0002:00011674       ??_R2DataDisplayPage@@8    0048c674     DataDisplayPage.obj
 0002:00011688       ??_R1A@?0A@EA@DataDisplayPage@@8 0048c688     DataDisplayPage.obj
 0002:000116ac       ??_R4DataDisplayPage@@6BQPaintDevice@@@ 0048c6ac     DataDisplayPage.obj
 0002:000116c4       ??_R4SizeDisplayPage@@6BQObject@@@ 0048c6c4     SizeDisplayPage.obj
 0002:000116dc       ??_R3SizeDisplayPage@@8    0048c6dc     SizeDisplayPage.obj
 0002:000116f0       ??_R2SizeDisplayPage@@8    0048c6f0     SizeDisplayPage.obj
 0002:00011704       ??_R1A@?0A@EA@SizeDisplayPage@@8 0048c704     SizeDisplayPage.obj
 0002:00011728       ??_R4SizeDisplayPage@@6BQPaintDevice@@@ 0048c728     SizeDisplayPage.obj
 0002:00011740       ??_R4DeviceAddPage@@6BQObject@@@ 0048c740     DeviceAddPage.obj
 0002:00011758       ??_R3DeviceAddPage@@8      0048c758     DeviceAddPage.obj
 0002:0001176c       ??_R2DeviceAddPage@@8      0048c76c     DeviceAddPage.obj
 0002:00011780       ??_R1A@?0A@EA@DeviceAddPage@@8 0048c780     DeviceAddPage.obj
 0002:000117a4       ??_R4DeviceAddPage@@6BQPaintDevice@@@ 0048c7a4     DeviceAddPage.obj
 0002:000117bc       ??_R4DeviceItemWidget@NM_DiskCalculator@@6BQObject@@@ 0048c7bc     DeviceItemWidget.obj
 0002:000117d4       ??_R3DeviceItemWidget@NM_DiskCalculator@@8 0048c7d4     DeviceItemWidget.obj
 0002:000117e8       ??_R2DeviceItemWidget@NM_DiskCalculator@@8 0048c7e8     DeviceItemWidget.obj
 0002:000117fc       ??_R1A@?0A@EA@DeviceItemWidget@NM_DiskCalculator@@8 0048c7fc     DeviceItemWidget.obj
 0002:00011820       ??_R4DeviceItemWidget@NM_DiskCalculator@@6BQPaintDevice@@@ 0048c820     DeviceItemWidget.obj
 0002:00011838       ??_R4QToolButton@@6BQObject@@@ 0048c838     DeviceItemWidget.obj
 0002:00011850       ??_R3QToolButton@@8        0048c850     DeviceItemWidget.obj
 0002:00011864       ??_R2QToolButton@@8        0048c864     DeviceItemWidget.obj
 0002:00011880       ??_R1A@?0A@EA@QToolButton@@8 0048c880     DeviceItemWidget.obj
 0002:000118a4       ??_R4QToolButton@@6BQPaintDevice@@@ 0048c8a4     DeviceItemWidget.obj
 0002:000118bc       ??_R4ButtonRadio@aptui@@6BQObject@@@ 0048c8bc     ButtonRadio.obj
 0002:000118d4       ??_R3ButtonRadio@aptui@@8  0048c8d4     ButtonRadio.obj
 0002:000118e8       ??_R2ButtonRadio@aptui@@8  0048c8e8     ButtonRadio.obj
 0002:00011908       ??_R1A@?0A@EA@ButtonRadio@aptui@@8 0048c908     ButtonRadio.obj
 0002:0001192c       ??_R4ButtonRadio@aptui@@6BQPaintDevice@@@ 0048c92c     ButtonRadio.obj
 0002:00011944       ??_R4UpdateDialog@@6BQObject@@@ 0048c944     UpdateDialog.obj
 0002:0001195c       ??_R3UpdateDialog@@8       0048c95c     UpdateDialog.obj
 0002:00011970       ??_R2UpdateDialog@@8       0048c970     UpdateDialog.obj
 0002:00011990       ??_R1A@?0A@EA@UpdateDialog@@8 0048c990     UpdateDialog.obj
 0002:000119b4       ??_R1A@?0A@EA@BaseDialog@aptui@@8 0048c9b4     UpdateDialog.obj
 0002:000119d8       ??_R3BaseDialog@aptui@@8   0048c9d8     UpdateDialog.obj
 0002:000119ec       ??_R2BaseDialog@aptui@@8   0048c9ec     UpdateDialog.obj
 0002:00011a08       ??_R1A@?0A@EA@QDialog@@8   0048ca08     UpdateDialog.obj
 0002:00011a2c       ??_R3QDialog@@8            0048ca2c     UpdateDialog.obj
 0002:00011a40       ??_R2QDialog@@8            0048ca40     UpdateDialog.obj
 0002:00011a54       ??_R4UpdateDialog@@6BQPaintDevice@@@ 0048ca54     UpdateDialog.obj
 0002:00011a6c       ??_R4WarningDialog@NM_DiskCalculator@@6BQObject@@@ 0048ca6c     WarningDialog.obj
 0002:00011a84       ??_R3WarningDialog@NM_DiskCalculator@@8 0048ca84     WarningDialog.obj
 0002:00011a98       ??_R2WarningDialog@NM_DiskCalculator@@8 0048ca98     WarningDialog.obj
 0002:00011ab4       ??_R1A@?0A@EA@WarningDialog@NM_DiskCalculator@@8 0048cab4     WarningDialog.obj
 0002:00011ad8       ??_R4WarningDialog@NM_DiskCalculator@@6BQPaintDevice@@@ 0048cad8     WarningDialog.obj
 0002:00011af0       ??_R4TipDialog@NM_DiskCalculator@@6BQObject@@@ 0048caf0     TipDialog.obj
 0002:00011b08       ??_R3TipDialog@NM_DiskCalculator@@8 0048cb08     TipDialog.obj
 0002:00011b1c       ??_R2TipDialog@NM_DiskCalculator@@8 0048cb1c     TipDialog.obj
 0002:00011b3c       ??_R1A@?0A@EA@TipDialog@NM_DiskCalculator@@8 0048cb3c     TipDialog.obj
 0002:00011b60       ??_R4TipDialog@NM_DiskCalculator@@6BQPaintDevice@@@ 0048cb60     TipDialog.obj
 0002:00011b78       ??_R4BaseTitle@aptui@@6BQObject@@@ 0048cb78     BaseTitle.obj
 0002:00011b90       ??_R3BaseTitle@aptui@@8    0048cb90     BaseTitle.obj
 0002:00011ba4       ??_R2BaseTitle@aptui@@8    0048cba4     BaseTitle.obj
 0002:00011bc8       ??_R1A@?0A@EA@BaseTitle@aptui@@8 0048cbc8     BaseTitle.obj
 0002:00011bec       ??_R1A@?0A@EA@CFancyTitle@iVMSGUIToolkit@@8 0048cbec     BaseTitle.obj
 0002:00011c10       ??_R3CFancyTitle@iVMSGUIToolkit@@8 0048cc10     BaseTitle.obj
 0002:00011c24       ??_R2CFancyTitle@iVMSGUIToolkit@@8 0048cc24     BaseTitle.obj
 0002:00011c44       ??_R1BE@?0A@EA@CWidgetSizeFactory@iVMSGUIToolkit@@8 0048cc44     BaseTitle.obj
 0002:00011c68       ??_R3CWidgetSizeFactory@iVMSGUIToolkit@@8 0048cc68     BaseTitle.obj
 0002:00011c7c       ??_R2CWidgetSizeFactory@iVMSGUIToolkit@@8 0048cc7c     BaseTitle.obj
 0002:00011c84       ??_R1A@?0A@EA@CWidgetSizeFactory@iVMSGUIToolkit@@8 0048cc84     BaseTitle.obj
 0002:00011ca8       ??_R4BaseTitle@aptui@@6BQPaintDevice@@@ 0048cca8     BaseTitle.obj
 0002:00011cc0       ??_R4BaseTitle@aptui@@6B@  0048ccc0     BaseTitle.obj
 0002:00011cd8       ??_R4WindowTitle@aptui@@6BQObject@@@ 0048ccd8     WindowTitle.obj
 0002:00011cf0       ??_R3WindowTitle@aptui@@8  0048ccf0     WindowTitle.obj
 0002:00011d04       ??_R2WindowTitle@aptui@@8  0048cd04     WindowTitle.obj
 0002:00011d28       ??_R1A@?0A@EA@WindowTitle@aptui@@8 0048cd28     WindowTitle.obj
 0002:00011d4c       ??_R4WindowTitle@aptui@@6BQPaintDevice@@@ 0048cd4c     WindowTitle.obj
 0002:00011d64       ??_R4WindowTitle@aptui@@6B@ 0048cd64     WindowTitle.obj
 0002:00011d7c       ??_R4CHBoxLayout@iVMSGUIToolkit@@6BQObject@@@ 0048cd7c     WindowTitle.obj
 0002:00011d94       ??_R3CHBoxLayout@iVMSGUIToolkit@@8 0048cd94     WindowTitle.obj
 0002:00011da8       ??_R2CHBoxLayout@iVMSGUIToolkit@@8 0048cda8     WindowTitle.obj
 0002:00011dc8       ??_R1A@?0A@EA@CHBoxLayout@iVMSGUIToolkit@@8 0048cdc8     WindowTitle.obj
 0002:00011dec       ??_R1BA@?0A@EA@CLayoutFunction@iVMSGUIToolkit@@8 0048cdec     WindowTitle.obj
 0002:00011e10       ??_R3CLayoutFunction@iVMSGUIToolkit@@8 0048ce10     WindowTitle.obj
 0002:00011e24       ??_R2CLayoutFunction@iVMSGUIToolkit@@8 0048ce24     WindowTitle.obj
 0002:00011e2c       ??_R1A@?0A@EA@CLayoutFunction@iVMSGUIToolkit@@8 0048ce2c     WindowTitle.obj
 0002:00011e50       ??_R4CHBoxLayout@iVMSGUIToolkit@@6BQLayoutItem@@@ 0048ce50     WindowTitle.obj
 0002:00011e68       ??_R4CWidgetItem@iVMSGUIToolkit@@6B@ 0048ce68     WindowTitle.obj
 0002:00011e80       ??_R3CWidgetItem@iVMSGUIToolkit@@8 0048ce80     WindowTitle.obj
 0002:00011e94       ??_R2CWidgetItem@iVMSGUIToolkit@@8 0048ce94     WindowTitle.obj
 0002:00011ea4       ??_R1A@?0A@EA@CWidgetItem@iVMSGUIToolkit@@8 0048cea4     WindowTitle.obj
 0002:00011ec8       ??_R1A@?0A@EA@QWidgetItem@@8 0048cec8     WindowTitle.obj
 0002:00011eec       ??_R3QWidgetItem@@8        0048ceec     WindowTitle.obj
 0002:00011f00       ??_R2QWidgetItem@@8        0048cf00     WindowTitle.obj
 0002:00011f0c       ??_R4Menu@aptui@@6BQObject@@@ 0048cf0c     Menu.obj
 0002:00011f24       ??_R3Menu@aptui@@8         0048cf24     Menu.obj
 0002:00011f38       ??_R2Menu@aptui@@8         0048cf38     Menu.obj
 0002:00011f54       ??_R1A@?0A@EA@Menu@aptui@@8 0048cf54     Menu.obj
 0002:00011f78       ??_R1A@?0A@EA@QMenu@@8     0048cf78     Menu.obj
 0002:00011f9c       ??_R3QMenu@@8              0048cf9c     Menu.obj
 0002:00011fb0       ??_R2QMenu@@8              0048cfb0     Menu.obj
 0002:00011fc4       ??_R4Menu@aptui@@6BQPaintDevice@@@ 0048cfc4     Menu.obj
 0002:00011fdc       ??_R4CCustomStyle@Menu@aptui@@6B@ 0048cfdc     Menu.obj
 0002:00011ff4       ??_R3CCustomStyle@Menu@aptui@@8 0048cff4     Menu.obj
 0002:00012008       ??_R2CCustomStyle@Menu@aptui@@8 0048d008     Menu.obj
 0002:00012024       ??_R1A@?0A@EA@CCustomStyle@Menu@aptui@@8 0048d024     Menu.obj
 0002:00012048       ??_R1A@?0A@EA@QProxyStyle@@8 0048d048     Menu.obj
 0002:0001206c       ??_R3QProxyStyle@@8        0048d06c     Menu.obj
 0002:00012080       ??_R2QProxyStyle@@8        0048d080     Menu.obj
 0002:00012094       ??_R1A@?0A@EA@QCommonStyle@@8 0048d094     Menu.obj
 0002:000120b8       ??_R3QCommonStyle@@8       0048d0b8     Menu.obj
 0002:000120cc       ??_R2QCommonStyle@@8       0048d0cc     Menu.obj
 0002:000120dc       ??_R1A@?0A@EA@QStyle@@8    0048d0dc     Menu.obj
 0002:00012100       ??_R3QStyle@@8             0048d100     Menu.obj
 0002:00012114       ??_R2QStyle@@8             0048d114     Menu.obj
 0002:00012120       ??_R4SystemMenu@aptui@@6BQObject@@@ 0048d120     TitleMenu.obj
 0002:00012138       ??_R3SystemMenu@aptui@@8   0048d138     TitleMenu.obj
 0002:0001214c       ??_R2SystemMenu@aptui@@8   0048d14c     TitleMenu.obj
 0002:0001216c       ??_R1A@?0A@EA@SystemMenu@aptui@@8 0048d16c     TitleMenu.obj
 0002:00012190       ??_R1A@?0A@EA@CMenu@iVMSGUIToolkit@@8 0048d190     TitleMenu.obj
 0002:000121b4       ??_R3CMenu@iVMSGUIToolkit@@8 0048d1b4     TitleMenu.obj
 0002:000121c8       ??_R2CMenu@iVMSGUIToolkit@@8 0048d1c8     TitleMenu.obj
 0002:000121e4       ??_R4SystemMenu@aptui@@6BQPaintDevice@@@ 0048d1e4     TitleMenu.obj
 0002:000121fc       ??_R4LineEditInterger@aptui@@6BQObject@@@ 0048d1fc     LineEditInterger.obj
 0002:00012214       ??_R3LineEditInterger@aptui@@8 0048d214     LineEditInterger.obj
 0002:00012228       ??_R2LineEditInterger@aptui@@8 0048d228     LineEditInterger.obj
 0002:00012248       ??_R1A@?0A@EA@LineEditInterger@aptui@@8 0048d248     LineEditInterger.obj
 0002:0001226c       ??_R1A@?0A@EA@QSpinBox@@8  0048d26c     LineEditInterger.obj
 0002:00012290       ??_R3QSpinBox@@8           0048d290     LineEditInterger.obj
 0002:000122a4       ??_R2QSpinBox@@8           0048d2a4     LineEditInterger.obj
 0002:000122c0       ??_R1A@?0A@EA@QAbstractSpinBox@@8 0048d2c0     LineEditInterger.obj
 0002:000122e4       ??_R3QAbstractSpinBox@@8   0048d2e4     LineEditInterger.obj
 0002:000122f8       ??_R2QAbstractSpinBox@@8   0048d2f8     LineEditInterger.obj
 0002:0001230c       ??_R4LineEditInterger@aptui@@6BQPaintDevice@@@ 0048d30c     LineEditInterger.obj
 0002:00012324       ??_R4TabWidget@aptui@@6BQObject@@@ 0048d324     TabWidget.obj
 0002:0001233c       ??_R3TabWidget@aptui@@8    0048d33c     TabWidget.obj
 0002:00012350       ??_R2TabWidget@aptui@@8    0048d350     TabWidget.obj
 0002:0001236c       ??_R1A@?0A@EA@TabWidget@aptui@@8 0048d36c     TabWidget.obj
 0002:00012390       ??_R1A@?0A@EA@QTabWidget@@8 0048d390     TabWidget.obj
 0002:000123b4       ??_R3QTabWidget@@8         0048d3b4     TabWidget.obj
 0002:000123c8       ??_R2QTabWidget@@8         0048d3c8     TabWidget.obj
 0002:000123dc       ??_R4TabWidget@aptui@@6BQPaintDevice@@@ 0048d3dc     TabWidget.obj
 0002:000123f4       ??_R4Line@aptui@@6BQObject@@@ 0048d3f4     Line.obj
 0002:0001240c       ??_R3Line@aptui@@8         0048d40c     Line.obj
 0002:00012420       ??_R2Line@aptui@@8         0048d420     Line.obj
 0002:0001243c       ??_R1A@?0A@EA@Line@aptui@@8 0048d43c     Line.obj
 0002:00012460       ??_R4Line@aptui@@6BQPaintDevice@@@ 0048d460     Line.obj
 0002:00012478       ??_R4CDlgAbout@aptui@@6B@  0048d478     DlgAbout.obj
 0002:00012490       ??_R4Switch@aptui@@6BQObject@@@ 0048d490     Switch.obj
 0002:000124a8       ??_R3Switch@aptui@@8       0048d4a8     Switch.obj
 0002:000124bc       ??_R2Switch@aptui@@8       0048d4bc     Switch.obj
 0002:000124d0       ??_R1A@?0A@EA@Switch@aptui@@8 0048d4d0     Switch.obj
 0002:000124f4       ??_R4Switch@aptui@@6BQPaintDevice@@@ 0048d4f4     Switch.obj
 0002:0001250c       ??_R4CoverWidget@aptui@@6BQObject@@@ 0048d50c     CoverWidget.obj
 0002:00012524       ??_R3CoverWidget@aptui@@8  0048d524     CoverWidget.obj
 0002:00012538       ??_R2CoverWidget@aptui@@8  0048d538     CoverWidget.obj
 0002:00012554       ??_R1A@?0A@EA@CoverWidget@aptui@@8 0048d554     CoverWidget.obj
 0002:00012578       ??_R1A@?0A@EA@Widget@aptui@@8 0048d578     CoverWidget.obj
 0002:0001259c       ??_R3Widget@aptui@@8       0048d59c     CoverWidget.obj
 0002:000125b0       ??_R2Widget@aptui@@8       0048d5b0     CoverWidget.obj
 0002:000125c4       ??_R4CoverWidget@aptui@@6BQPaintDevice@@@ 0048d5c4     CoverWidget.obj
 0002:000125dc       ??_R4Widget@aptui@@6BQObject@@@ 0048d5dc     Widget.obj
 0002:000125f4       ??_R4Widget@aptui@@6BQPaintDevice@@@ 0048d5f4     Widget.obj
 0002:0001260c       ??_R4MultiStatePushButton@aptui@@6BQObject@@@ 0048d60c     MultiStatePushButton.obj
 0002:00012624       ??_R3MultiStatePushButton@aptui@@8 0048d624     MultiStatePushButton.obj
 0002:00012638       ??_R2MultiStatePushButton@aptui@@8 0048d638     MultiStatePushButton.obj
 0002:00012658       ??_R1A@?0A@EA@MultiStatePushButton@aptui@@8 0048d658     MultiStatePushButton.obj
 0002:0001267c       ??_R4MultiStatePushButton@aptui@@6BQPaintDevice@@@ 0048d67c     MultiStatePushButton.obj
 0002:00012694       ??_R4BaseDialog@aptui@@6BQObject@@@ 0048d694     BaseDialog.obj
 0002:000126ac       ??_R4BaseDialog@aptui@@6BQPaintDevice@@@ 0048d6ac     BaseDialog.obj
 0002:000126c4       ??_R4Label@aptui@@6BQObject@@@ 0048d6c4     Label.obj
 0002:000126dc       ??_R3Label@aptui@@8        0048d6dc     Label.obj
 0002:000126f0       ??_R2Label@aptui@@8        0048d6f0     Label.obj
 0002:00012710       ??_R1A@?0A@EA@Label@aptui@@8 0048d710     Label.obj
 0002:00012734       ??_R4Label@aptui@@6BQPaintDevice@@@ 0048d734     Label.obj
 0002:0001274c       ??_R4EditableLabel@aptui@@6BQObject@@@ 0048d74c     Label.obj
 0002:00012764       ??_R3EditableLabel@aptui@@8 0048d764     Label.obj
 0002:00012778       ??_R2EditableLabel@aptui@@8 0048d778     Label.obj
 0002:0001279c       ??_R1A@?0A@EA@EditableLabel@aptui@@8 0048d79c     Label.obj
 0002:000127c0       ??_R4EditableLabel@aptui@@6BQPaintDevice@@@ 0048d7c0     Label.obj
 0002:000127d8       ??_R4ColorLabel@aptui@@6BQObject@@@ 0048d7d8     Label.obj
 0002:000127f0       ??_R3ColorLabel@aptui@@8   0048d7f0     Label.obj
 0002:00012804       ??_R2ColorLabel@aptui@@8   0048d804     Label.obj
 0002:00012828       ??_R1A@?0A@EA@ColorLabel@aptui@@8 0048d828     Label.obj
 0002:0001284c       ??_R4ColorLabel@aptui@@6BQPaintDevice@@@ 0048d84c     Label.obj
 0002:00012864       ??_R4QColorDialog@@6BQObject@@@ 0048d864     Label.obj
 0002:0001287c       ??_R3QColorDialog@@8       0048d87c     Label.obj
 0002:00012890       ??_R2QColorDialog@@8       0048d890     Label.obj
 0002:000128ac       ??_R1A@?0A@EA@QColorDialog@@8 0048d8ac     Label.obj
 0002:000128d0       ??_R4QColorDialog@@6BQPaintDevice@@@ 0048d8d0     Label.obj
 0002:000128e8       ??_R4QtLockedFile@SharedTools@@6B@ 0048d8e8     qtlockedfile.obj
 0002:00012900       ??_R3QtLockedFile@SharedTools@@8 0048d900     qtlockedfile.obj
 0002:00012914       ??_R2QtLockedFile@SharedTools@@8 0048d914     qtlockedfile.obj
 0002:00012928       ??_R1A@?0A@EA@QtLockedFile@SharedTools@@8 0048d928     qtlockedfile.obj
 0002:0001294c       ??_R1A@?0A@EA@QFile@@8     0048d94c     qtlockedfile.obj
 0002:00012970       ??_R3QFile@@8              0048d970     qtlockedfile.obj
 0002:00012984       ??_R2QFile@@8              0048d984     qtlockedfile.obj
 0002:00012994       ??_R1A@?0A@EA@QIODevice@@8 0048d994     qtlockedfile.obj
 0002:000129b8       ??_R3QIODevice@@8          0048d9b8     qtlockedfile.obj
 0002:000129cc       ??_R2QIODevice@@8          0048d9cc     qtlockedfile.obj
 0002:000129d8       ??_R4QtLocalPeer@SharedTools@@6B@ 0048d9d8     qtlocalpeer.obj
 0002:000129f0       ??_R3QtLocalPeer@SharedTools@@8 0048d9f0     qtlocalpeer.obj
 0002:00012a04       ??_R2QtLocalPeer@SharedTools@@8 0048da04     qtlocalpeer.obj
 0002:00012a10       ??_R1A@?0A@EA@QtLocalPeer@SharedTools@@8 0048da10     qtlocalpeer.obj
 0002:00012a34       ??_R4QLocalServer@@6B@     0048da34     qtlocalpeer.obj
 0002:00012a4c       ??_R3QLocalServer@@8       0048da4c     qtlocalpeer.obj
 0002:00012a60       ??_R2QLocalServer@@8       0048da60     qtlocalpeer.obj
 0002:00012a6c       ??_R1A@?0A@EA@QLocalServer@@8 0048da6c     qtlocalpeer.obj
 0002:00012a90       ??_R4QtSingleApplication@SharedTools@@6B@ 0048da90     qtsingleapplication.obj
 0002:00012aa8       ??_R4QtSingleCoreApplication@SharedTools@@6B@ 0048daa8     qtsinglecoreapplication.obj
 0002:00012ac0       ??_R3QtSingleCoreApplication@SharedTools@@8 0048dac0     qtsinglecoreapplication.obj
 0002:00012ad4       ??_R2QtSingleCoreApplication@SharedTools@@8 0048dad4     qtsinglecoreapplication.obj
 0002:00012ae4       ??_R1A@?0A@EA@QtSingleCoreApplication@SharedTools@@8 0048dae4     qtsinglecoreapplication.obj
 0002:00012b08       ??_R4type_info@@6B@        0048db08     MSVCRT:ti_inst.obj
 0002:00012b1c       ??_R3type_info@@8          0048db1c     MSVCRT:ti_inst.obj
 0002:00012b2c       ??_R2type_info@@8          0048db2c     MSVCRT:ti_inst.obj
 0002:00012b34       ??_R1A@?0A@EA@type_info@@8 0048db34     MSVCRT:ti_inst.obj
 0002:00012d60       ___safe_se_handler_table   0048dd60     <linker-defined>
 0002:000134e8       ___rtc_iaa                 0048e4e8     MSVCRT:_initsect_.obj
 0002:000135ec       ___rtc_izz                 0048e5ec     MSVCRT:_initsect_.obj
 0002:000136f0       ___rtc_taa                 0048e6f0     MSVCRT:_initsect_.obj
 0002:000137f4       ___rtc_tzz                 0048e7f4     MSVCRT:_initsect_.obj
 0003:00000004       ??_R0?AVbad_alloc@std@@@8  0049a004     BitrateCalculate.obj
 0003:00000028       ??_R0?AVConfigure@apt@@@8  0049a028     ConfigManager.obj
 0003:0000004c       ??_R0?AVConfigureManager@apt@@@8 0049a04c     ConfigManager.obj
 0003:00000078       ??_R0?AV?$CUiSingleton@VConfigureManager@apt@@@iVMSGUIToolkit@@@8 0049a078     ConfigManager.obj
 0003:000000cc       ??_R0?AVLanaguageManager@apt@@@8 0049a0cc     ConfigManager.obj
 0003:000000f8       ??_R0?AV?$CUiSingleton@VLanaguageManager@apt@@@iVMSGUIToolkit@@@8 0049a0f8     ConfigManager.obj
 0003:0000014c       ??_R0?AVQTranslator@@@8    0049a14c     ConfigManager.obj
 0003:0000016c       ??_R0?AVQObject@@@8        0049a16c     ConfigManager.obj
 0003:00000188       ??_R0?AVToolsApplication@apt@@@8 0049a188     ToolsApplication.obj
 0003:000001b4       ??_R0?AVQtSingleApplication@SharedTools@@@8 0049a1b4     ToolsApplication.obj
 0003:000001ec       ??_R0?AVQApplication@@@8   0049a1ec     ToolsApplication.obj
 0003:0000020c       ??_R0?AVQCoreApplication@@@8 0049a20c     ToolsApplication.obj
 0003:00000234       ??_R0?AVDiskCalculatorMainPage@@@8 0049a234     DiskCalculatorMainPage.obj
 0003:00000260       ??_R0?AVQMainWindow@@@8    0049a260     DiskCalculatorMainPage.obj
 0003:00000280       ??_R0?AVQWidget@@@8        0049a280     DiskCalculatorMainPage.obj
 0003:0000029c       ??_R0?AVQPaintDevice@@@8   0049a29c     DiskCalculatorMainPage.obj
 0003:000002bc       ??_R0?AVQGridLayout@@@8    0049a2bc     DiskCalculatorMainPage.obj
 0003:000002dc       ??_R0?AVQLayout@@@8        0049a2dc     DiskCalculatorMainPage.obj
 0003:000002f8       ??_R0?AVQLayoutItem@@@8    0049a2f8     DiskCalculatorMainPage.obj
 0003:00000318       ??_R0?AVQScrollArea@@@8    0049a318     DiskCalculatorMainPage.obj
 0003:00000338       ??_R0?AVQAbstractScrollArea@@@8 0049a338     DiskCalculatorMainPage.obj
 0003:00000360       ??_R0?AVQFrame@@@8         0049a360     DiskCalculatorMainPage.obj
 0003:0000037c       ??_R0?AVQVBoxLayout@@@8    0049a37c     DiskCalculatorMainPage.obj
 0003:0000039c       ??_R0?AVQBoxLayout@@@8     0049a39c     DiskCalculatorMainPage.obj
 0003:000003bc       ??_R0?AVQHBoxLayout@@@8    0049a3bc     DiskCalculatorMainPage.obj
 0003:000003dc       ??_R0?AVAboutDialog@@@8    0049a3dc     AboutDialog.obj
 0003:000003fc       ??_R0?AVCDlgAbout@aptui@@@8 0049a3fc     AboutDialog.obj
 0003:00000420       ??_R0?AVQWidgetAction@@@8  0049a420     AboutDialog.obj
 0003:00000444       ??_R0?AVQAction@@@8        0049a444     AboutDialog.obj
 0003:00000460       ??_R0?AVDeviceEditor@@@8   0049a460     DeviceEditor.obj
 0003:00000480       ??_R0?AVCIntValidator@iVMSGUIToolkit@@@8 0049a480     DeviceEditor.obj
 0003:000004b4       ??_R0?AVQIntValidator@@@8  0049a4b4     DeviceEditor.obj
 0003:000004d8       ??_R0?AVQValidator@@@8     0049a4d8     DeviceEditor.obj
 0003:000004f8       ??_R0?AVQSpacerItem@@@8    0049a4f8     DeviceEditor.obj
 0003:00000518       ??_R0?AVQCheckBox@@@8      0049a518     DeviceEditor.obj
 0003:00000534       ??_R0?AVQAbstractButton@@@8 0049a534     DeviceEditor.obj
 0003:00000558       ??_R0?AVQLabel@@@8         0049a558     DeviceEditor.obj
 0003:00000574       ??_R0?AVCLineEdit@iVMSGUIToolkit@@@8 0049a574     DeviceEditor.obj
 0003:000005a4       ??_R0?AVQLineEdit@@@8      0049a5a4     DeviceEditor.obj
 0003:000005c0       ??_R0?AVCComboBox@iVMSGUIToolkit@@@8 0049a5c0     DeviceEditor.obj
 0003:000005f0       ??_R0?AVQComboBox@@@8      0049a5f0     DeviceEditor.obj
 0003:0000060c       ??_R0?AVCRadioButton@iVMSGUIToolkit@@@8 0049a60c     DeviceEditor.obj
 0003:00000640       ??_R0?AVQRadioButton@@@8   0049a640     DeviceEditor.obj
 0003:00000660       ??_R0?AVCPushButton@iVMSGUIToolkit@@@8 0049a660     DeviceEditor.obj
 0003:00000694       ??_R0?AVQPushButton@@@8    0049a694     DeviceEditor.obj
 0003:000006b4       ??_R0?AVDeviceInfoManager@@@8 0049a6b4     DeviceInfoManager.obj
 0003:000006dc       ??_R0?AVScenceSelector@@@8 0049a6dc     ScenceSelector.obj
 0003:00000700       ??_R0?AVQListWidget@@@8    0049a700     ScenceSelector.obj
 0003:00000720       ??_R0?AVQListView@@@8      0049a720     ScenceSelector.obj
 0003:0000073c       ??_R0?AVQAbstractItemView@@@8 0049a73c     ScenceSelector.obj
 0003:00000764       ??_R0?AVScenceQRaidoButton@ScenceSelector@@@8 0049a764     ScenceSelector.obj
 0003:000007a0       ??_R0?AVCapacityCalculation@@@8 0049a7a0     CapacityCalculation.obj
 0003:000007c8       ??_R0?AVWidgetDeviceListBorder@@@8 0049a7c8     WidgetDeviceListBorder.obj
 0003:000007f4       ??_R0?AVBandWidthPage@@@8  0049a7f4     BandWidthPage.obj
 0003:00000818       ??_R0?AVDataCalculatorPage@@@8 0049a818     DataCalculatorPage.obj
 0003:00000840       ??_R0?AVQStackedWidget@@@8 0049a840     DataCalculatorPage.obj
 0003:00000864       ??_R0?AVCSlider@iVMSGUIToolkit@@@8 0049a864     DataCalculatorPage.obj
 0003:00000890       ??_R0?AVQSlider@@@8        0049a890     DataCalculatorPage.obj
 0003:000008ac       ??_R0?AVQAbstractSlider@@@8 0049a8ac     DataCalculatorPage.obj
 0003:000008d0       ??_R0?AVDataDisplayPage@@@8 0049a8d0     DataDisplayPage.obj
 0003:000008f4       ??_R0?AVSizeDisplayPage@@@8 0049a8f4     SizeDisplayPage.obj
 0003:00000918       ??_R0?AVDeviceAddPage@@@8  0049a918     DeviceAddPage.obj
 0003:0000093c       ??_R0?AVDeviceItemWidget@NM_DiskCalculator@@@8 0049a93c     DeviceItemWidget.obj
 0003:00000978       ??_R0?AVQToolButton@@@8    0049a978     DeviceItemWidget.obj
 0003:00000998       ??_R0?AVButtonRadio@aptui@@@8 0049a998     ButtonRadio.obj
 0003:000009c0       ??_R0?AVUpdateDialog@@@8   0049a9c0     UpdateDialog.obj
 0003:000009e0       ??_R0?AVBaseDialog@aptui@@@8 0049a9e0     UpdateDialog.obj
 0003:00000a08       ??_R0?AVQDialog@@@8        0049aa08     UpdateDialog.obj
 0003:00000a24       ??_R0?AVWarningDialog@NM_DiskCalculator@@@8 0049aa24     WarningDialog.obj
 0003:00000a5c       ??_R0?AVTipDialog@NM_DiskCalculator@@@8 0049aa5c     TipDialog.obj
 0003:00000a90       ??_R0?AVBaseTitle@aptui@@@8 0049aa90     BaseTitle.obj
 0003:00000ab4       ??_R0?AVCFancyTitle@iVMSGUIToolkit@@@8 0049aab4     BaseTitle.obj
 0003:00000ae8       ??_R0?AVCWidgetSizeFactory@iVMSGUIToolkit@@@8 0049aae8     BaseTitle.obj
 0003:00000b24       ??_R0?AVWindowTitle@aptui@@@8 0049ab24     WindowTitle.obj
 0003:00000b4c       ??_R0?AVCHBoxLayout@iVMSGUIToolkit@@@8 0049ab4c     WindowTitle.obj
 0003:00000b80       ??_R0?AVCLayoutFunction@iVMSGUIToolkit@@@8 0049ab80     WindowTitle.obj
 0003:00000bb8       ??_R0?AVCWidgetItem@iVMSGUIToolkit@@@8 0049abb8     WindowTitle.obj
 0003:00000bec       ??_R0?AVQWidgetItem@@@8    0049abec     WindowTitle.obj
 0003:00000c0c       ??_R0?AVMenu@aptui@@@8     0049ac0c     Menu.obj
 0003:00000c2c       ??_R0?AVQMenu@@@8          0049ac2c     Menu.obj
 0003:00000c48       ??_R0?AVCCustomStyle@Menu@aptui@@@8 0049ac48     Menu.obj
 0003:00000c78       ??_R0?AVQProxyStyle@@@8    0049ac78     Menu.obj
 0003:00000c98       ??_R0?AVQCommonStyle@@@8   0049ac98     Menu.obj
 0003:00000cb8       ??_R0?AVQStyle@@@8         0049acb8     Menu.obj
 0003:00000cd4       ??_R0?AVSystemMenu@aptui@@@8 0049acd4     TitleMenu.obj
 0003:00000cfc       ??_R0?AVCMenu@iVMSGUIToolkit@@@8 0049acfc     TitleMenu.obj
 0003:00000d28       ??_R0?AVLineEditInterger@aptui@@@8 0049ad28     LineEditInterger.obj
 0003:00000d54       ??_R0?AVQSpinBox@@@8       0049ad54     LineEditInterger.obj
 0003:00000d70       ??_R0?AVQAbstractSpinBox@@@8 0049ad70     LineEditInterger.obj
 0003:00000d98       ??_R0?AVTabWidget@aptui@@@8 0049ad98     TabWidget.obj
 0003:00000dbc       ??_R0?AVQTabWidget@@@8     0049adbc     TabWidget.obj
 0003:00000ddc       ??_R0?AVLine@aptui@@@8     0049addc     Line.obj
 0003:00000dfc       ??_R0?AVSwitch@aptui@@@8   0049adfc     Switch.obj
 0003:00000e1c       ??_R0?AVCoverWidget@aptui@@@8 0049ae1c     CoverWidget.obj
 0003:00000e44       ??_R0?AVWidget@aptui@@@8   0049ae44     CoverWidget.obj
 0003:00000e64       ??_R0?AVMultiStatePushButton@aptui@@@8 0049ae64     MultiStatePushButton.obj
 0003:00000e98       ??_R0?AVLabel@aptui@@@8    0049ae98     Label.obj
 0003:00000eb8       ??_R0?AVEditableLabel@aptui@@@8 0049aeb8     Label.obj
 0003:00000ee0       ??_R0?AVColorLabel@aptui@@@8 0049aee0     Label.obj
 0003:00000f08       ??_R0?AVQColorDialog@@@8   0049af08     Label.obj
 0003:00000f28       ??_R0?AVQtLockedFile@SharedTools@@@8 0049af28     qtlockedfile.obj
 0003:00000f58       ??_R0?AVQFile@@@8          0049af58     qtlockedfile.obj
 0003:00000f70       ??_R0?AVQIODevice@@@8      0049af70     qtlockedfile.obj
 0003:00000f8c       ?ack@QtLocalPeer@SharedTools@@0PBDB 0049af8c     qtlocalpeer.obj
 0003:00000f90       ??_R0?AVQtLocalPeer@SharedTools@@@8 0049af90     qtlocalpeer.obj
 0003:00000fc0       ??_R0?AVQLocalServer@@@8   0049afc0     qtlocalpeer.obj
 0003:00000fe0       ??_R0?AVQtSingleCoreApplication@SharedTools@@@8 0049afe0     qtsinglecoreapplication.obj
 0003:00001020       ___security_cookie         0049b020     MSVCRT:gs_cookie.obj
 0003:00001024       ___security_cookie_complement 0049b024     MSVCRT:gs_cookie.obj
 0003:00001030       ??_R0?AVtype_info@@@8      0049b030     MSVCRT:ti_inst.obj
 0003:00001050       ___native_dllmain_reason   0049b050     MSVCRT:natstart.obj
 0003:00001054       ___native_vcclrit_reason   0049b054     MSVCRT:natstart.obj
 0003:00001058       ___globallocalestatus      0049b058     MSVCRT:xthdloc.obj
 0003:0000105c       ___defaultmatherr          0049b05c     MSVCRT:merr.obj
 0003:000011b8       ?staticMetaObject@BandWidthPage@@2UQMetaObject@@B 0049b1b8     moc_BandWidthPage.obj
 0003:000011cc       ?staticMetaObject@BaseDialog@aptui@@2UQMetaObject@@B 0049b1cc     moc_BaseDialog.obj
 0003:000011e0       ?staticMetaObject@BaseTitle@aptui@@2UQMetaObject@@B 0049b1e0     moc_BaseTitle.obj
 0003:000011f4       ?staticMetaObject@ButtonRadio@aptui@@2UQMetaObject@@B 0049b1f4     moc_ButtonRadio.obj
 0003:00001208       ?staticMetaObject@CapacityCalculation@@2UQMetaObject@@B 0049b208     moc_CapacityCalculation.obj
 0003:0000121c       ?staticMetaObject@DataCalculatorPage@@2UQMetaObject@@B 0049b21c     moc_DataCalculatorPage.obj
 0003:00001230       ?staticMetaObject@DataDisplayPage@@2UQMetaObject@@B 0049b230     moc_DataDisplayPage.obj
 0003:00001244       ?staticMetaObject@DeviceAddPage@@2UQMetaObject@@B 0049b244     moc_DeviceAddPage.obj
 0003:00001258       ?staticMetaObject@DeviceEditor@@2UQMetaObject@@B 0049b258     moc_DeviceEditor.obj
 0003:0000126c       ?staticMetaObject@DeviceInfoManager@@2UQMetaObject@@B 0049b26c     moc_DeviceInfoManager.obj
 0003:00001280       ?staticMetaObject@DeviceItemWidget@NM_DiskCalculator@@2UQMetaObject@@B 0049b280     moc_DeviceItemWidget.obj
 0003:00001294       ?staticMetaObject@DiskCalculatorMainPage@@2UQMetaObject@@B 0049b294     moc_DiskCalculatorMainPage.obj
 0003:000012a8       ?staticMetaObject@CDlgAbout@aptui@@2UQMetaObject@@B 0049b2a8     moc_DlgAbout.obj
 0003:000012bc       ?staticMetaObject@Label@aptui@@2UQMetaObject@@B 0049b2bc     moc_Label.obj
 0003:000012d0       ?staticMetaObject@Line@aptui@@2UQMetaObject@@B 0049b2d0     moc_Line.obj
 0003:000012e4       ?staticMetaObject@LineEditInterger@aptui@@2UQMetaObject@@B 0049b2e4     moc_LineEditInterger.obj
 0003:000012f8       ?staticMetaObject@Menu@aptui@@2UQMetaObject@@B 0049b2f8     moc_Menu.obj
 0003:00001308       ?staticMetaObject@CCustomStyle@Menu@aptui@@2UQMetaObject@@B 0049b308     moc_Menu.obj
 0003:00001320       ?staticMetaObject@MultiStatePushButton@aptui@@2UQMetaObject@@B 0049b320     moc_MultiStatePushButton.obj
 0003:00001334       ?staticMetaObject@QtLocalPeer@SharedTools@@2UQMetaObject@@B 0049b334     moc_qtlocalpeer.obj
 0003:00001348       ?staticMetaObject@QtSingleApplication@SharedTools@@2UQMetaObject@@B 0049b348     moc_qtsingleapplication.obj
 0003:0000135c       ?staticMetaObject@QtSingleCoreApplication@SharedTools@@2UQMetaObject@@B 0049b35c     moc_qtsinglecoreapplication.obj
 0003:00001370       ?staticMetaObject@ScenceSelector@@2UQMetaObject@@B 0049b370     moc_ScenceSelector.obj
 0003:00001380       ?staticMetaObject@ScenceQRaidoButton@ScenceSelector@@2UQMetaObject@@B 0049b380     moc_ScenceSelector.obj
 0003:00001398       ?staticMetaObject@SizeDisplayPage@@2UQMetaObject@@B 0049b398     moc_SizeDisplayPage.obj
 0003:000013ac       ?staticMetaObject@Switch@aptui@@2UQMetaObject@@B 0049b3ac     moc_Switch.obj
 0003:000013c0       ?staticMetaObject@TabWidget@aptui@@2UQMetaObject@@B 0049b3c0     moc_TabWidget.obj
 0003:000013d4       ?staticMetaObject@SystemMenu@aptui@@2UQMetaObject@@B 0049b3d4     moc_TitleMenu.obj
 0003:000013e8       ?staticMetaObject@WarningDialog@NM_DiskCalculator@@2UQMetaObject@@B 0049b3e8     moc_WarningDialog.obj
 0003:000013fc       ?staticMetaObject@Widget@aptui@@2UQMetaObject@@B 0049b3fc     moc_Widget.obj
 0003:00001410       ?staticMetaObject@WidgetDeviceListBorder@@2UQMetaObject@@B 0049b410     moc_WidgetDeviceListBorder.obj
 0003:00001424       ?staticMetaObject@WindowTitle@aptui@@2UQMetaObject@@B 0049b424     moc_WindowTitle.obj
 0003:00001438       ?m_mutex@?1??Instance@?$CUiSingleton@VConfigureManager@apt@@@iVMSGUIToolkit@@SAAAVConfigureManager@apt@@XZ@4VQMutex@@A 0049b438     ConfigManager.obj
 0003:0000143c       ?s_instance@?1??Instance@?$CUiSingleton@VConfigureManager@apt@@@iVMSGUIToolkit@@SAAAVConfigureManager@apt@@XZ@4V?$auto_ptr@VConfigureManager@apt@@@std@@A 0049b43c     ConfigManager.obj
 0003:00001440       ??_B?1??Instance@?$CUiSingleton@VConfigureManager@apt@@@iVMSGUIToolkit@@SAAAVConfigureManager@apt@@XZ@51 0049b440     ConfigManager.obj
 0003:00001444       ?m_mutex@?1??Instance@?$CUiSingleton@VLanaguageManager@apt@@@iVMSGUIToolkit@@SAAAVLanaguageManager@apt@@XZ@4VQMutex@@A 0049b444     ToolsApplication.obj
 0003:00001448       ?s_instance@?1??Instance@?$CUiSingleton@VLanaguageManager@apt@@@iVMSGUIToolkit@@SAAAVLanaguageManager@apt@@XZ@4V?$auto_ptr@VLanaguageManager@apt@@@std@@A 0049b448     ToolsApplication.obj
 0003:0000144c       ??_B?1??Instance@?$CUiSingleton@VLanaguageManager@apt@@@iVMSGUIToolkit@@SAAAVLanaguageManager@apt@@XZ@51 0049b44c     ToolsApplication.obj
 0003:000014d0       ?nothrow@std@@3Unothrow_t@1@B 0049b4d0     msvcprt:nothrow.obj
 0003:0000181c       __forceCRTManifestRTM      0049b81c     MSVCRT:crtmanifestrtm.obj
 0003:00001820       __dowildcard               0049b820     MSVCRT:wildcard.obj
 0003:00001824       __newmode                  0049b824     MSVCRT:_newmode.obj
 0003:00001828       __commode                  0049b828     MSVCRT:xncommod.obj
 0003:0000182c       __fmode                    0049b82c     MSVCRT:xtxtmode.obj
 0003:00001830       __adjust_fdiv              0049b830     <common>
 0003:0000183c       ___native_startup_state    0049b83c     <common>
 0003:0000184c       ___native_startup_lock     0049b84c     <common>
 0003:00001850       ___sse2_available          0049b850     <common>
 0003:0000185c       ___dyn_tls_init_callback   0049b85c     <common>
 0003:00001860       ___onexitend               0049b860     <common>
 0003:00001870       ___onexitbegin             0049b870     <common>
 0004:00000000       __IMPORT_DESCRIPTOR_QtCore4 0049c000     QtCore4:QtCore4.dll
 0004:00000014       __IMPORT_DESCRIPTOR_QtGui4 0049c014     QtGui4:QtGui4.dll
 0004:00000028       __IMPORT_DESCRIPTOR_QtXml4 0049c028     QtXml4:QtXml4.dll
 0004:0000003c       __IMPORT_DESCRIPTOR_iVMSGUIToolkit 0049c03c     iVMSGUIToolkit:iVMSGUIToolkit.dll
 0004:00000050       __IMPORT_DESCRIPTOR_QtNetwork4 0049c050     QtNetwork4:QtNetwork4.dll
 0004:00000064       __IMPORT_DESCRIPTOR_ToolGuiToolkit 0049c064     ToolGuiToolkit:ToolGuiToolkit.dll
 0004:00000078       __IMPORT_DESCRIPTOR_KERNEL32 0049c078     kernel32:KERNEL32.dll
 0004:0000008c       __IMPORT_DESCRIPTOR_USER32 0049c08c     user32:USER32.dll
 0004:000000a0       __IMPORT_DESCRIPTOR_MSVCP90 0049c0a0     msvcprt:MSVCP90.dll
 0004:000000b4       __IMPORT_DESCRIPTOR_MSVCR90 0049c0b4     MSVCRT:MSVCR90.dll
 0004:000000c8       __NULL_IMPORT_DESCRIPTOR   0049c0c8     QtCore4:QtCore4.dll
 0004:00001ad8       __imp__GetCommandLineW@0   0049dad8     kernel32:KERNEL32.dll
 0004:00001adc       __imp__ReleaseSemaphore@12 0049dadc     kernel32:KERNEL32.dll
 0004:00001ae0       __imp__WaitForSingleObject@8 0049dae0     kernel32:KERNEL32.dll
 0004:00001ae4       __imp__CreateMutexW@12     0049dae4     kernel32:KERNEL32.dll
 0004:00001ae8       __imp__GetLastError@0      0049dae8     kernel32:KERNEL32.dll
 0004:00001aec       __imp__CreateSemaphoreW@16 0049daec     kernel32:KERNEL32.dll
 0004:00001af0       __imp__LocalFree@4         0049daf0     kernel32:KERNEL32.dll
 0004:00001af4       __imp__FormatMessageA@28   0049daf4     kernel32:KERNEL32.dll
 0004:00001af8       __imp__CloseHandle@4       0049daf8     kernel32:KERNEL32.dll
 0004:00001afc       __imp__GetCurrentProcessId@0 0049dafc     kernel32:KERNEL32.dll
 0004:00001b00       __imp__Sleep@4             0049db00     kernel32:KERNEL32.dll
 0004:00001b04       __imp__InterlockedExchange@8 0049db04     kernel32:KERNEL32.dll
 0004:00001b08       __imp__InterlockedCompareExchange@12 0049db08     kernel32:KERNEL32.dll
 0004:00001b0c       __imp__GetStartupInfoA@4   0049db0c     kernel32:KERNEL32.dll
 0004:00001b10       __imp__TerminateProcess@8  0049db10     kernel32:KERNEL32.dll
 0004:00001b14       __imp__GetCurrentProcess@0 0049db14     kernel32:KERNEL32.dll
 0004:00001b18       __imp__UnhandledExceptionFilter@4 0049db18     kernel32:KERNEL32.dll
 0004:00001b1c       __imp__SetUnhandledExceptionFilter@4 0049db1c     kernel32:KERNEL32.dll
 0004:00001b20       __imp__IsDebuggerPresent@0 0049db20     kernel32:KERNEL32.dll
 0004:00001b24       __imp__QueryPerformanceCounter@4 0049db24     kernel32:KERNEL32.dll
 0004:00001b28       __imp__GetTickCount@0      0049db28     kernel32:KERNEL32.dll
 0004:00001b2c       __imp__GetCurrentThreadId@0 0049db2c     kernel32:KERNEL32.dll
 0004:00001b30       __imp__GetSystemTimeAsFileTime@4 0049db30     kernel32:KERNEL32.dll
 0004:00001b34       __imp__ReleaseMutex@4      0049db34     kernel32:KERNEL32.dll
 0004:00001b38       \177KERNEL32_NULL_THUNK_DATA 0049db38     kernel32:KERNEL32.dll
 0004:00001b74       __imp_??1?$basic_string@DU?$char_traits@D@std@@V?$allocator@D@2@@std@@QAE@XZ 0049db74     msvcprt:MSVCP90.dll
 0004:00001b78       __imp_?c_str@?$basic_string@DU?$char_traits@D@std@@V?$allocator@D@2@@std@@QBEPBDXZ 0049db78     msvcprt:MSVCP90.dll
 0004:00001b7c       \177MSVCP90_NULL_THUNK_DATA 0049db7c     msvcprt:MSVCP90.dll
 0004:00001ba8       __imp__strcmp              0049dba8     MSVCRT:MSVCR90.dll
 0004:00001bac       __imp_??3@YAXPAX@Z         0049dbac     MSVCRT:MSVCR90.dll
 0004:00001bb0       __imp___CxxThrowException@8 0049dbb0     MSVCRT:MSVCR90.dll
 0004:00001bb4       __imp_??2@YAPAXI@Z         0049dbb4     MSVCRT:MSVCR90.dll
 0004:00001bb8       __imp__pow                 0049dbb8     MSVCRT:MSVCR90.dll
 0004:00001bbc       __imp__memcpy              0049dbbc     MSVCRT:MSVCR90.dll
 0004:00001bc0       __imp__memset              0049dbc0     MSVCRT:MSVCR90.dll
 0004:00001bc4       __imp__memmove             0049dbc4     MSVCRT:MSVCR90.dll
 0004:00001bc8       __imp__ceil                0049dbc8     MSVCRT:MSVCR90.dll
 0004:00001bcc       __imp____RTDynamicCast     0049dbcc     MSVCRT:MSVCR90.dll
 0004:00001bd0       __imp__strlen              0049dbd0     MSVCRT:MSVCR90.dll
 0004:00001bd4       __imp___unlock             0049dbd4     MSVCRT:MSVCR90.dll
 0004:00001bd8       __imp____dllonexit         0049dbd8     MSVCRT:MSVCR90.dll
 0004:00001bdc       __imp___encode_pointer     0049dbdc     MSVCRT:MSVCR90.dll
 0004:00001be0       __imp___lock               0049dbe0     MSVCRT:MSVCR90.dll
 0004:00001be4       __imp___onexit             0049dbe4     MSVCRT:MSVCR90.dll
 0004:00001be8       __imp___decode_pointer     0049dbe8     MSVCRT:MSVCR90.dll
 0004:00001bec       __imp___amsg_exit          0049dbec     MSVCRT:MSVCR90.dll
 0004:00001bf0       __imp____getmainargs       0049dbf0     MSVCRT:MSVCR90.dll
 0004:00001bf4       __imp___cexit              0049dbf4     MSVCRT:MSVCR90.dll
 0004:00001bf8       __imp___exit               0049dbf8     MSVCRT:MSVCR90.dll
 0004:00001bfc       __imp___XcptFilter         0049dbfc     MSVCRT:MSVCR90.dll
 0004:00001c00       __imp___ismbblead          0049dc00     MSVCRT:MSVCR90.dll
 0004:00001c04       __imp__exit                0049dc04     MSVCRT:MSVCR90.dll
 0004:00001c08       __imp___acmdln             0049dc08     MSVCRT:MSVCR90.dll
 0004:00001c0c       __imp___initterm           0049dc0c     MSVCRT:MSVCR90.dll
 0004:00001c10       __imp___initterm_e         0049dc10     MSVCRT:MSVCR90.dll
 0004:00001c14       __imp___configthreadlocale 0049dc14     MSVCRT:MSVCR90.dll
 0004:00001c18       __imp____setusermatherr    0049dc18     MSVCRT:MSVCR90.dll
 0004:00001c1c       __imp___adjust_fdiv        0049dc1c     MSVCRT:MSVCR90.dll
 0004:00001c20       __imp____p__commode        0049dc20     MSVCRT:MSVCR90.dll
 0004:00001c24       __imp____p__fmode          0049dc24     MSVCRT:MSVCR90.dll
 0004:00001c28       __imp____set_app_type      0049dc28     MSVCRT:MSVCR90.dll
 0004:00001c2c       __imp___crt_debugger_hook  0049dc2c     MSVCRT:MSVCR90.dll
 0004:00001c30       __imp_?terminate@@YAXXZ    0049dc30     MSVCRT:MSVCR90.dll
 0004:00001c34       __imp_?_type_info_dtor_internal_method@type_info@@QAEXXZ 0049dc34     MSVCRT:MSVCR90.dll
 0004:00001c38       __imp___except_handler4_common 0049dc38     MSVCRT:MSVCR90.dll
 0004:00001c3c       __imp___invoke_watson      0049dc3c     MSVCRT:MSVCR90.dll
 0004:00001c40       __imp___controlfp_s        0049dc40     MSVCRT:MSVCR90.dll
 0004:00001c44       __imp____CxxFrameHandler3  0049dc44     MSVCRT:MSVCR90.dll
 0004:00001c48       \177MSVCR90_NULL_THUNK_DATA 0049dc48     MSVCRT:MSVCR90.dll
 0004:00001c94       __imp_?qMemSet@@YAPAXPAXHI@Z 0049dc94     QtCore4:QtCore4.dll
 0004:00001c98       __imp_??4QBasicAtomicInt@@QAEAAV0@H@Z 0049dc98     QtCore4:QtCore4.dll
 0004:00001c9c       __imp_?reallocate@QVectorData@@SAPAU1@PAU1@HHH@Z 0049dc9c     QtCore4:QtCore4.dll
 0004:00001ca0       __imp_?qBadAlloc@@YAXXZ    0049dca0     QtCore4:QtCore4.dll
 0004:00001ca4       __imp_??8QBasicAtomicInt@@QBE_NH@Z 0049dca4     QtCore4:QtCore4.dll
 0004:00001ca8       __imp_?qFree@@YAXPAX@Z     0049dca8     QtCore4:QtCore4.dll
 0004:00001cac       __imp_?allocate@QVectorData@@SAPAU1@HH@Z 0049dcac     QtCore4:QtCore4.dll
 0004:00001cb0       __imp_??MQString@@QBE_NABV0@@Z 0049dcb0     QtCore4:QtCore4.dll
 0004:00001cb4       __imp_??1QFileInfo@@QAE@XZ 0049dcb4     QtCore4:QtCore4.dll
 0004:00001cb8       __imp_?shared_null@QListData@@2UData@1@A 0049dcb8     QtCore4:QtCore4.dll
 0004:00001cbc       __imp_?append@QListData@@QAEPAPAXXZ 0049dcbc     QtCore4:QtCore4.dll
 0004:00001cc0       __imp_?end@QListData@@QBEPAPAXXZ 0049dcc0     QtCore4:QtCore4.dll
 0004:00001cc4       __imp_?detach_grow@QListData@@QAEPAUData@1@PAHH@Z 0049dcc4     QtCore4:QtCore4.dll
 0004:00001cc8       __imp_?begin@QListData@@QBEPAPAXXZ 0049dcc8     QtCore4:QtCore4.dll
 0004:00001ccc       __imp_?detach@QListData@@QAEPAUData@1@H@Z 0049dccc     QtCore4:QtCore4.dll
 0004:00001cd0       __imp_?flush@QTextStream@@QAEXXZ 0049dcd0     QtCore4:QtCore4.dll
 0004:00001cd4       __imp_??6QTextStream@@QAEAAV0@ABVQString@@@Z 0049dcd4     QtCore4:QtCore4.dll
 0004:00001cd8       __imp_?remove@QFile@@SA_NABVQString@@@Z 0049dcd8     QtCore4:QtCore4.dll
 0004:00001cdc       __imp_?exists@QFileInfo@@QBE_NXZ 0049dcdc     QtCore4:QtCore4.dll
 0004:00001ce0       __imp_??0QFileInfo@@QAE@ABVQString@@@Z 0049dce0     QtCore4:QtCore4.dll
 0004:00001ce4       __imp_?fileName@QFile@@QBE?AVQString@@XZ 0049dce4     QtCore4:QtCore4.dll
 0004:00001ce8       __imp_?fileName@QFileInfo@@QBE?AVQString@@XZ 0049dce8     QtCore4:QtCore4.dll
 0004:00001cec       __imp_?append@QString@@QAEAAV1@PBD@Z 0049dcec     QtCore4:QtCore4.dll
 0004:00001cf0       __imp_?QStringList_contains@QtPrivate@@YA?AVQBool@@PBVQStringList@@ABVQString@@W4CaseSensitivity@Qt@@@Z 0049dcf0     QtCore4:QtCore4.dll
 0004:00001cf4       __imp_?toUInt@QString@@QBEIPA_NH@Z 0049dcf4     QtCore4:QtCore4.dll
 0004:00001cf8       __imp_??0QLocale@@QAE@XZ   0049dcf8     QtCore4:QtCore4.dll
 0004:00001cfc       __imp_?installTranslator@QCoreApplication@@SAXPAVQTranslator@@@Z 0049dcfc     QtCore4:QtCore4.dll
 0004:00001d00       __imp_?load@QTranslator@@QAE_NABVQString@@000@Z 0049dd00     QtCore4:QtCore4.dll
 0004:00001d04       __imp_??0QTranslator@@QAE@PAVQObject@@@Z 0049dd04     QtCore4:QtCore4.dll
 0004:00001d08       __imp_??4QLocale@@QAEAAV0@ABV0@@Z 0049dd08     QtCore4:QtCore4.dll
 0004:00001d0c       __imp_??0QLocale@@QAE@W4Language@0@W4Country@0@@Z 0049dd0c     QtCore4:QtCore4.dll
 0004:00001d10       __imp_?metaObject@QTranslator@@UBEPBUQMetaObject@@XZ 0049dd10     QtCore4:QtCore4.dll
 0004:00001d14       __imp_?qt_metacast@QTranslator@@UAEPAXPBD@Z 0049dd14     QtCore4:QtCore4.dll
 0004:00001d18       __imp_?qt_metacall@QTranslator@@UAEHW4Call@QMetaObject@@HPAPAX@Z 0049dd18     QtCore4:QtCore4.dll
 0004:00001d1c       __imp_?event@QObject@@UAE_NPAVQEvent@@@Z 0049dd1c     QtCore4:QtCore4.dll
 0004:00001d20       __imp_?eventFilter@QObject@@UAE_NPAV1@PAVQEvent@@@Z 0049dd20     QtCore4:QtCore4.dll
 0004:00001d24       __imp_?timerEvent@QObject@@MAEXPAVQTimerEvent@@@Z 0049dd24     QtCore4:QtCore4.dll
 0004:00001d28       __imp_?childEvent@QObject@@MAEXPAVQChildEvent@@@Z 0049dd28     QtCore4:QtCore4.dll
 0004:00001d2c       __imp_?customEvent@QObject@@MAEXPAVQEvent@@@Z 0049dd2c     QtCore4:QtCore4.dll
 0004:00001d30       __imp_?connectNotify@QObject@@MAEXPBD@Z 0049dd30     QtCore4:QtCore4.dll
 0004:00001d34       __imp_?disconnectNotify@QObject@@MAEXPBD@Z 0049dd34     QtCore4:QtCore4.dll
 0004:00001d38       __imp_?translate@QTranslator@@UBE?AVQString@@PBD00@Z 0049dd38     QtCore4:QtCore4.dll
 0004:00001d3c       __imp_?isEmpty@QTranslator@@UBE_NXZ 0049dd3c     QtCore4:QtCore4.dll
 0004:00001d40       __imp_??1QTranslator@@UAE@XZ 0049dd40     QtCore4:QtCore4.dll
 0004:00001d44       __imp_??0QLocale@@QAE@ABV0@@Z 0049dd44     QtCore4:QtCore4.dll
 0004:00001d48       __imp_??1QMutexLocker@@QAE@XZ 0049dd48     QtCore4:QtCore4.dll
 0004:00001d4c       __imp_??0QMutexLocker@@QAE@PAVQMutex@@@Z 0049dd4c     QtCore4:QtCore4.dll
 0004:00001d50       __imp_??0QMutex@@QAE@W4RecursionMode@0@@Z 0049dd50     QtCore4:QtCore4.dll
 0004:00001d54       __imp_??1QMutex@@QAE@XZ    0049dd54     QtCore4:QtCore4.dll
 0004:00001d58       __imp_?winEventFilter@QCoreApplication@@UAE_NPAUtagMSG@@PAJ@Z 0049dd58     QtCore4:QtCore4.dll
 0004:00001d5c       __imp_?toString@QVariant@@QBE?AVQString@@XZ 0049dd5c     QtCore4:QtCore4.dll
 0004:00001d60       __imp_?inherits@QObject@@QBE_NPBD@Z 0049dd60     QtCore4:QtCore4.dll
 0004:00001d64       __imp_??1QVariant@@QAE@XZ  0049dd64     QtCore4:QtCore4.dll
 0004:00001d68       __imp_?isNull@QVariant@@QBE_NXZ 0049dd68     QtCore4:QtCore4.dll
 0004:00001d6c       __imp_?property@QObject@@QBE?AVQVariant@@PBD@Z 0049dd6c     QtCore4:QtCore4.dll
 0004:00001d70       __imp_?type@QEvent@@QBE?AW4Type@1@XZ 0049dd70     QtCore4:QtCore4.dll
 0004:00001d74       __imp_?setObjectName@QObject@@QAEXABVQString@@@Z 0049dd74     QtCore4:QtCore4.dll
 0004:00001d78       __imp_?tr@QMetaObject@@QBE?AVQString@@PBD0@Z 0049dd78     QtCore4:QtCore4.dll
 0004:00001d7c       __imp_?qWarning@@YAXPBDZZ  0049dd7c     QtCore4:QtCore4.dll
 0004:00001d80       __imp_?toStdString@QString@@QBE?AV?$basic_string@DU?$char_traits@D@std@@V?$allocator@D@2@@std@@XZ 0049dd80     QtCore4:QtCore4.dll
 0004:00001d84       __imp_?fromUtf8@QString@@SA?AV1@PBDH@Z 0049dd84     QtCore4:QtCore4.dll
 0004:00001d88       __imp_?append@QString@@QAEAAV1@ABV1@@Z 0049dd88     QtCore4:QtCore4.dll
 0004:00001d8c       __imp_?entryList@QDir@@QBE?AVQStringList@@V?$QFlags@W4Filter@QDir@@@@V?$QFlags@W4SortFlag@QDir@@@@@Z 0049dd8c     QtCore4:QtCore4.dll
 0004:00001d90       __imp_?qDebug@@YAXPBDZZ    0049dd90     QtCore4:QtCore4.dll
 0004:00001d94       __imp_?codecForLocale@QTextCodec@@SAPAV1@XZ 0049dd94     QtCore4:QtCore4.dll
 0004:00001d98       __imp_?bottom@QRect@@QBEHXZ 0049dd98     QtCore4:QtCore4.dll
 0004:00001d9c       __imp_?right@QRect@@QBEHXZ 0049dd9c     QtCore4:QtCore4.dll
 0004:00001da0       __imp_?load@QPluginLoader@@QAE_NXZ 0049dda0     QtCore4:QtCore4.dll
 0004:00001da4       __imp_??1QPluginLoader@@UAE@XZ 0049dda4     QtCore4:QtCore4.dll
 0004:00001da8       __imp_?instance@QPluginLoader@@QAEPAVQObject@@XZ 0049dda8     QtCore4:QtCore4.dll
 0004:00001dac       __imp_?isLoaded@QPluginLoader@@QBE_NXZ 0049ddac     QtCore4:QtCore4.dll
 0004:00001db0       __imp_??0QPluginLoader@@QAE@ABVQString@@PAVQObject@@@Z 0049ddb0     QtCore4:QtCore4.dll
 0004:00001db4       __imp_?cleanPath@QDir@@SA?AVQString@@ABV2@@Z 0049ddb4     QtCore4:QtCore4.dll
 0004:00001db8       __imp_??0QChar@@QAE@UQLatin1Char@@@Z 0049ddb8     QtCore4:QtCore4.dll
 0004:00001dbc       __imp_?remove@QListData@@QAEXH@Z 0049ddbc     QtCore4:QtCore4.dll
 0004:00001dc0       __imp_?connectSlotsByName@QMetaObject@@SAXPAVQObject@@@Z 0049ddc0     QtCore4:QtCore4.dll
 0004:00001dc4       __imp_??0QRect@@QAE@HHHH@Z 0049ddc4     QtCore4:QtCore4.dll
 0004:00001dc8       __imp_??0QSize@@QAE@HH@Z   0049ddc8     QtCore4:QtCore4.dll
 0004:00001dcc       __imp_?objectName@QObject@@QBE?AVQString@@XZ 0049ddcc     QtCore4:QtCore4.dll
 0004:00001dd0       __imp_?translate@QCoreApplication@@SA?AVQString@@PBD00W4Encoding@1@@Z 0049ddd0     QtCore4:QtCore4.dll
 0004:00001dd4       __imp_?connect@QObject@@SA_NPBV1@PBD01W4ConnectionType@Qt@@@Z 0049ddd4     QtCore4:QtCore4.dll
 0004:00001dd8       __imp_??0QPoint@@QAE@HH@Z  0049ddd8     QtCore4:QtCore4.dll
 0004:00001ddc       __imp_?x@QPoint@@QBEHXZ    0049dddc     QtCore4:QtCore4.dll
 0004:00001de0       __imp_?y@QPoint@@QBEHXZ    0049dde0     QtCore4:QtCore4.dll
 0004:00001de4       __imp_?ignore@QEvent@@QAEXXZ 0049dde4     QtCore4:QtCore4.dll
 0004:00001de8       __imp_?accept@QEvent@@QAEXXZ 0049dde8     QtCore4:QtCore4.dll
 0004:00001dec       __imp_?setNum@QString@@QAEAAV1@KH@Z 0049ddec     QtCore4:QtCore4.dll
 0004:00001df0       __imp_??1QUrl@@QAE@XZ      0049ddf0     QtCore4:QtCore4.dll
 0004:00001df4       __imp_??0QUrl@@QAE@ABVQString@@@Z 0049ddf4     QtCore4:QtCore4.dll
 0004:00001df8       __imp_??YQString@@QAEAAV0@PBD@Z 0049ddf8     QtCore4:QtCore4.dll
 0004:00001dfc       __imp_?toUnicode@QTextCodec@@QBE?AVQString@@PBD@Z 0049ddfc     QtCore4:QtCore4.dll
 0004:00001e00       __imp_?currentPath@QDir@@SA?AVQString@@XZ 0049de00     QtCore4:QtCore4.dll
 0004:00001e04       __imp_?disconnect@QObject@@SA_NPBV1@PBD01@Z 0049de04     QtCore4:QtCore4.dll
 0004:00001e08       __imp_?sender@QObject@@IBEPAV1@XZ 0049de08     QtCore4:QtCore4.dll
 0004:00001e0c       __imp_??0QVariant@@QAE@H@Z 0049de0c     QtCore4:QtCore4.dll
 0004:00001e10       __imp_??0QVariant@@QAE@XZ  0049de10     QtCore4:QtCore4.dll
 0004:00001e14       __imp_?QStringList_sort@QtPrivate@@YAXPAVQStringList@@@Z 0049de14     QtCore4:QtCore4.dll
 0004:00001e18       __imp_??1QObject@@UAE@XZ   0049de18     QtCore4:QtCore4.dll
 0004:00001e1c       __imp_??0QObject@@QAE@PAV0@@Z 0049de1c     QtCore4:QtCore4.dll
 0004:00001e20       __imp_?arg@QString@@QBE?AV1@ABV1@HABVQChar@@@Z 0049de20     QtCore4:QtCore4.dll
 0004:00001e24       __imp_?exists@QFile@@SA_NABVQString@@@Z 0049de24     QtCore4:QtCore4.dll
 0004:00001e28       __imp_??6QDebug@@QAEAAV0@PBD@Z 0049de28     QtCore4:QtCore4.dll
 0004:00001e2c       __imp_?number@QString@@SA?AV1@_JH@Z 0049de2c     QtCore4:QtCore4.dll
 0004:00001e30       __imp_?setY@QPoint@@QAEXH@Z 0049de30     QtCore4:QtCore4.dll
 0004:00001e34       __imp_?setX@QPoint@@QAEXH@Z 0049de34     QtCore4:QtCore4.dll
 0004:00001e38       __imp_??0QPoint@@QAE@XZ    0049de38     QtCore4:QtCore4.dll
 0004:00001e3c       __imp_?parent@QObject@@QBEPAV1@XZ 0049de3c     QtCore4:QtCore4.dll
 0004:00001e40       __imp_?sprintf@QString@@QAAAAV1@PBDZZ 0049de40     QtCore4:QtCore4.dll
 0004:00001e44       __imp_?unlock@QMutex@@QAEXXZ 0049de44     QtCore4:QtCore4.dll
 0004:00001e48       __imp_?separator@QDir@@SA?AVQChar@@XZ 0049de48     QtCore4:QtCore4.dll
 0004:00001e4c       __imp_?blockSignals@QObject@@QAE_N_N@Z 0049de4c     QtCore4:QtCore4.dll
 0004:00001e50       __imp_??8QString@@QBE_NPBD@Z 0049de50     QtCore4:QtCore4.dll
 0004:00001e54       __imp_??0QSizeF@@QAE@NN@Z  0049de54     QtCore4:QtCore4.dll
 0004:00001e58       __imp_?number@QString@@SA?AV1@NDH@Z 0049de58     QtCore4:QtCore4.dll
 0004:00001e5c       __imp_??8QString@@QBE_NABVQLatin1String@@@Z 0049de5c     QtCore4:QtCore4.dll
 0004:00001e60       __imp_?free@QVectorData@@SAXPAU1@H@Z 0049de60     QtCore4:QtCore4.dll
 0004:00001e64       __imp_?codecForCStrings@QString@@0PAVQTextCodec@@A 0049de64     QtCore4:QtCore4.dll
 0004:00001e68       __imp_?toUpper@QString@@QBE?AV1@XZ 0049de68     QtCore4:QtCore4.dll
 0004:00001e6c       __imp_??6QDebug@@QAEAAV0@H@Z 0049de6c     QtCore4:QtCore4.dll
 0004:00001e70       __imp_?copy@QFile@@SA_NABVQString@@0@Z 0049de70     QtCore4:QtCore4.dll
 0004:00001e74       __imp_??0QSize@@QAE@XZ     0049de74     QtCore4:QtCore4.dll
 0004:00001e78       __imp_??9QString@@QBE_NPBD@Z 0049de78     QtCore4:QtCore4.dll
 0004:00001e7c       __imp_?top@QRect@@QBEHXZ   0049de7c     QtCore4:QtCore4.dll
 0004:00001e80       __imp_?width@QRect@@QBEHXZ 0049de80     QtCore4:QtCore4.dll
 0004:00001e84       __imp_?left@QString@@QBE?AV1@H@Z 0049de84     QtCore4:QtCore4.dll
 0004:00001e88       __imp_?mid@QString@@QBE?AV1@HH@Z 0049de88     QtCore4:QtCore4.dll
 0004:00001e8c       __imp_??0QRect@@QAE@ABVQPoint@@0@Z 0049de8c     QtCore4:QtCore4.dll
 0004:00001e90       __imp_?topRight@QRect@@QBE?AVQPoint@@XZ 0049de90     QtCore4:QtCore4.dll
 0004:00001e94       __imp_??BQIncompatibleFlag@@QBEHXZ 0049de94     QtCore4:QtCore4.dll
 0004:00001e98       __imp_?indexOf@QString@@QBEHVQChar@@HW4CaseSensitivity@Qt@@@Z 0049de98     QtCore4:QtCore4.dll
 0004:00001e9c       __imp_?getRect@QRect@@QBEXPAH000@Z 0049de9c     QtCore4:QtCore4.dll
 0004:00001ea0       __imp_?topLeft@QRect@@QBE?AVQPoint@@XZ 0049dea0     QtCore4:QtCore4.dll
 0004:00001ea4       __imp_?moveCenter@QRect@@QAEXABVQPoint@@@Z 0049dea4     QtCore4:QtCore4.dll
 0004:00001ea8       __imp_?x@QRect@@QBEHXZ     0049dea8     QtCore4:QtCore4.dll
 0004:00001eac       __imp_?y@QRect@@QBEHXZ     0049deac     QtCore4:QtCore4.dll
 0004:00001eb0       __imp_?height@QRect@@QBEHXZ 0049deb0     QtCore4:QtCore4.dll
 0004:00001eb4       __imp_?left@QRect@@QBEHXZ  0049deb4     QtCore4:QtCore4.dll
 0004:00001eb8       __imp_?center@QRect@@QBE?AVQPoint@@XZ 0049deb8     QtCore4:QtCore4.dll
 0004:00001ebc       __imp_?adjusted@QRect@@QBE?AV1@HHHH@Z 0049debc     QtCore4:QtCore4.dll
 0004:00001ec0       __imp_?cast@QMetaObject@@QBEPBVQObject@@PBV2@@Z 0049dec0     QtCore4:QtCore4.dll
 0004:00001ec4       __imp_??0QIncompatibleFlag@@QAE@H@Z 0049dec4     QtCore4:QtCore4.dll
 0004:00001ec8       __imp_?setProperty@QObject@@QAE_NPBDABVQVariant@@@Z 0049dec8     QtCore4:QtCore4.dll
 0004:00001ecc       __imp_??0QVariant@@QAE@ABVQString@@@Z 0049decc     QtCore4:QtCore4.dll
 0004:00001ed0       __imp_?registerType@QMetaType@@SAHPBDP6AXPAX@ZP6APAXPBX@Z@Z 0049ded0     QtCore4:QtCore4.dll
 0004:00001ed4       __imp_?registerTypedef@QMetaType@@SAHPBDH@Z 0049ded4     QtCore4:QtCore4.dll
 0004:00001ed8       __imp_?append@?$QVector@VQPoint@@@@QAEXABVQPoint@@@Z 0049ded8     QtCore4:QtCore4.dll
 0004:00001edc       __imp_?clear@?$QVector@VQPoint@@@@QAEXXZ 0049dedc     QtCore4:QtCore4.dll
 0004:00001ee0       __imp_?arg@QString@@QBE?AV1@HHHABVQChar@@@Z 0049dee0     QtCore4:QtCore4.dll
 0004:00001ee4       __imp_?metaObject@QFile@@UBEPBUQMetaObject@@XZ 0049dee4     QtCore4:QtCore4.dll
 0004:00001ee8       __imp_?qt_metacast@QFile@@UAEPAXPBD@Z 0049dee8     QtCore4:QtCore4.dll
 0004:00001eec       __imp_?qt_metacall@QFile@@UAEHW4Call@QMetaObject@@HPAPAX@Z 0049deec     QtCore4:QtCore4.dll
 0004:00001ef0       __imp_?isSequential@QFile@@UBE_NXZ 0049def0     QtCore4:QtCore4.dll
 0004:00001ef4       __imp_?pos@QFile@@UBE_JXZ  0049def4     QtCore4:QtCore4.dll
 0004:00001ef8       __imp_?size@QFile@@UBE_JXZ 0049def8     QtCore4:QtCore4.dll
 0004:00001efc       __imp_?seek@QFile@@UAE_N_J@Z 0049defc     QtCore4:QtCore4.dll
 0004:00001f00       __imp_?atEnd@QFile@@UBE_NXZ 0049df00     QtCore4:QtCore4.dll
 0004:00001f04       __imp_?reset@QIODevice@@UAE_NXZ 0049df04     QtCore4:QtCore4.dll
 0004:00001f08       __imp_?bytesAvailable@QIODevice@@UBE_JXZ 0049df08     QtCore4:QtCore4.dll
 0004:00001f0c       __imp_?bytesToWrite@QIODevice@@UBE_JXZ 0049df0c     QtCore4:QtCore4.dll
 0004:00001f10       __imp_?canReadLine@QIODevice@@UBE_NXZ 0049df10     QtCore4:QtCore4.dll
 0004:00001f14       __imp_?waitForReadyRead@QIODevice@@UAE_NH@Z 0049df14     QtCore4:QtCore4.dll
 0004:00001f18       __imp_?waitForBytesWritten@QIODevice@@UAE_NH@Z 0049df18     QtCore4:QtCore4.dll
 0004:00001f1c       __imp_?readData@QFile@@MAE_JPAD_J@Z 0049df1c     QtCore4:QtCore4.dll
 0004:00001f20       __imp_?readLineData@QFile@@MAE_JPAD_J@Z 0049df20     QtCore4:QtCore4.dll
 0004:00001f24       __imp_?writeData@QFile@@MAE_JPBD_J@Z 0049df24     QtCore4:QtCore4.dll
 0004:00001f28       __imp_?fileEngine@QFile@@UBEPAVQAbstractFileEngine@@XZ 0049df28     QtCore4:QtCore4.dll
 0004:00001f2c       __imp_??1QByteArray@@QAE@XZ 0049df2c     QtCore4:QtCore4.dll
 0004:00001f30       __imp_?constData@QByteArray@@QBEPBDXZ 0049df30     QtCore4:QtCore4.dll
 0004:00001f34       __imp_?toLatin1@QString@@QBE?AVQByteArray@@XZ 0049df34     QtCore4:QtCore4.dll
 0004:00001f38       __imp_?utf16@QString@@QBEPBGXZ 0049df38     QtCore4:QtCore4.dll
 0004:00001f3c       __imp_?fromLatin1@QString@@SA?AV1@PBDH@Z 0049df3c     QtCore4:QtCore4.dll
 0004:00001f40       __imp_?toLower@QString@@QBE?AV1@XZ 0049df40     QtCore4:QtCore4.dll
 0004:00001f44       __imp_??0QFileInfo@@QAE@ABVQFile@@@Z 0049df44     QtCore4:QtCore4.dll
 0004:00001f48       __imp_?isOpen@QIODevice@@QBE_NXZ 0049df48     QtCore4:QtCore4.dll
 0004:00001f4c       __imp_?truncate@QString@@QAEXH@Z 0049df4c     QtCore4:QtCore4.dll
 0004:00001f50       __imp_?length@QString@@QBEHXZ 0049df50     QtCore4:QtCore4.dll
 0004:00001f54       __imp_?endsWith@QString@@QBE_NABVQChar@@W4CaseSensitivity@Qt@@@Z 0049df54     QtCore4:QtCore4.dll
 0004:00001f58       __imp_??0QChar@@QAE@D@Z    0049df58     QtCore4:QtCore4.dll
 0004:00001f5c       __imp_?fromLocal8Bit@QString@@SA?AV1@PBDH@Z 0049df5c     QtCore4:QtCore4.dll
 0004:00001f60       __imp_?absolutePath@QDir@@QBE?AVQString@@XZ 0049df60     QtCore4:QtCore4.dll
 0004:00001f64       __imp_?tempPath@QDir@@SA?AVQString@@XZ 0049df64     QtCore4:QtCore4.dll
 0004:00001f68       __imp_?number@QString@@SA?AV1@KH@Z 0049df68     QtCore4:QtCore4.dll
 0004:00001f6c       __imp_??1QLibrary@@UAE@XZ  0049df6c     QtCore4:QtCore4.dll
 0004:00001f70       __imp_?resolve@QLibrary@@QAEPAXPBD@Z 0049df70     QtCore4:QtCore4.dll
 0004:00001f74       __imp_??0QLibrary@@QAE@ABVQString@@PAVQObject@@@Z 0049df74     QtCore4:QtCore4.dll
 0004:00001f78       __imp_??0QString@@QAE@ABVQLatin1String@@@Z 0049df78     QtCore4:QtCore4.dll
 0004:00001f7c       __imp_?qChecksum@@YAGPBDI@Z 0049df7c     QtCore4:QtCore4.dll
 0004:00001f80       __imp_?size@QByteArray@@QBEHXZ 0049df80     QtCore4:QtCore4.dll
 0004:00001f84       __imp_?toUtf8@QString@@QBE?AVQByteArray@@XZ 0049df84     QtCore4:QtCore4.dll
 0004:00001f88       __imp_?applicationFilePath@QCoreApplication@@SA?AVQString@@XZ 0049df88     QtCore4:QtCore4.dll
 0004:00001f8c       __imp_?connect@QObject@@QBE_NPBV1@PBD1W4ConnectionType@Qt@@@Z 0049df8c     QtCore4:QtCore4.dll
 0004:00001f90       __imp_?toLocal8Bit@QString@@QBE?AVQByteArray@@XZ 0049df90     QtCore4:QtCore4.dll
 0004:00001f94       __imp_??1QDataStream@@UAE@XZ 0049df94     QtCore4:QtCore4.dll
 0004:00001f98       __imp_?read@QIODevice@@QAE?AVQByteArray@@_J@Z 0049df98     QtCore4:QtCore4.dll
 0004:00001f9c       __imp_?writeBytes@QDataStream@@QAEAAV1@PBDI@Z 0049df9c     QtCore4:QtCore4.dll
 0004:00001fa0       __imp_??0QDataStream@@QAE@PAVQIODevice@@@Z 0049dfa0     QtCore4:QtCore4.dll
 0004:00001fa4       __imp_?write@QIODevice@@QAE_JPBD_J@Z 0049dfa4     QtCore4:QtCore4.dll
 0004:00001fa8       __imp_?qWarning@@YA?AVQDebug@@XZ 0049dfa8     QtCore4:QtCore4.dll
 0004:00001fac       __imp_?errorString@QIODevice@@QBE?AVQString@@XZ 0049dfac     QtCore4:QtCore4.dll
 0004:00001fb0       __imp_?readRawData@QDataStream@@QAEHPADH@Z 0049dfb0     QtCore4:QtCore4.dll
 0004:00001fb4       __imp_?data@QByteArray@@QAEPADXZ 0049dfb4     QtCore4:QtCore4.dll
 0004:00001fb8       __imp_?resize@QByteArray@@QAEXH@Z 0049dfb8     QtCore4:QtCore4.dll
 0004:00001fbc       __imp_??5QDataStream@@QAEAAV0@AAI@Z 0049dfbc     QtCore4:QtCore4.dll
 0004:00001fc0       __imp_??0QByteArray@@QAE@XZ 0049dfc0     QtCore4:QtCore4.dll
 0004:00001fc4       __imp_?isEmpty@QByteArray@@QBE_NXZ 0049dfc4     QtCore4:QtCore4.dll
 0004:00001fc8       __imp_?qstrcmp@@YAHABVQByteArray@@PBD@Z 0049dfc8     QtCore4:QtCore4.dll
 0004:00001fcc       __imp_??0QString@@QAE@VQChar@@@Z 0049dfcc     QtCore4:QtCore4.dll
 0004:00001fd0       __imp_?applicationPid@QCoreApplication@@SA_JXZ 0049dfd0     QtCore4:QtCore4.dll
 0004:00001fd4       __imp_??1QCoreApplication@@UAE@XZ 0049dfd4     QtCore4:QtCore4.dll
 0004:00001fd8       __imp_??0QCoreApplication@@QAE@AAHPAPADH@Z 0049dfd8     QtCore4:QtCore4.dll
 0004:00001fdc       __imp_?event@QCoreApplication@@MAE_NPAVQEvent@@@Z 0049dfdc     QtCore4:QtCore4.dll
 0004:00001fe0       __imp_?notify@QCoreApplication@@UAE_NPAVQObject@@PAVQEvent@@@Z 0049dfe0     QtCore4:QtCore4.dll
 0004:00001fe4       __imp_?compressEvent@QCoreApplication@@MAE_NPAVQEvent@@PAVQObject@@PAVQPostEventList@@@Z 0049dfe4     QtCore4:QtCore4.dll
 0004:00001fe8       __imp_?isWidgetType@QObject@@QBE_NXZ 0049dfe8     QtCore4:QtCore4.dll
 0004:00001fec       __imp_?applicationDirPath@QCoreApplication@@SA?AVQString@@XZ 0049dfec     QtCore4:QtCore4.dll
 0004:00001ff0       __imp_?toNativeSeparators@QDir@@SA?AVQString@@ABV2@@Z 0049dff0     QtCore4:QtCore4.dll
 0004:00001ff4       __imp_?instance@QCoreApplication@@SAPAV1@XZ 0049dff4     QtCore4:QtCore4.dll
 0004:00001ff8       __imp_?addLibraryPath@QCoreApplication@@SAXABVQString@@@Z 0049dff8     QtCore4:QtCore4.dll
 0004:00001ffc       __imp_?exit@QCoreApplication@@SAXH@Z 0049dffc     QtCore4:QtCore4.dll
 0004:00002000       __imp_?size@QRect@@QBE?AVQSize@@XZ 0049e000     QtCore4:QtCore4.dll
 0004:00002004       __imp_?width@QSize@@QBEHXZ 0049e004     QtCore4:QtCore4.dll
 0004:00002008       __imp_?height@QSize@@QBEHXZ 0049e008     QtCore4:QtCore4.dll
 0004:0000200c       __imp_?staticMetaObject@QCoreApplication@@2UQMetaObject@@B 0049e00c     QtCore4:QtCore4.dll
 0004:00002010       __imp_?qt_metacall@QCoreApplication@@UAEHW4Call@QMetaObject@@HPAPAX@Z 0049e010     QtCore4:QtCore4.dll
 0004:00002014       __imp_?qt_metacast@QCoreApplication@@UAEPAXPBD@Z 0049e014     QtCore4:QtCore4.dll
 0004:00002018       __imp_?staticMetaObject@QObject@@2UQMetaObject@@B 0049e018     QtCore4:QtCore4.dll
 0004:0000201c       __imp_?fromWCharArray@QString@@SA?AV1@PBGH@Z 0049e01c     QtCore4:QtCore4.dll
 0004:00002020       __imp_?free@QString@@CAXPAUData@1@@Z 0049e020     QtCore4:QtCore4.dll
 0004:00002024       __imp_?detach@QByteArray@@QAEXXZ 0049e024     QtCore4:QtCore4.dll
 0004:00002028       __imp_?qWinMain@@YAXPAUHINSTANCE__@@0PADHAAHAAV?$QVector@PAD@@@Z 0049e028     QtCore4:QtCore4.dll
 0004:0000202c       __imp_??9QBasicAtomicInt@@QBE_NH@Z 0049e02c     QtCore4:QtCore4.dll
 0004:00002030       __imp_?grow@QVectorData@@SAHHHH_N@Z 0049e030     QtCore4:QtCore4.dll
 0004:00002034       __imp_?at@QListData@@QBEPAPAXH@Z 0049e034     QtCore4:QtCore4.dll
 0004:00002038       __imp_?size@QListData@@QBEHXZ 0049e038     QtCore4:QtCore4.dll
 0004:0000203c       __imp_?shared_null@QMapData@@2U1@A 0049e03c     QtCore4:QtCore4.dll
 0004:00002040       __imp_?shared_null@QVectorData@@2U1@A 0049e040     QtCore4:QtCore4.dll
 0004:00002044       __imp_??0QFile@@QAE@XZ     0049e044     QtCore4:QtCore4.dll
 0004:00002048       __imp_?setFileName@QFile@@QAEXABVQString@@@Z 0049e048     QtCore4:QtCore4.dll
 0004:0000204c       __imp_?atEnd@QTextStream@@QBE_NXZ 0049e04c     QtCore4:QtCore4.dll
 0004:00002050       __imp_?readLine@QTextStream@@QAE?AVQString@@_J@Z 0049e050     QtCore4:QtCore4.dll
 0004:00002054       __imp_?split@QString@@QBE?AVQStringList@@ABV1@W4SplitBehavior@1@W4CaseSensitivity@Qt@@@Z 0049e054     QtCore4:QtCore4.dll
 0004:00002058       __imp_?endl@@YAAAVQTextStream@@AAV1@@Z 0049e058     QtCore4:QtCore4.dll
 0004:0000205c       __imp_?qDebug@@YA?AVQDebug@@XZ 0049e05c     QtCore4:QtCore4.dll
 0004:00002060       __imp_??6QDebug@@QAEAAV0@ABVQString@@@Z 0049e060     QtCore4:QtCore4.dll
 0004:00002064       __imp_??6QDebug@@QAEAAV0@P6AAAVQTextStream@@AAV1@@Z@Z 0049e064     QtCore4:QtCore4.dll
 0004:00002068       __imp_??1QDebug@@QAE@XZ    0049e068     QtCore4:QtCore4.dll
 0004:0000206c       __imp_?toDouble@QString@@QBENPA_N@Z 0049e06c     QtCore4:QtCore4.dll
 0004:00002070       __imp_?isEmpty@QString@@QBE_NXZ 0049e070     QtCore4:QtCore4.dll
 0004:00002074       __imp_?toInt@QString@@QBEHPA_NH@Z 0049e074     QtCore4:QtCore4.dll
 0004:00002078       __imp_??0QDir@@QAE@ABVQString@@@Z 0049e078     QtCore4:QtCore4.dll
 0004:0000207c       __imp_?entryInfoList@QDir@@QBE?AV?$QList@VQFileInfo@@@@V?$QFlags@W4Filter@QDir@@@@V?$QFlags@W4SortFlag@QDir@@@@@Z 0049e07c     QtCore4:QtCore4.dll
 0004:00002080       __imp_?completeBaseName@QFileInfo@@QBE?AVQString@@XZ 0049e080     QtCore4:QtCore4.dll
 0004:00002084       __imp_?absoluteFilePath@QFileInfo@@QBE?AVQString@@XZ 0049e084     QtCore4:QtCore4.dll
 0004:00002088       __imp_??1QDir@@QAE@XZ      0049e088     QtCore4:QtCore4.dll
 0004:0000208c       __imp_??8QString@@QBE_NABV0@@Z 0049e08c     QtCore4:QtCore4.dll
 0004:00002090       __imp_?number@QString@@SA?AV1@HH@Z 0049e090     QtCore4:QtCore4.dll
 0004:00002094       __imp_??0QTextStream@@QAE@PAVQIODevice@@@Z 0049e094     QtCore4:QtCore4.dll
 0004:00002098       __imp_?codecForName@QTextCodec@@SAPAV1@PBD@Z 0049e098     QtCore4:QtCore4.dll
 0004:0000209c       __imp_?setCodec@QTextStream@@QAEXPAVQTextCodec@@@Z 0049e09c     QtCore4:QtCore4.dll
 0004:000020a0       __imp_??1QTextStream@@UAE@XZ 0049e0a0     QtCore4:QtCore4.dll
 0004:000020a4       __imp_?isNull@QString@@QBE_NXZ 0049e0a4     QtCore4:QtCore4.dll
 0004:000020a8       __imp_??0QFile@@QAE@ABVQString@@@Z 0049e0a8     QtCore4:QtCore4.dll
 0004:000020ac       __imp_?open@QFile@@UAE_NV?$QFlags@W4OpenModeFlag@QIODevice@@@@@Z 0049e0ac     QtCore4:QtCore4.dll
 0004:000020b0       __imp_??1QFile@@UAE@XZ     0049e0b0     QtCore4:QtCore4.dll
 0004:000020b4       __imp_?close@QFile@@UAEXXZ 0049e0b4     QtCore4:QtCore4.dll
 0004:000020b8       __imp_??0QString@@QAE@XZ   0049e0b8     QtCore4:QtCore4.dll
 0004:000020bc       __imp_??0QString@@QAE@PBD@Z 0049e0bc     QtCore4:QtCore4.dll
 0004:000020c0       __imp_??4QString@@QAEAAV0@PBD@Z 0049e0c0     QtCore4:QtCore4.dll
 0004:000020c4       __imp_?fromAscii@QString@@SA?AV1@PBDH@Z 0049e0c4     QtCore4:QtCore4.dll
 0004:000020c8       __imp_??YQString@@QAEAAV0@VQChar@@@Z 0049e0c8     QtCore4:QtCore4.dll
 0004:000020cc       __imp_??YQString@@QAEAAV0@ABV0@@Z 0049e0cc     QtCore4:QtCore4.dll
 0004:000020d0       __imp_?tr@QObject@@SA?AVQString@@PBD0@Z 0049e0d0     QtCore4:QtCore4.dll
 0004:000020d4       __imp_??0QLatin1String@@QAE@PBD@Z 0049e0d4     QtCore4:QtCore4.dll
 0004:000020d8       __imp_?setApplicationName@QCoreApplication@@SAXABVQString@@@Z 0049e0d8     QtCore4:QtCore4.dll
 0004:000020dc       __imp_?qt_metacall@QObject@@UAEHW4Call@QMetaObject@@HPAPAX@Z 0049e0dc     QtCore4:QtCore4.dll
 0004:000020e0       __imp_?qt_metacast@QObject@@UAEPAXPBD@Z 0049e0e0     QtCore4:QtCore4.dll
 0004:000020e4       __imp_?node_create@QMapData@@QAEPAUNode@1@QAPAU21@HH@Z 0049e0e4     QtCore4:QtCore4.dll
 0004:000020e8       __imp_?node_delete@QMapData@@QAEXQAPAUNode@1@HPAU21@@Z 0049e0e8     QtCore4:QtCore4.dll
 0004:000020ec       __imp_?createData@QMapData@@SAPAU1@H@Z 0049e0ec     QtCore4:QtCore4.dll
 0004:000020f0       __imp_?continueFreeData@QMapData@@QAEXH@Z 0049e0f0     QtCore4:QtCore4.dll
 0004:000020f4       __imp_?ref@QBasicAtomicInt@@QAE_NXZ 0049e0f4     QtCore4:QtCore4.dll
 0004:000020f8       __imp_?deref@QBasicAtomicInt@@QAE_NXZ 0049e0f8     QtCore4:QtCore4.dll
 0004:000020fc       __imp_??0QString@@QAE@ABV0@@Z 0049e0fc     QtCore4:QtCore4.dll
 0004:00002100       __imp_??4QString@@QAEAAV0@ABV0@@Z 0049e100     QtCore4:QtCore4.dll
 0004:00002104       __imp_??1QString@@QAE@XZ   0049e104     QtCore4:QtCore4.dll
 0004:00002108       __imp_?lock@QMutex@@QAEXXZ 0049e108     QtCore4:QtCore4.dll
 0004:0000210c       __imp_?activate@QMetaObject@@SAXPAVQObject@@PBU1@HPAPAX@Z 0049e10c     QtCore4:QtCore4.dll
 0004:00002110       \177QtCore4_NULL_THUNK_DATA 0049e110     QtCore4:QtCore4.dll
 0004:00002220       __imp_?sizeHint@QWidget@@UBE?AVQSize@@XZ 0049e220     QtGui4:QtGui4.dll
 0004:00002224       __imp_?minimumSizeHint@QWidget@@UBE?AVQSize@@XZ 0049e224     QtGui4:QtGui4.dll
 0004:00002228       __imp_?heightForWidth@QWidget@@UBEHH@Z 0049e228     QtGui4:QtGui4.dll
 0004:0000222c       __imp_?mousePressEvent@QWidget@@MAEXPAVQMouseEvent@@@Z 0049e22c     QtGui4:QtGui4.dll
 0004:00002230       __imp_?mouseReleaseEvent@QWidget@@MAEXPAVQMouseEvent@@@Z 0049e230     QtGui4:QtGui4.dll
 0004:00002234       __imp_?mouseDoubleClickEvent@QWidget@@MAEXPAVQMouseEvent@@@Z 0049e234     QtGui4:QtGui4.dll
 0004:00002238       __imp_?mouseMoveEvent@QWidget@@MAEXPAVQMouseEvent@@@Z 0049e238     QtGui4:QtGui4.dll
 0004:0000223c       __imp_?wheelEvent@QWidget@@MAEXPAVQWheelEvent@@@Z 0049e23c     QtGui4:QtGui4.dll
 0004:00002240       __imp_?keyReleaseEvent@QWidget@@MAEXPAVQKeyEvent@@@Z 0049e240     QtGui4:QtGui4.dll
 0004:00002244       __imp_?focusInEvent@QWidget@@MAEXPAVQFocusEvent@@@Z 0049e244     QtGui4:QtGui4.dll
 0004:00002248       __imp_?focusOutEvent@QWidget@@MAEXPAVQFocusEvent@@@Z 0049e248     QtGui4:QtGui4.dll
 0004:0000224c       __imp_?enterEvent@QWidget@@MAEXPAVQEvent@@@Z 0049e24c     QtGui4:QtGui4.dll
 0004:00002250       __imp_?leaveEvent@QWidget@@MAEXPAVQEvent@@@Z 0049e250     QtGui4:QtGui4.dll
 0004:00002254       __imp_?paintEvent@QWidget@@MAEXPAVQPaintEvent@@@Z 0049e254     QtGui4:QtGui4.dll
 0004:00002258       __imp_?moveEvent@QWidget@@MAEXPAVQMoveEvent@@@Z 0049e258     QtGui4:QtGui4.dll
 0004:0000225c       __imp_?contextMenuEvent@QMainWindow@@MAEXPAVQContextMenuEvent@@@Z 0049e25c     QtGui4:QtGui4.dll
 0004:00002260       __imp_?tabletEvent@QWidget@@MAEXPAVQTabletEvent@@@Z 0049e260     QtGui4:QtGui4.dll
 0004:00002264       __imp_?actionEvent@QWidget@@MAEXPAVQActionEvent@@@Z 0049e264     QtGui4:QtGui4.dll
 0004:00002268       __imp_?dragEnterEvent@QWidget@@MAEXPAVQDragEnterEvent@@@Z 0049e268     QtGui4:QtGui4.dll
 0004:0000226c       __imp_?dragMoveEvent@QWidget@@MAEXPAVQDragMoveEvent@@@Z 0049e26c     QtGui4:QtGui4.dll
 0004:00002270       __imp_?dragLeaveEvent@QWidget@@MAEXPAVQDragLeaveEvent@@@Z 0049e270     QtGui4:QtGui4.dll
 0004:00002274       __imp_?dropEvent@QWidget@@MAEXPAVQDropEvent@@@Z 0049e274     QtGui4:QtGui4.dll
 0004:00002278       __imp_?showEvent@QWidget@@MAEXPAVQShowEvent@@@Z 0049e278     QtGui4:QtGui4.dll
 0004:0000227c       __imp_?hideEvent@QWidget@@MAEXPAVQHideEvent@@@Z 0049e27c     QtGui4:QtGui4.dll
 0004:00002280       __imp_?winEvent@QWidget@@MAE_NPAUtagMSG@@PAJ@Z 0049e280     QtGui4:QtGui4.dll
 0004:00002284       __imp_?changeEvent@QWidget@@MAEXPAVQEvent@@@Z 0049e284     QtGui4:QtGui4.dll
 0004:00002288       __imp_?inputMethodEvent@QWidget@@MAEXPAVQInputMethodEvent@@@Z 0049e288     QtGui4:QtGui4.dll
 0004:0000228c       __imp_?inputMethodQuery@QWidget@@UBE?AVQVariant@@W4InputMethodQuery@Qt@@@Z 0049e28c     QtGui4:QtGui4.dll
 0004:00002290       __imp_?focusNextPrevChild@QWidget@@MAE_N_N@Z 0049e290     QtGui4:QtGui4.dll
 0004:00002294       __imp_?styleChange@QWidget@@MAEXAAVQStyle@@@Z 0049e294     QtGui4:QtGui4.dll
 0004:00002298       __imp_?enabledChange@QWidget@@MAEX_N@Z 0049e298     QtGui4:QtGui4.dll
 0004:0000229c       __imp_?paletteChange@QWidget@@MAEXABVQPalette@@@Z 0049e29c     QtGui4:QtGui4.dll
 0004:000022a0       __imp_?fontChange@QWidget@@MAEXABVQFont@@@Z 0049e2a0     QtGui4:QtGui4.dll
 0004:000022a4       __imp_?windowActivationChange@QWidget@@MAEX_N@Z 0049e2a4     QtGui4:QtGui4.dll
 0004:000022a8       __imp_?languageChange@QWidget@@MAEXXZ 0049e2a8     QtGui4:QtGui4.dll
 0004:000022ac       __imp_?createPopupMenu@QMainWindow@@UAEPAVQMenu@@XZ 0049e2ac     QtGui4:QtGui4.dll
 0004:000022b0       __imp_?devType@QWidget@@UBEHXZ 0049e2b0     QtGui4:QtGui4.dll
 0004:000022b4       __imp_?paintEngine@QWidget@@UBEPAVQPaintEngine@@XZ 0049e2b4     QtGui4:QtGui4.dll
 0004:000022b8       __imp_?getDC@QWidget@@UBEPAUHDC__@@XZ 0049e2b8     QtGui4:QtGui4.dll
 0004:000022bc       __imp_?releaseDC@QWidget@@UBEXPAUHDC__@@@Z 0049e2bc     QtGui4:QtGui4.dll
 0004:000022c0       __imp_?metric@QWidget@@MBEHW4PaintDeviceMetric@QPaintDevice@@@Z 0049e2c0     QtGui4:QtGui4.dll
 0004:000022c4       __imp_?setCentralWidget@QMainWindow@@QAEXPAVQWidget@@@Z 0049e2c4     QtGui4:QtGui4.dll
 0004:000022c8       __imp_?addWidget@QGridLayout@@QAEXPAVQWidget@@HHHHV?$QFlags@W4AlignmentFlag@Qt@@@@@Z 0049e2c8     QtGui4:QtGui4.dll
 0004:000022cc       __imp_?setWidget@QScrollArea@@QAEXPAVQWidget@@@Z 0049e2cc     QtGui4:QtGui4.dll
 0004:000022d0       __imp_?addLayout@QGridLayout@@QAEXPAVQLayout@@HHHHV?$QFlags@W4AlignmentFlag@Qt@@@@@Z 0049e2d0     QtGui4:QtGui4.dll
 0004:000022d4       __imp_?setSpacing@QBoxLayout@@QAEXH@Z 0049e2d4     QtGui4:QtGui4.dll
 0004:000022d8       __imp_??0QVBoxLayout@@QAE@XZ 0049e2d8     QtGui4:QtGui4.dll
 0004:000022dc       __imp_?setGeometry@QWidget@@QAEXABVQRect@@@Z 0049e2dc     QtGui4:QtGui4.dll
 0004:000022e0       __imp_?setWidgetResizable@QScrollArea@@QAEX_N@Z 0049e2e0     QtGui4:QtGui4.dll
 0004:000022e4       __imp_??0QScrollArea@@QAE@PAVQWidget@@@Z 0049e2e4     QtGui4:QtGui4.dll
 0004:000022e8       __imp_?setContentsMargins@QLayout@@QAEXHHHH@Z 0049e2e8     QtGui4:QtGui4.dll
 0004:000022ec       __imp_?setSpacing@QGridLayout@@QAEXH@Z 0049e2ec     QtGui4:QtGui4.dll
 0004:000022f0       __imp_??0QGridLayout@@QAE@PAVQWidget@@@Z 0049e2f0     QtGui4:QtGui4.dll
 0004:000022f4       __imp_??0QWidget@@QAE@PAV0@V?$QFlags@W4WindowType@Qt@@@@@Z 0049e2f4     QtGui4:QtGui4.dll
 0004:000022f8       __imp_?setMaximumSize@QWidget@@QAEXABVQSize@@@Z 0049e2f8     QtGui4:QtGui4.dll
 0004:000022fc       __imp_?setWindowModality@QWidget@@QAEXW4WindowModality@Qt@@@Z 0049e2fc     QtGui4:QtGui4.dll
 0004:00002300       __imp_?metaObject@QWidget@@UBEPBUQMetaObject@@XZ 0049e300     QtGui4:QtGui4.dll
 0004:00002304       __imp_?event@QWidget@@MAE_NPAVQEvent@@@Z 0049e304     QtGui4:QtGui4.dll
 0004:00002308       __imp_?keyPressEvent@QWidget@@MAEXPAVQKeyEvent@@@Z 0049e308     QtGui4:QtGui4.dll
 0004:0000230c       __imp_?resizeEvent@QWidget@@MAEXPAVQResizeEvent@@@Z 0049e30c     QtGui4:QtGui4.dll
 0004:00002310       __imp_?closeEvent@QWidget@@MAEXPAVQCloseEvent@@@Z 0049e310     QtGui4:QtGui4.dll
 0004:00002314       __imp_?contextMenuEvent@QWidget@@MAEXPAVQContextMenuEvent@@@Z 0049e314     QtGui4:QtGui4.dll
 0004:00002318       __imp_?metaObject@QGridLayout@@UBEPBUQMetaObject@@XZ 0049e318     QtGui4:QtGui4.dll
 0004:0000231c       __imp_?qt_metacast@QGridLayout@@UAEPAXPBD@Z 0049e31c     QtGui4:QtGui4.dll
 0004:00002320       __imp_?qt_metacall@QGridLayout@@UAEHW4Call@QMetaObject@@HPAPAX@Z 0049e320     QtGui4:QtGui4.dll
 0004:00002324       __imp_?childEvent@QLayout@@MAEXPAVQChildEvent@@@Z 0049e324     QtGui4:QtGui4.dll
 0004:00002328       __imp_?addItem@QGridLayout@@MAEXPAVQLayoutItem@@@Z 0049e328     QtGui4:QtGui4.dll
 0004:0000232c       __imp_?itemAt@QGridLayout@@UBEPAVQLayoutItem@@H@Z 0049e32c     QtGui4:QtGui4.dll
 0004:00002330       __imp_?takeAt@QGridLayout@@UAEPAVQLayoutItem@@H@Z 0049e330     QtGui4:QtGui4.dll
 0004:00002334       __imp_?indexOf@QLayout@@UBEHPAVQWidget@@@Z 0049e334     QtGui4:QtGui4.dll
 0004:00002338       __imp_?count@QGridLayout@@UBEHXZ 0049e338     QtGui4:QtGui4.dll
 0004:0000233c       __imp_?sizeHint@QGridLayout@@UBE?AVQSize@@XZ 0049e33c     QtGui4:QtGui4.dll
 0004:00002340       __imp_?minimumSize@QGridLayout@@UBE?AVQSize@@XZ 0049e340     QtGui4:QtGui4.dll
 0004:00002344       __imp_?maximumSize@QGridLayout@@UBE?AVQSize@@XZ 0049e344     QtGui4:QtGui4.dll
 0004:00002348       __imp_?expandingDirections@QGridLayout@@UBE?AV?$QFlags@W4Orientation@Qt@@@@XZ 0049e348     QtGui4:QtGui4.dll
 0004:0000234c       __imp_?setGeometry@QGridLayout@@UAEXABVQRect@@@Z 0049e34c     QtGui4:QtGui4.dll
 0004:00002350       __imp_?geometry@QLayout@@UBE?AVQRect@@XZ 0049e350     QtGui4:QtGui4.dll
 0004:00002354       __imp_?isEmpty@QLayout@@UBE_NXZ 0049e354     QtGui4:QtGui4.dll
 0004:00002358       __imp_?hasHeightForWidth@QGridLayout@@UBE_NXZ 0049e358     QtGui4:QtGui4.dll
 0004:0000235c       __imp_?heightForWidth@QGridLayout@@UBEHH@Z 0049e35c     QtGui4:QtGui4.dll
 0004:00002360       __imp_?minimumHeightForWidth@QGridLayout@@UBEHH@Z 0049e360     QtGui4:QtGui4.dll
 0004:00002364       __imp_?invalidate@QGridLayout@@UAEXXZ 0049e364     QtGui4:QtGui4.dll
 0004:00002368       __imp_?widget@QLayoutItem@@UAEPAVQWidget@@XZ 0049e368     QtGui4:QtGui4.dll
 0004:0000236c       __imp_?layout@QLayout@@UAEPAV1@XZ 0049e36c     QtGui4:QtGui4.dll
 0004:00002370       __imp_?spacerItem@QLayoutItem@@UAEPAVQSpacerItem@@XZ 0049e370     QtGui4:QtGui4.dll
 0004:00002374       __imp_?metaObject@QScrollArea@@UBEPBUQMetaObject@@XZ 0049e374     QtGui4:QtGui4.dll
 0004:00002378       __imp_?qt_metacast@QScrollArea@@UAEPAXPBD@Z 0049e378     QtGui4:QtGui4.dll
 0004:0000237c       __imp_?qt_metacall@QScrollArea@@UAEHW4Call@QMetaObject@@HPAPAX@Z 0049e37c     QtGui4:QtGui4.dll
 0004:00002380       __imp_?event@QScrollArea@@MAE_NPAVQEvent@@@Z 0049e380     QtGui4:QtGui4.dll
 0004:00002384       __imp_?eventFilter@QScrollArea@@MAE_NPAVQObject@@PAVQEvent@@@Z 0049e384     QtGui4:QtGui4.dll
 0004:00002388       __imp_?sizeHint@QScrollArea@@UBE?AVQSize@@XZ 0049e388     QtGui4:QtGui4.dll
 0004:0000238c       __imp_?minimumSizeHint@QAbstractScrollArea@@UBE?AVQSize@@XZ 0049e38c     QtGui4:QtGui4.dll
 0004:00002390       __imp_?mousePressEvent@QAbstractScrollArea@@MAEXPAVQMouseEvent@@@Z 0049e390     QtGui4:QtGui4.dll
 0004:00002394       __imp_?mouseReleaseEvent@QAbstractScrollArea@@MAEXPAVQMouseEvent@@@Z 0049e394     QtGui4:QtGui4.dll
 0004:00002398       __imp_?mouseDoubleClickEvent@QAbstractScrollArea@@MAEXPAVQMouseEvent@@@Z 0049e398     QtGui4:QtGui4.dll
 0004:0000239c       __imp_?mouseMoveEvent@QAbstractScrollArea@@MAEXPAVQMouseEvent@@@Z 0049e39c     QtGui4:QtGui4.dll
 0004:000023a0       __imp_?wheelEvent@QAbstractScrollArea@@MAEXPAVQWheelEvent@@@Z 0049e3a0     QtGui4:QtGui4.dll
 0004:000023a4       __imp_?keyPressEvent@QAbstractScrollArea@@MAEXPAVQKeyEvent@@@Z 0049e3a4     QtGui4:QtGui4.dll
 0004:000023a8       __imp_?paintEvent@QAbstractScrollArea@@MAEXPAVQPaintEvent@@@Z 0049e3a8     QtGui4:QtGui4.dll
 0004:000023ac       __imp_?resizeEvent@QScrollArea@@MAEXPAVQResizeEvent@@@Z 0049e3ac     QtGui4:QtGui4.dll
 0004:000023b0       __imp_?contextMenuEvent@QAbstractScrollArea@@MAEXPAVQContextMenuEvent@@@Z 0049e3b0     QtGui4:QtGui4.dll
 0004:000023b4       __imp_?dragEnterEvent@QAbstractScrollArea@@MAEXPAVQDragEnterEvent@@@Z 0049e3b4     QtGui4:QtGui4.dll
 0004:000023b8       __imp_?dragMoveEvent@QAbstractScrollArea@@MAEXPAVQDragMoveEvent@@@Z 0049e3b8     QtGui4:QtGui4.dll
 0004:000023bc       __imp_?dragLeaveEvent@QAbstractScrollArea@@MAEXPAVQDragLeaveEvent@@@Z 0049e3bc     QtGui4:QtGui4.dll
 0004:000023c0       __imp_?dropEvent@QAbstractScrollArea@@MAEXPAVQDropEvent@@@Z 0049e3c0     QtGui4:QtGui4.dll
 0004:000023c4       __imp_?changeEvent@QFrame@@MAEXPAVQEvent@@@Z 0049e3c4     QtGui4:QtGui4.dll
 0004:000023c8       __imp_?focusNextPrevChild@QScrollArea@@UAE_N_N@Z 0049e3c8     QtGui4:QtGui4.dll
 0004:000023cc       __imp_?viewportEvent@QAbstractScrollArea@@MAE_NPAVQEvent@@@Z 0049e3cc     QtGui4:QtGui4.dll
 0004:000023d0       __imp_?scrollContentsBy@QScrollArea@@MAEXHH@Z 0049e3d0     QtGui4:QtGui4.dll
 0004:000023d4       __imp_?metaObject@QVBoxLayout@@UBEPBUQMetaObject@@XZ 0049e3d4     QtGui4:QtGui4.dll
 0004:000023d8       __imp_?qt_metacast@QVBoxLayout@@UAEPAXPBD@Z 0049e3d8     QtGui4:QtGui4.dll
 0004:000023dc       __imp_?qt_metacall@QVBoxLayout@@UAEHW4Call@QMetaObject@@HPAPAX@Z 0049e3dc     QtGui4:QtGui4.dll
 0004:000023e0       __imp_?addItem@QBoxLayout@@UAEXPAVQLayoutItem@@@Z 0049e3e0     QtGui4:QtGui4.dll
 0004:000023e4       __imp_?itemAt@QBoxLayout@@UBEPAVQLayoutItem@@H@Z 0049e3e4     QtGui4:QtGui4.dll
 0004:000023e8       __imp_?takeAt@QBoxLayout@@UAEPAVQLayoutItem@@H@Z 0049e3e8     QtGui4:QtGui4.dll
 0004:000023ec       __imp_?count@QBoxLayout@@UBEHXZ 0049e3ec     QtGui4:QtGui4.dll
 0004:000023f0       __imp_?sizeHint@QBoxLayout@@UBE?AVQSize@@XZ 0049e3f0     QtGui4:QtGui4.dll
 0004:000023f4       __imp_?minimumSize@QBoxLayout@@UBE?AVQSize@@XZ 0049e3f4     QtGui4:QtGui4.dll
 0004:000023f8       __imp_?maximumSize@QBoxLayout@@UBE?AVQSize@@XZ 0049e3f8     QtGui4:QtGui4.dll
 0004:000023fc       __imp_?expandingDirections@QBoxLayout@@UBE?AV?$QFlags@W4Orientation@Qt@@@@XZ 0049e3fc     QtGui4:QtGui4.dll
 0004:00002400       __imp_?setGeometry@QBoxLayout@@UAEXABVQRect@@@Z 0049e400     QtGui4:QtGui4.dll
 0004:00002404       __imp_?hasHeightForWidth@QBoxLayout@@UBE_NXZ 0049e404     QtGui4:QtGui4.dll
 0004:00002408       __imp_?heightForWidth@QBoxLayout@@UBEHH@Z 0049e408     QtGui4:QtGui4.dll
 0004:0000240c       __imp_?minimumHeightForWidth@QBoxLayout@@UBEHH@Z 0049e40c     QtGui4:QtGui4.dll
 0004:00002410       __imp_?invalidate@QBoxLayout@@UAEXXZ 0049e410     QtGui4:QtGui4.dll
 0004:00002414       __imp_?setWindowTitle@QWidget@@QAEXABVQString@@@Z 0049e414     QtGui4:QtGui4.dll
 0004:00002418       __imp_??1QWidget@@UAE@XZ   0049e418     QtGui4:QtGui4.dll
 0004:0000241c       __imp_??1QGridLayout@@UAE@XZ 0049e41c     QtGui4:QtGui4.dll
 0004:00002420       __imp_??1QScrollArea@@UAE@XZ 0049e420     QtGui4:QtGui4.dll
 0004:00002424       __imp_??1QVBoxLayout@@UAE@XZ 0049e424     QtGui4:QtGui4.dll
 0004:00002428       __imp_?lower@QWidget@@QAEXXZ 0049e428     QtGui4:QtGui4.dll
 0004:0000242c       __imp_?addLayout@QBoxLayout@@QAEXPAVQLayout@@H@Z 0049e42c     QtGui4:QtGui4.dll
 0004:00002430       __imp_?addWidget@QBoxLayout@@QAEXPAVQWidget@@HV?$QFlags@W4AlignmentFlag@Qt@@@@@Z 0049e430     QtGui4:QtGui4.dll
 0004:00002434       __imp_?setFocusPolicy@QWidget@@QAEXW4FocusPolicy@Qt@@@Z 0049e434     QtGui4:QtGui4.dll
 0004:00002438       __imp_?setAttribute@QWidget@@QAEXW4WidgetAttribute@Qt@@_N@Z 0049e438     QtGui4:QtGui4.dll
 0004:0000243c       __imp_?addAction@QWidget@@QAEXPAVQAction@@@Z 0049e43c     QtGui4:QtGui4.dll
 0004:00002440       __imp_??0QHBoxLayout@@QAE@XZ 0049e440     QtGui4:QtGui4.dll
 0004:00002444       __imp_?setWindowFlags@QWidget@@QAEXV?$QFlags@W4WindowType@Qt@@@@@Z 0049e444     QtGui4:QtGui4.dll
 0004:00002448       __imp_?metaObject@QHBoxLayout@@UBEPBUQMetaObject@@XZ 0049e448     QtGui4:QtGui4.dll
 0004:0000244c       __imp_?qt_metacast@QHBoxLayout@@UAEPAXPBD@Z 0049e44c     QtGui4:QtGui4.dll
 0004:00002450       __imp_?qt_metacall@QHBoxLayout@@UAEHW4Call@QMetaObject@@HPAPAX@Z 0049e450     QtGui4:QtGui4.dll
 0004:00002454       __imp_??1QHBoxLayout@@UAE@XZ 0049e454     QtGui4:QtGui4.dll
 0004:00002458       __imp_?raise@QWidget@@QAEXXZ 0049e458     QtGui4:QtGui4.dll
 0004:0000245c       __imp_?size@QResizeEvent@@QBEABVQSize@@XZ 0049e45c     QtGui4:QtGui4.dll
 0004:00002460       __imp_?popup@QMenu@@QAEXABVQPoint@@PAVQAction@@@Z 0049e460     QtGui4:QtGui4.dll
 0004:00002464       __imp_?pos@QCursor@@SA?AVQPoint@@XZ 0049e464     QtGui4:QtGui4.dll
 0004:00002468       __imp_?close@QWidget@@QAE_NXZ 0049e468     QtGui4:QtGui4.dll
 0004:0000246c       __imp_?width@QWidget@@QBEHXZ 0049e46c     QtGui4:QtGui4.dll
 0004:00002470       __imp_?height@QWidget@@QBEHXZ 0049e470     QtGui4:QtGui4.dll
 0004:00002474       __imp_?pos@QWidget@@QBE?AVQPoint@@XZ 0049e474     QtGui4:QtGui4.dll
 0004:00002478       __imp_?key@QKeyEvent@@QBEHXZ 0049e478     QtGui4:QtGui4.dll
 0004:0000247c       __imp_?event@QWidgetAction@@MAE_NPAVQEvent@@@Z 0049e47c     QtGui4:QtGui4.dll
 0004:00002480       __imp_?eventFilter@QWidgetAction@@MAE_NPAVQObject@@PAVQEvent@@@Z 0049e480     QtGui4:QtGui4.dll
 0004:00002484       __imp_?createWidget@QWidgetAction@@MAEPAVQWidget@@PAV2@@Z 0049e484     QtGui4:QtGui4.dll
 0004:00002488       __imp_?deleteWidget@QWidgetAction@@MAEXPAVQWidget@@@Z 0049e488     QtGui4:QtGui4.dll
 0004:0000248c       __imp_?openUrl@QDesktopServices@@SA_NABVQUrl@@@Z 0049e48c     QtGui4:QtGui4.dll
 0004:00002490       __imp_?setMaxLength@QLineEdit@@QAEXH@Z 0049e490     QtGui4:QtGui4.dll
 0004:00002494       __imp_?setValidator@QLineEdit@@QAEXPBVQValidator@@@Z 0049e494     QtGui4:QtGui4.dll
 0004:00002498       __imp_?setFixedWidth@QWidget@@QAEXH@Z 0049e498     QtGui4:QtGui4.dll
 0004:0000249c       __imp_?fixup@QIntValidator@@UBEXAAVQString@@@Z 0049e49c     QtGui4:QtGui4.dll
 0004:000024a0       __imp_?setRange@QIntValidator@@UAEXHH@Z 0049e4a0     QtGui4:QtGui4.dll
 0004:000024a4       __imp_?setTabOrder@QWidget@@SAXPAV1@0@Z 0049e4a4     QtGui4:QtGui4.dll
 0004:000024a8       __imp_?setFrameShape@QFrame@@QAEXW4Shape@1@@Z 0049e4a8     QtGui4:QtGui4.dll
 0004:000024ac       __imp_??0QFrame@@QAE@PAVQWidget@@V?$QFlags@W4WindowType@Qt@@@@@Z 0049e4ac     QtGui4:QtGui4.dll
 0004:000024b0       __imp_?setFrame@QComboBox@@QAEX_N@Z 0049e4b0     QtGui4:QtGui4.dll
 0004:000024b4       __imp_?setDuplicatesEnabled@QComboBox@@QAEX_N@Z 0049e4b4     QtGui4:QtGui4.dll
 0004:000024b8       __imp_?setEditable@QComboBox@@QAEX_N@Z 0049e4b8     QtGui4:QtGui4.dll
 0004:000024bc       __imp_?setMinimumSize@QWidget@@QAEXABVQSize@@@Z 0049e4bc     QtGui4:QtGui4.dll
 0004:000024c0       __imp_?setSizePolicy@QWidget@@QAEXVQSizePolicy@@@Z 0049e4c0     QtGui4:QtGui4.dll
 0004:000024c4       __imp_?setHeightForWidth@QSizePolicy@@QAEX_N@Z 0049e4c4     QtGui4:QtGui4.dll
 0004:000024c8       __imp_?hasHeightForWidth@QSizePolicy@@QBE_NXZ 0049e4c8     QtGui4:QtGui4.dll
 0004:000024cc       __imp_?sizePolicy@QWidget@@QBE?AVQSizePolicy@@XZ 0049e4cc     QtGui4:QtGui4.dll
 0004:000024d0       __imp_?setVerticalStretch@QSizePolicy@@QAEXE@Z 0049e4d0     QtGui4:QtGui4.dll
 0004:000024d4       __imp_?setHorizontalStretch@QSizePolicy@@QAEXE@Z 0049e4d4     QtGui4:QtGui4.dll
 0004:000024d8       __imp_??0QSizePolicy@@QAE@W4Policy@0@0@Z 0049e4d8     QtGui4:QtGui4.dll
 0004:000024dc       __imp_??0QLabel@@QAE@PAVQWidget@@V?$QFlags@W4WindowType@Qt@@@@@Z 0049e4dc     QtGui4:QtGui4.dll
 0004:000024e0       __imp_?setVerticalSpacing@QGridLayout@@QAEXH@Z 0049e4e0     QtGui4:QtGui4.dll
 0004:000024e4       __imp_?setHorizontalSpacing@QGridLayout@@QAEXH@Z 0049e4e4     QtGui4:QtGui4.dll
 0004:000024e8       __imp_?setChecked@QAbstractButton@@QAEX_N@Z 0049e4e8     QtGui4:QtGui4.dll
 0004:000024ec       __imp_??0QCheckBox@@QAE@PAVQWidget@@@Z 0049e4ec     QtGui4:QtGui4.dll
 0004:000024f0       __imp_??0QSpacerItem@@QAE@HHW4Policy@QSizePolicy@@0@Z 0049e4f0     QtGui4:QtGui4.dll
 0004:000024f4       __imp_??0QVBoxLayout@@QAE@PAVQWidget@@@Z 0049e4f4     QtGui4:QtGui4.dll
 0004:000024f8       __imp_??0QGridLayout@@QAE@XZ 0049e4f8     QtGui4:QtGui4.dll
 0004:000024fc       __imp_?setStyleSheet@QWidget@@QAEXABVQString@@@Z 0049e4fc     QtGui4:QtGui4.dll
 0004:00002500       __imp_?sizeHint@QSpacerItem@@UBE?AVQSize@@XZ 0049e500     QtGui4:QtGui4.dll
 0004:00002504       __imp_?minimumSize@QSpacerItem@@UBE?AVQSize@@XZ 0049e504     QtGui4:QtGui4.dll
 0004:00002508       __imp_?maximumSize@QSpacerItem@@UBE?AVQSize@@XZ 0049e508     QtGui4:QtGui4.dll
 0004:0000250c       __imp_?expandingDirections@QSpacerItem@@UBE?AV?$QFlags@W4Orientation@Qt@@@@XZ 0049e50c     QtGui4:QtGui4.dll
 0004:00002510       __imp_?setGeometry@QSpacerItem@@UAEXABVQRect@@@Z 0049e510     QtGui4:QtGui4.dll
 0004:00002514       __imp_?geometry@QSpacerItem@@UBE?AVQRect@@XZ 0049e514     QtGui4:QtGui4.dll
 0004:00002518       __imp_?isEmpty@QSpacerItem@@UBE_NXZ 0049e518     QtGui4:QtGui4.dll
 0004:0000251c       __imp_?hasHeightForWidth@QLayoutItem@@UBE_NXZ 0049e51c     QtGui4:QtGui4.dll
 0004:00002520       __imp_?heightForWidth@QLayoutItem@@UBEHH@Z 0049e520     QtGui4:QtGui4.dll
 0004:00002524       __imp_?minimumHeightForWidth@QLayoutItem@@UBEHH@Z 0049e524     QtGui4:QtGui4.dll
 0004:00002528       __imp_?invalidate@QLayoutItem@@UAEXXZ 0049e528     QtGui4:QtGui4.dll
 0004:0000252c       __imp_?layout@QLayoutItem@@UAEPAVQLayout@@XZ 0049e52c     QtGui4:QtGui4.dll
 0004:00002530       __imp_?spacerItem@QSpacerItem@@UAEPAV1@XZ 0049e530     QtGui4:QtGui4.dll
 0004:00002534       __imp_?metaObject@QCheckBox@@UBEPBUQMetaObject@@XZ 0049e534     QtGui4:QtGui4.dll
 0004:00002538       __imp_?qt_metacast@QCheckBox@@UAEPAXPBD@Z 0049e538     QtGui4:QtGui4.dll
 0004:0000253c       __imp_?qt_metacall@QCheckBox@@UAEHW4Call@QMetaObject@@HPAPAX@Z 0049e53c     QtGui4:QtGui4.dll
 0004:00002540       __imp_?event@QCheckBox@@MAE_NPAVQEvent@@@Z 0049e540     QtGui4:QtGui4.dll
 0004:00002544       __imp_?timerEvent@QAbstractButton@@MAEXPAVQTimerEvent@@@Z 0049e544     QtGui4:QtGui4.dll
 0004:00002548       __imp_?sizeHint@QCheckBox@@UBE?AVQSize@@XZ 0049e548     QtGui4:QtGui4.dll
 0004:0000254c       __imp_?minimumSizeHint@QCheckBox@@UBE?AVQSize@@XZ 0049e54c     QtGui4:QtGui4.dll
 0004:00002550       __imp_?mousePressEvent@QAbstractButton@@MAEXPAVQMouseEvent@@@Z 0049e550     QtGui4:QtGui4.dll
 0004:00002554       __imp_?mouseReleaseEvent@QAbstractButton@@MAEXPAVQMouseEvent@@@Z 0049e554     QtGui4:QtGui4.dll
 0004:00002558       __imp_?mouseMoveEvent@QCheckBox@@MAEXPAVQMouseEvent@@@Z 0049e558     QtGui4:QtGui4.dll
 0004:0000255c       __imp_?keyPressEvent@QAbstractButton@@MAEXPAVQKeyEvent@@@Z 0049e55c     QtGui4:QtGui4.dll
 0004:00002560       __imp_?keyReleaseEvent@QAbstractButton@@MAEXPAVQKeyEvent@@@Z 0049e560     QtGui4:QtGui4.dll
 0004:00002564       __imp_?focusInEvent@QAbstractButton@@MAEXPAVQFocusEvent@@@Z 0049e564     QtGui4:QtGui4.dll
 0004:00002568       __imp_?focusOutEvent@QAbstractButton@@MAEXPAVQFocusEvent@@@Z 0049e568     QtGui4:QtGui4.dll
 0004:0000256c       __imp_?paintEvent@QCheckBox@@MAEXPAVQPaintEvent@@@Z 0049e56c     QtGui4:QtGui4.dll
 0004:00002570       __imp_?changeEvent@QAbstractButton@@MAEXPAVQEvent@@@Z 0049e570     QtGui4:QtGui4.dll
 0004:00002574       __imp_?hitButton@QCheckBox@@MBE_NABVQPoint@@@Z 0049e574     QtGui4:QtGui4.dll
 0004:00002578       __imp_?checkStateSet@QCheckBox@@MAEXXZ 0049e578     QtGui4:QtGui4.dll
 0004:0000257c       __imp_?nextCheckState@QCheckBox@@MAEXXZ 0049e57c     QtGui4:QtGui4.dll
 0004:00002580       __imp_?metaObject@QLabel@@UBEPBUQMetaObject@@XZ 0049e580     QtGui4:QtGui4.dll
 0004:00002584       __imp_?event@QLabel@@MAE_NPAVQEvent@@@Z 0049e584     QtGui4:QtGui4.dll
 0004:00002588       __imp_?sizeHint@QLabel@@UBE?AVQSize@@XZ 0049e588     QtGui4:QtGui4.dll
 0004:0000258c       __imp_?minimumSizeHint@QLabel@@UBE?AVQSize@@XZ 0049e58c     QtGui4:QtGui4.dll
 0004:00002590       __imp_?heightForWidth@QLabel@@UBEHH@Z 0049e590     QtGui4:QtGui4.dll
 0004:00002594       __imp_?mousePressEvent@QLabel@@MAEXPAVQMouseEvent@@@Z 0049e594     QtGui4:QtGui4.dll
 0004:00002598       __imp_?mouseReleaseEvent@QLabel@@MAEXPAVQMouseEvent@@@Z 0049e598     QtGui4:QtGui4.dll
 0004:0000259c       __imp_?mouseMoveEvent@QLabel@@MAEXPAVQMouseEvent@@@Z 0049e59c     QtGui4:QtGui4.dll
 0004:000025a0       __imp_?keyPressEvent@QLabel@@MAEXPAVQKeyEvent@@@Z 0049e5a0     QtGui4:QtGui4.dll
 0004:000025a4       __imp_?focusInEvent@QLabel@@MAEXPAVQFocusEvent@@@Z 0049e5a4     QtGui4:QtGui4.dll
 0004:000025a8       __imp_?focusOutEvent@QLabel@@MAEXPAVQFocusEvent@@@Z 0049e5a8     QtGui4:QtGui4.dll
 0004:000025ac       __imp_?paintEvent@QLabel@@MAEXPAVQPaintEvent@@@Z 0049e5ac     QtGui4:QtGui4.dll
 0004:000025b0       __imp_?contextMenuEvent@QLabel@@MAEXPAVQContextMenuEvent@@@Z 0049e5b0     QtGui4:QtGui4.dll
 0004:000025b4       __imp_?changeEvent@QLabel@@MAEXPAVQEvent@@@Z 0049e5b4     QtGui4:QtGui4.dll
 0004:000025b8       __imp_?focusNextPrevChild@QLabel@@MAE_N_N@Z 0049e5b8     QtGui4:QtGui4.dll
 0004:000025bc       __imp_?event@QLineEdit@@UAE_NPAVQEvent@@@Z 0049e5bc     QtGui4:QtGui4.dll
 0004:000025c0       __imp_?sizeHint@QLineEdit@@UBE?AVQSize@@XZ 0049e5c0     QtGui4:QtGui4.dll
 0004:000025c4       __imp_?minimumSizeHint@QLineEdit@@UBE?AVQSize@@XZ 0049e5c4     QtGui4:QtGui4.dll
 0004:000025c8       __imp_?mouseReleaseEvent@QLineEdit@@MAEXPAVQMouseEvent@@@Z 0049e5c8     QtGui4:QtGui4.dll
 0004:000025cc       __imp_?mouseDoubleClickEvent@QLineEdit@@MAEXPAVQMouseEvent@@@Z 0049e5cc     QtGui4:QtGui4.dll
 0004:000025d0       __imp_?mouseMoveEvent@QLineEdit@@MAEXPAVQMouseEvent@@@Z 0049e5d0     QtGui4:QtGui4.dll
 0004:000025d4       __imp_?keyPressEvent@QLineEdit@@MAEXPAVQKeyEvent@@@Z 0049e5d4     QtGui4:QtGui4.dll
 0004:000025d8       __imp_?focusOutEvent@QLineEdit@@MAEXPAVQFocusEvent@@@Z 0049e5d8     QtGui4:QtGui4.dll
 0004:000025dc       __imp_?paintEvent@QLineEdit@@MAEXPAVQPaintEvent@@@Z 0049e5dc     QtGui4:QtGui4.dll
 0004:000025e0       __imp_?contextMenuEvent@QLineEdit@@MAEXPAVQContextMenuEvent@@@Z 0049e5e0     QtGui4:QtGui4.dll
 0004:000025e4       __imp_?dragEnterEvent@QLineEdit@@MAEXPAVQDragEnterEvent@@@Z 0049e5e4     QtGui4:QtGui4.dll
 0004:000025e8       __imp_?dragMoveEvent@QLineEdit@@MAEXPAVQDragMoveEvent@@@Z 0049e5e8     QtGui4:QtGui4.dll
 0004:000025ec       __imp_?dragLeaveEvent@QLineEdit@@MAEXPAVQDragLeaveEvent@@@Z 0049e5ec     QtGui4:QtGui4.dll
 0004:000025f0       __imp_?dropEvent@QLineEdit@@MAEXPAVQDropEvent@@@Z 0049e5f0     QtGui4:QtGui4.dll
 0004:000025f4       __imp_?changeEvent@QLineEdit@@MAEXPAVQEvent@@@Z 0049e5f4     QtGui4:QtGui4.dll
 0004:000025f8       __imp_?inputMethodEvent@QLineEdit@@MAEXPAVQInputMethodEvent@@@Z 0049e5f8     QtGui4:QtGui4.dll
 0004:000025fc       __imp_?inputMethodQuery@QLineEdit@@UBE?AVQVariant@@W4InputMethodQuery@Qt@@@Z 0049e5fc     QtGui4:QtGui4.dll
 0004:00002600       __imp_?event@QComboBox@@UAE_NPAVQEvent@@@Z 0049e600     QtGui4:QtGui4.dll
 0004:00002604       __imp_?sizeHint@QComboBox@@UBE?AVQSize@@XZ 0049e604     QtGui4:QtGui4.dll
 0004:00002608       __imp_?minimumSizeHint@QComboBox@@UBE?AVQSize@@XZ 0049e608     QtGui4:QtGui4.dll
 0004:0000260c       __imp_?mousePressEvent@QComboBox@@MAEXPAVQMouseEvent@@@Z 0049e60c     QtGui4:QtGui4.dll
 0004:00002610       __imp_?mouseReleaseEvent@QComboBox@@MAEXPAVQMouseEvent@@@Z 0049e610     QtGui4:QtGui4.dll
 0004:00002614       __imp_?wheelEvent@QComboBox@@MAEXPAVQWheelEvent@@@Z 0049e614     QtGui4:QtGui4.dll
 0004:00002618       __imp_?keyPressEvent@QComboBox@@MAEXPAVQKeyEvent@@@Z 0049e618     QtGui4:QtGui4.dll
 0004:0000261c       __imp_?keyReleaseEvent@QComboBox@@MAEXPAVQKeyEvent@@@Z 0049e61c     QtGui4:QtGui4.dll
 0004:00002620       __imp_?focusInEvent@QComboBox@@MAEXPAVQFocusEvent@@@Z 0049e620     QtGui4:QtGui4.dll
 0004:00002624       __imp_?focusOutEvent@QComboBox@@MAEXPAVQFocusEvent@@@Z 0049e624     QtGui4:QtGui4.dll
 0004:00002628       __imp_?paintEvent@QComboBox@@MAEXPAVQPaintEvent@@@Z 0049e628     QtGui4:QtGui4.dll
 0004:0000262c       __imp_?resizeEvent@QComboBox@@MAEXPAVQResizeEvent@@@Z 0049e62c     QtGui4:QtGui4.dll
 0004:00002630       __imp_?contextMenuEvent@QComboBox@@MAEXPAVQContextMenuEvent@@@Z 0049e630     QtGui4:QtGui4.dll
 0004:00002634       __imp_?showEvent@QComboBox@@MAEXPAVQShowEvent@@@Z 0049e634     QtGui4:QtGui4.dll
 0004:00002638       __imp_?hideEvent@QComboBox@@MAEXPAVQHideEvent@@@Z 0049e638     QtGui4:QtGui4.dll
 0004:0000263c       __imp_?changeEvent@QComboBox@@MAEXPAVQEvent@@@Z 0049e63c     QtGui4:QtGui4.dll
 0004:00002640       __imp_?inputMethodEvent@QComboBox@@MAEXPAVQInputMethodEvent@@@Z 0049e640     QtGui4:QtGui4.dll
 0004:00002644       __imp_?inputMethodQuery@QComboBox@@MBE?AVQVariant@@W4InputMethodQuery@Qt@@@Z 0049e644     QtGui4:QtGui4.dll
 0004:00002648       __imp_?showPopup@QComboBox@@UAEXXZ 0049e648     QtGui4:QtGui4.dll
 0004:0000264c       __imp_?hidePopup@QComboBox@@UAEXXZ 0049e64c     QtGui4:QtGui4.dll
 0004:00002650       __imp_?event@QRadioButton@@MAE_NPAVQEvent@@@Z 0049e650     QtGui4:QtGui4.dll
 0004:00002654       __imp_?sizeHint@QRadioButton@@UBE?AVQSize@@XZ 0049e654     QtGui4:QtGui4.dll
 0004:00002658       __imp_?minimumSizeHint@QRadioButton@@UBE?AVQSize@@XZ 0049e658     QtGui4:QtGui4.dll
 0004:0000265c       __imp_?mouseMoveEvent@QRadioButton@@MAEXPAVQMouseEvent@@@Z 0049e65c     QtGui4:QtGui4.dll
 0004:00002660       __imp_?paintEvent@QRadioButton@@MAEXPAVQPaintEvent@@@Z 0049e660     QtGui4:QtGui4.dll
 0004:00002664       __imp_?hitButton@QRadioButton@@MBE_NABVQPoint@@@Z 0049e664     QtGui4:QtGui4.dll
 0004:00002668       __imp_?checkStateSet@QAbstractButton@@MAEXXZ 0049e668     QtGui4:QtGui4.dll
 0004:0000266c       __imp_?nextCheckState@QAbstractButton@@MAEXXZ 0049e66c     QtGui4:QtGui4.dll
 0004:00002670       __imp_?event@QPushButton@@MAE_NPAVQEvent@@@Z 0049e670     QtGui4:QtGui4.dll
 0004:00002674       __imp_?sizeHint@QPushButton@@UBE?AVQSize@@XZ 0049e674     QtGui4:QtGui4.dll
 0004:00002678       __imp_?minimumSizeHint@QPushButton@@UBE?AVQSize@@XZ 0049e678     QtGui4:QtGui4.dll
 0004:0000267c       __imp_?mouseMoveEvent@QAbstractButton@@MAEXPAVQMouseEvent@@@Z 0049e67c     QtGui4:QtGui4.dll
 0004:00002680       __imp_?keyPressEvent@QPushButton@@MAEXPAVQKeyEvent@@@Z 0049e680     QtGui4:QtGui4.dll
 0004:00002684       __imp_?focusInEvent@QPushButton@@MAEXPAVQFocusEvent@@@Z 0049e684     QtGui4:QtGui4.dll
 0004:00002688       __imp_?focusOutEvent@QPushButton@@MAEXPAVQFocusEvent@@@Z 0049e688     QtGui4:QtGui4.dll
 0004:0000268c       __imp_?hitButton@QAbstractButton@@MBE_NABVQPoint@@@Z 0049e68c     QtGui4:QtGui4.dll
 0004:00002690       __imp_?metaObject@QFrame@@UBEPBUQMetaObject@@XZ 0049e690     QtGui4:QtGui4.dll
 0004:00002694       __imp_?event@QFrame@@MAE_NPAVQEvent@@@Z 0049e694     QtGui4:QtGui4.dll
 0004:00002698       __imp_?sizeHint@QFrame@@UBE?AVQSize@@XZ 0049e698     QtGui4:QtGui4.dll
 0004:0000269c       __imp_?paintEvent@QFrame@@MAEXPAVQPaintEvent@@@Z 0049e69c     QtGui4:QtGui4.dll
 0004:000026a0       __imp_?insertItems@QComboBox@@QAEXHABVQStringList@@@Z 0049e6a0     QtGui4:QtGui4.dll
 0004:000026a4       __imp_?clear@QComboBox@@QAEXXZ 0049e6a4     QtGui4:QtGui4.dll
 0004:000026a8       __imp_?setText@QLabel@@QAEXABVQString@@@Z 0049e6a8     QtGui4:QtGui4.dll
 0004:000026ac       __imp_?setText@QAbstractButton@@QAEXABVQString@@@Z 0049e6ac     QtGui4:QtGui4.dll
 0004:000026b0       __imp_??1QCheckBox@@UAE@XZ 0049e6b0     QtGui4:QtGui4.dll
 0004:000026b4       __imp_??1QLabel@@UAE@XZ    0049e6b4     QtGui4:QtGui4.dll
 0004:000026b8       __imp_??1QFrame@@UAE@XZ    0049e6b8     QtGui4:QtGui4.dll
 0004:000026bc       __imp_?hide@QWidget@@QAEXXZ 0049e6bc     QtGui4:QtGui4.dll
 0004:000026c0       __imp_?addItems@QComboBox@@QAEXABVQStringList@@@Z 0049e6c0     QtGui4:QtGui4.dll
 0004:000026c4       __imp_?setVisible@QWidget@@UAEX_N@Z 0049e6c4     QtGui4:QtGui4.dll
 0004:000026c8       __imp_?currentIndex@QComboBox@@QBEHXZ 0049e6c8     QtGui4:QtGui4.dll
 0004:000026cc       __imp_?isChecked@QAbstractButton@@QBE_NXZ 0049e6cc     QtGui4:QtGui4.dll
 0004:000026d0       __imp_?currentText@QComboBox@@QBE?AVQString@@XZ 0049e6d0     QtGui4:QtGui4.dll
 0004:000026d4       __imp_?text@QLineEdit@@QBE?AVQString@@XZ 0049e6d4     QtGui4:QtGui4.dll
 0004:000026d8       __imp_?setCurrentIndex@QComboBox@@QAEXH@Z 0049e6d8     QtGui4:QtGui4.dll
 0004:000026dc       __imp_?setItemData@QComboBox@@QAEXHABVQVariant@@H@Z 0049e6dc     QtGui4:QtGui4.dll
 0004:000026e0       __imp_?count@QComboBox@@QBEHXZ 0049e6e0     QtGui4:QtGui4.dll
 0004:000026e4       __imp_?addItem@QComboBox@@QAEXABVQString@@ABVQVariant@@@Z 0049e6e4     QtGui4:QtGui4.dll
 0004:000026e8       __imp_??1QSpacerItem@@UAE@XZ 0049e6e8     QtGui4:QtGui4.dll
 0004:000026ec       __imp_?setSpacing@QListView@@QAEXH@Z 0049e6ec     QtGui4:QtGui4.dll
 0004:000026f0       __imp_?addItem@QGridLayout@@QAEXPAVQLayoutItem@@HHHHV?$QFlags@W4AlignmentFlag@Qt@@@@@Z 0049e6f0     QtGui4:QtGui4.dll
 0004:000026f4       __imp_?setStretch@QBoxLayout@@QAEXHH@Z 0049e6f4     QtGui4:QtGui4.dll
 0004:000026f8       __imp_?setFrameShadow@QFrame@@QAEXW4Shadow@1@@Z 0049e6f8     QtGui4:QtGui4.dll
 0004:000026fc       __imp_??0QListWidget@@QAE@PAVQWidget@@@Z 0049e6fc     QtGui4:QtGui4.dll
 0004:00002700       __imp_?setMargin@QLabel@@QAEXH@Z 0049e700     QtGui4:QtGui4.dll
 0004:00002704       __imp_?metaObject@QListWidget@@UBEPBUQMetaObject@@XZ 0049e704     QtGui4:QtGui4.dll
 0004:00002708       __imp_?qt_metacast@QListWidget@@UAEPAXPBD@Z 0049e708     QtGui4:QtGui4.dll
 0004:0000270c       __imp_?qt_metacall@QListWidget@@UAEHW4Call@QMetaObject@@HPAPAX@Z 0049e70c     QtGui4:QtGui4.dll
 0004:00002710       __imp_?event@QListWidget@@MAE_NPAVQEvent@@@Z 0049e710     QtGui4:QtGui4.dll
 0004:00002714       __imp_?timerEvent@QListView@@MAEXPAVQTimerEvent@@@Z 0049e714     QtGui4:QtGui4.dll
 0004:00002718       __imp_?sizeHint@QAbstractScrollArea@@UBE?AVQSize@@XZ 0049e718     QtGui4:QtGui4.dll
 0004:0000271c       __imp_?mousePressEvent@QAbstractItemView@@MAEXPAVQMouseEvent@@@Z 0049e71c     QtGui4:QtGui4.dll
 0004:00002720       __imp_?mouseReleaseEvent@QListView@@MAEXPAVQMouseEvent@@@Z 0049e720     QtGui4:QtGui4.dll
 0004:00002724       __imp_?mouseDoubleClickEvent@QAbstractItemView@@MAEXPAVQMouseEvent@@@Z 0049e724     QtGui4:QtGui4.dll
 0004:00002728       __imp_?mouseMoveEvent@QListView@@MAEXPAVQMouseEvent@@@Z 0049e728     QtGui4:QtGui4.dll
 0004:0000272c       __imp_?keyPressEvent@QAbstractItemView@@MAEXPAVQKeyEvent@@@Z 0049e72c     QtGui4:QtGui4.dll
 0004:00002730       __imp_?focusInEvent@QAbstractItemView@@MAEXPAVQFocusEvent@@@Z 0049e730     QtGui4:QtGui4.dll
 0004:00002734       __imp_?focusOutEvent@QAbstractItemView@@MAEXPAVQFocusEvent@@@Z 0049e734     QtGui4:QtGui4.dll
 0004:00002738       __imp_?paintEvent@QListView@@MAEXPAVQPaintEvent@@@Z 0049e738     QtGui4:QtGui4.dll
 0004:0000273c       __imp_?resizeEvent@QListView@@MAEXPAVQResizeEvent@@@Z 0049e73c     QtGui4:QtGui4.dll
 0004:00002740       __imp_?dragEnterEvent@QAbstractItemView@@MAEXPAVQDragEnterEvent@@@Z 0049e740     QtGui4:QtGui4.dll
 0004:00002744       __imp_?dragMoveEvent@QListView@@MAEXPAVQDragMoveEvent@@@Z 0049e744     QtGui4:QtGui4.dll
 0004:00002748       __imp_?dragLeaveEvent@QListView@@MAEXPAVQDragLeaveEvent@@@Z 0049e748     QtGui4:QtGui4.dll
 0004:0000274c       __imp_?dropEvent@QListWidget@@UAEXPAVQDropEvent@@@Z 0049e74c     QtGui4:QtGui4.dll
 0004:00002750       __imp_?inputMethodEvent@QAbstractItemView@@MAEXPAVQInputMethodEvent@@@Z 0049e750     QtGui4:QtGui4.dll
 0004:00002754       __imp_?inputMethodQuery@QAbstractItemView@@UBE?AVQVariant@@W4InputMethodQuery@Qt@@@Z 0049e754     QtGui4:QtGui4.dll
 0004:00002758       __imp_?focusNextPrevChild@QAbstractItemView@@MAE_N_N@Z 0049e758     QtGui4:QtGui4.dll
 0004:0000275c       __imp_?viewportEvent@QAbstractItemView@@MAE_NPAVQEvent@@@Z 0049e75c     QtGui4:QtGui4.dll
 0004:00002760       __imp_?scrollContentsBy@QListView@@MAEXHH@Z 0049e760     QtGui4:QtGui4.dll
 0004:00002764       __imp_?setModel@QListWidget@@EAEXPAVQAbstractItemModel@@@Z 0049e764     QtGui4:QtGui4.dll
 0004:00002768       __imp_?setSelectionModel@QAbstractItemView@@UAEXPAVQItemSelectionModel@@@Z 0049e768     QtGui4:QtGui4.dll
 0004:0000276c       __imp_?keyboardSearch@QAbstractItemView@@UAEXABVQString@@@Z 0049e76c     QtGui4:QtGui4.dll
 0004:00002770       __imp_?visualRect@QListView@@UBE?AVQRect@@ABVQModelIndex@@@Z 0049e770     QtGui4:QtGui4.dll
 0004:00002774       __imp_?scrollTo@QListView@@UAEXABVQModelIndex@@W4ScrollHint@QAbstractItemView@@@Z 0049e774     QtGui4:QtGui4.dll
 0004:00002778       __imp_?indexAt@QListView@@UBE?AVQModelIndex@@ABVQPoint@@@Z 0049e778     QtGui4:QtGui4.dll
 0004:0000277c       __imp_?sizeHintForRow@QAbstractItemView@@UBEHH@Z 0049e77c     QtGui4:QtGui4.dll
 0004:00002780       __imp_?sizeHintForColumn@QAbstractItemView@@UBEHH@Z 0049e780     QtGui4:QtGui4.dll
 0004:00002784       __imp_?reset@QListView@@UAEXXZ 0049e784     QtGui4:QtGui4.dll
 0004:00002788       __imp_?setRootIndex@QListView@@UAEXABVQModelIndex@@@Z 0049e788     QtGui4:QtGui4.dll
 0004:0000278c       __imp_?doItemsLayout@QListView@@UAEXXZ 0049e78c     QtGui4:QtGui4.dll
 0004:00002790       __imp_?selectAll@QAbstractItemView@@UAEXXZ 0049e790     QtGui4:QtGui4.dll
 0004:00002794       __imp_?edit@QAbstractItemView@@MAE_NABVQModelIndex@@W4EditTrigger@1@PAVQEvent@@@Z 0049e794     QtGui4:QtGui4.dll
 0004:00002798       __imp_?dataChanged@QListView@@MAEXABVQModelIndex@@0@Z 0049e798     QtGui4:QtGui4.dll
 0004:0000279c       __imp_?rowsInserted@QListView@@MAEXABVQModelIndex@@HH@Z 0049e79c     QtGui4:QtGui4.dll
 0004:000027a0       __imp_?rowsAboutToBeRemoved@QListView@@MAEXABVQModelIndex@@HH@Z 0049e7a0     QtGui4:QtGui4.dll
 0004:000027a4       __imp_?selectionChanged@QListView@@MAEXABVQItemSelection@@0@Z 0049e7a4     QtGui4:QtGui4.dll
 0004:000027a8       __imp_?currentChanged@QListView@@MAEXABVQModelIndex@@0@Z 0049e7a8     QtGui4:QtGui4.dll
 0004:000027ac       __imp_?updateEditorData@QAbstractItemView@@MAEXXZ 0049e7ac     QtGui4:QtGui4.dll
 0004:000027b0       __imp_?updateEditorGeometries@QAbstractItemView@@MAEXXZ 0049e7b0     QtGui4:QtGui4.dll
 0004:000027b4       __imp_?updateGeometries@QListView@@MAEXXZ 0049e7b4     QtGui4:QtGui4.dll
 0004:000027b8       __imp_?verticalScrollbarAction@QAbstractItemView@@MAEXH@Z 0049e7b8     QtGui4:QtGui4.dll
 0004:000027bc       __imp_?horizontalScrollbarAction@QAbstractItemView@@MAEXH@Z 0049e7bc     QtGui4:QtGui4.dll
 0004:000027c0       __imp_?verticalScrollbarValueChanged@QAbstractItemView@@MAEXH@Z 0049e7c0     QtGui4:QtGui4.dll
 0004:000027c4       __imp_?horizontalScrollbarValueChanged@QAbstractItemView@@MAEXH@Z 0049e7c4     QtGui4:QtGui4.dll
 0004:000027c8       __imp_?closeEditor@QAbstractItemView@@MAEXPAVQWidget@@W4EndEditHint@QAbstractItemDelegate@@@Z 0049e7c8     QtGui4:QtGui4.dll
 0004:000027cc       __imp_?commitData@QAbstractItemView@@MAEXPAVQWidget@@@Z 0049e7cc     QtGui4:QtGui4.dll
 0004:000027d0       __imp_?editorDestroyed@QAbstractItemView@@MAEXPAVQObject@@@Z 0049e7d0     QtGui4:QtGui4.dll
 0004:000027d4       __imp_?moveCursor@QListView@@MAE?AVQModelIndex@@W4CursorAction@QAbstractItemView@@V?$QFlags@W4KeyboardModifier@Qt@@@@@Z 0049e7d4     QtGui4:QtGui4.dll
 0004:000027d8       __imp_?horizontalOffset@QListView@@MBEHXZ 0049e7d8     QtGui4:QtGui4.dll
 0004:000027dc       __imp_?verticalOffset@QListView@@MBEHXZ 0049e7dc     QtGui4:QtGui4.dll
 0004:000027e0       __imp_?isIndexHidden@QListView@@MBE_NABVQModelIndex@@@Z 0049e7e0     QtGui4:QtGui4.dll
 0004:000027e4       __imp_?setSelection@QListView@@MAEXABVQRect@@V?$QFlags@W4SelectionFlag@QItemSelectionModel@@@@@Z 0049e7e4     QtGui4:QtGui4.dll
 0004:000027e8       __imp_?visualRegionForSelection@QListView@@MBE?AVQRegion@@ABVQItemSelection@@@Z 0049e7e8     QtGui4:QtGui4.dll
 0004:000027ec       __imp_?selectedIndexes@QListView@@MBE?AV?$QList@VQModelIndex@@@@XZ 0049e7ec     QtGui4:QtGui4.dll
 0004:000027f0       __imp_?selectionCommand@QAbstractItemView@@MBE?AV?$QFlags@W4SelectionFlag@QItemSelectionModel@@@@ABVQModelIndex@@PBVQEvent@@@Z 0049e7f0     QtGui4:QtGui4.dll
 0004:000027f4       __imp_?startDrag@QListView@@MAEXV?$QFlags@W4DropAction@Qt@@@@@Z 0049e7f4     QtGui4:QtGui4.dll
 0004:000027f8       __imp_?viewOptions@QListView@@MBE?AVQStyleOptionViewItem@@XZ 0049e7f8     QtGui4:QtGui4.dll
 0004:000027fc       __imp_?mimeTypes@QListWidget@@MBE?AVQStringList@@XZ 0049e7fc     QtGui4:QtGui4.dll
 0004:00002800       __imp_?mimeData@QListWidget@@MBEPAVQMimeData@@V?$QList@PAVQListWidgetItem@@@@@Z 0049e800     QtGui4:QtGui4.dll
 0004:00002804       __imp_?dropMimeData@QListWidget@@MAE_NHPBVQMimeData@@W4DropAction@Qt@@@Z 0049e804     QtGui4:QtGui4.dll
 0004:00002808       __imp_?supportedDropActions@QListWidget@@MBE?AV?$QFlags@W4DropAction@Qt@@@@XZ 0049e808     QtGui4:QtGui4.dll
 0004:0000280c       __imp_??1QListWidget@@UAE@XZ 0049e80c     QtGui4:QtGui4.dll
 0004:00002810       __imp_?setCheckable@QAbstractButton@@QAEX_N@Z 0049e810     QtGui4:QtGui4.dll
 0004:00002814       __imp_?setItemWidget@QListWidget@@QAEXPAVQListWidgetItem@@PAVQWidget@@@Z 0049e814     QtGui4:QtGui4.dll
 0004:00002818       __imp_?setSizeHint@QListWidgetItem@@QAEXABVQSize@@@Z 0049e818     QtGui4:QtGui4.dll
 0004:0000281c       __imp_?item@QListWidget@@QBEPAVQListWidgetItem@@H@Z 0049e81c     QtGui4:QtGui4.dll
 0004:00002820       __imp_?count@QListWidget@@QBEHXZ 0049e820     QtGui4:QtGui4.dll
 0004:00002824       __imp_?setToolTip@QWidget@@QAEXABVQString@@@Z 0049e824     QtGui4:QtGui4.dll
 0004:00002828       __imp_?addItem@QListWidget@@QAEXABVQString@@@Z 0049e828     QtGui4:QtGui4.dll
 0004:0000282c       __imp_??1QPushButton@@UAE@XZ 0049e82c     QtGui4:QtGui4.dll
 0004:00002830       __imp_??0QPushButton@@QAE@PAVQWidget@@@Z 0049e830     QtGui4:QtGui4.dll
 0004:00002834       __imp_?paintEvent@QPushButton@@MAEXPAVQPaintEvent@@@Z 0049e834     QtGui4:QtGui4.dll
 0004:00002838       __imp_?update@QWidget@@QAEXXZ 0049e838     QtGui4:QtGui4.dll
 0004:0000283c       __imp_?style@QWidget@@QBEPAVQStyle@@XZ 0049e83c     QtGui4:QtGui4.dll
 0004:00002840       __imp_??1QImage@@UAE@XZ    0049e840     QtGui4:QtGui4.dll
 0004:00002844       __imp_??1QPixmap@@UAE@XZ   0049e844     QtGui4:QtGui4.dll
 0004:00002848       __imp_?setPixmap@QLabel@@QAEXABVQPixmap@@@Z 0049e848     QtGui4:QtGui4.dll
 0004:0000284c       __imp_?fromImage@QPixmap@@SA?AV1@ABVQImage@@V?$QFlags@W4ImageConversionFlag@Qt@@@@@Z 0049e84c     QtGui4:QtGui4.dll
 0004:00002850       __imp_?scaled@QImage@@QBE?AV1@ABVQSize@@W4AspectRatioMode@Qt@@W4TransformationMode@4@@Z 0049e850     QtGui4:QtGui4.dll
 0004:00002854       __imp_??0QImage@@QAE@ABVQString@@PBD@Z 0049e854     QtGui4:QtGui4.dll
 0004:00002858       __imp_?size@QWidget@@QBE?AVQSize@@XZ 0049e858     QtGui4:QtGui4.dll
 0004:0000285c       __imp_?clear@QLabel@@QAEXXZ 0049e85c     QtGui4:QtGui4.dll
 0004:00002860       __imp_?clear@QListWidget@@QAEXXZ 0049e860     QtGui4:QtGui4.dll
 0004:00002864       __imp_?setLayout@QWidget@@QAEXPAVQLayout@@@Z 0049e864     QtGui4:QtGui4.dll
 0004:00002868       __imp_??0QHBoxLayout@@QAE@PAVQWidget@@@Z 0049e868     QtGui4:QtGui4.dll
 0004:0000286c       __imp_?metaObject@QPushButton@@UBEPBUQMetaObject@@XZ 0049e86c     QtGui4:QtGui4.dll
 0004:00002870       __imp_?setCurrentIndex@QStackedWidget@@QAEXH@Z 0049e870     QtGui4:QtGui4.dll
 0004:00002874       __imp_?addWidget@QStackedWidget@@QAEHPAVQWidget@@@Z 0049e874     QtGui4:QtGui4.dll
 0004:00002878       __imp_?setMaximum@QSpinBox@@QAEXH@Z 0049e878     QtGui4:QtGui4.dll
 0004:0000287c       __imp_?setOrientation@QAbstractSlider@@QAEXW4Orientation@Qt@@@Z 0049e87c     QtGui4:QtGui4.dll
 0004:00002880       __imp_?setPageStep@QAbstractSlider@@QAEXH@Z 0049e880     QtGui4:QtGui4.dll
 0004:00002884       __imp_?setMaximum@QAbstractSlider@@QAEXH@Z 0049e884     QtGui4:QtGui4.dll
 0004:00002888       __imp_?setLayoutDirection@QWidget@@QAEXW4LayoutDirection@Qt@@@Z 0049e888     QtGui4:QtGui4.dll
 0004:0000288c       __imp_??0QStackedWidget@@QAE@PAVQWidget@@@Z 0049e88c     QtGui4:QtGui4.dll
 0004:00002890       __imp_?setAutoFillBackground@QWidget@@QAEX_N@Z 0049e890     QtGui4:QtGui4.dll
 0004:00002894       __imp_?metaObject@QStackedWidget@@UBEPBUQMetaObject@@XZ 0049e894     QtGui4:QtGui4.dll
 0004:00002898       __imp_?qt_metacast@QStackedWidget@@UAEPAXPBD@Z 0049e898     QtGui4:QtGui4.dll
 0004:0000289c       __imp_?qt_metacall@QStackedWidget@@UAEHW4Call@QMetaObject@@HPAPAX@Z 0049e89c     QtGui4:QtGui4.dll
 0004:000028a0       __imp_?event@QStackedWidget@@MAE_NPAVQEvent@@@Z 0049e8a0     QtGui4:QtGui4.dll
 0004:000028a4       __imp_?event@QSlider@@UAE_NPAVQEvent@@@Z 0049e8a4     QtGui4:QtGui4.dll
 0004:000028a8       __imp_?timerEvent@QAbstractSlider@@MAEXPAVQTimerEvent@@@Z 0049e8a8     QtGui4:QtGui4.dll
 0004:000028ac       __imp_?sizeHint@QSlider@@UBE?AVQSize@@XZ 0049e8ac     QtGui4:QtGui4.dll
 0004:000028b0       __imp_?minimumSizeHint@QSlider@@UBE?AVQSize@@XZ 0049e8b0     QtGui4:QtGui4.dll
 0004:000028b4       __imp_?mouseMoveEvent@QSlider@@MAEXPAVQMouseEvent@@@Z 0049e8b4     QtGui4:QtGui4.dll
 0004:000028b8       __imp_?wheelEvent@QAbstractSlider@@MAEXPAVQWheelEvent@@@Z 0049e8b8     QtGui4:QtGui4.dll
 0004:000028bc       __imp_?keyPressEvent@QAbstractSlider@@MAEXPAVQKeyEvent@@@Z 0049e8bc     QtGui4:QtGui4.dll
 0004:000028c0       __imp_?paintEvent@QSlider@@MAEXPAVQPaintEvent@@@Z 0049e8c0     QtGui4:QtGui4.dll
 0004:000028c4       __imp_?changeEvent@QAbstractSlider@@MAEXPAVQEvent@@@Z 0049e8c4     QtGui4:QtGui4.dll
 0004:000028c8       __imp_?sliderChange@QAbstractSlider@@MAEXW4SliderChange@1@@Z 0049e8c8     QtGui4:QtGui4.dll
 0004:000028cc       __imp_??1QStackedWidget@@UAE@XZ 0049e8cc     QtGui4:QtGui4.dll
 0004:000028d0       __imp_?setValue@QAbstractSlider@@QAEXH@Z 0049e8d0     QtGui4:QtGui4.dll
 0004:000028d4       __imp_?setValue@QSpinBox@@QAEXH@Z 0049e8d4     QtGui4:QtGui4.dll
 0004:000028d8       __imp_?text@QAbstractSpinBox@@QBE?AVQString@@XZ 0049e8d8     QtGui4:QtGui4.dll
 0004:000028dc       __imp_?currentIndex@QStackedWidget@@QBEHXZ 0049e8dc     QtGui4:QtGui4.dll
 0004:000028e0       __imp_?mapToGlobal@QWidget@@QBE?AVQPoint@@ABV2@@Z 0049e8e0     QtGui4:QtGui4.dll
 0004:000028e4       __imp_?setAlignment@QLabel@@QAEXV?$QFlags@W4AlignmentFlag@Qt@@@@@Z 0049e8e4     QtGui4:QtGui4.dll
 0004:000028e8       __imp_?setSizeIncrement@QWidget@@QAEXABVQSize@@@Z 0049e8e8     QtGui4:QtGui4.dll
 0004:000028ec       __imp_?setFlow@QListView@@QAEXW4Flow@1@@Z 0049e8ec     QtGui4:QtGui4.dll
 0004:000028f0       __imp_?setAutoScrollMargin@QAbstractItemView@@QAEXH@Z 0049e8f0     QtGui4:QtGui4.dll
 0004:000028f4       __imp_?setLineWidth@QFrame@@QAEXH@Z 0049e8f4     QtGui4:QtGui4.dll
 0004:000028f8       __imp_?takeItem@QListWidget@@QAEPAVQListWidgetItem@@H@Z 0049e8f8     QtGui4:QtGui4.dll
 0004:000028fc       __imp_?itemWidget@QListWidget@@QBEPAVQWidget@@PAVQListWidgetItem@@@Z 0049e8fc     QtGui4:QtGui4.dll
 0004:00002900       __imp_??1QTextEdit@@UAE@XZ 0049e900     QtGui4:QtGui4.dll
 0004:00002904       __imp_??1QPrinter@@UAE@XZ  0049e904     QtGui4:QtGui4.dll
 0004:00002908       __imp_??1QPrintDialog@@UAE@XZ 0049e908     QtGui4:QtGui4.dll
 0004:0000290c       __imp_?print@QTextDocument@@QBEXPAVQPrinter@@@Z 0049e90c     QtGui4:QtGui4.dll
 0004:00002910       __imp_?document@QTextEdit@@QBEPAVQTextDocument@@XZ 0049e910     QtGui4:QtGui4.dll
 0004:00002914       __imp_?setOutputFileName@QPrinter@@QAEXABVQString@@@Z 0049e914     QtGui4:QtGui4.dll
 0004:00002918       __imp_?setOutputFormat@QPrinter@@QAEXW4OutputFormat@1@@Z 0049e918     QtGui4:QtGui4.dll
 0004:0000291c       __imp_??0QPrintDialog@@QAE@PAVQPrinter@@PAVQWidget@@@Z 0049e91c     QtGui4:QtGui4.dll
 0004:00002920       __imp_?setPaperSize@QPrinter@@QAEXABVQSizeF@@W4Unit@1@@Z 0049e920     QtGui4:QtGui4.dll
 0004:00002924       __imp_?setPageSize@QPrinter@@QAEXW4PageSize@1@@Z 0049e924     QtGui4:QtGui4.dll
 0004:00002928       __imp_?setFullPage@QPrinter@@QAEX_N@Z 0049e928     QtGui4:QtGui4.dll
 0004:0000292c       __imp_??0QPrinter@@QAE@W4PrinterMode@0@@Z 0049e92c     QtGui4:QtGui4.dll
 0004:00002930       __imp_?insertHtml@QTextEdit@@QAEXABVQString@@@Z 0049e930     QtGui4:QtGui4.dll
 0004:00002934       __imp_??0QTextEdit@@QAE@PAVQWidget@@@Z 0049e934     QtGui4:QtGui4.dll
 0004:00002938       __imp_?getSaveFileName@QFileDialog@@SA?AVQString@@PAVQWidget@@ABV2@11PAV2@V?$QFlags@W4Option@QFileDialog@@@@@Z 0049e938     QtGui4:QtGui4.dll
 0004:0000293c       __imp_??0QLabel@@QAE@ABVQString@@PAVQWidget@@V?$QFlags@W4WindowType@Qt@@@@@Z 0049e93c     QtGui4:QtGui4.dll
 0004:00002940       __imp_?setScaledContents@QLabel@@QAEX_N@Z 0049e940     QtGui4:QtGui4.dll
 0004:00002944       __imp_?setContextMenuPolicy@QWidget@@QAEXW4ContextMenuPolicy@Qt@@@Z 0049e944     QtGui4:QtGui4.dll
 0004:00002948       __imp_?setSizeConstraint@QLayout@@QAEXW4SizeConstraint@1@@Z 0049e948     QtGui4:QtGui4.dll
 0004:0000294c       __imp_??0QToolButton@@QAE@PAVQWidget@@@Z 0049e94c     QtGui4:QtGui4.dll
 0004:00002950       __imp_?metaObject@QToolButton@@UBEPBUQMetaObject@@XZ 0049e950     QtGui4:QtGui4.dll
 0004:00002954       __imp_?qt_metacast@QToolButton@@UAEPAXPBD@Z 0049e954     QtGui4:QtGui4.dll
 0004:00002958       __imp_?qt_metacall@QToolButton@@UAEHW4Call@QMetaObject@@HPAPAX@Z 0049e958     QtGui4:QtGui4.dll
 0004:0000295c       __imp_?event@QToolButton@@MAE_NPAVQEvent@@@Z 0049e95c     QtGui4:QtGui4.dll
 0004:00002960       __imp_?timerEvent@QToolButton@@MAEXPAVQTimerEvent@@@Z 0049e960     QtGui4:QtGui4.dll
 0004:00002964       __imp_?sizeHint@QToolButton@@UBE?AVQSize@@XZ 0049e964     QtGui4:QtGui4.dll
 0004:00002968       __imp_?minimumSizeHint@QToolButton@@UBE?AVQSize@@XZ 0049e968     QtGui4:QtGui4.dll
 0004:0000296c       __imp_?mousePressEvent@QToolButton@@MAEXPAVQMouseEvent@@@Z 0049e96c     QtGui4:QtGui4.dll
 0004:00002970       __imp_?mouseReleaseEvent@QToolButton@@MAEXPAVQMouseEvent@@@Z 0049e970     QtGui4:QtGui4.dll
 0004:00002974       __imp_?enterEvent@QToolButton@@MAEXPAVQEvent@@@Z 0049e974     QtGui4:QtGui4.dll
 0004:00002978       __imp_?leaveEvent@QToolButton@@MAEXPAVQEvent@@@Z 0049e978     QtGui4:QtGui4.dll
 0004:0000297c       __imp_?paintEvent@QToolButton@@MAEXPAVQPaintEvent@@@Z 0049e97c     QtGui4:QtGui4.dll
 0004:00002980       __imp_?actionEvent@QToolButton@@MAEXPAVQActionEvent@@@Z 0049e980     QtGui4:QtGui4.dll
 0004:00002984       __imp_?changeEvent@QToolButton@@MAEXPAVQEvent@@@Z 0049e984     QtGui4:QtGui4.dll
 0004:00002988       __imp_?hitButton@QToolButton@@MBE_NABVQPoint@@@Z 0049e988     QtGui4:QtGui4.dll
 0004:0000298c       __imp_?nextCheckState@QToolButton@@MAEXXZ 0049e98c     QtGui4:QtGui4.dll
 0004:00002990       __imp_??1QToolButton@@UAE@XZ 0049e990     QtGui4:QtGui4.dll
 0004:00002994       __imp_?setFocus@QWidget@@QAEXW4FocusReason@Qt@@@Z 0049e994     QtGui4:QtGui4.dll
 0004:00002998       __imp_??1QFontMetrics@@QAE@XZ 0049e998     QtGui4:QtGui4.dll
 0004:0000299c       __imp_?elidedText@QFontMetrics@@QBE?AVQString@@ABV2@W4TextElideMode@Qt@@HH@Z 0049e99c     QtGui4:QtGui4.dll
 0004:000029a0       __imp_?width@QFontMetrics@@QBEHABVQString@@H@Z 0049e9a0     QtGui4:QtGui4.dll
 0004:000029a4       __imp_??0QFontMetrics@@QAE@ABVQFont@@@Z 0049e9a4     QtGui4:QtGui4.dll
 0004:000029a8       __imp_??0QRadioButton@@QAE@PAVQWidget@@@Z 0049e9a8     QtGui4:QtGui4.dll
 0004:000029ac       __imp_??1QRadioButton@@UAE@XZ 0049e9ac     QtGui4:QtGui4.dll
 0004:000029b0       __imp_?eventFilter@QDialog@@MAE_NPAVQObject@@PAVQEvent@@@Z 0049e9b0     QtGui4:QtGui4.dll
 0004:000029b4       __imp_?setVisible@QDialog@@UAEX_N@Z 0049e9b4     QtGui4:QtGui4.dll
 0004:000029b8       __imp_?sizeHint@QDialog@@UBE?AVQSize@@XZ 0049e9b8     QtGui4:QtGui4.dll
 0004:000029bc       __imp_?minimumSizeHint@QDialog@@UBE?AVQSize@@XZ 0049e9bc     QtGui4:QtGui4.dll
 0004:000029c0       __imp_?keyPressEvent@QDialog@@MAEXPAVQKeyEvent@@@Z 0049e9c0     QtGui4:QtGui4.dll
 0004:000029c4       __imp_?resizeEvent@QDialog@@MAEXPAVQResizeEvent@@@Z 0049e9c4     QtGui4:QtGui4.dll
 0004:000029c8       __imp_?closeEvent@QDialog@@MAEXPAVQCloseEvent@@@Z 0049e9c8     QtGui4:QtGui4.dll
 0004:000029cc       __imp_?contextMenuEvent@QDialog@@MAEXPAVQContextMenuEvent@@@Z 0049e9cc     QtGui4:QtGui4.dll
 0004:000029d0       __imp_?showEvent@QDialog@@MAEXPAVQShowEvent@@@Z 0049e9d0     QtGui4:QtGui4.dll
 0004:000029d4       __imp_?done@QDialog@@UAEXH@Z 0049e9d4     QtGui4:QtGui4.dll
 0004:000029d8       __imp_?accept@QDialog@@UAEXXZ 0049e9d8     QtGui4:QtGui4.dll
 0004:000029dc       __imp_?reject@QDialog@@UAEXXZ 0049e9dc     QtGui4:QtGui4.dll
 0004:000029e0       __imp_?setWordWrap@QLabel@@QAEX_N@Z 0049e9e0     QtGui4:QtGui4.dll
 0004:000029e4       __imp_??0QImage@@QAE@PBD0@Z 0049e9e4     QtGui4:QtGui4.dll
 0004:000029e8       __imp_??0QPixmap@@QAE@XZ   0049e9e8     QtGui4:QtGui4.dll
 0004:000029ec       __imp_?getOpenFileName@QFileDialog@@SA?AVQString@@PAVQWidget@@ABV2@11PAV2@V?$QFlags@W4Option@QFileDialog@@@@@Z 0049e9ec     QtGui4:QtGui4.dll
 0004:000029f0       __imp_??1QDialog@@UAE@XZ   0049e9f0     QtGui4:QtGui4.dll
 0004:000029f4       __imp_??0QDialog@@QAE@PAVQWidget@@V?$QFlags@W4WindowType@Qt@@@@@Z 0049e9f4     QtGui4:QtGui4.dll
 0004:000029f8       __imp_?scaled@QImage@@QBE?AV1@HHW4AspectRatioMode@Qt@@W4TransformationMode@3@@Z 0049e9f8     QtGui4:QtGui4.dll
 0004:000029fc       __imp_?move@QWidget@@QAEXABVQPoint@@@Z 0049e9fc     QtGui4:QtGui4.dll
 0004:00002a00       __imp_?setEnabled@QWidget@@QAEX_N@Z 0049ea00     QtGui4:QtGui4.dll
 0004:00002a04       __imp_?setIcon@QAbstractButton@@QAEXABVQIcon@@@Z 0049ea04     QtGui4:QtGui4.dll
 0004:00002a08       __imp_?addSpacerItem@QBoxLayout@@QAEXPAVQSpacerItem@@@Z 0049ea08     QtGui4:QtGui4.dll
 0004:00002a0c       __imp_?addStretch@QBoxLayout@@QAEXH@Z 0049ea0c     QtGui4:QtGui4.dll
 0004:00002a10       __imp_??1QKeySequence@@QAE@XZ 0049ea10     QtGui4:QtGui4.dll
 0004:00002a14       __imp_?setShortcut@QAbstractButton@@QAEXABVQKeySequence@@@Z 0049ea14     QtGui4:QtGui4.dll
 0004:00002a18       __imp_??0QKeySequence@@QAE@HHHH@Z 0049ea18     QtGui4:QtGui4.dll
 0004:00002a1c       __imp_?setFixedHeight@QWidget@@QAEXH@Z 0049ea1c     QtGui4:QtGui4.dll
 0004:00002a20       __imp_?metaObject@QBoxLayout@@UBEPBUQMetaObject@@XZ 0049ea20     QtGui4:QtGui4.dll
 0004:00002a24       __imp_?qt_metacast@QBoxLayout@@UAEPAXPBD@Z 0049ea24     QtGui4:QtGui4.dll
 0004:00002a28       __imp_?qt_metacall@QBoxLayout@@UAEHW4Call@QMetaObject@@HPAPAX@Z 0049ea28     QtGui4:QtGui4.dll
 0004:00002a2c       __imp_?sizeHint@QWidgetItem@@UBE?AVQSize@@XZ 0049ea2c     QtGui4:QtGui4.dll
 0004:00002a30       __imp_?minimumSize@QWidgetItem@@UBE?AVQSize@@XZ 0049ea30     QtGui4:QtGui4.dll
 0004:00002a34       __imp_?maximumSize@QWidgetItem@@UBE?AVQSize@@XZ 0049ea34     QtGui4:QtGui4.dll
 0004:00002a38       __imp_?expandingDirections@QWidgetItem@@UBE?AV?$QFlags@W4Orientation@Qt@@@@XZ 0049ea38     QtGui4:QtGui4.dll
 0004:00002a3c       __imp_?geometry@QWidgetItem@@UBE?AVQRect@@XZ 0049ea3c     QtGui4:QtGui4.dll
 0004:00002a40       __imp_?isEmpty@QWidgetItem@@UBE_NXZ 0049ea40     QtGui4:QtGui4.dll
 0004:00002a44       __imp_?hasHeightForWidth@QWidgetItem@@UBE_NXZ 0049ea44     QtGui4:QtGui4.dll
 0004:00002a48       __imp_?heightForWidth@QWidgetItem@@UBEHH@Z 0049ea48     QtGui4:QtGui4.dll
 0004:00002a4c       __imp_?widget@QWidgetItem@@UAEPAVQWidget@@XZ 0049ea4c     QtGui4:QtGui4.dll
 0004:00002a50       __imp_?showMinimized@QWidget@@QAEXXZ 0049ea50     QtGui4:QtGui4.dll
 0004:00002a54       __imp_?button@QMouseEvent@@QBE?AW4MouseButton@Qt@@XZ 0049ea54     QtGui4:QtGui4.dll
 0004:00002a58       __imp_??1QMenu@@UAE@XZ     0049ea58     QtGui4:QtGui4.dll
 0004:00002a5c       __imp_??0QMenu@@QAE@ABVQString@@PAVQWidget@@@Z 0049ea5c     QtGui4:QtGui4.dll
 0004:00002a60       __imp_?timerEvent@QMenu@@MAEXPAVQTimerEvent@@@Z 0049ea60     QtGui4:QtGui4.dll
 0004:00002a64       __imp_?sizeHint@QMenu@@UBE?AVQSize@@XZ 0049ea64     QtGui4:QtGui4.dll
 0004:00002a68       __imp_?mousePressEvent@QMenu@@MAEXPAVQMouseEvent@@@Z 0049ea68     QtGui4:QtGui4.dll
 0004:00002a6c       __imp_?mouseReleaseEvent@QMenu@@MAEXPAVQMouseEvent@@@Z 0049ea6c     QtGui4:QtGui4.dll
 0004:00002a70       __imp_?mouseMoveEvent@QMenu@@MAEXPAVQMouseEvent@@@Z 0049ea70     QtGui4:QtGui4.dll
 0004:00002a74       __imp_?wheelEvent@QMenu@@MAEXPAVQWheelEvent@@@Z 0049ea74     QtGui4:QtGui4.dll
 0004:00002a78       __imp_?keyPressEvent@QMenu@@MAEXPAVQKeyEvent@@@Z 0049ea78     QtGui4:QtGui4.dll
 0004:00002a7c       __imp_?enterEvent@QMenu@@MAEXPAVQEvent@@@Z 0049ea7c     QtGui4:QtGui4.dll
 0004:00002a80       __imp_?leaveEvent@QMenu@@MAEXPAVQEvent@@@Z 0049ea80     QtGui4:QtGui4.dll
 0004:00002a84       __imp_?paintEvent@QMenu@@MAEXPAVQPaintEvent@@@Z 0049ea84     QtGui4:QtGui4.dll
 0004:00002a88       __imp_?actionEvent@QMenu@@MAEXPAVQActionEvent@@@Z 0049ea88     QtGui4:QtGui4.dll
 0004:00002a8c       __imp_?hideEvent@QMenu@@MAEXPAVQHideEvent@@@Z 0049ea8c     QtGui4:QtGui4.dll
 0004:00002a90       __imp_?changeEvent@QMenu@@MAEXPAVQEvent@@@Z 0049ea90     QtGui4:QtGui4.dll
 0004:00002a94       __imp_?focusNextPrevChild@QMenu@@MAE_N_N@Z 0049ea94     QtGui4:QtGui4.dll
 0004:00002a98       __imp_??0QMenu@@QAE@PAVQWidget@@@Z 0049ea98     QtGui4:QtGui4.dll
 0004:00002a9c       __imp_?event@QMenu@@MAE_NPAVQEvent@@@Z 0049ea9c     QtGui4:QtGui4.dll
 0004:00002aa0       __imp_?winId@QWidget@@QBEPAUHWND__@@XZ 0049eaa0     QtGui4:QtGui4.dll
 0004:00002aa4       __imp_?addMenu@QMenu@@QAEPAVQAction@@PAV1@@Z 0049eaa4     QtGui4:QtGui4.dll
 0004:00002aa8       __imp_?menuAction@QMenu@@QBEPAVQAction@@XZ 0049eaa8     QtGui4:QtGui4.dll
 0004:00002aac       __imp_?setIcon@QMenu@@QAEXABVQIcon@@@Z 0049eaac     QtGui4:QtGui4.dll
 0004:00002ab0       __imp_??1QPainter@@QAE@XZ  0049eab0     QtGui4:QtGui4.dll
 0004:00002ab4       __imp_??0QPixmap@@QAE@ABV0@@Z 0049eab4     QtGui4:QtGui4.dll
 0004:00002ab8       __imp_?end@QPainter@@QAE_NXZ 0049eab8     QtGui4:QtGui4.dll
 0004:00002abc       __imp_?drawPixmap@QPainter@@QAEXABVQRect@@ABVQPixmap@@0@Z 0049eabc     QtGui4:QtGui4.dll
 0004:00002ac0       __imp_?height@QPixmap@@QBEHXZ 0049eac0     QtGui4:QtGui4.dll
 0004:00002ac4       __imp_?width@QPixmap@@QBEHXZ 0049eac4     QtGui4:QtGui4.dll
 0004:00002ac8       __imp_?begin@QPainter@@QAE_NPAVQPaintDevice@@@Z 0049eac8     QtGui4:QtGui4.dll
 0004:00002acc       __imp_??0QPainter@@QAE@XZ  0049eacc     QtGui4:QtGui4.dll
 0004:00002ad0       __imp_?fill@QPixmap@@QAEXABVQColor@@@Z 0049ead0     QtGui4:QtGui4.dll
 0004:00002ad4       __imp_??0QColor@@QAE@HHHH@Z 0049ead4     QtGui4:QtGui4.dll
 0004:00002ad8       __imp_??0QPixmap@@QAE@ABVQSize@@@Z 0049ead8     QtGui4:QtGui4.dll
 0004:00002adc       __imp_??1QProxyStyle@@UAE@XZ 0049eadc     QtGui4:QtGui4.dll
 0004:00002ae0       __imp_?load@QPixmap@@QAE_NABVQString@@PBDV?$QFlags@W4ImageConversionFlag@Qt@@@@@Z 0049eae0     QtGui4:QtGui4.dll
 0004:00002ae4       __imp_??0QProxyStyle@@QAE@PAVQStyle@@@Z 0049eae4     QtGui4:QtGui4.dll
 0004:00002ae8       __imp_?event@QProxyStyle@@MAE_NPAVQEvent@@@Z 0049eae8     QtGui4:QtGui4.dll
 0004:00002aec       __imp_?polish@QProxyStyle@@UAEXAAVQPalette@@@Z 0049eaec     QtGui4:QtGui4.dll
 0004:00002af0       __imp_?polish@QProxyStyle@@UAEXPAVQApplication@@@Z 0049eaf0     QtGui4:QtGui4.dll
 0004:00002af4       __imp_?polish@QProxyStyle@@UAEXPAVQWidget@@@Z 0049eaf4     QtGui4:QtGui4.dll
 0004:00002af8       __imp_?unpolish@QProxyStyle@@UAEXPAVQApplication@@@Z 0049eaf8     QtGui4:QtGui4.dll
 0004:00002afc       __imp_?unpolish@QProxyStyle@@UAEXPAVQWidget@@@Z 0049eafc     QtGui4:QtGui4.dll
 0004:00002b00       __imp_?itemTextRect@QProxyStyle@@UBE?AVQRect@@ABVQFontMetrics@@ABV2@H_NABVQString@@@Z 0049eb00     QtGui4:QtGui4.dll
 0004:00002b04       __imp_?itemPixmapRect@QProxyStyle@@UBE?AVQRect@@ABV2@HABVQPixmap@@@Z 0049eb04     QtGui4:QtGui4.dll
 0004:00002b08       __imp_?drawItemText@QProxyStyle@@UBEXPAVQPainter@@ABVQRect@@HABVQPalette@@_NABVQString@@W4ColorRole@4@@Z 0049eb08     QtGui4:QtGui4.dll
 0004:00002b0c       __imp_?drawItemPixmap@QProxyStyle@@UBEXPAVQPainter@@ABVQRect@@HABVQPixmap@@@Z 0049eb0c     QtGui4:QtGui4.dll
 0004:00002b10       __imp_?standardPalette@QProxyStyle@@UBE?AVQPalette@@XZ 0049eb10     QtGui4:QtGui4.dll
 0004:00002b14       __imp_?subElementRect@QProxyStyle@@UBE?AVQRect@@W4SubElement@QStyle@@PBVQStyleOption@@PBVQWidget@@@Z 0049eb14     QtGui4:QtGui4.dll
 0004:00002b18       __imp_?drawComplexControl@QProxyStyle@@UBEXW4ComplexControl@QStyle@@PBVQStyleOptionComplex@@PAVQPainter@@PBVQWidget@@@Z 0049eb18     QtGui4:QtGui4.dll
 0004:00002b1c       __imp_?hitTestComplexControl@QProxyStyle@@UBE?AW4SubControl@QStyle@@W4ComplexControl@3@PBVQStyleOptionComplex@@ABVQPoint@@PBVQWidget@@@Z 0049eb1c     QtGui4:QtGui4.dll
 0004:00002b20       __imp_?subControlRect@QProxyStyle@@UBE?AVQRect@@W4ComplexControl@QStyle@@PBVQStyleOptionComplex@@W4SubControl@4@PBVQWidget@@@Z 0049eb20     QtGui4:QtGui4.dll
 0004:00002b24       __imp_?sizeFromContents@QProxyStyle@@UBE?AVQSize@@W4ContentsType@QStyle@@PBVQStyleOption@@ABV2@PBVQWidget@@@Z 0049eb24     QtGui4:QtGui4.dll
 0004:00002b28       __imp_?styleHint@QProxyStyle@@UBEHW4StyleHint@QStyle@@PBVQStyleOption@@PBVQWidget@@PAVQStyleHintReturn@@@Z 0049eb28     QtGui4:QtGui4.dll
 0004:00002b2c       __imp_?standardPixmap@QProxyStyle@@UBE?AVQPixmap@@W4StandardPixmap@QStyle@@PBVQStyleOption@@PBVQWidget@@@Z 0049eb2c     QtGui4:QtGui4.dll
 0004:00002b30       __imp_?generatedIconPixmap@QProxyStyle@@UBE?AVQPixmap@@W4Mode@QIcon@@ABV2@PBVQStyleOption@@@Z 0049eb30     QtGui4:QtGui4.dll
 0004:00002b34       __imp_?drawPixmap@QPainter@@QAEXABVQRect@@ABVQPixmap@@@Z 0049eb34     QtGui4:QtGui4.dll
 0004:00002b38       __imp_?drawPrimitive@QProxyStyle@@UBEXW4PrimitiveElement@QStyle@@PBVQStyleOption@@PAVQPainter@@PBVQWidget@@@Z 0049eb38     QtGui4:QtGui4.dll
 0004:00002b3c       __imp_?restore@QPainter@@QAEXXZ 0049eb3c     QtGui4:QtGui4.dll
 0004:00002b40       __imp_?isNull@QPixmap@@QBE_NXZ 0049eb40     QtGui4:QtGui4.dll
 0004:00002b44       __imp_?save@QPainter@@QAEXXZ 0049eb44     QtGui4:QtGui4.dll
 0004:00002b48       __imp_?pixelMetric@QProxyStyle@@UBEHW4PixelMetric@QStyle@@PBVQStyleOption@@PBVQWidget@@@Z 0049eb48     QtGui4:QtGui4.dll
 0004:00002b4c       __imp_?drawControl@QProxyStyle@@UBEXW4ControlElement@QStyle@@PBVQStyleOption@@PAVQPainter@@PBVQWidget@@@Z 0049eb4c     QtGui4:QtGui4.dll
 0004:00002b50       __imp_??1QStyleOptionMenuItem@@QAE@XZ 0049eb50     QtGui4:QtGui4.dll
 0004:00002b54       __imp_?setColor@QPalette@@QAEXW4ColorRole@1@ABVQColor@@@Z 0049eb54     QtGui4:QtGui4.dll
 0004:00002b58       __imp_??0QStyleOptionMenuItem@@QAE@ABV0@@Z 0049eb58     QtGui4:QtGui4.dll
 0004:00002b5c       __imp_?color@QBrush@@QBEABVQColor@@XZ 0049eb5c     QtGui4:QtGui4.dll
 0004:00002b60       __imp_?light@QPalette@@QBEABVQBrush@@XZ 0049eb60     QtGui4:QtGui4.dll
 0004:00002b64       __imp_?setBold@QFont@@QAEX_N@Z 0049eb64     QtGui4:QtGui4.dll
 0004:00002b68       __imp_??1QFontInfo@@QAE@XZ 0049eb68     QtGui4:QtGui4.dll
 0004:00002b6c       __imp_?setPointSizeF@QFont@@QAEXN@Z 0049eb6c     QtGui4:QtGui4.dll
 0004:00002b70       __imp_?pointSizeF@QFontInfo@@QBENXZ 0049eb70     QtGui4:QtGui4.dll
 0004:00002b74       __imp_??0QFontInfo@@QAE@ABVQFont@@@Z 0049eb74     QtGui4:QtGui4.dll
 0004:00002b78       __imp_??0QFont@@QAE@ABV0@@Z 0049eb78     QtGui4:QtGui4.dll
 0004:00002b7c       __imp_?drawText@QPainter@@QAEXABVQRect@@HABVQString@@PAV2@@Z 0049eb7c     QtGui4:QtGui4.dll
 0004:00002b80       __imp_??4QColor@@QAEAAV0@ABV0@@Z 0049eb80     QtGui4:QtGui4.dll
 0004:00002b84       __imp_??0QColor@@QAE@XZ    0049eb84     QtGui4:QtGui4.dll
 0004:00002b88       __imp_?drawPixmap@QPainter@@QAEXABVQPoint@@ABVQPixmap@@@Z 0049eb88     QtGui4:QtGui4.dll
 0004:00002b8c       __imp_??1QStyleOption@@QAE@XZ 0049eb8c     QtGui4:QtGui4.dll
 0004:00002b90       __imp_?setBrush@QPalette@@QAEXW4ColorRole@1@ABVQBrush@@@Z 0049eb90     QtGui4:QtGui4.dll
 0004:00002b94       __imp_??0QStyleOption@@QAE@ABV0@@Z 0049eb94     QtGui4:QtGui4.dll
 0004:00002b98       __imp_??4QPixmap@@QAEAAV0@ABV0@@Z 0049eb98     QtGui4:QtGui4.dll
 0004:00002b9c       __imp_?pixmap@QIcon@@QBE?AVQPixmap@@ABVQSize@@W4Mode@1@W4State@1@@Z 0049eb9c     QtGui4:QtGui4.dll
 0004:00002ba0       __imp_?iconSize@QComboBox@@QBE?AVQSize@@XZ 0049eba0     QtGui4:QtGui4.dll
 0004:00002ba4       __imp_??1QStyleOptionButton@@QAE@XZ 0049eba4     QtGui4:QtGui4.dll
 0004:00002ba8       __imp_??4QStyleOption@@QAEAAV0@ABV0@@Z 0049eba8     QtGui4:QtGui4.dll
 0004:00002bac       __imp_??0QStyleOptionButton@@QAE@XZ 0049ebac     QtGui4:QtGui4.dll
 0004:00002bb0       __imp_?isNull@QIcon@@QBE_NXZ 0049ebb0     QtGui4:QtGui4.dll
 0004:00002bb4       __imp_?visualRect@QStyle@@SA?AVQRect@@W4LayoutDirection@Qt@@ABV2@1@Z 0049ebb4     QtGui4:QtGui4.dll
 0004:00002bb8       __imp_?fillRect@QPainter@@QAEXABVQRect@@ABVQColor@@@Z 0049ebb8     QtGui4:QtGui4.dll
 0004:00002bbc       __imp_?drawLine@QPainter@@QAEXHHHH@Z 0049ebbc     QtGui4:QtGui4.dll
 0004:00002bc0       __imp_?proxy@QStyle@@QBEPBV1@XZ 0049ebc0     QtGui4:QtGui4.dll
 0004:00002bc4       __imp_?setFont@QPainter@@QAEXABVQFont@@@Z 0049ebc4     QtGui4:QtGui4.dll
 0004:00002bc8       __imp_?drawRect@QPainter@@QAEXABVQRect@@@Z 0049ebc8     QtGui4:QtGui4.dll
 0004:00002bcc       __imp_??1QBrush@@QAE@XZ    0049ebcc     QtGui4:QtGui4.dll
 0004:00002bd0       __imp_?setBrush@QPainter@@QAEXABVQBrush@@@Z 0049ebd0     QtGui4:QtGui4.dll
 0004:00002bd4       __imp_??0QBrush@@QAE@ABVQColor@@W4BrushStyle@Qt@@@Z 0049ebd4     QtGui4:QtGui4.dll
 0004:00002bd8       __imp_?setPen@QPainter@@QAEXABVQColor@@@Z 0049ebd8     QtGui4:QtGui4.dll
 0004:00002bdc       __imp_?setBlue@QColor@@QAEXH@Z 0049ebdc     QtGui4:QtGui4.dll
 0004:00002be0       __imp_?blue@QColor@@QBEHXZ 0049ebe0     QtGui4:QtGui4.dll
 0004:00002be4       __imp_?setGreen@QColor@@QAEXH@Z 0049ebe4     QtGui4:QtGui4.dll
 0004:00002be8       __imp_?green@QColor@@QBEHXZ 0049ebe8     QtGui4:QtGui4.dll
 0004:00002bec       __imp_?setRed@QColor@@QAEXH@Z 0049ebec     QtGui4:QtGui4.dll
 0004:00002bf0       __imp_?red@QColor@@QBEHXZ  0049ebf0     QtGui4:QtGui4.dll
 0004:00002bf4       __imp_??0QColor@@QAE@ABV0@@Z 0049ebf4     QtGui4:QtGui4.dll
 0004:00002bf8       __imp_?staticMetaObject@QComboBox@@2UQMetaObject@@B 0049ebf8     QtGui4:QtGui4.dll
 0004:00002bfc       __imp_??0QSpinBox@@QAE@PAVQWidget@@@Z 0049ebfc     QtGui4:QtGui4.dll
 0004:00002c00       __imp_?event@QSpinBox@@MAE_NPAVQEvent@@@Z 0049ec00     QtGui4:QtGui4.dll
 0004:00002c04       __imp_?timerEvent@QAbstractSpinBox@@MAEXPAVQTimerEvent@@@Z 0049ec04     QtGui4:QtGui4.dll
 0004:00002c08       __imp_?sizeHint@QAbstractSpinBox@@UBE?AVQSize@@XZ 0049ec08     QtGui4:QtGui4.dll
 0004:00002c0c       __imp_?minimumSizeHint@QAbstractSpinBox@@UBE?AVQSize@@XZ 0049ec0c     QtGui4:QtGui4.dll
 0004:00002c10       __imp_?mousePressEvent@QAbstractSpinBox@@MAEXPAVQMouseEvent@@@Z 0049ec10     QtGui4:QtGui4.dll
 0004:00002c14       __imp_?mouseReleaseEvent@QAbstractSpinBox@@MAEXPAVQMouseEvent@@@Z 0049ec14     QtGui4:QtGui4.dll
 0004:00002c18       __imp_?mouseMoveEvent@QAbstractSpinBox@@MAEXPAVQMouseEvent@@@Z 0049ec18     QtGui4:QtGui4.dll
 0004:00002c1c       __imp_?wheelEvent@QAbstractSpinBox@@MAEXPAVQWheelEvent@@@Z 0049ec1c     QtGui4:QtGui4.dll
 0004:00002c20       __imp_?keyPressEvent@QAbstractSpinBox@@MAEXPAVQKeyEvent@@@Z 0049ec20     QtGui4:QtGui4.dll
 0004:00002c24       __imp_?keyReleaseEvent@QAbstractSpinBox@@MAEXPAVQKeyEvent@@@Z 0049ec24     QtGui4:QtGui4.dll
 0004:00002c28       __imp_?focusInEvent@QAbstractSpinBox@@MAEXPAVQFocusEvent@@@Z 0049ec28     QtGui4:QtGui4.dll
 0004:00002c2c       __imp_?focusOutEvent@QAbstractSpinBox@@MAEXPAVQFocusEvent@@@Z 0049ec2c     QtGui4:QtGui4.dll
 0004:00002c30       __imp_?paintEvent@QAbstractSpinBox@@MAEXPAVQPaintEvent@@@Z 0049ec30     QtGui4:QtGui4.dll
 0004:00002c34       __imp_?resizeEvent@QAbstractSpinBox@@MAEXPAVQResizeEvent@@@Z 0049ec34     QtGui4:QtGui4.dll
 0004:00002c38       __imp_?closeEvent@QAbstractSpinBox@@MAEXPAVQCloseEvent@@@Z 0049ec38     QtGui4:QtGui4.dll
 0004:00002c3c       __imp_?contextMenuEvent@QAbstractSpinBox@@MAEXPAVQContextMenuEvent@@@Z 0049ec3c     QtGui4:QtGui4.dll
 0004:00002c40       __imp_?showEvent@QAbstractSpinBox@@MAEXPAVQShowEvent@@@Z 0049ec40     QtGui4:QtGui4.dll
 0004:00002c44       __imp_?hideEvent@QAbstractSpinBox@@MAEXPAVQHideEvent@@@Z 0049ec44     QtGui4:QtGui4.dll
 0004:00002c48       __imp_?changeEvent@QAbstractSpinBox@@MAEXPAVQEvent@@@Z 0049ec48     QtGui4:QtGui4.dll
 0004:00002c4c       __imp_?inputMethodQuery@QAbstractSpinBox@@UBE?AVQVariant@@W4InputMethodQuery@Qt@@@Z 0049ec4c     QtGui4:QtGui4.dll
 0004:00002c50       __imp_?validate@QSpinBox@@MBE?AW4State@QValidator@@AAVQString@@AAH@Z 0049ec50     QtGui4:QtGui4.dll
 0004:00002c54       __imp_?fixup@QSpinBox@@MBEXAAVQString@@@Z 0049ec54     QtGui4:QtGui4.dll
 0004:00002c58       __imp_?stepBy@QAbstractSpinBox@@UAEXH@Z 0049ec58     QtGui4:QtGui4.dll
 0004:00002c5c       __imp_?clear@QAbstractSpinBox@@UAEXXZ 0049ec5c     QtGui4:QtGui4.dll
 0004:00002c60       __imp_?stepEnabled@QAbstractSpinBox@@MBE?AV?$QFlags@W4StepEnabledFlag@QAbstractSpinBox@@@@XZ 0049ec60     QtGui4:QtGui4.dll
 0004:00002c64       __imp_?valueFromText@QSpinBox@@MBEHABVQString@@@Z 0049ec64     QtGui4:QtGui4.dll
 0004:00002c68       __imp_?textFromValue@QSpinBox@@MBE?AVQString@@H@Z 0049ec68     QtGui4:QtGui4.dll
 0004:00002c6c       __imp_??1QSpinBox@@UAE@XZ  0049ec6c     QtGui4:QtGui4.dll
 0004:00002c70       __imp_?setExpanding@QTabBar@@QAEX_N@Z 0049ec70     QtGui4:QtGui4.dll
 0004:00002c74       __imp_?tabBar@QTabWidget@@IBEPAVQTabBar@@XZ 0049ec74     QtGui4:QtGui4.dll
 0004:00002c78       __imp_??1QTabWidget@@UAE@XZ 0049ec78     QtGui4:QtGui4.dll
 0004:00002c7c       __imp_??0QTabWidget@@QAE@PAVQWidget@@@Z 0049ec7c     QtGui4:QtGui4.dll
 0004:00002c80       __imp_?event@QTabWidget@@MAE_NPAVQEvent@@@Z 0049ec80     QtGui4:QtGui4.dll
 0004:00002c84       __imp_?sizeHint@QTabWidget@@UBE?AVQSize@@XZ 0049ec84     QtGui4:QtGui4.dll
 0004:00002c88       __imp_?minimumSizeHint@QTabWidget@@UBE?AVQSize@@XZ 0049ec88     QtGui4:QtGui4.dll
 0004:00002c8c       __imp_?heightForWidth@QTabWidget@@UBEHH@Z 0049ec8c     QtGui4:QtGui4.dll
 0004:00002c90       __imp_?keyPressEvent@QTabWidget@@MAEXPAVQKeyEvent@@@Z 0049ec90     QtGui4:QtGui4.dll
 0004:00002c94       __imp_?paintEvent@QTabWidget@@MAEXPAVQPaintEvent@@@Z 0049ec94     QtGui4:QtGui4.dll
 0004:00002c98       __imp_?showEvent@QTabWidget@@MAEXPAVQShowEvent@@@Z 0049ec98     QtGui4:QtGui4.dll
 0004:00002c9c       __imp_?changeEvent@QTabWidget@@MAEXPAVQEvent@@@Z 0049ec9c     QtGui4:QtGui4.dll
 0004:00002ca0       __imp_?tabInserted@QTabWidget@@MAEXH@Z 0049eca0     QtGui4:QtGui4.dll
 0004:00002ca4       __imp_?tabRemoved@QTabWidget@@MAEXH@Z 0049eca4     QtGui4:QtGui4.dll
 0004:00002ca8       __imp_?resizeEvent@QTabWidget@@MAEXPAVQResizeEvent@@@Z 0049eca8     QtGui4:QtGui4.dll
 0004:00002cac       __imp_??1QWidgetAction@@UAE@XZ 0049ecac     QtGui4:QtGui4.dll
 0004:00002cb0       __imp_?setDefaultWidget@QWidgetAction@@QAEXPAVQWidget@@@Z 0049ecb0     QtGui4:QtGui4.dll
 0004:00002cb4       __imp_??0QWidgetAction@@QAE@PAVQObject@@@Z 0049ecb4     QtGui4:QtGui4.dll
 0004:00002cb8       __imp_?setFont@QWidget@@QAEXABVQFont@@@Z 0049ecb8     QtGui4:QtGui4.dll
 0004:00002cbc       __imp_?isVisible@QWidget@@QBE_NXZ 0049ecbc     QtGui4:QtGui4.dll
 0004:00002cc0       __imp_?fill@QImage@@QAEXI@Z 0049ecc0     QtGui4:QtGui4.dll
 0004:00002cc4       __imp_?rgb@QColor@@QBEIXZ  0049ecc4     QtGui4:QtGui4.dll
 0004:00002cc8       __imp_??0QColor@@QAE@W4GlobalColor@Qt@@@Z 0049ecc8     QtGui4:QtGui4.dll
 0004:00002ccc       __imp_??0QImage@@QAE@HHW4Format@0@@Z 0049eccc     QtGui4:QtGui4.dll
 0004:00002cd0       __imp_?setIconSize@QAbstractButton@@QAEXABVQSize@@@Z 0049ecd0     QtGui4:QtGui4.dll
 0004:00002cd4       __imp_?setMargin@QLayout@@QAEXH@Z 0049ecd4     QtGui4:QtGui4.dll
 0004:00002cd8       __imp_??0QPainter@@QAE@PAVQPaintDevice@@@Z 0049ecd8     QtGui4:QtGui4.dll
 0004:00002cdc       __imp_?init@QStyleOption@@QAEXPBVQWidget@@@Z 0049ecdc     QtGui4:QtGui4.dll
 0004:00002ce0       __imp_??0QStyleOption@@QAE@HH@Z 0049ece0     QtGui4:QtGui4.dll
 0004:00002ce4       __imp_?showMaximized@QWidget@@QAEXXZ 0049ece4     QtGui4:QtGui4.dll
 0004:00002ce8       __imp_?showNormal@QWidget@@QAEXXZ 0049ece8     QtGui4:QtGui4.dll
 0004:00002cec       __imp_?isMaximized@QWidget@@QBE_NXZ 0049ecec     QtGui4:QtGui4.dll
 0004:00002cf0       __imp_??1QPolygon@@QAE@XZ  0049ecf0     QtGui4:QtGui4.dll
 0004:00002cf4       __imp_??0QPolygon@@QAE@XZ  0049ecf4     QtGui4:QtGui4.dll
 0004:00002cf8       __imp_?pos@QMouseEvent@@QBEABVQPoint@@XZ 0049ecf8     QtGui4:QtGui4.dll
 0004:00002cfc       __imp_?drawPolyline@QPainter@@QAEXABVQPolygon@@@Z 0049ecfc     QtGui4:QtGui4.dll
 0004:00002d00       __imp_??1QPen@@QAE@XZ      0049ed00     QtGui4:QtGui4.dll
 0004:00002d04       __imp_?setPen@QPainter@@QAEXABVQPen@@@Z 0049ed04     QtGui4:QtGui4.dll
 0004:00002d08       __imp_??0QPen@@QAE@ABVQColor@@@Z 0049ed08     QtGui4:QtGui4.dll
 0004:00002d0c       __imp_??1QCursor@@QAE@XZ   0049ed0c     QtGui4:QtGui4.dll
 0004:00002d10       __imp_?setCursor@QWidget@@QAEXABVQCursor@@@Z 0049ed10     QtGui4:QtGui4.dll
 0004:00002d14       __imp_??0QCursor@@QAE@ABVQPixmap@@HH@Z 0049ed14     QtGui4:QtGui4.dll
 0004:00002d18       __imp_??0QPixmap@@QAE@ABVQString@@PBDV?$QFlags@W4ImageConversionFlag@Qt@@@@@Z 0049ed18     QtGui4:QtGui4.dll
 0004:00002d1c       __imp_??0QCursor@@QAE@W4CursorShape@Qt@@@Z 0049ed1c     QtGui4:QtGui4.dll
 0004:00002d20       __imp_?currentColor@QColorDialog@@QBE?AVQColor@@XZ 0049ed20     QtGui4:QtGui4.dll
 0004:00002d24       __imp_?setCurrentColor@QColorDialog@@QAEXABVQColor@@@Z 0049ed24     QtGui4:QtGui4.dll
 0004:00002d28       __imp_??0QColorDialog@@QAE@PAVQWidget@@@Z 0049ed28     QtGui4:QtGui4.dll
 0004:00002d2c       __imp_?isEnabled@QWidget@@QBE_NXZ 0049ed2c     QtGui4:QtGui4.dll
 0004:00002d30       __imp_?metaObject@QColorDialog@@UBEPBUQMetaObject@@XZ 0049ed30     QtGui4:QtGui4.dll
 0004:00002d34       __imp_?qt_metacast@QColorDialog@@UAEPAXPBD@Z 0049ed34     QtGui4:QtGui4.dll
 0004:00002d38       __imp_?qt_metacall@QColorDialog@@UAEHW4Call@QMetaObject@@HPAPAX@Z 0049ed38     QtGui4:QtGui4.dll
 0004:00002d3c       __imp_?setVisible@QColorDialog@@UAEX_N@Z 0049ed3c     QtGui4:QtGui4.dll
 0004:00002d40       __imp_?changeEvent@QColorDialog@@MAEXPAVQEvent@@@Z 0049ed40     QtGui4:QtGui4.dll
 0004:00002d44       __imp_?done@QColorDialog@@MAEXH@Z 0049ed44     QtGui4:QtGui4.dll
 0004:00002d48       __imp_??1QColorDialog@@UAE@XZ 0049ed48     QtGui4:QtGui4.dll
 0004:00002d4c       __imp_??0QPolygon@@QAE@ABV0@@Z 0049ed4c     QtGui4:QtGui4.dll
 0004:00002d50       __imp_??0QApplication@@QAE@AAHPAPAD_NH@Z 0049ed50     QtGui4:QtGui4.dll
 0004:00002d54       __imp_??0QApplication@@QAE@AAHPAPADH@Z 0049ed54     QtGui4:QtGui4.dll
 0004:00002d58       __imp_?event@QApplication@@MAE_NPAVQEvent@@@Z 0049ed58     QtGui4:QtGui4.dll
 0004:00002d5c       __imp_?file@QFileOpenEvent@@QBE?AVQString@@XZ 0049ed5c     QtGui4:QtGui4.dll
 0004:00002d60       __imp_?activateWindow@QWidget@@QAEXXZ 0049ed60     QtGui4:QtGui4.dll
 0004:00002d64       __imp_?setWindowState@QWidget@@QAEXV?$QFlags@W4WindowState@Qt@@@@@Z 0049ed64     QtGui4:QtGui4.dll
 0004:00002d68       __imp_?windowState@QWidget@@QBE?AV?$QFlags@W4WindowState@Qt@@@@XZ 0049ed68     QtGui4:QtGui4.dll
 0004:00002d6c       __imp_?addItem@QListWidget@@QAEXPAVQListWidgetItem@@@Z 0049ed6c     QtGui4:QtGui4.dll
 0004:00002d70       __imp_?qt_metacast@QWidget@@UAEPAXPBD@Z 0049ed70     QtGui4:QtGui4.dll
 0004:00002d74       __imp_?qt_metacall@QWidget@@UAEHW4Call@QMetaObject@@HPAPAX@Z 0049ed74     QtGui4:QtGui4.dll
 0004:00002d78       __imp_?staticMetaObject@QWidget@@2UQMetaObject@@B 0049ed78     QtGui4:QtGui4.dll
 0004:00002d7c       __imp_?qt_metacast@QDialog@@UAEPAXPBD@Z 0049ed7c     QtGui4:QtGui4.dll
 0004:00002d80       __imp_?qt_metacall@QDialog@@UAEHW4Call@QMetaObject@@HPAPAX@Z 0049ed80     QtGui4:QtGui4.dll
 0004:00002d84       __imp_?staticMetaObject@QDialog@@2UQMetaObject@@B 0049ed84     QtGui4:QtGui4.dll
 0004:00002d88       __imp_?qt_metacast@QRadioButton@@UAEPAXPBD@Z 0049ed88     QtGui4:QtGui4.dll
 0004:00002d8c       __imp_?qt_metacall@QRadioButton@@UAEHW4Call@QMetaObject@@HPAPAX@Z 0049ed8c     QtGui4:QtGui4.dll
 0004:00002d90       __imp_?staticMetaObject@QRadioButton@@2UQMetaObject@@B 0049ed90     QtGui4:QtGui4.dll
 0004:00002d94       __imp_?qt_metacast@QMainWindow@@UAEPAXPBD@Z 0049ed94     QtGui4:QtGui4.dll
 0004:00002d98       __imp_?qt_metacall@QMainWindow@@UAEHW4Call@QMetaObject@@HPAPAX@Z 0049ed98     QtGui4:QtGui4.dll
 0004:00002d9c       __imp_?staticMetaObject@QMainWindow@@2UQMetaObject@@B 0049ed9c     QtGui4:QtGui4.dll
 0004:00002da0       __imp_?qt_metacast@QWidgetAction@@UAEPAXPBD@Z 0049eda0     QtGui4:QtGui4.dll
 0004:00002da4       __imp_?qt_metacall@QWidgetAction@@UAEHW4Call@QMetaObject@@HPAPAX@Z 0049eda4     QtGui4:QtGui4.dll
 0004:00002da8       __imp_?staticMetaObject@QWidgetAction@@2UQMetaObject@@B 0049eda8     QtGui4:QtGui4.dll
 0004:00002dac       __imp_?qt_metacast@QLabel@@UAEPAXPBD@Z 0049edac     QtGui4:QtGui4.dll
 0004:00002db0       __imp_?qt_metacall@QLabel@@UAEHW4Call@QMetaObject@@HPAPAX@Z 0049edb0     QtGui4:QtGui4.dll
 0004:00002db4       __imp_?staticMetaObject@QLabel@@2UQMetaObject@@B 0049edb4     QtGui4:QtGui4.dll
 0004:00002db8       __imp_?qt_metacast@QFrame@@UAEPAXPBD@Z 0049edb8     QtGui4:QtGui4.dll
 0004:00002dbc       __imp_?qt_metacall@QFrame@@UAEHW4Call@QMetaObject@@HPAPAX@Z 0049edbc     QtGui4:QtGui4.dll
 0004:00002dc0       __imp_?staticMetaObject@QFrame@@2UQMetaObject@@B 0049edc0     QtGui4:QtGui4.dll
 0004:00002dc4       __imp_?qt_metacast@QSpinBox@@UAEPAXPBD@Z 0049edc4     QtGui4:QtGui4.dll
 0004:00002dc8       __imp_?qt_metacall@QSpinBox@@UAEHW4Call@QMetaObject@@HPAPAX@Z 0049edc8     QtGui4:QtGui4.dll
 0004:00002dcc       __imp_?staticMetaObject@QSpinBox@@2UQMetaObject@@B 0049edcc     QtGui4:QtGui4.dll
 0004:00002dd0       __imp_?qt_metacast@QMenu@@UAEPAXPBD@Z 0049edd0     QtGui4:QtGui4.dll
 0004:00002dd4       __imp_?qt_metacall@QMenu@@UAEHW4Call@QMetaObject@@HPAPAX@Z 0049edd4     QtGui4:QtGui4.dll
 0004:00002dd8       __imp_?qt_metacast@QProxyStyle@@UAEPAXPBD@Z 0049edd8     QtGui4:QtGui4.dll
 0004:00002ddc       __imp_?qt_metacall@QProxyStyle@@UAEHW4Call@QMetaObject@@HPAPAX@Z 0049eddc     QtGui4:QtGui4.dll
 0004:00002de0       __imp_?staticMetaObject@QMenu@@2UQMetaObject@@B 0049ede0     QtGui4:QtGui4.dll
 0004:00002de4       __imp_?staticMetaObject@QProxyStyle@@2UQMetaObject@@B 0049ede4     QtGui4:QtGui4.dll
 0004:00002de8       __imp_?qt_metacast@QPushButton@@UAEPAXPBD@Z 0049ede8     QtGui4:QtGui4.dll
 0004:00002dec       __imp_?qt_metacall@QPushButton@@UAEHW4Call@QMetaObject@@HPAPAX@Z 0049edec     QtGui4:QtGui4.dll
 0004:00002df0       __imp_?staticMetaObject@QPushButton@@2UQMetaObject@@B 0049edf0     QtGui4:QtGui4.dll
 0004:00002df4       __imp_?qt_metacast@QApplication@@UAEPAXPBD@Z 0049edf4     QtGui4:QtGui4.dll
 0004:00002df8       __imp_?qt_metacall@QApplication@@UAEHW4Call@QMetaObject@@HPAPAX@Z 0049edf8     QtGui4:QtGui4.dll
 0004:00002dfc       __imp_?staticMetaObject@QApplication@@2UQMetaObject@@B 0049edfc     QtGui4:QtGui4.dll
 0004:00002e00       __imp_?qt_metacast@QTabWidget@@UAEPAXPBD@Z 0049ee00     QtGui4:QtGui4.dll
 0004:00002e04       __imp_?qt_metacall@QTabWidget@@UAEHW4Call@QMetaObject@@HPAPAX@Z 0049ee04     QtGui4:QtGui4.dll
 0004:00002e08       __imp_?staticMetaObject@QTabWidget@@2UQMetaObject@@B 0049ee08     QtGui4:QtGui4.dll
 0004:00002e0c       __imp_?exec@QApplication@@SAHXZ 0049ee0c     QtGui4:QtGui4.dll
 0004:00002e10       __imp_?show@QWidget@@QAEXXZ 0049ee10     QtGui4:QtGui4.dll
 0004:00002e14       __imp_?move@QWidget@@QAEXHH@Z 0049ee14     QtGui4:QtGui4.dll
 0004:00002e18       __imp_?resize@QWidget@@QAEXABVQSize@@@Z 0049ee18     QtGui4:QtGui4.dll
 0004:00002e1c       __imp_?resize@QWidget@@QAEXHH@Z 0049ee1c     QtGui4:QtGui4.dll
 0004:00002e20       __imp_?availableGeometry@QDesktopWidget@@QBE?BVQRect@@H@Z 0049ee20     QtGui4:QtGui4.dll
 0004:00002e24       __imp_?desktop@QApplication@@SAPAVQDesktopWidget@@XZ 0049ee24     QtGui4:QtGui4.dll
 0004:00002e28       __imp_?compressEvent@QApplication@@MAE_NPAVQEvent@@PAVQObject@@PAVQPostEventList@@@Z 0049ee28     QtGui4:QtGui4.dll
 0004:00002e2c       __imp_?commitData@QApplication@@UAEXAAVQSessionManager@@@Z 0049ee2c     QtGui4:QtGui4.dll
 0004:00002e30       __imp_?saveState@QApplication@@UAEXAAVQSessionManager@@@Z 0049ee30     QtGui4:QtGui4.dll
 0004:00002e34       __imp_??1QApplication@@UAE@XZ 0049ee34     QtGui4:QtGui4.dll
 0004:00002e38       __imp_?notify@QApplication@@UAE_NPAVQObject@@PAVQEvent@@@Z 0049ee38     QtGui4:QtGui4.dll
 0004:00002e3c       __imp_?showText@QToolTip@@SAXABVQPoint@@ABVQString@@PAVQWidget@@@Z 0049ee3c     QtGui4:QtGui4.dll
 0004:00002e40       __imp_?globalPos@QHelpEvent@@QBEABVQPoint@@XZ 0049ee40     QtGui4:QtGui4.dll
 0004:00002e44       __imp_??1QIcon@@QAE@XZ     0049ee44     QtGui4:QtGui4.dll
 0004:00002e48       __imp_?setWindowIcon@QApplication@@SAXABVQIcon@@@Z 0049ee48     QtGui4:QtGui4.dll
 0004:00002e4c       __imp_??0QIcon@@QAE@ABVQString@@@Z 0049ee4c     QtGui4:QtGui4.dll
 0004:00002e50       __imp_?exec@QDialog@@QAEHXZ 0049ee50     QtGui4:QtGui4.dll
 0004:00002e54       __imp_?setFixedSize@QWidget@@QAEXHH@Z 0049ee54     QtGui4:QtGui4.dll
 0004:00002e58       __imp_??1QFont@@QAE@XZ     0049ee58     QtGui4:QtGui4.dll
 0004:00002e5c       __imp_?setFont@QApplication@@SAXABVQFont@@PBD@Z 0049ee5c     QtGui4:QtGui4.dll
 0004:00002e60       __imp_?setStyleHint@QFont@@QAEXW4StyleHint@1@W4StyleStrategy@1@@Z 0049ee60     QtGui4:QtGui4.dll
 0004:00002e64       __imp_?setPointSize@QFont@@QAEXH@Z 0049ee64     QtGui4:QtGui4.dll
 0004:00002e68       __imp_?setFamily@QFont@@QAEXABVQString@@@Z 0049ee68     QtGui4:QtGui4.dll
 0004:00002e6c       __imp_??0QFont@@QAE@XZ     0049ee6c     QtGui4:QtGui4.dll
 0004:00002e70       __imp_?setStyleSheet@QApplication@@QAEXABVQString@@@Z 0049ee70     QtGui4:QtGui4.dll
 0004:00002e74       __imp_?setStyle@QApplication@@SAXPAVQStyle@@@Z 0049ee74     QtGui4:QtGui4.dll
 0004:00002e78       __imp_?create@QStyleFactory@@SAPAVQStyle@@ABVQString@@@Z 0049ee78     QtGui4:QtGui4.dll
 0004:00002e7c       __imp_?screenGeometry@QDesktopWidget@@QBE?BVQRect@@H@Z 0049ee7c     QtGui4:QtGui4.dll
 0004:00002e80       __imp_?screenCount@QDesktopWidget@@QBEHXZ 0049ee80     QtGui4:QtGui4.dll
 0004:00002e84       __imp_??1QMainWindow@@UAE@XZ 0049ee84     QtGui4:QtGui4.dll
 0004:00002e88       __imp_??0QMainWindow@@QAE@PAVQWidget@@V?$QFlags@W4WindowType@Qt@@@@@Z 0049ee88     QtGui4:QtGui4.dll
 0004:00002e8c       __imp_?event@QMainWindow@@MAE_NPAVQEvent@@@Z 0049ee8c     QtGui4:QtGui4.dll
 0004:00002e90       __imp_?setText@QLineEdit@@QAEXABVQString@@@Z 0049ee90     QtGui4:QtGui4.dll
 0004:00002e94       \177QtGui4_NULL_THUNK_DATA 0049ee94     QtGui4:QtGui4.dll
 0004:0000313c       __imp_?qt_metacall@QLocalServer@@UAEHW4Call@QMetaObject@@HPAPAX@Z 0049f13c     QtNetwork4:QtNetwork4.dll
 0004:00003140       __imp_?qt_metacast@QLocalServer@@UAEPAXPBD@Z 0049f140     QtNetwork4:QtNetwork4.dll
 0004:00003144       __imp_?metaObject@QLocalServer@@UBEPBUQMetaObject@@XZ 0049f144     QtNetwork4:QtNetwork4.dll
 0004:00003148       __imp_??0QLocalServer@@QAE@PAVQObject@@@Z 0049f148     QtNetwork4:QtNetwork4.dll
 0004:0000314c       __imp_?nextPendingConnection@QLocalServer@@UAEPAVQLocalSocket@@XZ 0049f14c     QtNetwork4:QtNetwork4.dll
 0004:00003150       __imp_?incomingConnection@QLocalServer@@MAEXI@Z 0049f150     QtNetwork4:QtNetwork4.dll
 0004:00003154       __imp_??1QLocalServer@@UAE@XZ 0049f154     QtNetwork4:QtNetwork4.dll
 0004:00003158       __imp_?errorString@QLocalServer@@QBE?AVQString@@XZ 0049f158     QtNetwork4:QtNetwork4.dll
 0004:0000315c       __imp_?listen@QLocalServer@@QAE_NABVQString@@@Z 0049f15c     QtNetwork4:QtNetwork4.dll
 0004:00003160       __imp_?removeServer@QLocalServer@@SA_NABVQString@@@Z 0049f160     QtNetwork4:QtNetwork4.dll
 0004:00003164       __imp_?waitForReadyRead@QLocalSocket@@UAE_NH@Z 0049f164     QtNetwork4:QtNetwork4.dll
 0004:00003168       __imp_?waitForBytesWritten@QLocalSocket@@UAE_NH@Z 0049f168     QtNetwork4:QtNetwork4.dll
 0004:0000316c       __imp_??1QLocalSocket@@UAE@XZ 0049f16c     QtNetwork4:QtNetwork4.dll
 0004:00003170       __imp_?waitForConnected@QLocalSocket@@QAE_NH@Z 0049f170     QtNetwork4:QtNetwork4.dll
 0004:00003174       __imp_?connectToServer@QLocalSocket@@QAEXABVQString@@V?$QFlags@W4OpenModeFlag@QIODevice@@@@@Z 0049f174     QtNetwork4:QtNetwork4.dll
 0004:00003178       __imp_??0QLocalSocket@@QAE@PAVQObject@@@Z 0049f178     QtNetwork4:QtNetwork4.dll
 0004:0000317c       __imp_?hasPendingConnections@QLocalServer@@UBE_NXZ 0049f17c     QtNetwork4:QtNetwork4.dll
 0004:00003180       \177QtNetwork4_NULL_THUNK_DATA 0049f180     QtNetwork4:QtNetwork4.dll
 0004:000031b8       __imp_??0QDomElement@@QAE@ABV0@@Z 0049f1b8     QtXml4:QtXml4.dll
 0004:000031bc       __imp_??1QDomNodeList@@QAE@XZ 0049f1bc     QtXml4:QtXml4.dll
 0004:000031c0       __imp_?item@QDomNodeList@@QBE?AVQDomNode@@H@Z 0049f1c0     QtXml4:QtXml4.dll
 0004:000031c4       __imp_?count@QDomNodeList@@QBEHXZ 0049f1c4     QtXml4:QtXml4.dll
 0004:000031c8       __imp_?elementsByTagName@QDomElement@@QBE?AVQDomNodeList@@ABVQString@@@Z 0049f1c8     QtXml4:QtXml4.dll
 0004:000031cc       __imp_?nodeName@QDomNode@@QBE?AVQString@@XZ 0049f1cc     QtXml4:QtXml4.dll
 0004:000031d0       __imp_?createElement@QDomDocument@@QAE?AVQDomElement@@ABVQString@@@Z 0049f1d0     QtXml4:QtXml4.dll
 0004:000031d4       __imp_??1QDomProcessingInstruction@@QAE@XZ 0049f1d4     QtXml4:QtXml4.dll
 0004:000031d8       __imp_?appendChild@QDomNode@@QAE?AV1@ABV1@@Z 0049f1d8     QtXml4:QtXml4.dll
 0004:000031dc       __imp_?createProcessingInstruction@QDomDocument@@QAE?AVQDomProcessingInstruction@@ABVQString@@0@Z 0049f1dc     QtXml4:QtXml4.dll
 0004:000031e0       __imp_??0QDomNode@@QAE@ABV0@@Z 0049f1e0     QtXml4:QtXml4.dll
 0004:000031e4       __imp_?createTextNode@QDomDocument@@QAE?AVQDomText@@ABVQString@@@Z 0049f1e4     QtXml4:QtXml4.dll
 0004:000031e8       __imp_??0QDomDocument@@QAE@ABV0@@Z 0049f1e8     QtXml4:QtXml4.dll
 0004:000031ec       __imp_?setData@QDomCharacterData@@QAEXABVQString@@@Z 0049f1ec     QtXml4:QtXml4.dll
 0004:000031f0       __imp_?toText@QDomNode@@QBE?AVQDomText@@XZ 0049f1f0     QtXml4:QtXml4.dll
 0004:000031f4       __imp_?isText@QDomNode@@QBE_NXZ 0049f1f4     QtXml4:QtXml4.dll
 0004:000031f8       __imp_?setAttribute@QDomElement@@QAEXABVQString@@0@Z 0049f1f8     QtXml4:QtXml4.dll
 0004:000031fc       __imp_?data@QDomCharacterData@@QBE?AVQString@@XZ 0049f1fc     QtXml4:QtXml4.dll
 0004:00003200       __imp_?attribute@QDomElement@@QBE?AVQString@@ABV2@0@Z 0049f200     QtXml4:QtXml4.dll
 0004:00003204       __imp_?removeChild@QDomNode@@QAE?AV1@ABV1@@Z 0049f204     QtXml4:QtXml4.dll
 0004:00003208       __imp_?tagName@QDomElement@@QBE?AVQString@@XZ 0049f208     QtXml4:QtXml4.dll
 0004:0000320c       __imp_??1QDomElement@@QAE@XZ 0049f20c     QtXml4:QtXml4.dll
 0004:00003210       __imp_??0QDomDocument@@QAE@XZ 0049f210     QtXml4:QtXml4.dll
 0004:00003214       __imp_??0QDomElement@@QAE@XZ 0049f214     QtXml4:QtXml4.dll
 0004:00003218       __imp_?toElement@QDomNode@@QBE?AVQDomElement@@XZ 0049f218     QtXml4:QtXml4.dll
 0004:0000321c       __imp_??4QDomDocument@@QAEAAV0@ABV0@@Z 0049f21c     QtXml4:QtXml4.dll
 0004:00003220       __imp_?isNull@QDomNode@@QBE_NXZ 0049f220     QtXml4:QtXml4.dll
 0004:00003224       __imp_?hasChildNodes@QDomNode@@QBE_NXZ 0049f224     QtXml4:QtXml4.dll
 0004:00003228       __imp_?firstChild@QDomNode@@QBE?AV1@XZ 0049f228     QtXml4:QtXml4.dll
 0004:0000322c       __imp_?nextSibling@QDomNode@@QBE?AV1@XZ 0049f22c     QtXml4:QtXml4.dll
 0004:00003230       __imp_??4QDomNode@@QAEAAV0@ABV0@@Z 0049f230     QtXml4:QtXml4.dll
 0004:00003234       __imp_??1QDomNode@@QAE@XZ  0049f234     QtXml4:QtXml4.dll
 0004:00003238       __imp_?isElement@QDomNode@@QBE_NXZ 0049f238     QtXml4:QtXml4.dll
 0004:0000323c       __imp_?save@QDomNode@@QBEXAAVQTextStream@@H@Z 0049f23c     QtXml4:QtXml4.dll
 0004:00003240       __imp_?setContent@QDomDocument@@QAE_NPAVQIODevice@@PAVQString@@PAH2@Z 0049f240     QtXml4:QtXml4.dll
 0004:00003244       __imp_?documentElement@QDomDocument@@QBE?AVQDomElement@@XZ 0049f244     QtXml4:QtXml4.dll
 0004:00003248       __imp_??4QDomElement@@QAEAAV0@ABV0@@Z 0049f248     QtXml4:QtXml4.dll
 0004:0000324c       __imp_??1QDomDocument@@QAE@XZ 0049f24c     QtXml4:QtXml4.dll
 0004:00003250       __imp_??1QDomText@@QAE@XZ  0049f250     QtXml4:QtXml4.dll
 0004:00003254       \177QtXml4_NULL_THUNK_DATA 0049f254     QtXml4:QtXml4.dll
 0004:0000329c       __imp_??0GenericDS@aptui@@QAE@XZ 0049f29c     ToolGuiToolkit:ToolGuiToolkit.dll
 0004:000032a0       __imp_??1GenericDS@aptui@@UAE@XZ 0049f2a0     ToolGuiToolkit:ToolGuiToolkit.dll
 0004:000032a4       \177ToolGuiToolkit_NULL_THUNK_DATA 0049f2a4     ToolGuiToolkit:ToolGuiToolkit.dll
 0004:000032d0       __imp__SetClassLongW@12    0049f2d0     user32:USER32.dll
 0004:000032d4       __imp__GetClassLongW@8     0049f2d4     user32:USER32.dll
 0004:000032d8       \177USER32_NULL_THUNK_DATA 0049f2d8     user32:USER32.dll
 0004:00003304       __imp_?IsFullScreen@CWidgetSizeFactory@iVMSGUIToolkit@@QBE_NPAVQWidget@@@Z 0049f304     iVMSGUIToolkit:iVMSGUIToolkit.dll
 0004:00003308       __imp_?SignalWndSizeStatusChanged@CFancyTitle@iVMSGUIToolkit@@IAEXXZ 0049f308     iVMSGUIToolkit:iVMSGUIToolkit.dll
 0004:0000330c       __imp_?IsMaximized@CWidgetSizeFactory@iVMSGUIToolkit@@QBE_NPAVQWidget@@@Z 0049f30c     iVMSGUIToolkit:iVMSGUIToolkit.dll
 0004:00003310       __imp_?ShowNormal@CWidgetSizeFactory@iVMSGUIToolkit@@QAEXPAVQWidget@@ABVQSize@@@Z 0049f310     iVMSGUIToolkit:iVMSGUIToolkit.dll
 0004:00003314       __imp_?ShowMaximized@CWidgetSizeFactory@iVMSGUIToolkit@@QAEXPAVQWidget@@@Z 0049f314     iVMSGUIToolkit:iVMSGUIToolkit.dll
 0004:00003318       __imp_?GetIndependentWindow@iVMSGUIToolkit@@YAPAVQWidget@@PAV2@PBD@Z 0049f318     iVMSGUIToolkit:iVMSGUIToolkit.dll
 0004:0000331c       __imp_??1CWidgetItem@iVMSGUIToolkit@@UAE@XZ 0049f31c     iVMSGUIToolkit:iVMSGUIToolkit.dll
 0004:00003320       __imp_??1CHBoxLayout@iVMSGUIToolkit@@UAE@XZ 0049f320     iVMSGUIToolkit:iVMSGUIToolkit.dll
 0004:00003324       __imp_?setGeometry@CWidgetItem@iVMSGUIToolkit@@UAEXABVQRect@@@Z 0049f324     iVMSGUIToolkit:iVMSGUIToolkit.dll
 0004:00003328       __imp_??0CHBoxLayout@iVMSGUIToolkit@@QAE@PAVQWidget@@@Z 0049f328     iVMSGUIToolkit:iVMSGUIToolkit.dll
 0004:0000332c       __imp_?SetLayoutContentsMargins@CHBoxLayout@iVMSGUIToolkit@@QAEXHHHH@Z 0049f32c     iVMSGUIToolkit:iVMSGUIToolkit.dll
 0004:00003330       __imp_?SetLayoutSpacing@CHBoxLayout@iVMSGUIToolkit@@QAEXH@Z 0049f330     iVMSGUIToolkit:iVMSGUIToolkit.dll
 0004:00003334       __imp_??0CMenu@iVMSGUIToolkit@@QAE@PAVQWidget@@@Z 0049f334     iVMSGUIToolkit:iVMSGUIToolkit.dll
 0004:00003338       __imp_??0CLineEdit@iVMSGUIToolkit@@QAE@PAVQWidget@@@Z 0049f338     iVMSGUIToolkit:iVMSGUIToolkit.dll
 0004:0000333c       __imp_??0CComboBox@iVMSGUIToolkit@@QAE@PAVQWidget@@@Z 0049f33c     iVMSGUIToolkit:iVMSGUIToolkit.dll
 0004:00003340       __imp_??0CRadioButton@iVMSGUIToolkit@@QAE@PAVQWidget@@@Z 0049f340     iVMSGUIToolkit:iVMSGUIToolkit.dll
 0004:00003344       __imp_??0CPushButton@iVMSGUIToolkit@@QAE@PAVQWidget@@@Z 0049f344     iVMSGUIToolkit:iVMSGUIToolkit.dll
 0004:00003348       __imp_?validate@CIntValidator@iVMSGUIToolkit@@UBE?AW4State@QValidator@@AAVQString@@AAH@Z 0049f348     iVMSGUIToolkit:iVMSGUIToolkit.dll
 0004:0000334c       __imp_?qt_metacall@CIntValidator@iVMSGUIToolkit@@UAEHW4Call@QMetaObject@@HPAPAX@Z 0049f34c     iVMSGUIToolkit:iVMSGUIToolkit.dll
 0004:00003350       __imp_?qt_metacast@CIntValidator@iVMSGUIToolkit@@UAEPAXPBD@Z 0049f350     iVMSGUIToolkit:iVMSGUIToolkit.dll
 0004:00003354       __imp_?metaObject@CIntValidator@iVMSGUIToolkit@@UBEPBUQMetaObject@@XZ 0049f354     iVMSGUIToolkit:iVMSGUIToolkit.dll
 0004:00003358       __imp_??0CIntValidator@iVMSGUIToolkit@@QAE@HHPAVQObject@@@Z 0049f358     iVMSGUIToolkit:iVMSGUIToolkit.dll
 0004:0000335c       __imp_?InitGuiTextCodec@iVMSGUIToolkit@@YAXPAVQTextCodec@@@Z 0049f35c     iVMSGUIToolkit:iVMSGUIToolkit.dll
 0004:00003360       __imp_?InitGuiLocale@iVMSGUIToolkit@@YAXABVQLocale@@@Z 0049f360     iVMSGUIToolkit:iVMSGUIToolkit.dll
 0004:00003364       __imp_?ReadAll@CFile@iVMSGUIToolkit@@SA?AVQString@@ABVQStringList@@ABV3@@Z 0049f364     iVMSGUIToolkit:iVMSGUIToolkit.dll
 0004:00003368       __imp_??1CMenu@iVMSGUIToolkit@@UAE@XZ 0049f368     iVMSGUIToolkit:iVMSGUIToolkit.dll
 0004:0000336c       __imp_?AddWidget@CHBoxLayout@iVMSGUIToolkit@@QAEXPAVQWidget@@@Z 0049f36c     iVMSGUIToolkit:iVMSGUIToolkit.dll
 0004:00003370       __imp_?ReadAll@CFile@iVMSGUIToolkit@@SA?AVQString@@ABV3@@Z 0049f370     iVMSGUIToolkit:iVMSGUIToolkit.dll
 0004:00003374       __imp_?GetTargetPath@iVMSGUIToolkit@@YA?AVQString@@XZ 0049f374     iVMSGUIToolkit:iVMSGUIToolkit.dll
 0004:00003378       __imp_?SetValue@CGenericDS@iVMSGUIToolkit@@QAE_NABVQString@@@Z 0049f378     iVMSGUIToolkit:iVMSGUIToolkit.dll
 0004:0000337c       __imp_?SaveXML@CGenericDS@iVMSGUIToolkit@@QAE_NABVQString@@@Z 0049f37c     iVMSGUIToolkit:iVMSGUIToolkit.dll
 0004:00003380       __imp_??0CGenericDS@iVMSGUIToolkit@@QAE@XZ 0049f380     iVMSGUIToolkit:iVMSGUIToolkit.dll
 0004:00003384       __imp_?LoadXML@CGenericDS@iVMSGUIToolkit@@QAE_NABVQString@@@Z 0049f384     iVMSGUIToolkit:iVMSGUIToolkit.dll
 0004:00003388       __imp_??1CGenericDS@iVMSGUIToolkit@@QAE@XZ 0049f388     iVMSGUIToolkit:iVMSGUIToolkit.dll
 0004:0000338c       __imp_?GetChildrenCount@CGenericDS@iVMSGUIToolkit@@QBEHXZ 0049f38c     iVMSGUIToolkit:iVMSGUIToolkit.dll
 0004:00003390       __imp_?GetChild@CGenericDS@iVMSGUIToolkit@@QBE?AV12@H@Z 0049f390     iVMSGUIToolkit:iVMSGUIToolkit.dll
 0004:00003394       __imp_?GetName@CGenericDS@iVMSGUIToolkit@@QBE?AVQString@@XZ 0049f394     iVMSGUIToolkit:iVMSGUIToolkit.dll
 0004:00003398       __imp_?GetChildByName@CGenericDS@iVMSGUIToolkit@@QBE?AV12@ABVQString@@@Z 0049f398     iVMSGUIToolkit:iVMSGUIToolkit.dll
 0004:0000339c       __imp_??4CGenericDS@iVMSGUIToolkit@@QAEAAV01@ABV01@@Z 0049f39c     iVMSGUIToolkit:iVMSGUIToolkit.dll
 0004:000033a0       __imp_?GetValue@CGenericDS@iVMSGUIToolkit@@QBE?AVQString@@XZ 0049f3a0     iVMSGUIToolkit:iVMSGUIToolkit.dll
 0004:000033a4       __imp_?GetTargetPathFile@iVMSGUIToolkit@@YA?AVQString@@ABV2@@Z 0049f3a4     iVMSGUIToolkit:iVMSGUIToolkit.dll
 0004:000033a8       __imp_?staticMetaObject@CMenu@iVMSGUIToolkit@@2UQMetaObject@@B 0049f3a8     iVMSGUIToolkit:iVMSGUIToolkit.dll
 0004:000033ac       __imp_?qt_metacall@CMenu@iVMSGUIToolkit@@UAEHW4Call@QMetaObject@@HPAPAX@Z 0049f3ac     iVMSGUIToolkit:iVMSGUIToolkit.dll
 0004:000033b0       __imp_?qt_metacast@CMenu@iVMSGUIToolkit@@UAEPAXPBD@Z 0049f3b0     iVMSGUIToolkit:iVMSGUIToolkit.dll
 0004:000033b4       __imp_?staticMetaObject@CFancyTitle@iVMSGUIToolkit@@2UQMetaObject@@B 0049f3b4     iVMSGUIToolkit:iVMSGUIToolkit.dll
 0004:000033b8       __imp_?qt_metacall@CFancyTitle@iVMSGUIToolkit@@UAEHW4Call@QMetaObject@@HPAPAX@Z 0049f3b8     iVMSGUIToolkit:iVMSGUIToolkit.dll
 0004:000033bc       __imp_?qt_metacast@CFancyTitle@iVMSGUIToolkit@@UAEPAXPBD@Z 0049f3bc     iVMSGUIToolkit:iVMSGUIToolkit.dll
 0004:000033c0       __imp_??0CWidgetItem@iVMSGUIToolkit@@QAE@PAVQWidget@@V?$QFlags@W4AlignmentFlag@Qt@@@@@Z 0049f3c0     iVMSGUIToolkit:iVMSGUIToolkit.dll
 0004:000033c4       __imp_?AddItem@CHBoxLayout@iVMSGUIToolkit@@QAEXPAVQLayoutItem@@H@Z 0049f3c4     iVMSGUIToolkit:iVMSGUIToolkit.dll
 0004:000033c8       __imp_?SetOpenDoubleClickEnable@CFancyTitle@iVMSGUIToolkit@@QAEX_N@Z 0049f3c8     iVMSGUIToolkit:iVMSGUIToolkit.dll
 0004:000033cc       __imp_?resizeEvent@CFancyTitle@iVMSGUIToolkit@@EAEXPAVQResizeEvent@@@Z 0049f3cc     iVMSGUIToolkit:iVMSGUIToolkit.dll
 0004:000033d0       __imp_?mouseMoveEvent@CFancyTitle@iVMSGUIToolkit@@EAEXPAVQMouseEvent@@@Z 0049f3d0     iVMSGUIToolkit:iVMSGUIToolkit.dll
 0004:000033d4       __imp_?mouseDoubleClickEvent@CFancyTitle@iVMSGUIToolkit@@EAEXPAVQMouseEvent@@@Z 0049f3d4     iVMSGUIToolkit:iVMSGUIToolkit.dll
 0004:000033d8       __imp_?mouseReleaseEvent@CFancyTitle@iVMSGUIToolkit@@EAEXPAVQMouseEvent@@@Z 0049f3d8     iVMSGUIToolkit:iVMSGUIToolkit.dll
 0004:000033dc       __imp_?mousePressEvent@CFancyTitle@iVMSGUIToolkit@@EAEXPAVQMouseEvent@@@Z 0049f3dc     iVMSGUIToolkit:iVMSGUIToolkit.dll
 0004:000033e0       __imp_??0CFancyTitle@iVMSGUIToolkit@@QAE@PAVQWidget@@@Z 0049f3e0     iVMSGUIToolkit:iVMSGUIToolkit.dll
 0004:000033e4       __imp_??1CFancyTitle@iVMSGUIToolkit@@UAE@XZ 0049f3e4     iVMSGUIToolkit:iVMSGUIToolkit.dll
 0004:000033e8       __imp_??1CSlider@iVMSGUIToolkit@@UAE@XZ 0049f3e8     iVMSGUIToolkit:iVMSGUIToolkit.dll
 0004:000033ec       __imp_?OnShowToolTip@CSlider@iVMSGUIToolkit@@MAEXH@Z 0049f3ec     iVMSGUIToolkit:iVMSGUIToolkit.dll
 0004:000033f0       __imp_?enterEvent@CSlider@iVMSGUIToolkit@@MAEXPAVQEvent@@@Z 0049f3f0     iVMSGUIToolkit:iVMSGUIToolkit.dll
 0004:000033f4       __imp_?mouseReleaseEvent@CSlider@iVMSGUIToolkit@@MAEXPAVQMouseEvent@@@Z 0049f3f4     iVMSGUIToolkit:iVMSGUIToolkit.dll
 0004:000033f8       __imp_?mousePressEvent@CSlider@iVMSGUIToolkit@@MAEXPAVQMouseEvent@@@Z 0049f3f8     iVMSGUIToolkit:iVMSGUIToolkit.dll
 0004:000033fc       __imp_?qt_metacall@CSlider@iVMSGUIToolkit@@UAEHW4Call@QMetaObject@@HPAPAX@Z 0049f3fc     iVMSGUIToolkit:iVMSGUIToolkit.dll
 0004:00003400       __imp_?qt_metacast@CSlider@iVMSGUIToolkit@@UAEPAXPBD@Z 0049f400     iVMSGUIToolkit:iVMSGUIToolkit.dll
 0004:00003404       __imp_?metaObject@CSlider@iVMSGUIToolkit@@UBEPBUQMetaObject@@XZ 0049f404     iVMSGUIToolkit:iVMSGUIToolkit.dll
 0004:00003408       __imp_??0CSlider@iVMSGUIToolkit@@QAE@PAVQWidget@@@Z 0049f408     iVMSGUIToolkit:iVMSGUIToolkit.dll
 0004:0000340c       __imp_??1CIntValidator@iVMSGUIToolkit@@UAE@XZ 0049f40c     iVMSGUIToolkit:iVMSGUIToolkit.dll
 0004:00003410       __imp_??1CPushButton@iVMSGUIToolkit@@UAE@XZ 0049f410     iVMSGUIToolkit:iVMSGUIToolkit.dll
 0004:00003414       __imp_??1CRadioButton@iVMSGUIToolkit@@UAE@XZ 0049f414     iVMSGUIToolkit:iVMSGUIToolkit.dll
 0004:00003418       __imp_??1CComboBox@iVMSGUIToolkit@@UAE@XZ 0049f418     iVMSGUIToolkit:iVMSGUIToolkit.dll
 0004:0000341c       __imp_??1CLineEdit@iVMSGUIToolkit@@UAE@XZ 0049f41c     iVMSGUIToolkit:iVMSGUIToolkit.dll
 0004:00003420       __imp_?paintEvent@CPushButton@iVMSGUIToolkit@@MAEXPAVQPaintEvent@@@Z 0049f420     iVMSGUIToolkit:iVMSGUIToolkit.dll
 0004:00003424       __imp_?leaveEvent@CPushButton@iVMSGUIToolkit@@MAEXPAVQEvent@@@Z 0049f424     iVMSGUIToolkit:iVMSGUIToolkit.dll
 0004:00003428       __imp_?enterEvent@CPushButton@iVMSGUIToolkit@@MAEXPAVQEvent@@@Z 0049f428     iVMSGUIToolkit:iVMSGUIToolkit.dll
 0004:0000342c       __imp_?qt_metacall@CPushButton@iVMSGUIToolkit@@UAEHW4Call@QMetaObject@@HPAPAX@Z 0049f42c     iVMSGUIToolkit:iVMSGUIToolkit.dll
 0004:00003430       __imp_?qt_metacast@CPushButton@iVMSGUIToolkit@@UAEPAXPBD@Z 0049f430     iVMSGUIToolkit:iVMSGUIToolkit.dll
 0004:00003434       __imp_?metaObject@CPushButton@iVMSGUIToolkit@@UBEPBUQMetaObject@@XZ 0049f434     iVMSGUIToolkit:iVMSGUIToolkit.dll
 0004:00003438       __imp_?qt_metacall@CRadioButton@iVMSGUIToolkit@@UAEHW4Call@QMetaObject@@HPAPAX@Z 0049f438     iVMSGUIToolkit:iVMSGUIToolkit.dll
 0004:0000343c       __imp_?qt_metacast@CRadioButton@iVMSGUIToolkit@@UAEPAXPBD@Z 0049f43c     iVMSGUIToolkit:iVMSGUIToolkit.dll
 0004:00003440       __imp_?metaObject@CRadioButton@iVMSGUIToolkit@@UBEPBUQMetaObject@@XZ 0049f440     iVMSGUIToolkit:iVMSGUIToolkit.dll
 0004:00003444       __imp_?qt_metacall@CComboBox@iVMSGUIToolkit@@UAEHW4Call@QMetaObject@@HPAPAX@Z 0049f444     iVMSGUIToolkit:iVMSGUIToolkit.dll
 0004:00003448       __imp_?qt_metacast@CComboBox@iVMSGUIToolkit@@UAEPAXPBD@Z 0049f448     iVMSGUIToolkit:iVMSGUIToolkit.dll
 0004:0000344c       __imp_?metaObject@CComboBox@iVMSGUIToolkit@@UBEPBUQMetaObject@@XZ 0049f44c     iVMSGUIToolkit:iVMSGUIToolkit.dll
 0004:00003450       __imp_?focusInEvent@CLineEdit@iVMSGUIToolkit@@MAEXPAVQFocusEvent@@@Z 0049f450     iVMSGUIToolkit:iVMSGUIToolkit.dll
 0004:00003454       __imp_?mousePressEvent@CLineEdit@iVMSGUIToolkit@@MAEXPAVQMouseEvent@@@Z 0049f454     iVMSGUIToolkit:iVMSGUIToolkit.dll
 0004:00003458       __imp_?qt_metacall@CLineEdit@iVMSGUIToolkit@@UAEHW4Call@QMetaObject@@HPAPAX@Z 0049f458     iVMSGUIToolkit:iVMSGUIToolkit.dll
 0004:0000345c       __imp_?qt_metacast@CLineEdit@iVMSGUIToolkit@@UAEPAXPBD@Z 0049f45c     iVMSGUIToolkit:iVMSGUIToolkit.dll
 0004:00003460       __imp_?metaObject@CLineEdit@iVMSGUIToolkit@@UBEPBUQMetaObject@@XZ 0049f460     iVMSGUIToolkit:iVMSGUIToolkit.dll
 0004:00003464       \177iVMSGUIToolkit_NULL_THUNK_DATA 0049f464     iVMSGUIToolkit:iVMSGUIToolkit.dll

 entry point at        0001:000691bf


 Exports

  ordinal    name

        1    ??4_Init_locks@std@@QAEAAV01@ABV01@@Z (public: class std::_Init_locks & __thiscall std::_Init_locks::operator=(class std::_Init_locks const &))
